LX51 LINKER/LOCATER V4.66.1.0                                                           03/23/2017  15:15:44  PAGE 1


LX51 LINKER/LOCATER V4.66.1.0, INVOKED BY:
C:\KEIL_V4\C51\BIN\LX51.EXE .\Output\main.obj, .\Output\Interrupt.obj, .\Output\MotorControl.obj, .\Output\SPWM.obj, .\O
>> utput\SinCos.obj, .\Output\MDU.obj, .\Output\LPF.obj, .\Output\BuzzerScan.obj, .\Output\IRScan.obj, .\Output\KeyScan.
>> obj, .\Output\PWMScan.obj, .\Output\UARTScan.obj, .\Output\LED.obj, .\Output\PID.obj, .\Output\UARTInit.obj, .\Output
>> \TimerInit.obj, .\Output\SPIInit.obj, .\Output\GPIOInit.obj, .\Output\ADCInit.obj, .\Output\CMPInit.obj, .\Output\AMP
>> Init.obj, .\Output\DriverInit.obj, .\Output\SystemInit.obj, .\Output\InterruptInit.obj, ..\Library\FU68xx_Hardware_Dr
>> iver\Source\FU68xx_System.LIB TO .\Output\FU68xx_SPWM_OnePhase PRINT (.\Listing\FU68xx_SPWM_OnePhase.map) REMOVEUNUSE
>> D


CPU MODE:     8051 MODE
MEMORY MODEL: LARGE WITH FLOATING POINT ARITHMETIC


INPUT MODULES INCLUDED:
  .\Output\main.obj (MAIN)
         COMMENT TYPE 0: C51 V9.52.0.0
  .\Output\Interrupt.obj (INTERRUPT)
         COMMENT TYPE 0: C51 V9.52.0.0
  .\Output\MotorControl.obj (MOTORCONTROL)
         COMMENT TYPE 0: C51 V9.52.0.0
  .\Output\SPWM.obj (SPWM)
         COMMENT TYPE 0: C51 V9.52.0.0
  .\Output\SinCos.obj (SINCOS)
         COMMENT TYPE 0: C51 V9.52.0.0
  .\Output\MDU.obj (MDU)
         COMMENT TYPE 0: C51 V9.52.0.0
  .\Output\LPF.obj (LPF)
         COMMENT TYPE 0: C51 V9.52.0.0
  .\Output\BuzzerScan.obj (BUZZERSCAN)
         COMMENT TYPE 0: C51 V9.52.0.0
  .\Output\IRScan.obj (IRSCAN)
         COMMENT TYPE 0: C51 V9.52.0.0
  .\Output\KeyScan.obj (KEYSCAN)
         COMMENT TYPE 0: C51 V9.52.0.0
  .\Output\PWMScan.obj (PWMSCAN)
         COMMENT TYPE 0: C51 V9.52.0.0
  .\Output\UARTScan.obj (UARTSCAN)
         COMMENT TYPE 0: C51 V9.52.0.0
  .\Output\LED.obj (LED)
         COMMENT TYPE 0: C51 V9.52.0.0
  .\Output\PID.obj (PID)
         COMMENT TYPE 0: C51 V9.52.0.0
  .\Output\UARTInit.obj (UARTINIT)
         COMMENT TYPE 0: C51 V9.52.0.0
  .\Output\TimerInit.obj (TIMERINIT)
         COMMENT TYPE 0: C51 V9.52.0.0
  .\Output\SPIInit.obj (SPIINIT)
         COMMENT TYPE 0: C51 V9.52.0.0
  .\Output\GPIOInit.obj (GPIOINIT)
         COMMENT TYPE 0: C51 V9.52.0.0
  .\Output\ADCInit.obj (ADCINIT)
         COMMENT TYPE 0: C51 V9.52.0.0
  .\Output\CMPInit.obj (CMPINIT)
         COMMENT TYPE 0: C51 V9.52.0.0
  .\Output\AMPInit.obj (AMPINIT)
         COMMENT TYPE 0: C51 V9.52.0.0
  .\Output\DriverInit.obj (DRIVERINIT)
         COMMENT TYPE 0: C51 V9.52.0.0
  .\Output\SystemInit.obj (SYSTEMINIT)
         COMMENT TYPE 0: C51 V9.52.0.0
  .\Output\InterruptInit.obj (INTERRUPTINIT)
         COMMENT TYPE 0: C51 V9.52.0.0
  ..\Library\FU68xx_Hardware_Driver\Source\FU68xx_System.LIB (FU68XX_SYSTEM)
         COMMENT TYPE 0: C51 V9.54
  C:\KEIL_V4\C51\LIB\C51FPL.LIB (?C?FPADD)
LX51 LINKER/LOCATER V4.66.1.0                                                         03/23/2017  15:15:44  PAGE 2


         COMMENT TYPE 1: A51 / ASM51 Assembler
  C:\KEIL_V4\C51\LIB\C51FPL.LIB (?C?FPMUL)
         COMMENT TYPE 1: A51 / ASM51 Assembler
  C:\KEIL_V4\C51\LIB\C51FPL.LIB (?C?FPDIV)
         COMMENT TYPE 1: A51 / ASM51 Assembler
  C:\KEIL_V4\C51\LIB\C51FPL.LIB (?C?FCAST)
         COMMENT TYPE 1: A51 / ASM51 Assembler
  C:\KEIL_V4\C51\LIB\C51FPL.LIB (?C?CASTF)
         COMMENT TYPE 1: A51 / ASM51 Assembler
  C:\KEIL_V4\C51\LIB\C51FPL.LIB (?C?FPGETOPN)
         COMMENT TYPE 1: A51 / ASM51 Assembler
  C:\KEIL_V4\C51\LIB\C51L.LIB (?C_STARTUP)
         COMMENT TYPE 1: A51 / ASM51 Assembler
  C:\KEIL_V4\C51\LIB\C51L.LIB (?C?ULDIV)
         COMMENT TYPE 1: A51 / ASM51 Assembler
  C:\KEIL_V4\C51\LIB\C51L.LIB (?C?LNEG)
         COMMENT TYPE 1: A51 / ASM51 Assembler
  C:\KEIL_V4\C51\LIB\C51L.LIB (?C?SLCMP)
         COMMENT TYPE 1: A51 / ASM51 Assembler
  C:\KEIL_V4\C51\LIB\C51L.LIB (?C?ULCMP)
         COMMENT TYPE 1: A51 / ASM51 Assembler
  C:\KEIL_V4\C51\LIB\C51L.LIB (?C?SLSHR)
         COMMENT TYPE 1: A51 / ASM51 Assembler
  C:\KEIL_V4\C51\LIB\C51L.LIB (?C?LSTXDATA)
         COMMENT TYPE 1: A51 / ASM51 Assembler
  C:\KEIL_V4\C51\LIB\C51L.LIB (?C?LSTKXDATA)
         COMMENT TYPE 1: A51 / ASM51 Assembler
  C:\KEIL_V4\C51\LIB\C51L.LIB (?C?ICASE)
         COMMENT TYPE 1: A51 / ASM51 Assembler
  C:\KEIL_V4\C51\LIB\C51L.LIB (?C?LIMUL)
         COMMENT TYPE 1: A51 / ASM51 Assembler
  C:\KEIL_V4\C51\LIB\C51L.LIB (?C_INIT)
         COMMENT TYPE 1: A51 / ASM51 Assembler


ACTIVE MEMORY CLASSES OF MODULE:  .\Output\FU68xx_SPWM_OnePhase (MAIN)

BASE        START       END         USED      MEMORY CLASS
==========================================================
C:000000H   C:000000H   C:00FFFFH   001EA6H   CODE
X:000000H   X:000000H   X:00FFFFH   000190H   XDATA
I:000000H   I:000000H   I:0000FFH   000039H   IDATA
I:000020H.0 I:000020H.0 I:00002FH.7 000000H.3 BIT
I:000000H   I:000000H   I:00007FH   000008H   DATA


MEMORY MAP OF MODULE:  .\Output\FU68xx_SPWM_OnePhase (MAIN)


START     STOP      LENGTH    ALIGN  RELOC    MEMORY CLASS   SEGMENT NAME
=========================================================================

* * * * * * * * * * *   D A T A   M E M O R Y   * * * * * * * * * * * * *
000000H   000007H   000008H   ---    AT..     DATA           "REG BANK 0"
000008H.0 00001FH.7 000018H.0 ---    ---      **GAP**
000020H.0 000020H.1 000000H.2 BIT    UNIT     BIT            _BIT_GROUP_
000020H.2 000020H.2 000000H.1 BIT    UNIT     BIT            ?BI?PID
000020H.3 000020H   000000H.5 ---    ---      **GAP**
000021H   000058H   000038H   BYTE   UNIT     IDATA          ?ID?PID
000059H   000059H   000001H   BYTE   UNIT     IDATA          ?STACK

* * * * * * * * * * *   C O D E   M E M O R Y   * * * * * * * * * * * * *
000000H   000002H   000003H   ---    OFFS..   CODE           ?CO??C_STARTUP?0
000003H   000021H   00001FH   BYTE   UNIT     CODE           ?PR?SOFTWAREINIT?MAIN
000022H   000022H   000001H   ---    ---      **GAP**
LX51 LINKER/LOCATER V4.66.1.0                                                         03/23/2017  15:15:44  PAGE 3


000023H   000025H   000003H   BYTE   OFFS..   CODE           ?INTERRUPT?00023
000026H   000031H   00000CH   BYTE   UNIT     CODE           ?PR?MDUINIT?MDU
000032H   000032H   000001H   ---    ---      **GAP**
000033H   000035H   000003H   BYTE   OFFS..   CODE           ?INTERRUPT?00033
000036H   00003AH   000005H   ---    ---      **GAP**
00003BH   00003DH   000003H   BYTE   OFFS..   CODE           ?INTERRUPT?0003B
00003EH   000049H   00000CH   BYTE   UNIT     CODE           ?PR?BUZZERINIT?BUZZERSCAN
00004AH   00004AH   000001H   ---    ---      **GAP**
00004BH   00004DH   000003H   BYTE   OFFS..   CODE           ?INTERRUPT?0004B
00004EH   000052H   000005H   ---    ---      **GAP**
000053H   000055H   000003H   BYTE   OFFS..   CODE           ?INTERRUPT?00053
000056H   00005FH   00000AH   BYTE   UNIT     CODE           ?PR?MOTORINIT?MOTORCONTROL
000060H   000062H   000003H   ---    ---      **GAP**
000063H   000065H   000003H   BYTE   OFFS..   CODE           ?INTERRUPT?00063
000066H   000570H   00050BH   BYTE   UNIT     CODE           ?C?LIB_CODE
000571H   0007B1H   000241H   BYTE   UNIT     CODE           ?PR?FAULTDETECT?MOTORCONTROL
0007B2H   000994H   0001E3H   BYTE   UNIT     CODE           ?PR?SPWM?SPWM
000995H   000B40H   0001ACH   BYTE   UNIT     CODE           ?PR?SPEEDCONTROL?MOTORCONTROL
000B41H   000CACH   00016CH   BYTE   UNIT     CODE           ?PR?ADC_ISR?INTERRUPT
000CADH   000DF2H   000146H   BYTE   UNIT     CODE           ?PR?TIM0INIT?TIMERINIT
000DF3H   000F00H   00010EH   BYTE   UNIT     CODE           ?PR?MOTORPRECHARGE?MOTORCONTROL
000F01H   001005H   000105H   BYTE   UNIT     CODE           ?PR?IRSCANCONTROL?IRSCAN
001006H   0010FEH   0000F9H   BYTE   UNIT     CODE           ?PR?SYSTEMTICK?MOTORCONTROL
0010FFH   0011E9H   0000EBH   BYTE   UNIT     CODE           ?PR?MDUAPP?MDU
0011EAH   0012CEH   0000E5H   BYTE   UNIT     CODE           ?PR?PARAMETERINIT?MOTORCONTROL
0012CFH   00139BH   0000CDH   BYTE   UNIT     CODE           ?C_INITSEG
00139CH   00143BH   0000A0H   BYTE   UNIT     CODE           ?PR?ADCDATAINIT?ADCINIT
00143CH   0014D0H   000095H   BYTE   UNIT     CODE           ?PR?LEDCONTROL?LED
0014D1H   001562H   000092H   BYTE   UNIT     CODE           ?PR?KEYVALUE?KEYSCAN
001563H   0015EEH   00008CH   BYTE   UNIT     CODE           ?C_C51STARTUP
0015EFH   001671H   000083H   BYTE   UNIT     CODE           ?PR?ADCINIT?ADCINIT
001672H   0016DCH   00006BH   BYTE   UNIT     CODE           ?PR?TIM0_ISR?INTERRUPT
0016DDH   001740H   000064H   BYTE   UNIT     CODE           ?PR?TIM45_ISR?INTERRUPT
001741H   00179EH   00005EH   BYTE   UNIT     CODE           ?PR?RESTARTCONTROL?MOTORCONTROL
00179FH   0017F6H   000058H   BYTE   UNIT     CODE           ?PR?MAIN?MAIN
0017F7H   00184CH   000056H   BYTE   UNIT     CODE           ?PR?GPIOINIT?GPIOINIT
00184DH   00189BH   00004FH   BYTE   UNIT     CODE           ?PR?TIM4INIT?TIMERINIT
00189CH   0018E6H   00004BH   BYTE   UNIT     CODE           ?PR?SPIINIT?SPIINIT
0018E7H   00192DH   000047H   BYTE   UNIT     CODE           ?PR?TIM23_ISR?INTERRUPT
00192EH   001973H   000046H   BYTE   UNIT     CODE           ?PR?KEYINIT?KEYSCAN
001974H   0019B8H   000045H   BYTE   UNIT     CODE           ?PR?_VREFCONFIG?FU68XX_SYSTEM
0019B9H   0019F8H   000040H   BYTE   UNIT     CODE           ?PR?ONOFFCONTROL?MOTORCONTROL
0019F9H   001A37H   00003FH   BYTE   UNIT     CODE           ?PR?_MDU_MULA_U16?MDU
001A38H   001A75H   00003EH   BYTE   UNIT     CODE           ?PR?MOTORMAIN?MOTORCONTROL
001A76H   001AADH   000038H   BYTE   UNIT     CODE           ?PR?MOTORSTOP?MOTORCONTROL
001AAEH   001AE5H   000038H   BYTE   UNIT     CODE           ?PR?_MDU_MULA_S16?MDU
001AE6H   001B1CH   000037H   BYTE   UNIT     CODE           ?PR?TIM3INIT?TIMERINIT
001B1DH   001B53H   000037H   BYTE   UNIT     CODE           ?PR?_WATCHDOGCONFIG?FU68XX_SYSTEM
001B54H   001B89H   000036H   BYTE   UNIT     CODE           ?PR?BUZZERSCAN?BUZZERSCAN
001B8AH   001BBCH   000033H   BYTE   UNIT     CODE           ?PR?CMPIINT?CMPINIT
001BBDH   001BECH   000030H   BYTE   UNIT     CODE           ?PR?UARTSCANINIT?UARTSCAN
001BEDH   001C1BH   00002FH   BYTE   UNIT     CODE           ?PR?CMP_ISR?INTERRUPT
001C1CH   001C49H   00002EH   BYTE   UNIT     CODE           ?PR?IRINIT?IRSCAN
001C4AH   001C75H   00002CH   BYTE   UNIT     CODE           ?PR?UART_ISR?INTERRUPT
001C76H   001CA0H   00002BH   BYTE   UNIT     CODE           ?PR?MOTORNORMAL?MOTORCONTROL
001CA1H   001CC7H   000027H   BYTE   UNIT     CODE           ?PR?MOTORFAULT?MOTORCONTROL
001CC8H   001CECH   000025H   BYTE   UNIT     CODE           ?PR?INTERRUPTINIT?INTERRUPTINIT
001CEDH   001D10H   000024H   BYTE   UNIT     CODE           ?PR?HARDWAREINIT?MAIN
001D11H   001D32H   000022H   BYTE   UNIT     CODE           ?PR?_LPF?LPF
001D33H   001D54H   000022H   BYTE   UNIT     CODE           ?PR?KEYSCAN?KEYSCAN
001D55H   001D75H   000021H   BYTE   UNIT     CODE           ?PR?PWMSCAN?PWMSCAN
001D76H   001D96H   000021H   BYTE   UNIT     CODE           ?PR?SYSTEMINIT?SYSTEMINIT
001D97H   001DB4H   00001EH   BYTE   UNIT     CODE           ?PR?VHALFCONFIG?FU68XX_SYSTEM
001DB5H   001DD1H   00001DH   BYTE   UNIT     CODE           ?PR?DRIVERINIT?DRIVERINIT
001DD2H   001DEBH   00001AH   BYTE   UNIT     CODE           ?PR?_MDU_MUL_U16?MDU
LX51 LINKER/LOCATER V4.66.1.0                                                         03/23/2017  15:15:44  PAGE 4


001DECH   001E05H   00001AH   BYTE   UNIT     CODE           ?PR?MDUCONTROLINIT?MDU
001E06H   001E1EH   000019H   BYTE   UNIT     CODE           ?PR?PWMIN_INIT?PWMSCAN
001E1FH   001E36H   000018H   BYTE   UNIT     CODE           ?PR?_SINCOS?SINCOS
001E37H   001E4EH   000018H   BYTE   UNIT     CODE           ?PR?AMPIINT?AMPINIT
001E4FH   001E64H   000016H   BYTE   UNIT     CODE           ?PR?EXTERNALSLOWCLOCKCONFIG?FU68XX_SYSTEM
001E65H   001E77H   000013H   BYTE   UNIT     CODE           ?PR?MOTORSTART?MOTORCONTROL
001E78H   001E89H   000012H   BYTE   UNIT     CODE           ?PR?SINCOSINIT?SINCOS
001E8AH   001E98H   00000FH   BYTE   UNIT     CODE           ?PR?SYSTEMFASTCLOCKCONFIG?FU68XX_SYSTEM
001E99H   001EA6H   00000EH   BYTE   UNIT     CODE           ?PR?LEDCONTROLINIT?LED
001EA7H   001EAEH   000008H   BYTE   UNIT     CODE           ?PR?WATCHDOGREFRESH?FU68XX_SYSTEM
001EAFH   001EB5H   000007H   BYTE   UNIT     CODE           ?PR?MOTORREADY?MOTORCONTROL

* * * * * * * * * * *  X D A T A   M E M O R Y  * * * * * * * * * * * * *
000000H   0000B6H   0000B7H   BYTE   UNIT     XDATA          ?XD?MOTORCONTROL
0000B7H   0000FAH   000044H   BYTE   UNIT     XDATA          ?XD?ADCINIT
0000FBH   000114H   00001AH   BYTE   UNIT     XDATA          ?XD?SINCOS
000115H   00012CH   000018H   BYTE   UNIT     XDATA          _XDATA_GROUP_
00012DH   000141H   000015H   BYTE   UNIT     XDATA          ?XD?IRSCAN
000142H   000156H   000015H   BYTE   UNIT     XDATA          ?XD?UARTSCAN
000157H   000166H   000010H   BYTE   UNIT     XDATA          ?XD?INTERRUPT
000167H   00016FH   000009H   BYTE   UNIT     XDATA          ?XD?MDU
000170H   000178H   000009H   BYTE   UNIT     XDATA          ?XD?PWMSCAN
000179H   000180H   000008H   BYTE   UNIT     XDATA          ?XD?KEYSCAN
000181H   000186H   000006H   BYTE   UNIT     XDATA          ?XD?PID
000187H   00018BH   000005H   BYTE   UNIT     XDATA          ?XD?LED
00018CH   00018FH   000004H   BYTE   UNIT     XDATA          ?XD?BUZZERSCAN

* * * * * * * * *   R E M O V E D     S E G M E N T S   * * * * * * * *
   *DEL*:           000014H   BYTE   UNIT     CODE           ?PR?CURRENTCONTROL?MOTORCONTROL
   *DEL*:           00023CH   BYTE   UNIT     CODE           ?PR?_SIN?SINCOS
   *DEL*:           00000DH   BYTE   UNIT     XDATA          ?XD?_SIN?SINCOS
   *DEL*:           0002B2H   BYTE   UNIT     CODE           ?PR?_COS?SINCOS
   *DEL*:           000016H   BYTE   UNIT     XDATA          ?XD?_COS?SINCOS
   *DEL*:           00002EH   BYTE   UNIT     CODE           ?PR?_MDU_MUL_U32?MDU
   *DEL*:           00001AH   BYTE   UNIT     CODE           ?PR?_MDU_MUL_S16?MDU
   *DEL*:           00002EH   BYTE   UNIT     CODE           ?PR?_MDU_MUL_S32?MDU
   *DEL*:           000054H   BYTE   UNIT     CODE           ?PR?_MDU_MULA_U32?MDU
   *DEL*:           000007H   BYTE   UNIT     XDATA          ?XD?_MDU_MULA_U32?MDU
   *DEL*:           000054H   BYTE   UNIT     CODE           ?PR?_MDU_MULA_S32?MDU
   *DEL*:           000007H   BYTE   UNIT     XDATA          ?XD?_MDU_MULA_S32?MDU
   *DEL*:           000041H   BYTE   UNIT     CODE           ?PR?_MDU_DIV_U16?MDU
   *DEL*:           000064H   BYTE   UNIT     CODE           ?PR?_MDU_DIV_U32?MDU
   *DEL*:           000002H   BYTE   UNIT     XDATA          ?XD?_MDU_DIV_U32?MDU
   *DEL*:           0000C6H   BYTE   UNIT     CODE           ?PR?IRVALUE?IRSCAN
   *DEL*:           000001H   BYTE   UNIT     CODE           ?PR?UARTSCANCONTROL?UARTSCAN
   *DEL*:           0000CAH   BYTE   UNIT     CODE           ?PR?_SETCURRENT?PID
   *DEL*:           00001CH   BYTE   UNIT     CODE           ?PR?UARTINIT?UARTINIT
   *DEL*:           000028H   BYTE   UNIT     CODE           ?PR?_UARTSENDDATA?UARTINIT
   *DEL*:           0000F9H   BYTE   UNIT     CODE           ?PR?TIM1INIT?TIMERINIT
   *DEL*:           000054H   BYTE   UNIT     CODE           ?PR?TIM2INIT?TIMERINIT
   *DEL*:           00004FH   BYTE   UNIT     CODE           ?PR?TIM5INIT?TIMERINIT
   *DEL*:           00005CH   BYTE   UNIT     CODE           ?PR?_TIM5_TIMING_US?TIMERINIT
   *DEL*:           000051H   BYTE   UNIT     CODE           ?PR?_SPISENDDATA?SPIINIT
   *DEL*:           00007CH   BYTE   UNIT     CODE           ?PR?ADCGETCONVERSIONVALUE?ADCINIT
   *DEL*:           00001BH   BYTE   UNIT     CODE           ?PR?INTERNALFASTCLOCKCONFIG?FU68XX_SYSTEM
   *DEL*:           000000H.1 BIT    UNIT     BIT            ?BI?INTERNALFASTCLOCKCONFIG?FU68XX_SYSTEM
   *DEL*:           00000FH   BYTE   UNIT     CODE           ?PR?LVDPOWERDOWNDETECTCONFIG?FU68XX_SYSTEM
   *DEL*:           000000H.1 BIT    UNIT     BIT            ?BI?LVDPOWERDOWNDETECTCONFIG?FU68XX_SYSTEM
   *DEL*:           00000FH   BYTE   UNIT     CODE           ?PR?LVDPOWERDOWNWARNIECONFIG?FU68XX_SYSTEM
   *DEL*:           000000H.1 BIT    UNIT     BIT            ?BI?LVDPOWERDOWNWARNIECONFIG?FU68XX_SYSTEM
   *DEL*:           000031H   BYTE   UNIT     CODE           ?PR?_FLASH_SECTOR_ERASE?FU68XX_SYSTEM
   *DEL*:           000000H.1 BIT    UNIT     BIT            ?BI?_FLASH_SECTOR_ERASE?FU68XX_SYSTEM
   *DEL*:           000030H   BYTE   UNIT     CODE           ?PR?_FLASH_SECTOR_WRITE?FU68XX_SYSTEM
   *DEL*:           000000H.1 BIT    UNIT     BIT            ?BI?_FLASH_SECTOR_WRITE?FU68XX_SYSTEM

LX51 LINKER/LOCATER V4.66.1.0                                                         03/23/2017  15:15:44  PAGE 5




OVERLAY MAP OF MODULE:   .\Output\FU68xx_SPWM_OnePhase (MAIN)


FUNCTION/MODULE                              BIT_GROUP   XDATA_GROUP
--> CALLED FUNCTION/MODULE                  START  STOP  START  STOP
====================================================================
TIM0_ISR/INTERRUPT                          ----- -----  ----- -----
  +--> SYSTEMTICK/MOTORCONTROL
  +--> MDUAPP/MDU
  +--> SPWM/SPWM

SYSTEMTICK/MOTORCONTROL                     ----- -----  ----- -----

MDUAPP/MDU                                  ----- -----  ----- -----
  +--> _MDU_MULA_U16/MDU
  +--> _MDU_MUL_U16/MDU

_MDU_MULA_U16/MDU                           ----- -----  ----- -----

_MDU_MUL_U16/MDU                            ----- -----  ----- -----

SPWM/SPWM                                   ----- -----  0115H 0126H
  +--> _SINCOS/SINCOS
  +--> _MDU_MULA_S16/MDU

_SINCOS/SINCOS                              ----- -----  ----- -----

_MDU_MULA_S16/MDU                           ----- -----  ----- -----

*** NEW ROOT ******************************

TIM23_ISR/INTERRUPT                         ----- -----  ----- -----

*** NEW ROOT ******************************

TIM45_ISR/INTERRUPT                         ----- -----  ----- -----
  +--> FAULTDETECT/MOTORCONTROL
  +--> SPEEDCONTROL/MOTORCONTROL
  +--> ONOFFCONTROL/MOTORCONTROL
  +--> KEYSCAN/KEYSCAN
  +--> PWMSCAN/PWMSCAN
  +--> IRSCANCONTROL/IRSCAN
  +--> BUZZERSCAN/BUZZERSCAN
  +--> LEDCONTROL/LED

FAULTDETECT/MOTORCONTROL                    ----- -----  ----- -----

SPEEDCONTROL/MOTORCONTROL                   ----- -----  ----- -----

ONOFFCONTROL/MOTORCONTROL                   ----- -----  0127H 0128H

KEYSCAN/KEYSCAN                             ----- -----  ----- -----
  +--> KEYVALUE/KEYSCAN

KEYVALUE/KEYSCAN                            ----- -----  ----- -----

PWMSCAN/PWMSCAN                             ----- -----  ----- -----

IRSCANCONTROL/IRSCAN                        ----- -----  ----- -----

BUZZERSCAN/BUZZERSCAN                       ----- -----  ----- -----

LEDCONTROL/LED                              ----- -----  ----- -----
LX51 LINKER/LOCATER V4.66.1.0                                                         03/23/2017  15:15:44  PAGE 6



*** NEW ROOT ******************************

CMP_ISR/INTERRUPT                           ----- -----  ----- -----

*** NEW ROOT ******************************

ADC_ISR/INTERRUPT                           ----- -----  ----- -----
  +--> _LPF/LPF

_LPF/LPF                                    ----- -----  ----- -----

*** NEW ROOT ******************************

UART_ISR/INTERRUPT                          ----- -----  ----- -----

*** NEW ROOT ******************************

?C_C51STARTUP                               ----- -----  ----- -----
  +--> MAIN/MAIN
  +--> ?C_INITSEG

MAIN/MAIN                                   ----- -----  0129H 012CH
  +--> SYSTEMINIT/SYSTEMINIT
  +--> SOFTWAREINIT/MAIN
  +--> HARDWAREINIT/MAIN
  +--> MOTORMAIN/MOTORCONTROL
  +--> WATCHDOGREFRESH/FU68XX_SYSTEM

SYSTEMINIT/SYSTEMINIT                       ----- -----  ----- -----
  +--> SYSTEMFASTCLOCKCONFIG/FU68XX_SYSTEM
  +--> EXTERNALSLOWCLOCKCONFIG/FU68XX_SYSTEM
  +--> _VREFCONFIG/FU68XX_SYSTEM
  +--> VHALFCONFIG/FU68XX_SYSTEM
  +--> _WATCHDOGCONFIG/FU68XX_SYSTEM

SYSTEMFASTCLOCKCONFIG/FU68XX_SYSTEM         20H.0 20H.0  ----- -----

EXTERNALSLOWCLOCKCONFIG/FU68XX_SYSTEM       20H.0 20H.0  ----- -----

_VREFCONFIG/FU68XX_SYSTEM                   20H.0 20H.0  ----- -----

VHALFCONFIG/FU68XX_SYSTEM                   20H.0 20H.1  ----- -----

_WATCHDOGCONFIG/FU68XX_SYSTEM               20H.0 20H.0  ----- -----

SOFTWAREINIT/MAIN                           ----- -----  ----- -----
  +--> PARAMETERINIT/MOTORCONTROL
  +--> KEYINIT/KEYSCAN
  +--> IRINIT/IRSCAN
  +--> PWMIN_INIT/PWMSCAN
  +--> BUZZERINIT/BUZZERSCAN
  +--> UARTSCANINIT/UARTSCAN
  +--> LEDCONTROLINIT/LED

PARAMETERINIT/MOTORCONTROL                  ----- -----  ----- -----

KEYINIT/KEYSCAN                             ----- -----  ----- -----
  +--> KEYVALUE/KEYSCAN

IRINIT/IRSCAN                               ----- -----  ----- -----

PWMIN_INIT/PWMSCAN                          ----- -----  ----- -----

BUZZERINIT/BUZZERSCAN                       ----- -----  ----- -----
LX51 LINKER/LOCATER V4.66.1.0                                                         03/23/2017  15:15:44  PAGE 7



UARTSCANINIT/UARTSCAN                       ----- -----  ----- -----

LEDCONTROLINIT/LED                          ----- -----  ----- -----

HARDWAREINIT/MAIN                           ----- -----  ----- -----
  +--> GPIOINIT/GPIOINIT
  +--> SPIINIT/SPIINIT
  +--> CMPIINT/CMPINIT
  +--> AMPIINT/AMPINIT
  +--> MDUINIT/MDU
  +--> ADCINIT/ADCINIT
  +--> SINCOSINIT/SINCOS
  +--> DRIVERINIT/DRIVERINIT
  +--> TIM0INIT/TIMERINIT
  +--> TIM3INIT/TIMERINIT
  +--> TIM4INIT/TIMERINIT
  +--> INTERRUPTINIT/INTERRUPTINIT

GPIOINIT/GPIOINIT                           ----- -----  ----- -----

SPIINIT/SPIINIT                             ----- -----  ----- -----

CMPIINT/CMPINIT                             ----- -----  ----- -----

AMPIINT/AMPINIT                             ----- -----  ----- -----

MDUINIT/MDU                                 ----- -----  ----- -----
  +--> MDUCONTROLINIT/MDU

MDUCONTROLINIT/MDU                          ----- -----  ----- -----

ADCINIT/ADCINIT                             ----- -----  ----- -----
  +--> ADCDATAINIT/ADCINIT

ADCDATAINIT/ADCINIT                         ----- -----  ----- -----

SINCOSINIT/SINCOS                           ----- -----  ----- -----

DRIVERINIT/DRIVERINIT                       ----- -----  ----- -----

TIM0INIT/TIMERINIT                          ----- -----  ----- -----

TIM3INIT/TIMERINIT                          ----- -----  ----- -----

TIM4INIT/TIMERINIT                          ----- -----  ----- -----

INTERRUPTINIT/INTERRUPTINIT                 ----- -----  ----- -----

MOTORMAIN/MOTORCONTROL                      ----- -----  ----- -----
  +--> MOTORSTOP/MOTORCONTROL
  +--> MOTORINIT/MOTORCONTROL
  +--> MOTORREADY/MOTORCONTROL
  +--> MOTORPRECHARGE/MOTORCONTROL
  +--> MOTORSTART/MOTORCONTROL
  +--> MOTORNORMAL/MOTORCONTROL
  +--> MOTORFAULT/MOTORCONTROL

MOTORSTOP/MOTORCONTROL                      ----- -----  ----- -----

MOTORINIT/MOTORCONTROL                      ----- -----  ----- -----
  +--> PARAMETERINIT/MOTORCONTROL

MOTORREADY/MOTORCONTROL                     ----- -----  ----- -----

LX51 LINKER/LOCATER V4.66.1.0                                                         03/23/2017  15:15:44  PAGE 8


MOTORPRECHARGE/MOTORCONTROL                 ----- -----  ----- -----

MOTORSTART/MOTORCONTROL                     ----- -----  ----- -----

MOTORNORMAL/MOTORCONTROL                    ----- -----  ----- -----

MOTORFAULT/MOTORCONTROL                     ----- -----  ----- -----
  +--> RESTARTCONTROL/MOTORCONTROL

RESTARTCONTROL/MOTORCONTROL                 ----- -----  ----- -----

WATCHDOGREFRESH/FU68XX_SYSTEM               ----- -----  ----- -----

?C_INITSEG                                  ----- -----  ----- -----



PUBLIC SYMBOLS OF MODULE:  .\Output\FU68xx_SPWM_OnePhase (MAIN)


      VALUE       CLASS    TYPE      PUBLIC SYMBOL NAME
      =================================================
*DEL*:00000000H   XDATA    BYTE      ?_MDU_MULA_S32?BYTE
*DEL*:00000000H   XDATA    BYTE      ?_MDU_MULA_U32?BYTE
      00000020H.0 BIT      BIT       ?_VREFConfig?BIT
      00000020H.0 BIT      BIT       ?_WatchDogConfig?BIT
      01000342H   CODE     ---       ?C?CASTF
      00000000H   NUMBER   ---       ?C?CODESEG
      0100030EH   CODE     ---       ?C?FCASTC
      01000309H   CODE     ---       ?C?FCASTI
      01000304H   CODE     ---       ?C?FCASTL
      0100006DH   CODE     ---       ?C?FPADD
      01000267H   CODE     ---       ?C?FPDIV
      01000379H   CODE     ---       ?C?FPGETOPN2
      0100015EH   CODE     ---       ?C?FPMUL
      010003AEH   CODE     ---       ?C?FPNANRESULT
      010003B8H   CODE     ---       ?C?FPOVERFLOW
      01000390H   CODE     ---       ?C?FPRESULT
      010003A4H   CODE     ---       ?C?FPRESULT2
      01000069H   CODE     ---       ?C?FPSUB
      010003B5H   CODE     ---       ?C?FPUNDERFLOW
      01000517H   CODE     ---       ?C?ICASE
      01000544H   CODE     ---       ?C?LIMUL
      01000491H   CODE     ---       ?C?LNEG
      010004E6H   CODE     ---       ?C?LSTKXDATA
      010004DAH   CODE     ---       ?C?LSTXDATA
      0100049FH   CODE     ---       ?C?SLCMP
      010004C6H   CODE     ---       ?C?SLSHR
      010004B5H   CODE     ---       ?C?ULCMP
      010003FFH   CODE     ---       ?C?ULDIV
      00000000H   NUMBER   ---       ?C?XDATASEG
      010015AAH   CODE     ---       ?C_START
      01000000H   CODE     ---       ?C_STARTUP
      00000020H.0 BIT      BIT       ?ExternalSlowClockConfig?BIT
*DEL*:00000000H.0 BIT      BIT       ?InternalFastClockConfig?BIT
*DEL*:00000000H.0 BIT      BIT       ?LVDPowerDownDetectConfig?BIT
*DEL*:00000000H.0 BIT      BIT       ?LVDPowerDownWarnIEConfig?BIT
      00000020H.0 BIT      BIT       ?SystemFastClockConfig?BIT
      00000020H.0 BIT      BIT       ?VHALFConfig?BIT
*DEL*:00000000H   CODE     ---       _Cos
*DEL*:00000000H   CODE     ---       _Flash_Sector_Erase
*DEL*:00000000H   CODE     ---       _Flash_Sector_Write
      01001D11H   CODE     ---       _LPF
*DEL*:00000000H   CODE     ---       _MDU_DIV_U16
*DEL*:00000000H   CODE     ---       _MDU_DIV_U32
LX51 LINKER/LOCATER V4.66.1.0                                                         03/23/2017  15:15:44  PAGE 9


*DEL*:00000000H   CODE     ---       _MDU_MUL_S16
*DEL*:00000000H   CODE     ---       _MDU_MUL_S32
      01001DD2H   CODE     ---       _MDU_MUL_U16
*DEL*:00000000H   CODE     ---       _MDU_MUL_U32
      01001AAEH   CODE     ---       _MDU_MULA_S16
*DEL*:00000000H   CODE     ---       _MDU_MULA_S32
      01001A00H   CODE     ---       _MDU_MULA_U16
*DEL*:00000000H   CODE     ---       _MDU_MULA_U32
*DEL*:00000000H   CODE     ---       _SetCurrent
*DEL*:00000000H   CODE     ---       _Sin
      01001E1FH   CODE     ---       _SinCos
*DEL*:00000000H   CODE     ---       _SPISendData
*DEL*:00000000H   CODE     ---       _TIM5_Timing_us
*DEL*:00000000H   CODE     ---       _UARTSendData
      01001974H   CODE     ---       _VREFConfig
      01001B1DH   CODE     ---       _WatchDogConfig
*SFR* 000000D0H.6 DATA     BIT       AC
*SFR* 000000E0H   DATA     BYTE      ACC
      01000B41H   CODE     ---       ADC_ISR
      020000B7H   XDATA    ---       ADCData
      0100139CH   CODE     ---       ADCDataInit
*DEL*:00000000H   CODE     ---       ADCGetConversionValue
      010015EFH   CODE     ---       ADCInit
      01001E37H   CODE     ---       AMPIint
*SFR* 000000F0H   DATA     BYTE      B
      0100003EH   CODE     ---       BuzzerInit
      01001B54H   CODE     ---       BuzzerScan
      0200018CH   XDATA    ---       BZScan
*SFR* 000000D5H   DATA     BYTE      CMP_CR0
*SFR* 000000D6H   DATA     BYTE      CMP_CR1
*SFR* 000000DAH   DATA     BYTE      CMP_CR2
      01001BEDH   CODE     ---       CMP_ISR
*SFR* 000000D7H   DATA     BYTE      CMP_SR
      01001B8AH   CODE     ---       CMPIint
*DEL*:00000000H   CODE     ---       CurrentControl
      00000029H   IDATA    ---       CurrentPID
*SFR* 000000D0H.7 DATA     BIT       CY
      02000181H   XDATA    WORD      Delta_Current
      02000183H   XDATA    WORD      Delta_Speed
*SFR* 00000082H   DATA     WORD      DP
*SFR* 00000083H   DATA     BYTE      DPH
*SFR* 00000082H   DATA     BYTE      DPL
      01001DB5H   CODE     ---       DriverInit
*SFR* 000000F8H   DATA     BYTE      DRV_OUT
*SFR* 000000A8H.7 DATA     BIT       EA
*SFR* 000000A8H.4 DATA     BIT       ES0
*SFR* 000000D9H   DATA     BYTE      EVT_FILT
*SFR* 000000A8H   DATA     BIT       EX0
*SFR* 000000A8H.2 DATA     BIT       EX1
      01001E4FH   CODE     ---       ExternalSlowClockConfig
*SFR* 000000D0H.5 DATA     BIT       F0
*SFR* 000000D0H.1 DATA     BIT       F1
      01000571H   CODE     ---       FaultDetect
      02000166H   XDATA    BYTE      FlagSPI
      00000020H.2 BIT      BIT       FlagStartPI
*SFR* 00000084H   DATA     BYTE      FLKEY
*SFR* 000000E8H   DATA     BYTE      FOC_SET0
*SFR* 000000E9H   DATA     BYTE      FOC_SET1
*SFR* 000000E8H.7 DATA     BIT       FOCEN
*SFR* 00000080H   DATA     BIT       GP00
*SFR* 00000080H.1 DATA     BIT       GP01
*SFR* 00000080H.2 DATA     BIT       GP02
*SFR* 00000080H.3 DATA     BIT       GP03
*SFR* 00000080H.4 DATA     BIT       GP04
*SFR* 00000080H.5 DATA     BIT       GP05
LX51 LINKER/LOCATER V4.66.1.0                                                         03/23/2017  15:15:44  PAGE 10


*SFR* 00000080H.6 DATA     BIT       GP06
*SFR* 00000080H.7 DATA     BIT       GP07
*SFR* 00000090H   DATA     BIT       GP10
*SFR* 00000090H.1 DATA     BIT       GP11
*SFR* 00000090H.2 DATA     BIT       GP12
*SFR* 00000090H.3 DATA     BIT       GP13
*SFR* 00000090H.4 DATA     BIT       GP14
*SFR* 00000090H.5 DATA     BIT       GP15
*SFR* 00000090H.6 DATA     BIT       GP16
*SFR* 00000090H.7 DATA     BIT       GP17
*SFR* 000000A0H   DATA     BIT       GP20
*SFR* 000000A0H.1 DATA     BIT       GP21
*SFR* 000000A0H.2 DATA     BIT       GP22
*SFR* 000000A0H.3 DATA     BIT       GP23
*SFR* 000000A0H.4 DATA     BIT       GP24
*SFR* 000000A0H.5 DATA     BIT       GP25
*SFR* 000000A0H.6 DATA     BIT       GP26
*SFR* 000000A0H.7 DATA     BIT       GP27
*SFR* 000000B0H   DATA     BIT       GP30
*SFR* 000000B0H.1 DATA     BIT       GP31
*SFR* 000000B0H.2 DATA     BIT       GP32
*SFR* 000000B0H.3 DATA     BIT       GP33
*SFR* 000000B0H.4 DATA     BIT       GP34
*SFR* 000000B0H.5 DATA     BIT       GP35
*SFR* 000000B0H.6 DATA     BIT       GP36
*SFR* 000000B0H.7 DATA     BIT       GP37
      010017F7H   CODE     ---       GPIOInit
      01001CEDH   CODE     ---       HardwareInit
*SFR* 000000A8H   DATA     BYTE      IE
*SFR* 00000088H.2 DATA     BIT       IF0
*DEL*:00000000H   CODE     ---       InternalFastClockConfig
      01001CC8H   CODE     ---       InterruptInit
*SFR* 000000B8H   DATA     BYTE      IP0
*SFR* 000000C0H   DATA     BYTE      IP1
*SFR* 000000C8H   DATA     BYTE      IP2
*SFR* 000000D8H   DATA     BYTE      IP3
      0200012DH   XDATA    ---       IRControl
      01001C1CH   CODE     ---       IRInit
      02000136H   XDATA    ---       IRScan
      01000F01H   CODE     ---       IRScanControl
*DEL*:00000000H   CODE     ---       IRValue
*SFR* 00000088H   DATA     BIT       IT00
*SFR* 00000088H.1 DATA     BIT       IT01
*SFR* 00000088H.3 DATA     BIT       IT10
*SFR* 00000088H.4 DATA     BIT       IT11
      0100192EH   CODE     ---       KeyInit
      01001D33H   CODE     ---       KeyScan
      010014D1H   CODE     ---       KeyValue
      02000179H   XDATA    ---       KS
      0100143CH   CODE     ---       LEDControl
      01001E99H   CODE     ---       LEDControlInit
      02000187H   XDATA    ---       LEDCtl
*SFR* 000000DCH   DATA     WORD      LPF_K
*SFR* 000000DDH   DATA     BYTE      LPF_KH
*SFR* 000000DCH   DATA     BYTE      LPF_KL
*SFR* 000000DEH   DATA     WORD      LPF_X
*SFR* 000000DFH   DATA     BYTE      LPF_XH
*SFR* 000000DEH   DATA     BYTE      LPF_XL
*SFR* 000000E6H   DATA     WORD      LPF_Y
*SFR* 000000E7H   DATA     BYTE      LPF_YH
*SFR* 000000E6H   DATA     BYTE      LPF_YL
*DEL*:00000000H   CODE     ---       LVDPowerDownDetectConfig
*DEL*:00000000H   CODE     ---       LVDPowerDownWarnIEConfig
*SFR* 000000DBH   DATA     BYTE      LVSR
      0100179FH   CODE     ---       main
LX51 LINKER/LOCATER V4.66.1.0                                                         03/23/2017  15:15:44  PAGE 11


      02000026H   XDATA    ---       MC
*SFR* 000000A8H.5 DATA     BIT       MCDIE
*SFR* 00000088H.6 DATA     BIT       MCDIF
*SFR* 000000C4H   DATA     BYTE      MD_DA0
*SFR* 000000C5H   DATA     BYTE      MD_DA1
*SFR* 000000C6H   DATA     BYTE      MD_DA2
*SFR* 000000C7H   DATA     BYTE      MD_DA3
*SFR* 000000C6H   DATA     WORD      MD_DAH
*SFR* 000000C4H   DATA     WORD      MD_DAL
*SFR* 000000CCH   DATA     BYTE      MD_DB0
*SFR* 000000CDH   DATA     BYTE      MD_DB1
*SFR* 000000CEH   DATA     BYTE      MD_DB2
*SFR* 000000CFH   DATA     BYTE      MD_DB3
*SFR* 000000CEH   DATA     WORD      MD_DBH
*SFR* 000000CCH   DATA     WORD      MD_DBL
*SFR* 000000C2H   DATA     WORD      MD_MA
*SFR* 000000C3H   DATA     BYTE      MD_MAH
*SFR* 000000C2H   DATA     BYTE      MD_MAL
*SFR* 000000CAH   DATA     WORD      MD_MB
*SFR* 000000CBH   DATA     BYTE      MD_MBH
*SFR* 000000CAH   DATA     BYTE      MD_MBL
*SFR* 000000C1H   DATA     BYTE      MD_MODE
      010010FFH   CODE     ---       MDUAPP
      02000167H   XDATA    ---       MDUControl
      01001DECH   CODE     ---       MDUControlInit
      01000026H   CODE     ---       MDUInit
*SFR* 00000098H.6 DATA     BIT       MOD0
*SFR* 00000098H.7 DATA     BIT       MOD1
*SFR* 000000F8H.7 DATA     BIT       MOE
      01001CA1H   CODE     ---       MotorFault
      01000056H   CODE     ---       MotorInit
      01001A38H   CODE     ---       MotorMain
      01001C76H   CODE     ---       MotorNormal
      01000DF3H   CODE     ---       MotorPrecharge
      01001EAFH   CODE     ---       MotorReady
      01001E65H   CODE     ---       MotorStart
      01001A76H   CODE     ---       MotorStop
*SFR* 000000F8H.6 DATA     BIT       OIS4
*SFR* 000000F8H   DATA     BIT       OISUH
*SFR* 000000F8H.1 DATA     BIT       OISUL
*SFR* 000000F8H.2 DATA     BIT       OISVH
*SFR* 000000F8H.3 DATA     BIT       OISVL
*SFR* 000000F8H.4 DATA     BIT       OISWH
*SFR* 000000F8H.5 DATA     BIT       OISWL
      010019B9H   CODE     ---       ONOFFControl
*SFR* 000000F1H   DATA     BYTE      OSC_CFG
*SFR* 000000D0H.2 DATA     BIT       OV
*SFR* 000000D0H   DATA     BIT       P
*SFR* 00000080H   DATA     BYTE      P0
*SFR* 000000FCH   DATA     BYTE      P0_OE
*SFR* 00000090H   DATA     BYTE      P1
*SFR* 000000FDH   DATA     BYTE      P1_OE
*SFR* 000000D1H   DATA     BYTE      P1IE
*SFR* 000000D2H   DATA     BYTE      P1IF
*SFR* 000000A0H   DATA     BYTE      P2
*SFR* 000000FEH   DATA     BYTE      P2_OE
*SFR* 000000D3H   DATA     BYTE      P2IE
*SFR* 000000D4H   DATA     BYTE      P2IF
*SFR* 000000B0H   DATA     BYTE      P3
*SFR* 000000FFH   DATA     BYTE      P3_OE
*SFR* 000000C0H.4 DATA     BIT       PADC0
*SFR* 000000C0H.5 DATA     BIT       PADC1
      010011EAH   CODE     ---       ParameterInit
*SFR* 000000C0H.6 DATA     BIT       PCMP0
*SFR* 000000C0H.7 DATA     BIT       PCMP1
LX51 LINKER/LOCATER V4.66.1.0                                                         03/23/2017  15:15:44  PAGE 12


*SFR* 00000087H   DATA     BYTE      PCON
*SFR* 000000B8H.6 DATA     BIT       PFOC0
*SFR* 000000B8H.7 DATA     BIT       PFOC1
*SFR* 000000D8H.2 DATA     BIT       PI2C0
*SFR* 000000D8H.3 DATA     BIT       PI2C1
*SFR* 000000EAH   DATA     WORD      PI_EK
*SFR* 000000EBH   DATA     BYTE      PI_EKH
*SFR* 000000EAH   DATA     BYTE      PI_EKL
*SFR* 000000F2H   DATA     WORD      PI_KI
*SFR* 000000F3H   DATA     BYTE      PI_KIH
*SFR* 000000F2H   DATA     BYTE      PI_KIL
*SFR* 000000EEH   DATA     WORD      PI_KP
*SFR* 000000EFH   DATA     BYTE      PI_KPH
*SFR* 000000EEH   DATA     BYTE      PI_KPL
*SFR* 000000ECH   DATA     WORD      PI_UK
*SFR* 000000EDH   DATA     BYTE      PI_UKH
*SFR* 000000ECH   DATA     BYTE      PI_UKL
*SFR* 000000F4H   DATA     WORD      PI_UKMAX
*SFR* 000000F5H   DATA     BYTE      PI_UKMAXH
*SFR* 000000F4H   DATA     BYTE      PI_UKMAXL
*SFR* 000000F6H   DATA     WORD      PI_UKMIN
*SFR* 000000F7H   DATA     BYTE      PI_UKMINH
*SFR* 000000F6H   DATA     BYTE      PI_UKMINL
*SFR* 000000F9H   DATA     BYTE      PL_CR
*SFR* 000000B8H   DATA     BIT       PLVW0
*SFR* 000000B8H.1 DATA     BIT       PLVW1
*SFR* 000000D8H.6 DATA     BIT       PMCD0
*SFR* 000000D8H.7 DATA     BIT       PMCD1
      00000049H   IDATA    ---       PowerPID
*SFR* 000000C8H   DATA     BIT       PRTC0
*SFR* 000000C8H.1 DATA     BIT       PRTC1
*SFR* 00000085H   DATA     BYTE      PSCTL
*SFR* 000000D8H.4 DATA     BIT       PSPI0
*SFR* 000000D8H.5 DATA     BIT       PSPI1
*SFR* 000000D0H   DATA     BYTE      PSW
*SFR* 000000C0H   DATA     BIT       PTIM00
*SFR* 000000C0H.1 DATA     BIT       PTIM01
*SFR* 000000C0H.2 DATA     BIT       PTIM10
*SFR* 000000C0H.3 DATA     BIT       PTIM11
*SFR* 000000C8H.2 DATA     BIT       PTIM230
*SFR* 000000C8H.3 DATA     BIT       PTIM231
*SFR* 000000C8H.4 DATA     BIT       PTIM450
*SFR* 000000C8H.5 DATA     BIT       PTIM451
*SFR* 000000C8H.6 DATA     BIT       PTSD0
*SFR* 000000C8H.7 DATA     BIT       PTSD1
*SFR* 000000D8H   DATA     BIT       PUART0
*SFR* 000000D8H.1 DATA     BIT       PUART1
      01001E06H   CODE     ---       PWMIN_Init
      02000170H   XDATA    ---       PWMINCtl
      01001D55H   CODE     ---       PWMScan
*SFR* 000000B8H.2 DATA     BIT       PX00
*SFR* 000000B8H.3 DATA     BIT       PX01
*SFR* 000000B8H.4 DATA     BIT       PX10
*SFR* 000000B8H.5 DATA     BIT       PX11
*SFR* 00000098H.2 DATA     BIT       RB8
*SFR* 00000098H.4 DATA     BIT       REN
      01001741H   CODE     ---       RestartControl
*SFR* 00000098H   DATA     BIT       RI
*SFR* 000000D0H.3 DATA     BIT       RS0
*SFR* 000000D0H.4 DATA     BIT       RS1
*SFR* 000000C9H   DATA     BYTE      RSTSRC
*SFR* 000000A8H.6 DATA     BIT       RTCIE
      01001E78H   CODE     ---       SinCosInit
*SFR* 00000098H.5 DATA     BIT       SM2
      01000003H   CODE     ---       SoftwareInit
LX51 LINKER/LOCATER V4.66.1.0                                                         03/23/2017  15:15:44  PAGE 13


*SFR* 00000081H   DATA     BYTE      SP
      01000995H   CODE     ---       SpeedControl
      00000039H   IDATA    ---       SpeedPID
      00000021H   IDATA    ---       SpeedRamp
*SFR* 000000A8H.3 DATA     BIT       SPIIE
      0100189CH   CODE     ---       SPIInit
      010007B2H   CODE     ---       SPWM
*SFR* 000000E4H   DATA     WORD      SV_ANGLE
*SFR* 000000E5H   DATA     BYTE      SV_ANGLEH
*SFR* 000000E4H   DATA     BYTE      SV_ANGLEL
*SFR* 000000E1H   DATA     BYTE      SV_CR
*SFR* 000000E2H   DATA     WORD      SV_US
*SFR* 000000E3H   DATA     BYTE      SV_USH
*SFR* 000000E2H   DATA     BYTE      SV_USL
      01001E8AH   CODE     ---       SystemFastClockConfig
      01001D76H   CODE     ---       SystemInit
      01001006H   CODE     ---       SystemTick
      020000FBH   XDATA    ---       TanAngle
      0200008BH   XDATA    ---       TargetCurrentTable
      02000185H   XDATA    WORD      TargetSpeed
      020000A1H   XDATA    ---       TargetSpeedTable
      02000010H   XDATA    ---       TargetVSTable
*SFR* 00000098H.3 DATA     BIT       TB8
*SFR* 00000088H   DATA     BYTE      TCON
*SFR* 00000098H.1 DATA     BIT       TI
*SFR* 000000B6H   DATA     WORD      TIM0_CCR1
*SFR* 000000B7H   DATA     BYTE      TIM0_CCR1H
*SFR* 000000B6H   DATA     BYTE      TIM0_CCR1L
*SFR* 000000BAH   DATA     WORD      TIM0_CCR2
*SFR* 000000BBH   DATA     BYTE      TIM0_CCR2H
*SFR* 000000BAH   DATA     BYTE      TIM0_CCR2L
*SFR* 000000BCH   DATA     WORD      TIM0_CCR3
*SFR* 000000BDH   DATA     BYTE      TIM0_CCR3H
*SFR* 000000BCH   DATA     BYTE      TIM0_CCR3L
*SFR* 000000BEH   DATA     WORD      TIM0_CCR4
*SFR* 000000BFH   DATA     BYTE      TIM0_CCR4H
*SFR* 000000BEH   DATA     BYTE      TIM0_CCR4L
*SFR* 000000B9H   DATA     BYTE      TIM0_IER
      01001672H   CODE     ---       TIM0_ISR
*SFR* 000000B1H   DATA     BYTE      TIM0_SR1
      01000CADH   CODE     ---       TIM0Init
*DEL*:00000000H   CODE     ---       TIM1Init
      010018E7H   CODE     ---       TIM23_ISR
*SFR* 000000B4H   DATA     WORD      TIM2_ADTR
*SFR* 000000B5H   DATA     BYTE      TIM2_ADTRH
*SFR* 000000B4H   DATA     BYTE      TIM2_ADTRL
*SFR* 000000AEH   DATA     WORD      TIM2_ARR
*SFR* 000000AFH   DATA     BYTE      TIM2_ARRH
*SFR* 000000AEH   DATA     BYTE      TIM2_ARRL
*SFR* 000000B2H   DATA     WORD      TIM2_CMTR
*SFR* 000000B3H   DATA     BYTE      TIM2_CMTRH
*SFR* 000000B2H   DATA     BYTE      TIM2_CMTRL
*SFR* 000000AAH   DATA     WORD      TIM2_CNTR
*SFR* 000000ABH   DATA     BYTE      TIM2_CNTRH
*SFR* 000000AAH   DATA     BYTE      TIM2_CNTRL
*SFR* 000000A1H   DATA     BYTE      TIM2_CR0
*SFR* 000000A9H   DATA     BYTE      TIM2_CR1
*SFR* 000000ACH   DATA     WORD      TIM2_DR
*SFR* 000000ADH   DATA     BYTE      TIM2_DRH
*SFR* 000000ACH   DATA     BYTE      TIM2_DRL
*DEL*:00000000H   CODE     ---       TIM2Init
*SFR* 000000A6H   DATA     WORD      TIM3_ARR
*SFR* 000000A7H   DATA     BYTE      TIM3_ARRH
*SFR* 000000A6H   DATA     BYTE      TIM3_ARRL
*SFR* 000000A2H   DATA     WORD      TIM3_CNTR
LX51 LINKER/LOCATER V4.66.1.0                                                         03/23/2017  15:15:44  PAGE 14


*SFR* 000000A3H   DATA     BYTE      TIM3_CNTRH
*SFR* 000000A2H   DATA     BYTE      TIM3_CNTRL
*SFR* 0000009CH   DATA     BYTE      TIM3_CR0
*SFR* 0000009DH   DATA     BYTE      TIM3_CR1
*SFR* 000000A4H   DATA     WORD      TIM3_DR
*SFR* 000000A5H   DATA     BYTE      TIM3_DRH
*SFR* 000000A4H   DATA     BYTE      TIM3_DRL
      01001AE6H   CODE     ---       TIM3Init
      010016DDH   CODE     ---       TIM45_ISR
*SFR* 00000096H   DATA     WORD      TIM4_ARR
*SFR* 00000097H   DATA     BYTE      TIM4_ARRH
*SFR* 00000096H   DATA     BYTE      TIM4_ARRL
*SFR* 00000092H   DATA     WORD      TIM4_CNTR
*SFR* 00000093H   DATA     BYTE      TIM4_CNTRH
*SFR* 00000092H   DATA     BYTE      TIM4_CNTRL
*SFR* 0000009EH   DATA     BYTE      TIM4_CR0
*SFR* 0000009FH   DATA     BYTE      TIM4_CR1
*SFR* 00000094H   DATA     WORD      TIM4_DR
*SFR* 00000095H   DATA     BYTE      TIM4_DRH
*SFR* 00000094H   DATA     BYTE      TIM4_DRL
      0100184DH   CODE     ---       TIM4Init
*SFR* 0000008EH   DATA     WORD      TIM5_ARR
*SFR* 0000008FH   DATA     BYTE      TIM5_ARRH
*SFR* 0000008EH   DATA     BYTE      TIM5_ARRL
*SFR* 0000008AH   DATA     WORD      TIM5_CNTR
*SFR* 0000008BH   DATA     BYTE      TIM5_CNTRH
*SFR* 0000008AH   DATA     BYTE      TIM5_CNTRL
*SFR* 00000089H   DATA     BYTE      TIM5_CR0
*SFR* 00000091H   DATA     BYTE      TIM5_CR1
*SFR* 0000008CH   DATA     WORD      TIM5_DR
*SFR* 0000008DH   DATA     BYTE      TIM5_DRH
*SFR* 0000008CH   DATA     BYTE      TIM5_DRL
*DEL*:00000000H   CODE     ---       TIM5Init
*SFR* 000000A8H.1 DATA     BIT       TSDIE
*SFR* 00000088H.5 DATA     BIT       TSDIF
      01001C4AH   CODE     ---       UART_ISR
      02000142H   XDATA    ---       UARTControl
*DEL*:00000000H   CODE     ---       UARTInit
      02000155H   XDATA    ---       UARTScan
*DEL*:00000000H   CODE     ---       UARTScanControl
      01001BBDH   CODE     ---       UARTScanInit
*SFR* 0000009AH   DATA     WORD      UT_BAUD
*SFR* 0000009BH   DATA     BYTE      UT_BAUDH
*SFR* 0000009AH   DATA     BYTE      UT_BAUDL
*SFR* 00000098H   DATA     BYTE      UT_CR
*SFR* 00000099H   DATA     BYTE      UT_DR
      01001D97H   CODE     ---       VHALFConfig
      01001EA7H   CODE     ---       WatchDogRefresh



SYMBOL TABLE OF MODULE:  .\Output\FU68xx_SPWM_OnePhase (MAIN)

      VALUE       REP       CLASS    TYPE      SYMBOL NAME
      ====================================================
      ---         MODULE    ---      ---       MAIN
      01001CEDH   PUBLIC    CODE     ---       HardwareInit
      01000003H   PUBLIC    CODE     ---       SoftwareInit
      0100179FH   PUBLIC    CODE     ---       main
      000000E2H   SFRSYM    DATA     BYTE      SV_USL
      000000ABH   SFRSYM    DATA     BYTE      TIM2_CNTRH
      000000B0H.4 SFRSYM    DATA     BIT       GP34
      000000A0H.5 SFRSYM    DATA     BIT       GP25
      00000090H.6 SFRSYM    DATA     BIT       GP16
      00000080H.7 SFRSYM    DATA     BIT       GP07
LX51 LINKER/LOCATER V4.66.1.0                                                         03/23/2017  15:15:44  PAGE 15


      00000088H.1 SFRSYM    DATA     BIT       IT01
      00000088H.3 SFRSYM    DATA     BIT       IT10
      000000F6H   SFRSYM    DATA     WORD      PI_UKMIN
      000000C2H   SFRSYM    DATA     WORD      MD_MA
      000000A3H   SFRSYM    DATA     BYTE      TIM3_CNTRH
      000000B0H.5 SFRSYM    DATA     BIT       GP35
      000000A0H.6 SFRSYM    DATA     BIT       GP26
      00000090H.7 SFRSYM    DATA     BIT       GP17
      00000080H   SFRSYM    DATA     BYTE      P0
      00000088H.4 SFRSYM    DATA     BIT       IT11
      000000CAH   SFRSYM    DATA     WORD      MD_MB
      00000093H   SFRSYM    DATA     BYTE      TIM4_CNTRH
      000000B0H.6 SFRSYM    DATA     BIT       GP36
      000000A0H.7 SFRSYM    DATA     BIT       GP27
      00000090H   SFRSYM    DATA     BYTE      P1
      000000D9H   SFRSYM    DATA     BYTE      EVT_FILT
      000000F4H   SFRSYM    DATA     WORD      PI_UKMAX
      0000008BH   SFRSYM    DATA     BYTE      TIM5_CNTRH
      000000B2H   SFRSYM    DATA     BYTE      TIM2_CMTRL
      000000B0H.7 SFRSYM    DATA     BIT       GP37
      000000A0H   SFRSYM    DATA     BYTE      P2
      000000AAH   SFRSYM    DATA     BYTE      TIM2_CNTRL
      000000B0H   SFRSYM    DATA     BYTE      P3
      000000A2H   SFRSYM    DATA     BYTE      TIM3_CNTRL
      000000D0H.6 SFRSYM    DATA     BIT       AC
      00000092H   SFRSYM    DATA     BYTE      TIM4_CNTRL
      0000008AH   SFRSYM    DATA     BYTE      TIM5_CNTRL
      000000B6H   SFRSYM    DATA     WORD      TIM0_CCR1
      000000A8H.7 SFRSYM    DATA     BIT       EA
      000000D5H   SFRSYM    DATA     BYTE      CMP_CR0
      000000BAH   SFRSYM    DATA     WORD      TIM0_CCR2
      000000D6H   SFRSYM    DATA     BYTE      CMP_CR1
      000000BCH   SFRSYM    DATA     WORD      TIM0_CCR3
      00000085H   SFRSYM    DATA     BYTE      PSCTL
      000000DAH   SFRSYM    DATA     BYTE      CMP_CR2
      000000BEH   SFRSYM    DATA     WORD      TIM0_CCR4
      000000B8H.2 SFRSYM    DATA     BIT       PX00
      000000EAH   SFRSYM    DATA     WORD      PI_EK
      000000F8H   SFRSYM    DATA     BIT       OISUH
      000000B8H.3 SFRSYM    DATA     BIT       PX01
      000000B8H.4 SFRSYM    DATA     BIT       PX10
      000000F8H.2 SFRSYM    DATA     BIT       OISVH
      000000B8H.5 SFRSYM    DATA     BIT       PX11
      000000F8H.4 SFRSYM    DATA     BIT       OISWH
      000000DCH   SFRSYM    DATA     WORD      LPF_K
      000000F2H   SFRSYM    DATA     WORD      PI_KI
      000000F8H.1 SFRSYM    DATA     BIT       OISUL
      000000A8H   SFRSYM    DATA     BYTE      IE
      000000F8H.3 SFRSYM    DATA     BIT       OISVL
      000000F8H.5 SFRSYM    DATA     BIT       OISWL
      000000D1H   SFRSYM    DATA     BYTE      P1IE
      00000098H.6 SFRSYM    DATA     BIT       MOD0
      000000D3H   SFRSYM    DATA     BYTE      P2IE
      000000D2H   SFRSYM    DATA     BYTE      P1IF
      000000F9H   SFRSYM    DATA     BYTE      PL_CR
      00000098H.7 SFRSYM    DATA     BIT       MOD1
      000000D4H   SFRSYM    DATA     BYTE      P2IF
      000000ACH   SFRSYM    DATA     WORD      TIM2_DR
      00000082H   SFRSYM    DATA     WORD      DP
      000000EEH   SFRSYM    DATA     WORD      PI_KP
      000000A4H   SFRSYM    DATA     WORD      TIM3_DR
      00000094H   SFRSYM    DATA     WORD      TIM4_DR
      0000008CH   SFRSYM    DATA     WORD      TIM5_DR
      000000F1H   SFRSYM    DATA     BYTE      OSC_CFG
      000000C1H   SFRSYM    DATA     BYTE      MD_MODE
LX51 LINKER/LOCATER V4.66.1.0                                                         03/23/2017  15:15:44  PAGE 16


      000000ECH   SFRSYM    DATA     WORD      PI_UK
      000000DEH   SFRSYM    DATA     WORD      LPF_X
      00000098H   SFRSYM    DATA     BIT       RI
      000000E6H   SFRSYM    DATA     WORD      LPF_Y
      000000C0H   SFRSYM    DATA     BIT       PTIM00
      000000D0H.7 SFRSYM    DATA     BIT       CY
      00000098H.1 SFRSYM    DATA     BIT       TI
      000000C0H.1 SFRSYM    DATA     BIT       PTIM01
      000000C0H.2 SFRSYM    DATA     BIT       PTIM10
      000000C0H.3 SFRSYM    DATA     BIT       PTIM11
      000000E1H   SFRSYM    DATA     BYTE      SV_CR
      00000098H   SFRSYM    DATA     BYTE      UT_CR
      00000099H   SFRSYM    DATA     BYTE      UT_DR
      000000F8H.6 SFRSYM    DATA     BIT       OIS4
      00000081H   SFRSYM    DATA     BYTE      SP
      000000D0H.2 SFRSYM    DATA     BIT       OV
      000000C4H   SFRSYM    DATA     BYTE      MD_DA0
      0000009AH   SFRSYM    DATA     WORD      UT_BAUD
      000000CCH   SFRSYM    DATA     BYTE      MD_DB0
      000000C5H   SFRSYM    DATA     BYTE      MD_DA1
      000000CDH   SFRSYM    DATA     BYTE      MD_DB1
      000000C6H   SFRSYM    DATA     BYTE      MD_DA2
      000000CEH   SFRSYM    DATA     BYTE      MD_DB2
      000000C7H   SFRSYM    DATA     BYTE      MD_DA3
      000000B4H   SFRSYM    DATA     WORD      TIM2_ADTR
      000000CFH   SFRSYM    DATA     BYTE      MD_DB3
      000000AFH   SFRSYM    DATA     BYTE      TIM2_ARRH
      000000A7H   SFRSYM    DATA     BYTE      TIM3_ARRH
      00000097H   SFRSYM    DATA     BYTE      TIM4_ARRH
      0000008FH   SFRSYM    DATA     BYTE      TIM5_ARRH
      000000AEH   SFRSYM    DATA     BYTE      TIM2_ARRL
      000000A6H   SFRSYM    DATA     BYTE      TIM3_ARRL
      00000087H   SFRSYM    DATA     BYTE      PCON
      000000E2H   SFRSYM    DATA     WORD      SV_US
      00000096H   SFRSYM    DATA     BYTE      TIM4_ARRL
      0000008EH   SFRSYM    DATA     BYTE      TIM5_ARRL
      000000B2H   SFRSYM    DATA     WORD      TIM2_CMTR
      00000088H   SFRSYM    DATA     BYTE      TCON
      000000AAH   SFRSYM    DATA     WORD      TIM2_CNTR
      000000A2H   SFRSYM    DATA     WORD      TIM3_CNTR
      00000092H   SFRSYM    DATA     WORD      TIM4_CNTR
      0000008AH   SFRSYM    DATA     WORD      TIM5_CNTR
      000000E5H   SFRSYM    DATA     BYTE      SV_ANGLEH
      000000D8H   SFRSYM    DATA     BIT       PUART0
      000000E4H   SFRSYM    DATA     BYTE      SV_ANGLEL
      000000C6H   SFRSYM    DATA     WORD      MD_DAH
      000000D8H.1 SFRSYM    DATA     BIT       PUART1
      000000D8H.2 SFRSYM    DATA     BIT       PI2C0
      00000088H.2 SFRSYM    DATA     BIT       IF0
      000000CEH   SFRSYM    DATA     WORD      MD_DBH
      000000D8H.3 SFRSYM    DATA     BIT       PI2C1
      000000F0H   SFRSYM    DATA     BYTE      B
      000000C4H   SFRSYM    DATA     WORD      MD_DAL
      000000A1H   SFRSYM    DATA     BYTE      TIM2_CR0
      000000CCH   SFRSYM    DATA     WORD      MD_DBL
      0000009CH   SFRSYM    DATA     BYTE      TIM3_CR0
      000000A9H   SFRSYM    DATA     BYTE      TIM2_CR1
      0000009EH   SFRSYM    DATA     BYTE      TIM4_CR0
      0000009DH   SFRSYM    DATA     BYTE      TIM3_CR1
      00000089H   SFRSYM    DATA     BYTE      TIM5_CR0
      0000009FH   SFRSYM    DATA     BYTE      TIM4_CR1
      000000F8H   SFRSYM    DATA     BYTE      DRV_OUT
      00000091H   SFRSYM    DATA     BYTE      TIM5_CR1
      000000E0H   SFRSYM    DATA     BYTE      ACC
      000000F7H   SFRSYM    DATA     BYTE      PI_UKMINH
LX51 LINKER/LOCATER V4.66.1.0                                                         03/23/2017  15:15:44  PAGE 17


      000000C3H   SFRSYM    DATA     BYTE      MD_MAH
      000000A8H.4 SFRSYM    DATA     BIT       ES0
      000000DBH   SFRSYM    DATA     BYTE      LVSR
      000000CBH   SFRSYM    DATA     BYTE      MD_MBH
      000000C0H.4 SFRSYM    DATA     BIT       PADC0
      000000B8H   SFRSYM    DATA     BYTE      IP0
      000000F5H   SFRSYM    DATA     BYTE      PI_UKMAXH
      000000C0H.5 SFRSYM    DATA     BIT       PADC1
      000000C0H   SFRSYM    DATA     BYTE      IP1
      000000C8H   SFRSYM    DATA     BYTE      IP2
      000000F6H   SFRSYM    DATA     BYTE      PI_UKMINL
      000000C2H   SFRSYM    DATA     BYTE      MD_MAL
      00000098H.2 SFRSYM    DATA     BIT       RB8
      000000D8H   SFRSYM    DATA     BYTE      IP3
      000000CAH   SFRSYM    DATA     BYTE      MD_MBL
      000000A8H   SFRSYM    DATA     BIT       EX0
      000000F4H   SFRSYM    DATA     BYTE      PI_UKMAXL
      00000098H.3 SFRSYM    DATA     BIT       TB8
      000000B7H   SFRSYM    DATA     BYTE      TIM0_CCR1H
      000000A8H.2 SFRSYM    DATA     BIT       EX1
      000000BBH   SFRSYM    DATA     BYTE      TIM0_CCR2H
      000000D0H   SFRSYM    DATA     BIT       P
      000000BDH   SFRSYM    DATA     BYTE      TIM0_CCR3H
      000000BFH   SFRSYM    DATA     BYTE      TIM0_CCR4H
      000000C8H.2 SFRSYM    DATA     BIT       PTIM230
      000000EBH   SFRSYM    DATA     BYTE      PI_EKH
      00000098H.5 SFRSYM    DATA     BIT       SM2
      000000B6H   SFRSYM    DATA     BYTE      TIM0_CCR1L
      000000B1H   SFRSYM    DATA     BYTE      TIM0_SR1
      000000C8H.3 SFRSYM    DATA     BIT       PTIM231
      000000BAH   SFRSYM    DATA     BYTE      TIM0_CCR2L
      000000BCH   SFRSYM    DATA     BYTE      TIM0_CCR3L
      000000BEH   SFRSYM    DATA     BYTE      TIM0_CCR4L
      000000D8H.6 SFRSYM    DATA     BIT       PMCD0
      000000C8H.4 SFRSYM    DATA     BIT       PTIM450
      000000D0H.3 SFRSYM    DATA     BIT       RS0
      000000DDH   SFRSYM    DATA     BYTE      LPF_KH
      000000F3H   SFRSYM    DATA     BYTE      PI_KIH
      000000EAH   SFRSYM    DATA     BYTE      PI_EKL
      000000E8H   SFRSYM    DATA     BYTE      FOC_SET0
      000000D8H.7 SFRSYM    DATA     BIT       PMCD1
      000000C8H.5 SFRSYM    DATA     BIT       PTIM451
      000000D0H.4 SFRSYM    DATA     BIT       RS1
      000000E9H   SFRSYM    DATA     BYTE      FOC_SET1
      000000B8H.6 SFRSYM    DATA     BIT       PFOC0
      000000DCH   SFRSYM    DATA     BYTE      LPF_KL
      000000F2H   SFRSYM    DATA     BYTE      PI_KIL
      000000B8H.7 SFRSYM    DATA     BIT       PFOC1
      000000ADH   SFRSYM    DATA     BYTE      TIM2_DRH
      000000B9H   SFRSYM    DATA     BYTE      TIM0_IER
      00000083H   SFRSYM    DATA     BYTE      DPH
      000000EFH   SFRSYM    DATA     BYTE      PI_KPH
      000000A5H   SFRSYM    DATA     BYTE      TIM3_DRH
      00000095H   SFRSYM    DATA     BYTE      TIM4_DRH
      0000008DH   SFRSYM    DATA     BYTE      TIM5_DRH
      000000ACH   SFRSYM    DATA     BYTE      TIM2_DRL
      00000082H   SFRSYM    DATA     BYTE      DPL
      000000EEH   SFRSYM    DATA     BYTE      PI_KPL
      000000A4H   SFRSYM    DATA     BYTE      TIM3_DRL
      000000F8H.7 SFRSYM    DATA     BIT       MOE
      000000C0H.6 SFRSYM    DATA     BIT       PCMP0
      000000EDH   SFRSYM    DATA     BYTE      PI_UKH
      00000094H   SFRSYM    DATA     BYTE      TIM4_DRL
      000000C0H.7 SFRSYM    DATA     BIT       PCMP1
      000000DFH   SFRSYM    DATA     BYTE      LPF_XH
LX51 LINKER/LOCATER V4.66.1.0                                                         03/23/2017  15:15:44  PAGE 18


      0000008CH   SFRSYM    DATA     BYTE      TIM5_DRL
      000000AEH   SFRSYM    DATA     WORD      TIM2_ARR
      000000A8H.5 SFRSYM    DATA     BIT       MCDIE
      000000C9H   SFRSYM    DATA     BYTE      RSTSRC
      000000E7H   SFRSYM    DATA     BYTE      LPF_YH
      000000A6H   SFRSYM    DATA     WORD      TIM3_ARR
      00000088H.6 SFRSYM    DATA     BIT       MCDIF
      00000098H.4 SFRSYM    DATA     BIT       REN
      00000096H   SFRSYM    DATA     WORD      TIM4_ARR
      000000ECH   SFRSYM    DATA     BYTE      PI_UKL
      000000D7H   SFRSYM    DATA     BYTE      CMP_SR
      0000008EH   SFRSYM    DATA     WORD      TIM5_ARR
      000000DEH   SFRSYM    DATA     BYTE      LPF_XL
      000000E6H   SFRSYM    DATA     BYTE      LPF_YL
      000000C8H   SFRSYM    DATA     BIT       PRTC0
      000000C8H.1 SFRSYM    DATA     BIT       PRTC1
      000000E8H.7 SFRSYM    DATA     BIT       FOCEN
      000000C8H.6 SFRSYM    DATA     BIT       PTSD0
      000000D8H.4 SFRSYM    DATA     BIT       PSPI0
      000000C8H.7 SFRSYM    DATA     BIT       PTSD1
      000000D8H.5 SFRSYM    DATA     BIT       PSPI1
      0000009BH   SFRSYM    DATA     BYTE      UT_BAUDH
      000000E4H   SFRSYM    DATA     WORD      SV_ANGLE
      000000B5H   SFRSYM    DATA     BYTE      TIM2_ADTRH
      0000009AH   SFRSYM    DATA     BYTE      UT_BAUDL
      000000FCH   SFRSYM    DATA     BYTE      P0_OE
      000000FDH   SFRSYM    DATA     BYTE      P1_OE
      000000D0H.5 SFRSYM    DATA     BIT       F0
      000000B4H   SFRSYM    DATA     BYTE      TIM2_ADTRL
      000000FEH   SFRSYM    DATA     BYTE      P2_OE
      000000D0H.1 SFRSYM    DATA     BIT       F1
      00000080H   SFRSYM    DATA     BIT       GP00
      000000FFH   SFRSYM    DATA     BYTE      P3_OE
      00000090H   SFRSYM    DATA     BIT       GP10
      00000080H.1 SFRSYM    DATA     BIT       GP01
      000000A8H.6 SFRSYM    DATA     BIT       RTCIE
      000000A0H   SFRSYM    DATA     BIT       GP20
      00000090H.1 SFRSYM    DATA     BIT       GP11
      00000080H.2 SFRSYM    DATA     BIT       GP02
      000000E3H   SFRSYM    DATA     BYTE      SV_USH
      000000B0H   SFRSYM    DATA     BIT       GP30
      000000A0H.1 SFRSYM    DATA     BIT       GP21
      00000090H.2 SFRSYM    DATA     BIT       GP12
      00000080H.3 SFRSYM    DATA     BIT       GP03
      000000B8H   SFRSYM    DATA     BIT       PLVW0
      000000A8H.1 SFRSYM    DATA     BIT       TSDIE
      000000D0H   SFRSYM    DATA     BYTE      PSW
      000000B0H.1 SFRSYM    DATA     BIT       GP31
      000000A0H.2 SFRSYM    DATA     BIT       GP22
      00000090H.3 SFRSYM    DATA     BIT       GP13
      00000080H.4 SFRSYM    DATA     BIT       GP04
      000000B8H.1 SFRSYM    DATA     BIT       PLVW1
      000000A8H.3 SFRSYM    DATA     BIT       SPIIE
      00000088H.5 SFRSYM    DATA     BIT       TSDIF
      000000B0H.2 SFRSYM    DATA     BIT       GP32
      000000A0H.3 SFRSYM    DATA     BIT       GP23
      00000090H.4 SFRSYM    DATA     BIT       GP14
      00000080H.5 SFRSYM    DATA     BIT       GP05
      00000084H   SFRSYM    DATA     BYTE      FLKEY
      000000B3H   SFRSYM    DATA     BYTE      TIM2_CMTRH
      000000B0H.3 SFRSYM    DATA     BIT       GP33
      000000A0H.4 SFRSYM    DATA     BIT       GP24
      00000090H.5 SFRSYM    DATA     BIT       GP15
      00000080H.6 SFRSYM    DATA     BIT       GP06
      00000088H   SFRSYM    DATA     BIT       IT00
LX51 LINKER/LOCATER V4.66.1.0                                                         03/23/2017  15:15:44  PAGE 19



      0100179FH   BLOCK     CODE     ---       LVL=0
      0100179FH   BLOCK     CODE     NEAR LAB  LVL=1
      02000129H   SYMBOL    XDATA    DWORD     PowerUpCnt
      ---         BLOCKEND  ---      ---       LVL=1
      0100179FH   LINE      CODE     ---       #39
      0100179FH   LINE      CODE     ---       #40
      0100179FH   LINE      CODE     ---       #44
      010017E6H   LINE      CODE     ---       #47
      010017E9H   LINE      CODE     ---       #50
      010017ECH   LINE      CODE     ---       #53
      010017EFH   LINE      CODE     ---       #56
      010017EFH   LINE      CODE     ---       #57
      010017EFH   LINE      CODE     ---       #59
      010017F2H   LINE      CODE     ---       #64
      010017F5H   LINE      CODE     ---       #65
      ---         BLOCKEND  ---      ---       LVL=0

      01000003H   BLOCK     CODE     ---       LVL=0
      01000003H   LINE      CODE     ---       #74
      01000003H   LINE      CODE     ---       #75
      01000003H   LINE      CODE     ---       #78
      01000006H   LINE      CODE     ---       #81
      0100000BH   LINE      CODE     ---       #82
      01000010H   LINE      CODE     ---       #84
      01000013H   LINE      CODE     ---       #85
      01000016H   LINE      CODE     ---       #86
      01000019H   LINE      CODE     ---       #87
      0100001CH   LINE      CODE     ---       #88
      0100001FH   LINE      CODE     ---       #89
      ---         BLOCKEND  ---      ---       LVL=0

      01001CEDH   BLOCK     CODE     ---       LVL=0
      01001CEDH   LINE      CODE     ---       #98
      01001CEDH   LINE      CODE     ---       #99
      01001CEDH   LINE      CODE     ---       #101
      01001CF0H   LINE      CODE     ---       #107
      01001CF3H   LINE      CODE     ---       #110
      01001CF6H   LINE      CODE     ---       #113
      01001CF9H   LINE      CODE     ---       #116
      01001CFCH   LINE      CODE     ---       #119
      01001CFFH   LINE      CODE     ---       #122
      01001D02H   LINE      CODE     ---       #125
      01001D05H   LINE      CODE     ---       #128
      01001D08H   LINE      CODE     ---       #129
      01001D0BH   LINE      CODE     ---       #130
      01001D0EH   LINE      CODE     ---       #133
      ---         BLOCKEND  ---      ---       LVL=0

      ---         MODULE    ---      ---       INTERRUPT
      02000166H   PUBLIC    XDATA    BYTE      FlagSPI
      01001C4AH   PUBLIC    CODE     ---       UART_ISR
      01000B41H   PUBLIC    CODE     ---       ADC_ISR
      01001BEDH   PUBLIC    CODE     ---       CMP_ISR
      010016DDH   PUBLIC    CODE     ---       TIM45_ISR
      010018E7H   PUBLIC    CODE     ---       TIM23_ISR
      01001672H   PUBLIC    CODE     ---       TIM0_ISR
      000000E2H   SFRSYM    DATA     BYTE      SV_USL
      000000ABH   SFRSYM    DATA     BYTE      TIM2_CNTRH
      000000B0H.4 SFRSYM    DATA     BIT       GP34
      000000A0H.5 SFRSYM    DATA     BIT       GP25
      00000090H.6 SFRSYM    DATA     BIT       GP16
      00000080H.7 SFRSYM    DATA     BIT       GP07
      00000088H.1 SFRSYM    DATA     BIT       IT01
      00000088H.3 SFRSYM    DATA     BIT       IT10
LX51 LINKER/LOCATER V4.66.1.0                                                         03/23/2017  15:15:44  PAGE 20


      000000F6H   SFRSYM    DATA     WORD      PI_UKMIN
      000000C2H   SFRSYM    DATA     WORD      MD_MA
      000000A3H   SFRSYM    DATA     BYTE      TIM3_CNTRH
      000000B0H.5 SFRSYM    DATA     BIT       GP35
      000000A0H.6 SFRSYM    DATA     BIT       GP26
      00000090H.7 SFRSYM    DATA     BIT       GP17
      00000080H   SFRSYM    DATA     BYTE      P0
      00000088H.4 SFRSYM    DATA     BIT       IT11
      000000CAH   SFRSYM    DATA     WORD      MD_MB
      00000093H   SFRSYM    DATA     BYTE      TIM4_CNTRH
      000000B0H.6 SFRSYM    DATA     BIT       GP36
      000000A0H.7 SFRSYM    DATA     BIT       GP27
      00000090H   SFRSYM    DATA     BYTE      P1
      000000D9H   SFRSYM    DATA     BYTE      EVT_FILT
      000000F4H   SFRSYM    DATA     WORD      PI_UKMAX
      0000008BH   SFRSYM    DATA     BYTE      TIM5_CNTRH
      000000B2H   SFRSYM    DATA     BYTE      TIM2_CMTRL
      000000B0H.7 SFRSYM    DATA     BIT       GP37
      000000A0H   SFRSYM    DATA     BYTE      P2
      000000AAH   SFRSYM    DATA     BYTE      TIM2_CNTRL
      000000B0H   SFRSYM    DATA     BYTE      P3
      000000A2H   SFRSYM    DATA     BYTE      TIM3_CNTRL
      000000D0H.6 SFRSYM    DATA     BIT       AC
      00000092H   SFRSYM    DATA     BYTE      TIM4_CNTRL
      0000008AH   SFRSYM    DATA     BYTE      TIM5_CNTRL
      000000B6H   SFRSYM    DATA     WORD      TIM0_CCR1
      000000A8H.7 SFRSYM    DATA     BIT       EA
      000000D5H   SFRSYM    DATA     BYTE      CMP_CR0
      000000BAH   SFRSYM    DATA     WORD      TIM0_CCR2
      000000D6H   SFRSYM    DATA     BYTE      CMP_CR1
      000000BCH   SFRSYM    DATA     WORD      TIM0_CCR3
      00000085H   SFRSYM    DATA     BYTE      PSCTL
      000000DAH   SFRSYM    DATA     BYTE      CMP_CR2
      000000BEH   SFRSYM    DATA     WORD      TIM0_CCR4
      000000B8H.2 SFRSYM    DATA     BIT       PX00
      000000EAH   SFRSYM    DATA     WORD      PI_EK
      000000F8H   SFRSYM    DATA     BIT       OISUH
      000000B8H.3 SFRSYM    DATA     BIT       PX01
      000000B8H.4 SFRSYM    DATA     BIT       PX10
      000000F8H.2 SFRSYM    DATA     BIT       OISVH
      000000B8H.5 SFRSYM    DATA     BIT       PX11
      000000F8H.4 SFRSYM    DATA     BIT       OISWH
      000000DCH   SFRSYM    DATA     WORD      LPF_K
      000000F2H   SFRSYM    DATA     WORD      PI_KI
      000000F8H.1 SFRSYM    DATA     BIT       OISUL
      000000A8H   SFRSYM    DATA     BYTE      IE
      000000F8H.3 SFRSYM    DATA     BIT       OISVL
      000000F8H.5 SFRSYM    DATA     BIT       OISWL
      000000D1H   SFRSYM    DATA     BYTE      P1IE
      00000098H.6 SFRSYM    DATA     BIT       MOD0
      000000D3H   SFRSYM    DATA     BYTE      P2IE
      000000D2H   SFRSYM    DATA     BYTE      P1IF
      000000F9H   SFRSYM    DATA     BYTE      PL_CR
      00000098H.7 SFRSYM    DATA     BIT       MOD1
      000000D4H   SFRSYM    DATA     BYTE      P2IF
      000000ACH   SFRSYM    DATA     WORD      TIM2_DR
      00000082H   SFRSYM    DATA     WORD      DP
      000000EEH   SFRSYM    DATA     WORD      PI_KP
      000000A4H   SFRSYM    DATA     WORD      TIM3_DR
      00000094H   SFRSYM    DATA     WORD      TIM4_DR
      0000008CH   SFRSYM    DATA     WORD      TIM5_DR
      000000F1H   SFRSYM    DATA     BYTE      OSC_CFG
      000000C1H   SFRSYM    DATA     BYTE      MD_MODE
      000000ECH   SFRSYM    DATA     WORD      PI_UK
      000000DEH   SFRSYM    DATA     WORD      LPF_X
LX51 LINKER/LOCATER V4.66.1.0                                                         03/23/2017  15:15:44  PAGE 21


      00000098H   SFRSYM    DATA     BIT       RI
      000000E6H   SFRSYM    DATA     WORD      LPF_Y
      000000C0H   SFRSYM    DATA     BIT       PTIM00
      000000D0H.7 SFRSYM    DATA     BIT       CY
      00000098H.1 SFRSYM    DATA     BIT       TI
      000000C0H.1 SFRSYM    DATA     BIT       PTIM01
      000000C0H.2 SFRSYM    DATA     BIT       PTIM10
      000000C0H.3 SFRSYM    DATA     BIT       PTIM11
      000000E1H   SFRSYM    DATA     BYTE      SV_CR
      00000098H   SFRSYM    DATA     BYTE      UT_CR
      00000099H   SFRSYM    DATA     BYTE      UT_DR
      000000F8H.6 SFRSYM    DATA     BIT       OIS4
      00000081H   SFRSYM    DATA     BYTE      SP
      000000D0H.2 SFRSYM    DATA     BIT       OV
      000000C4H   SFRSYM    DATA     BYTE      MD_DA0
      0000009AH   SFRSYM    DATA     WORD      UT_BAUD
      000000CCH   SFRSYM    DATA     BYTE      MD_DB0
      000000C5H   SFRSYM    DATA     BYTE      MD_DA1
      000000CDH   SFRSYM    DATA     BYTE      MD_DB1
      000000C6H   SFRSYM    DATA     BYTE      MD_DA2
      000000CEH   SFRSYM    DATA     BYTE      MD_DB2
      000000C7H   SFRSYM    DATA     BYTE      MD_DA3
      000000B4H   SFRSYM    DATA     WORD      TIM2_ADTR
      000000CFH   SFRSYM    DATA     BYTE      MD_DB3
      000000AFH   SFRSYM    DATA     BYTE      TIM2_ARRH
      000000A7H   SFRSYM    DATA     BYTE      TIM3_ARRH
      00000097H   SFRSYM    DATA     BYTE      TIM4_ARRH
      0000008FH   SFRSYM    DATA     BYTE      TIM5_ARRH
      000000AEH   SFRSYM    DATA     BYTE      TIM2_ARRL
      000000A6H   SFRSYM    DATA     BYTE      TIM3_ARRL
      00000087H   SFRSYM    DATA     BYTE      PCON
      000000E2H   SFRSYM    DATA     WORD      SV_US
      00000096H   SFRSYM    DATA     BYTE      TIM4_ARRL
      0000008EH   SFRSYM    DATA     BYTE      TIM5_ARRL
      000000B2H   SFRSYM    DATA     WORD      TIM2_CMTR
      00000088H   SFRSYM    DATA     BYTE      TCON
      000000AAH   SFRSYM    DATA     WORD      TIM2_CNTR
      000000A2H   SFRSYM    DATA     WORD      TIM3_CNTR
      00000092H   SFRSYM    DATA     WORD      TIM4_CNTR
      0000008AH   SFRSYM    DATA     WORD      TIM5_CNTR
      000000E5H   SFRSYM    DATA     BYTE      SV_ANGLEH
      000000D8H   SFRSYM    DATA     BIT       PUART0
      000000E4H   SFRSYM    DATA     BYTE      SV_ANGLEL
      000000C6H   SFRSYM    DATA     WORD      MD_DAH
      000000D8H.1 SFRSYM    DATA     BIT       PUART1
      000000D8H.2 SFRSYM    DATA     BIT       PI2C0
      00000088H.2 SFRSYM    DATA     BIT       IF0
      000000CEH   SFRSYM    DATA     WORD      MD_DBH
      000000D8H.3 SFRSYM    DATA     BIT       PI2C1
      000000F0H   SFRSYM    DATA     BYTE      B
      000000C4H   SFRSYM    DATA     WORD      MD_DAL
      000000A1H   SFRSYM    DATA     BYTE      TIM2_CR0
      000000CCH   SFRSYM    DATA     WORD      MD_DBL
      0000009CH   SFRSYM    DATA     BYTE      TIM3_CR0
      000000A9H   SFRSYM    DATA     BYTE      TIM2_CR1
      0000009EH   SFRSYM    DATA     BYTE      TIM4_CR0
      0000009DH   SFRSYM    DATA     BYTE      TIM3_CR1
      00000089H   SFRSYM    DATA     BYTE      TIM5_CR0
      0000009FH   SFRSYM    DATA     BYTE      TIM4_CR1
      000000F8H   SFRSYM    DATA     BYTE      DRV_OUT
      00000091H   SFRSYM    DATA     BYTE      TIM5_CR1
      000000E0H   SFRSYM    DATA     BYTE      ACC
      000000F7H   SFRSYM    DATA     BYTE      PI_UKMINH
      000000C3H   SFRSYM    DATA     BYTE      MD_MAH
      000000A8H.4 SFRSYM    DATA     BIT       ES0
LX51 LINKER/LOCATER V4.66.1.0                                                         03/23/2017  15:15:44  PAGE 22


      000000DBH   SFRSYM    DATA     BYTE      LVSR
      000000CBH   SFRSYM    DATA     BYTE      MD_MBH
      000000C0H.4 SFRSYM    DATA     BIT       PADC0
      000000B8H   SFRSYM    DATA     BYTE      IP0
      000000F5H   SFRSYM    DATA     BYTE      PI_UKMAXH
      000000C0H.5 SFRSYM    DATA     BIT       PADC1
      000000C0H   SFRSYM    DATA     BYTE      IP1
      000000C8H   SFRSYM    DATA     BYTE      IP2
      000000F6H   SFRSYM    DATA     BYTE      PI_UKMINL
      000000C2H   SFRSYM    DATA     BYTE      MD_MAL
      00000098H.2 SFRSYM    DATA     BIT       RB8
      000000D8H   SFRSYM    DATA     BYTE      IP3
      000000CAH   SFRSYM    DATA     BYTE      MD_MBL
      000000A8H   SFRSYM    DATA     BIT       EX0
      000000F4H   SFRSYM    DATA     BYTE      PI_UKMAXL
      00000098H.3 SFRSYM    DATA     BIT       TB8
      000000B7H   SFRSYM    DATA     BYTE      TIM0_CCR1H
      000000A8H.2 SFRSYM    DATA     BIT       EX1
      000000BBH   SFRSYM    DATA     BYTE      TIM0_CCR2H
      000000D0H   SFRSYM    DATA     BIT       P
      000000BDH   SFRSYM    DATA     BYTE      TIM0_CCR3H
      000000BFH   SFRSYM    DATA     BYTE      TIM0_CCR4H
      000000C8H.2 SFRSYM    DATA     BIT       PTIM230
      000000EBH   SFRSYM    DATA     BYTE      PI_EKH
      00000098H.5 SFRSYM    DATA     BIT       SM2
      000000B6H   SFRSYM    DATA     BYTE      TIM0_CCR1L
      000000B1H   SFRSYM    DATA     BYTE      TIM0_SR1
      000000C8H.3 SFRSYM    DATA     BIT       PTIM231
      000000BAH   SFRSYM    DATA     BYTE      TIM0_CCR2L
      000000BCH   SFRSYM    DATA     BYTE      TIM0_CCR3L
      000000BEH   SFRSYM    DATA     BYTE      TIM0_CCR4L
      000000D8H.6 SFRSYM    DATA     BIT       PMCD0
      000000C8H.4 SFRSYM    DATA     BIT       PTIM450
      000000D0H.3 SFRSYM    DATA     BIT       RS0
      000000DDH   SFRSYM    DATA     BYTE      LPF_KH
      000000F3H   SFRSYM    DATA     BYTE      PI_KIH
      000000EAH   SFRSYM    DATA     BYTE      PI_EKL
      000000E8H   SFRSYM    DATA     BYTE      FOC_SET0
      000000D8H.7 SFRSYM    DATA     BIT       PMCD1
      000000C8H.5 SFRSYM    DATA     BIT       PTIM451
      000000D0H.4 SFRSYM    DATA     BIT       RS1
      000000E9H   SFRSYM    DATA     BYTE      FOC_SET1
      000000B8H.6 SFRSYM    DATA     BIT       PFOC0
      000000DCH   SFRSYM    DATA     BYTE      LPF_KL
      000000F2H   SFRSYM    DATA     BYTE      PI_KIL
      000000B8H.7 SFRSYM    DATA     BIT       PFOC1
      000000ADH   SFRSYM    DATA     BYTE      TIM2_DRH
      000000B9H   SFRSYM    DATA     BYTE      TIM0_IER
      00000083H   SFRSYM    DATA     BYTE      DPH
      000000EFH   SFRSYM    DATA     BYTE      PI_KPH
      000000A5H   SFRSYM    DATA     BYTE      TIM3_DRH
      00000095H   SFRSYM    DATA     BYTE      TIM4_DRH
      0000008DH   SFRSYM    DATA     BYTE      TIM5_DRH
      000000ACH   SFRSYM    DATA     BYTE      TIM2_DRL
      00000082H   SFRSYM    DATA     BYTE      DPL
      000000EEH   SFRSYM    DATA     BYTE      PI_KPL
      000000A4H   SFRSYM    DATA     BYTE      TIM3_DRL
      000000F8H.7 SFRSYM    DATA     BIT       MOE
      000000C0H.6 SFRSYM    DATA     BIT       PCMP0
      000000EDH   SFRSYM    DATA     BYTE      PI_UKH
      00000094H   SFRSYM    DATA     BYTE      TIM4_DRL
      000000C0H.7 SFRSYM    DATA     BIT       PCMP1
      000000DFH   SFRSYM    DATA     BYTE      LPF_XH
      0000008CH   SFRSYM    DATA     BYTE      TIM5_DRL
      000000AEH   SFRSYM    DATA     WORD      TIM2_ARR
LX51 LINKER/LOCATER V4.66.1.0                                                         03/23/2017  15:15:44  PAGE 23


      000000A8H.5 SFRSYM    DATA     BIT       MCDIE
      000000C9H   SFRSYM    DATA     BYTE      RSTSRC
      000000E7H   SFRSYM    DATA     BYTE      LPF_YH
      000000A6H   SFRSYM    DATA     WORD      TIM3_ARR
      00000088H.6 SFRSYM    DATA     BIT       MCDIF
      00000098H.4 SFRSYM    DATA     BIT       REN
      00000096H   SFRSYM    DATA     WORD      TIM4_ARR
      000000ECH   SFRSYM    DATA     BYTE      PI_UKL
      000000D7H   SFRSYM    DATA     BYTE      CMP_SR
      0000008EH   SFRSYM    DATA     WORD      TIM5_ARR
      000000DEH   SFRSYM    DATA     BYTE      LPF_XL
      000000E6H   SFRSYM    DATA     BYTE      LPF_YL
      000000C8H   SFRSYM    DATA     BIT       PRTC0
      000000C8H.1 SFRSYM    DATA     BIT       PRTC1
      000000E8H.7 SFRSYM    DATA     BIT       FOCEN
      000000C8H.6 SFRSYM    DATA     BIT       PTSD0
      000000D8H.4 SFRSYM    DATA     BIT       PSPI0
      000000C8H.7 SFRSYM    DATA     BIT       PTSD1
      000000D8H.5 SFRSYM    DATA     BIT       PSPI1
      0000009BH   SFRSYM    DATA     BYTE      UT_BAUDH
      000000E4H   SFRSYM    DATA     WORD      SV_ANGLE
      000000B5H   SFRSYM    DATA     BYTE      TIM2_ADTRH
      0000009AH   SFRSYM    DATA     BYTE      UT_BAUDL
      000000FCH   SFRSYM    DATA     BYTE      P0_OE
      000000FDH   SFRSYM    DATA     BYTE      P1_OE
      000000D0H.5 SFRSYM    DATA     BIT       F0
      000000B4H   SFRSYM    DATA     BYTE      TIM2_ADTRL
      000000FEH   SFRSYM    DATA     BYTE      P2_OE
      000000D0H.1 SFRSYM    DATA     BIT       F1
      00000080H   SFRSYM    DATA     BIT       GP00
      000000FFH   SFRSYM    DATA     BYTE      P3_OE
      00000090H   SFRSYM    DATA     BIT       GP10
      00000080H.1 SFRSYM    DATA     BIT       GP01
      000000A8H.6 SFRSYM    DATA     BIT       RTCIE
      000000A0H   SFRSYM    DATA     BIT       GP20
      00000090H.1 SFRSYM    DATA     BIT       GP11
      00000080H.2 SFRSYM    DATA     BIT       GP02
      000000E3H   SFRSYM    DATA     BYTE      SV_USH
      000000B0H   SFRSYM    DATA     BIT       GP30
      000000A0H.1 SFRSYM    DATA     BIT       GP21
      00000090H.2 SFRSYM    DATA     BIT       GP12
      00000080H.3 SFRSYM    DATA     BIT       GP03
      000000B8H   SFRSYM    DATA     BIT       PLVW0
      000000A8H.1 SFRSYM    DATA     BIT       TSDIE
      000000D0H   SFRSYM    DATA     BYTE      PSW
      000000B0H.1 SFRSYM    DATA     BIT       GP31
      000000A0H.2 SFRSYM    DATA     BIT       GP22
      00000090H.3 SFRSYM    DATA     BIT       GP13
      00000080H.4 SFRSYM    DATA     BIT       GP04
      000000B8H.1 SFRSYM    DATA     BIT       PLVW1
      000000A8H.3 SFRSYM    DATA     BIT       SPIIE
      00000088H.5 SFRSYM    DATA     BIT       TSDIF
      000000B0H.2 SFRSYM    DATA     BIT       GP32
      000000A0H.3 SFRSYM    DATA     BIT       GP23
      00000090H.4 SFRSYM    DATA     BIT       GP14
      00000080H.5 SFRSYM    DATA     BIT       GP05
      00000084H   SFRSYM    DATA     BYTE      FLKEY
      000000B3H   SFRSYM    DATA     BYTE      TIM2_CMTRH
      000000B0H.3 SFRSYM    DATA     BIT       GP33
      000000A0H.4 SFRSYM    DATA     BIT       GP24
      00000090H.5 SFRSYM    DATA     BIT       GP15
      00000080H.6 SFRSYM    DATA     BIT       GP06
      00000088H   SFRSYM    DATA     BIT       IT00

      01001672H   BLOCK     CODE     ---       LVL=0
LX51 LINKER/LOCATER V4.66.1.0                                                         03/23/2017  15:15:44  PAGE 24


      0100168FH   BLOCK     CODE     NEAR LAB  LVL=1
      02000157H   SYMBOL    XDATA    BYTE      SystemTickCnt
      ---         BLOCKEND  ---      ---       LVL=1
      01001672H   LINE      CODE     ---       #28
      0100168FH   LINE      CODE     ---       #32
      01001694H   LINE      CODE     ---       #33
      01001694H   LINE      CODE     ---       #35
      0100169BH   LINE      CODE     ---       #36
      0100169EH   LINE      CODE     ---       #37
      0100169EH   LINE      CODE     ---       #39
      010016A3H   LINE      CODE     ---       #40
      010016A3H   LINE      CODE     ---       #42
      010016A9H   LINE      CODE     ---       #43
      010016ADH   LINE      CODE     ---       #44
      010016ADH   LINE      CODE     ---       #45
      010016AFH   LINE      CODE     ---       #46
      010016B2H   LINE      CODE     ---       #47
      010016B2H   LINE      CODE     ---       #50
      010016B5H   LINE      CODE     ---       #52
      010016BCH   LINE      CODE     ---       #53
      010016BCH   LINE      CODE     ---       #55
      010016BFH   LINE      CODE     ---       #56
      010016BFH   LINE      CODE     ---       #69
      010016C2H   LINE      CODE     ---       #70
      010016C2H   LINE      CODE     ---       #72
      ---         BLOCKEND  ---      ---       LVL=0

      010018E7H   BLOCK     CODE     ---       LVL=0
      010018E7H   LINE      CODE     ---       #73
      010018EDH   LINE      CODE     ---       #77
      010018F2H   LINE      CODE     ---       #78
      010018F2H   LINE      CODE     ---       #84
      010018FAH   LINE      CODE     ---       #85
      010018FAH   LINE      CODE     ---       #86
      010018FFH   LINE      CODE     ---       #87
      010018FFH   LINE      CODE     ---       #92
      01001907H   LINE      CODE     ---       #93
      01001907H   LINE      CODE     ---       #94
      0100190CH   LINE      CODE     ---       #95
      0100190CH   LINE      CODE     ---       #96
      01001912H   LINE      CODE     ---       #97
      01001912H   LINE      CODE     ---       #98
      01001919H   LINE      CODE     ---       #100
      0100191BH   LINE      CODE     ---       #102
      0100191BH   LINE      CODE     ---       #103
      0100191FH   LINE      CODE     ---       #105
      0100191FH   LINE      CODE     ---       #106
      01001927H   LINE      CODE     ---       #107
      01001927H   LINE      CODE     ---       #109
      ---         BLOCKEND  ---      ---       LVL=0

      010016DDH   BLOCK     CODE     ---       LVL=0
      010016DDH   LINE      CODE     ---       #120
      010016FAH   LINE      CODE     ---       #122
      010016FFH   LINE      CODE     ---       #123
      010016FFH   LINE      CODE     ---       #125
      01001702H   LINE      CODE     ---       #127
      01001709H   LINE      CODE     ---       #128
      01001709H   LINE      CODE     ---       #130
      0100170CH   LINE      CODE     ---       #131
      0100170CH   LINE      CODE     ---       #134
      0100170FH   LINE      CODE     ---       #137
      01001712H   LINE      CODE     ---       #140
      01001715H   LINE      CODE     ---       #143
      01001718H   LINE      CODE     ---       #146
LX51 LINKER/LOCATER V4.66.1.0                                                         03/23/2017  15:15:44  PAGE 25


      0100171BH   LINE      CODE     ---       #149
      0100171EH   LINE      CODE     ---       #151
      01001726H   LINE      CODE     ---       #152
      01001726H   LINE      CODE     ---       #154
      ---         BLOCKEND  ---      ---       LVL=0

      01001BEDH   BLOCK     CODE     ---       LVL=0
      01001BEDH   LINE      CODE     ---       #162
      01001BF5H   LINE      CODE     ---       #164
      01001BFAH   LINE      CODE     ---       #165
      01001BFAH   LINE      CODE     ---       #166
      01001BFDH   LINE      CODE     ---       #167
      01001C04H   LINE      CODE     ---       #168
      01001C04H   LINE      CODE     ---       #169
      01001C07H   LINE      CODE     ---       #171
      01001C0DH   LINE      CODE     ---       #172
      01001C13H   LINE      CODE     ---       #173
      01001C13H   LINE      CODE     ---       #174
      01001C13H   LINE      CODE     ---       #175
      ---         BLOCKEND  ---      ---       LVL=0

      01000B41H   BLOCK     CODE     ---       LVL=0
      01000B5EH   BLOCK     CODE     NEAR LAB  LVL=1
      02000158H   SYMBOL    XDATA    WORD      ADCData_VoltageVTH
      0200015AH   SYMBOL    XDATA    WORD      ADCData_VoltageBUS
      0200015CH   SYMBOL    XDATA    WORD      ADCData_VoltageN
      0200015EH   SYMBOL    XDATA    WORD      ADCData_CurrentBUS
      02000160H   SYMBOL    XDATA    WORD      ADCData_RCCurrentBUS
      02000162H   SYMBOL    XDATA    WORD      ADCData_VoltageSREF0
      02000164H   SYMBOL    XDATA    WORD      ADCData_VoltageSREF1
      ---         BLOCKEND  ---      ---       LVL=1
      01000B41H   LINE      CODE     ---       #186
      01000B5EH   LINE      CODE     ---       #197
      01000B68H   LINE      CODE     ---       #198
      01000B68H   LINE      CODE     ---       #201
      01000B81H   LINE      CODE     ---       #202
      01000B9AH   LINE      CODE     ---       #203
      01000BB3H   LINE      CODE     ---       #204
      01000BCCH   LINE      CODE     ---       #205
      01000BE5H   LINE      CODE     ---       #208
      01000C04H   LINE      CODE     ---       #209
      01000C23H   LINE      CODE     ---       #210
      01000C42H   LINE      CODE     ---       #211
      01000C61H   LINE      CODE     ---       #212
      01000C80H   LINE      CODE     ---       #214
      01000C87H   LINE      CODE     ---       #215
      01000C87H   LINE      CODE     ---       #217
      01000C8EH   LINE      CODE     ---       #218
      01000C8EH   LINE      CODE     ---       #219
      01000C92H   LINE      CODE     ---       #220
      01000C92H   LINE      CODE     ---       #221
      ---         BLOCKEND  ---      ---       LVL=0

      01001C4AH   BLOCK     CODE     ---       LVL=0
      01001C4AH   LINE      CODE     ---       #229
      01001C57H   LINE      CODE     ---       #231
      01001C5AH   LINE      CODE     ---       #232
      01001C5AH   LINE      CODE     ---       #233
      01001C64H   LINE      CODE     ---       #234
      01001C66H   LINE      CODE     ---       #235
      01001C66H   LINE      CODE     ---       #236
      01001C69H   LINE      CODE     ---       #237
      01001C69H   LINE      CODE     ---       #238
      01001C6BH   LINE      CODE     ---       #239
      01001C6BH   LINE      CODE     ---       #241
LX51 LINKER/LOCATER V4.66.1.0                                                         03/23/2017  15:15:44  PAGE 26


      ---         BLOCKEND  ---      ---       LVL=0

      ---         MODULE    ---      ---       MOTORCONTROL
      020000A1H   PUBLIC    XDATA    ---       TargetSpeedTable
      0200008BH   PUBLIC    XDATA    ---       TargetCurrentTable
      02000026H   PUBLIC    XDATA    ---       MC
      02000010H   PUBLIC    XDATA    ---       TargetVSTable
      01001006H   PUBLIC    CODE     ---       SystemTick
      010019B9H   PUBLIC    CODE     ---       ONOFFControl
      01000995H   PUBLIC    CODE     ---       SpeedControl
      01001741H   PUBLIC    CODE     ---       RestartControl
      01000571H   PUBLIC    CODE     ---       FaultDetect
      010011EAH   PUBLIC    CODE     ---       ParameterInit
      01001CA1H   PUBLIC    CODE     ---       MotorFault
      01001C76H   PUBLIC    CODE     ---       MotorNormal
      01001E65H   PUBLIC    CODE     ---       MotorStart
      01000DF3H   PUBLIC    CODE     ---       MotorPrecharge
      01001EAFH   PUBLIC    CODE     ---       MotorReady
      01000056H   PUBLIC    CODE     ---       MotorInit
      01001A76H   PUBLIC    CODE     ---       MotorStop
      01001A38H   PUBLIC    CODE     ---       MotorMain
      000000E2H   SFRSYM    DATA     BYTE      SV_USL
      000000ABH   SFRSYM    DATA     BYTE      TIM2_CNTRH
      000000B0H.4 SFRSYM    DATA     BIT       GP34
      000000A0H.5 SFRSYM    DATA     BIT       GP25
      00000090H.6 SFRSYM    DATA     BIT       GP16
      00000080H.7 SFRSYM    DATA     BIT       GP07
      00000088H.1 SFRSYM    DATA     BIT       IT01
      00000088H.3 SFRSYM    DATA     BIT       IT10
      000000F6H   SFRSYM    DATA     WORD      PI_UKMIN
      000000C2H   SFRSYM    DATA     WORD      MD_MA
      000000A3H   SFRSYM    DATA     BYTE      TIM3_CNTRH
      000000B0H.5 SFRSYM    DATA     BIT       GP35
      000000A0H.6 SFRSYM    DATA     BIT       GP26
      00000090H.7 SFRSYM    DATA     BIT       GP17
      00000080H   SFRSYM    DATA     BYTE      P0
      00000088H.4 SFRSYM    DATA     BIT       IT11
      000000CAH   SFRSYM    DATA     WORD      MD_MB
      00000093H   SFRSYM    DATA     BYTE      TIM4_CNTRH
      000000B0H.6 SFRSYM    DATA     BIT       GP36
      000000A0H.7 SFRSYM    DATA     BIT       GP27
      00000090H   SFRSYM    DATA     BYTE      P1
      000000D9H   SFRSYM    DATA     BYTE      EVT_FILT
      000000F4H   SFRSYM    DATA     WORD      PI_UKMAX
      0000008BH   SFRSYM    DATA     BYTE      TIM5_CNTRH
      000000B2H   SFRSYM    DATA     BYTE      TIM2_CMTRL
      000000B0H.7 SFRSYM    DATA     BIT       GP37
      000000A0H   SFRSYM    DATA     BYTE      P2
      000000AAH   SFRSYM    DATA     BYTE      TIM2_CNTRL
      000000B0H   SFRSYM    DATA     BYTE      P3
      000000A2H   SFRSYM    DATA     BYTE      TIM3_CNTRL
      000000D0H.6 SFRSYM    DATA     BIT       AC
      00000092H   SFRSYM    DATA     BYTE      TIM4_CNTRL
      0000008AH   SFRSYM    DATA     BYTE      TIM5_CNTRL
      000000B6H   SFRSYM    DATA     WORD      TIM0_CCR1
      000000A8H.7 SFRSYM    DATA     BIT       EA
      000000D5H   SFRSYM    DATA     BYTE      CMP_CR0
      000000BAH   SFRSYM    DATA     WORD      TIM0_CCR2
      000000D6H   SFRSYM    DATA     BYTE      CMP_CR1
      000000BCH   SFRSYM    DATA     WORD      TIM0_CCR3
      00000085H   SFRSYM    DATA     BYTE      PSCTL
      000000DAH   SFRSYM    DATA     BYTE      CMP_CR2
      000000BEH   SFRSYM    DATA     WORD      TIM0_CCR4
      000000B8H.2 SFRSYM    DATA     BIT       PX00
      000000EAH   SFRSYM    DATA     WORD      PI_EK
LX51 LINKER/LOCATER V4.66.1.0                                                         03/23/2017  15:15:44  PAGE 27


      000000F8H   SFRSYM    DATA     BIT       OISUH
      000000B8H.3 SFRSYM    DATA     BIT       PX01
      000000B8H.4 SFRSYM    DATA     BIT       PX10
      000000F8H.2 SFRSYM    DATA     BIT       OISVH
      000000B8H.5 SFRSYM    DATA     BIT       PX11
      000000F8H.4 SFRSYM    DATA     BIT       OISWH
      000000DCH   SFRSYM    DATA     WORD      LPF_K
      000000F2H   SFRSYM    DATA     WORD      PI_KI
      000000F8H.1 SFRSYM    DATA     BIT       OISUL
      000000A8H   SFRSYM    DATA     BYTE      IE
      000000F8H.3 SFRSYM    DATA     BIT       OISVL
      000000F8H.5 SFRSYM    DATA     BIT       OISWL
      000000D1H   SFRSYM    DATA     BYTE      P1IE
      00000098H.6 SFRSYM    DATA     BIT       MOD0
      000000D3H   SFRSYM    DATA     BYTE      P2IE
      000000D2H   SFRSYM    DATA     BYTE      P1IF
      000000F9H   SFRSYM    DATA     BYTE      PL_CR
      00000098H.7 SFRSYM    DATA     BIT       MOD1
      000000D4H   SFRSYM    DATA     BYTE      P2IF
      000000ACH   SFRSYM    DATA     WORD      TIM2_DR
      00000082H   SFRSYM    DATA     WORD      DP
      000000EEH   SFRSYM    DATA     WORD      PI_KP
      000000A4H   SFRSYM    DATA     WORD      TIM3_DR
      00000094H   SFRSYM    DATA     WORD      TIM4_DR
      0000008CH   SFRSYM    DATA     WORD      TIM5_DR
      000000F1H   SFRSYM    DATA     BYTE      OSC_CFG
      000000C1H   SFRSYM    DATA     BYTE      MD_MODE
      000000ECH   SFRSYM    DATA     WORD      PI_UK
      000000DEH   SFRSYM    DATA     WORD      LPF_X
      00000098H   SFRSYM    DATA     BIT       RI
      000000E6H   SFRSYM    DATA     WORD      LPF_Y
      000000C0H   SFRSYM    DATA     BIT       PTIM00
      000000D0H.7 SFRSYM    DATA     BIT       CY
      00000098H.1 SFRSYM    DATA     BIT       TI
      000000C0H.1 SFRSYM    DATA     BIT       PTIM01
      000000C0H.2 SFRSYM    DATA     BIT       PTIM10
      000000C0H.3 SFRSYM    DATA     BIT       PTIM11
      000000E1H   SFRSYM    DATA     BYTE      SV_CR
      00000098H   SFRSYM    DATA     BYTE      UT_CR
      00000099H   SFRSYM    DATA     BYTE      UT_DR
      000000F8H.6 SFRSYM    DATA     BIT       OIS4
      00000081H   SFRSYM    DATA     BYTE      SP
      000000D0H.2 SFRSYM    DATA     BIT       OV
      000000C4H   SFRSYM    DATA     BYTE      MD_DA0
      0000009AH   SFRSYM    DATA     WORD      UT_BAUD
      000000CCH   SFRSYM    DATA     BYTE      MD_DB0
      000000C5H   SFRSYM    DATA     BYTE      MD_DA1
      000000CDH   SFRSYM    DATA     BYTE      MD_DB1
      000000C6H   SFRSYM    DATA     BYTE      MD_DA2
      000000CEH   SFRSYM    DATA     BYTE      MD_DB2
      000000C7H   SFRSYM    DATA     BYTE      MD_DA3
      000000B4H   SFRSYM    DATA     WORD      TIM2_ADTR
      000000CFH   SFRSYM    DATA     BYTE      MD_DB3
      000000AFH   SFRSYM    DATA     BYTE      TIM2_ARRH
      000000A7H   SFRSYM    DATA     BYTE      TIM3_ARRH
      00000097H   SFRSYM    DATA     BYTE      TIM4_ARRH
      0000008FH   SFRSYM    DATA     BYTE      TIM5_ARRH
      000000AEH   SFRSYM    DATA     BYTE      TIM2_ARRL
      000000A6H   SFRSYM    DATA     BYTE      TIM3_ARRL
      00000087H   SFRSYM    DATA     BYTE      PCON
      000000E2H   SFRSYM    DATA     WORD      SV_US
      00000096H   SFRSYM    DATA     BYTE      TIM4_ARRL
      0000008EH   SFRSYM    DATA     BYTE      TIM5_ARRL
      000000B2H   SFRSYM    DATA     WORD      TIM2_CMTR
      00000088H   SFRSYM    DATA     BYTE      TCON
LX51 LINKER/LOCATER V4.66.1.0                                                         03/23/2017  15:15:44  PAGE 28


      000000AAH   SFRSYM    DATA     WORD      TIM2_CNTR
      000000A2H   SFRSYM    DATA     WORD      TIM3_CNTR
      00000092H   SFRSYM    DATA     WORD      TIM4_CNTR
      0000008AH   SFRSYM    DATA     WORD      TIM5_CNTR
      000000E5H   SFRSYM    DATA     BYTE      SV_ANGLEH
      000000D8H   SFRSYM    DATA     BIT       PUART0
      000000E4H   SFRSYM    DATA     BYTE      SV_ANGLEL
      000000C6H   SFRSYM    DATA     WORD      MD_DAH
      000000D8H.1 SFRSYM    DATA     BIT       PUART1
      000000D8H.2 SFRSYM    DATA     BIT       PI2C0
      00000088H.2 SFRSYM    DATA     BIT       IF0
      000000CEH   SFRSYM    DATA     WORD      MD_DBH
      000000D8H.3 SFRSYM    DATA     BIT       PI2C1
      000000F0H   SFRSYM    DATA     BYTE      B
      000000C4H   SFRSYM    DATA     WORD      MD_DAL
      000000A1H   SFRSYM    DATA     BYTE      TIM2_CR0
      000000CCH   SFRSYM    DATA     WORD      MD_DBL
      0000009CH   SFRSYM    DATA     BYTE      TIM3_CR0
      000000A9H   SFRSYM    DATA     BYTE      TIM2_CR1
      0000009EH   SFRSYM    DATA     BYTE      TIM4_CR0
      0000009DH   SFRSYM    DATA     BYTE      TIM3_CR1
      00000089H   SFRSYM    DATA     BYTE      TIM5_CR0
      0000009FH   SFRSYM    DATA     BYTE      TIM4_CR1
      000000F8H   SFRSYM    DATA     BYTE      DRV_OUT
      00000091H   SFRSYM    DATA     BYTE      TIM5_CR1
      000000E0H   SFRSYM    DATA     BYTE      ACC
      000000F7H   SFRSYM    DATA     BYTE      PI_UKMINH
      000000C3H   SFRSYM    DATA     BYTE      MD_MAH
      000000A8H.4 SFRSYM    DATA     BIT       ES0
      000000DBH   SFRSYM    DATA     BYTE      LVSR
      000000CBH   SFRSYM    DATA     BYTE      MD_MBH
      000000C0H.4 SFRSYM    DATA     BIT       PADC0
      000000B8H   SFRSYM    DATA     BYTE      IP0
      000000F5H   SFRSYM    DATA     BYTE      PI_UKMAXH
      000000C0H.5 SFRSYM    DATA     BIT       PADC1
      000000C0H   SFRSYM    DATA     BYTE      IP1
      000000C8H   SFRSYM    DATA     BYTE      IP2
      000000F6H   SFRSYM    DATA     BYTE      PI_UKMINL
      000000C2H   SFRSYM    DATA     BYTE      MD_MAL
      00000098H.2 SFRSYM    DATA     BIT       RB8
      000000D8H   SFRSYM    DATA     BYTE      IP3
      000000CAH   SFRSYM    DATA     BYTE      MD_MBL
      000000A8H   SFRSYM    DATA     BIT       EX0
      000000F4H   SFRSYM    DATA     BYTE      PI_UKMAXL
      00000098H.3 SFRSYM    DATA     BIT       TB8
      000000B7H   SFRSYM    DATA     BYTE      TIM0_CCR1H
      000000A8H.2 SFRSYM    DATA     BIT       EX1
      000000BBH   SFRSYM    DATA     BYTE      TIM0_CCR2H
      000000D0H   SFRSYM    DATA     BIT       P
      000000BDH   SFRSYM    DATA     BYTE      TIM0_CCR3H
      000000BFH   SFRSYM    DATA     BYTE      TIM0_CCR4H
      000000C8H.2 SFRSYM    DATA     BIT       PTIM230
      000000EBH   SFRSYM    DATA     BYTE      PI_EKH
      00000098H.5 SFRSYM    DATA     BIT       SM2
      000000B6H   SFRSYM    DATA     BYTE      TIM0_CCR1L
      000000B1H   SFRSYM    DATA     BYTE      TIM0_SR1
      000000C8H.3 SFRSYM    DATA     BIT       PTIM231
      000000BAH   SFRSYM    DATA     BYTE      TIM0_CCR2L
      000000BCH   SFRSYM    DATA     BYTE      TIM0_CCR3L
      000000BEH   SFRSYM    DATA     BYTE      TIM0_CCR4L
      000000D8H.6 SFRSYM    DATA     BIT       PMCD0
      000000C8H.4 SFRSYM    DATA     BIT       PTIM450
      000000D0H.3 SFRSYM    DATA     BIT       RS0
      000000DDH   SFRSYM    DATA     BYTE      LPF_KH
      000000F3H   SFRSYM    DATA     BYTE      PI_KIH
LX51 LINKER/LOCATER V4.66.1.0                                                         03/23/2017  15:15:44  PAGE 29


      000000EAH   SFRSYM    DATA     BYTE      PI_EKL
      000000E8H   SFRSYM    DATA     BYTE      FOC_SET0
      000000D8H.7 SFRSYM    DATA     BIT       PMCD1
      000000C8H.5 SFRSYM    DATA     BIT       PTIM451
      000000D0H.4 SFRSYM    DATA     BIT       RS1
      000000E9H   SFRSYM    DATA     BYTE      FOC_SET1
      000000B8H.6 SFRSYM    DATA     BIT       PFOC0
      000000DCH   SFRSYM    DATA     BYTE      LPF_KL
      000000F2H   SFRSYM    DATA     BYTE      PI_KIL
      000000B8H.7 SFRSYM    DATA     BIT       PFOC1
      000000ADH   SFRSYM    DATA     BYTE      TIM2_DRH
      000000B9H   SFRSYM    DATA     BYTE      TIM0_IER
      00000083H   SFRSYM    DATA     BYTE      DPH
      000000EFH   SFRSYM    DATA     BYTE      PI_KPH
      000000A5H   SFRSYM    DATA     BYTE      TIM3_DRH
      00000095H   SFRSYM    DATA     BYTE      TIM4_DRH
      0000008DH   SFRSYM    DATA     BYTE      TIM5_DRH
      000000ACH   SFRSYM    DATA     BYTE      TIM2_DRL
      00000082H   SFRSYM    DATA     BYTE      DPL
      000000EEH   SFRSYM    DATA     BYTE      PI_KPL
      000000A4H   SFRSYM    DATA     BYTE      TIM3_DRL
      000000F8H.7 SFRSYM    DATA     BIT       MOE
      000000C0H.6 SFRSYM    DATA     BIT       PCMP0
      000000EDH   SFRSYM    DATA     BYTE      PI_UKH
      00000094H   SFRSYM    DATA     BYTE      TIM4_DRL
      000000C0H.7 SFRSYM    DATA     BIT       PCMP1
      000000DFH   SFRSYM    DATA     BYTE      LPF_XH
      0000008CH   SFRSYM    DATA     BYTE      TIM5_DRL
      000000AEH   SFRSYM    DATA     WORD      TIM2_ARR
      000000A8H.5 SFRSYM    DATA     BIT       MCDIE
      000000C9H   SFRSYM    DATA     BYTE      RSTSRC
      000000E7H   SFRSYM    DATA     BYTE      LPF_YH
      000000A6H   SFRSYM    DATA     WORD      TIM3_ARR
      00000088H.6 SFRSYM    DATA     BIT       MCDIF
      00000098H.4 SFRSYM    DATA     BIT       REN
      00000096H   SFRSYM    DATA     WORD      TIM4_ARR
      000000ECH   SFRSYM    DATA     BYTE      PI_UKL
      000000D7H   SFRSYM    DATA     BYTE      CMP_SR
      0000008EH   SFRSYM    DATA     WORD      TIM5_ARR
      000000DEH   SFRSYM    DATA     BYTE      LPF_XL
      000000E6H   SFRSYM    DATA     BYTE      LPF_YL
      000000C8H   SFRSYM    DATA     BIT       PRTC0
      000000C8H.1 SFRSYM    DATA     BIT       PRTC1
      000000E8H.7 SFRSYM    DATA     BIT       FOCEN
      000000C8H.6 SFRSYM    DATA     BIT       PTSD0
      000000D8H.4 SFRSYM    DATA     BIT       PSPI0
      000000C8H.7 SFRSYM    DATA     BIT       PTSD1
      000000D8H.5 SFRSYM    DATA     BIT       PSPI1
      0000009BH   SFRSYM    DATA     BYTE      UT_BAUDH
      000000E4H   SFRSYM    DATA     WORD      SV_ANGLE
      000000B5H   SFRSYM    DATA     BYTE      TIM2_ADTRH
      0000009AH   SFRSYM    DATA     BYTE      UT_BAUDL
      000000FCH   SFRSYM    DATA     BYTE      P0_OE
      000000FDH   SFRSYM    DATA     BYTE      P1_OE
      000000D0H.5 SFRSYM    DATA     BIT       F0
      000000B4H   SFRSYM    DATA     BYTE      TIM2_ADTRL
      000000FEH   SFRSYM    DATA     BYTE      P2_OE
      000000D0H.1 SFRSYM    DATA     BIT       F1
      00000080H   SFRSYM    DATA     BIT       GP00
      000000FFH   SFRSYM    DATA     BYTE      P3_OE
      00000090H   SFRSYM    DATA     BIT       GP10
      00000080H.1 SFRSYM    DATA     BIT       GP01
      000000A8H.6 SFRSYM    DATA     BIT       RTCIE
      000000A0H   SFRSYM    DATA     BIT       GP20
      00000090H.1 SFRSYM    DATA     BIT       GP11
LX51 LINKER/LOCATER V4.66.1.0                                                         03/23/2017  15:15:44  PAGE 30


      00000080H.2 SFRSYM    DATA     BIT       GP02
      000000E3H   SFRSYM    DATA     BYTE      SV_USH
      000000B0H   SFRSYM    DATA     BIT       GP30
      000000A0H.1 SFRSYM    DATA     BIT       GP21
      00000090H.2 SFRSYM    DATA     BIT       GP12
      00000080H.3 SFRSYM    DATA     BIT       GP03
      000000B8H   SFRSYM    DATA     BIT       PLVW0
      000000A8H.1 SFRSYM    DATA     BIT       TSDIE
      000000D0H   SFRSYM    DATA     BYTE      PSW
      000000B0H.1 SFRSYM    DATA     BIT       GP31
      000000A0H.2 SFRSYM    DATA     BIT       GP22
      00000090H.3 SFRSYM    DATA     BIT       GP13
      00000080H.4 SFRSYM    DATA     BIT       GP04
      000000B8H.1 SFRSYM    DATA     BIT       PLVW1
      000000A8H.3 SFRSYM    DATA     BIT       SPIIE
      00000088H.5 SFRSYM    DATA     BIT       TSDIF
      000000B0H.2 SFRSYM    DATA     BIT       GP32
      000000A0H.3 SFRSYM    DATA     BIT       GP23
      00000090H.4 SFRSYM    DATA     BIT       GP14
      00000080H.5 SFRSYM    DATA     BIT       GP05
      00000084H   SFRSYM    DATA     BYTE      FLKEY
      000000B3H   SFRSYM    DATA     BYTE      TIM2_CMTRH
      000000B0H.3 SFRSYM    DATA     BIT       GP33
      000000A0H.4 SFRSYM    DATA     BIT       GP24
      00000090H.5 SFRSYM    DATA     BIT       GP15
      00000080H.6 SFRSYM    DATA     BIT       GP06
      00000088H   SFRSYM    DATA     BIT       IT00

      01001A38H   BLOCK     CODE     ---       LVL=0
      01001A38H   LINE      CODE     ---       #33
      01001A38H   LINE      CODE     ---       #34
      01001A38H   LINE      CODE     ---       #35
      01001A60H   LINE      CODE     ---       #36
      01001A60H   LINE      CODE     ---       #37
      01001A60H   LINE      CODE     ---       #38
      01001A63H   LINE      CODE     ---       #39
      01001A63H   LINE      CODE     ---       #40
      01001A63H   LINE      CODE     ---       #41
      01001A66H   LINE      CODE     ---       #42
      01001A66H   LINE      CODE     ---       #43
      01001A66H   LINE      CODE     ---       #44
      01001A69H   LINE      CODE     ---       #45
      01001A69H   LINE      CODE     ---       #46
      01001A69H   LINE      CODE     ---       #47
      01001A6CH   LINE      CODE     ---       #48
      01001A6CH   LINE      CODE     ---       #49
      01001A6CH   LINE      CODE     ---       #50
      01001A6FH   LINE      CODE     ---       #51
      01001A6FH   LINE      CODE     ---       #52
      01001A6FH   LINE      CODE     ---       #53
      01001A72H   LINE      CODE     ---       #54
      01001A72H   LINE      CODE     ---       #55
      01001A72H   LINE      CODE     ---       #56
      01001A75H   LINE      CODE     ---       #57
      01001A75H   LINE      CODE     ---       #58
      01001A75H   LINE      CODE     ---       #59
      01001A75H   LINE      CODE     ---       #60
      01001A75H   LINE      CODE     ---       #61
      ---         BLOCKEND  ---      ---       LVL=0

      01001A76H   BLOCK     CODE     ---       LVL=0
      01001A76H   LINE      CODE     ---       #73
      01001A76H   LINE      CODE     ---       #74
      01001A76H   LINE      CODE     ---       #76
      01001A7CH   LINE      CODE     ---       #77
LX51 LINKER/LOCATER V4.66.1.0                                                         03/23/2017  15:15:44  PAGE 31


      01001A7CH   LINE      CODE     ---       #78
      01001A80H   LINE      CODE     ---       #79
      01001A85H   LINE      CODE     ---       #80
      01001A85H   LINE      CODE     ---       #82
      01001AA0H   LINE      CODE     ---       #83
      01001AA0H   LINE      CODE     ---       #84
      01001AAAH   LINE      CODE     ---       #85
      01001AAAH   LINE      CODE     ---       #87
      01001AADH   LINE      CODE     ---       #89
      ---         BLOCKEND  ---      ---       LVL=0

      01000056H   BLOCK     CODE     ---       LVL=0
      01000056H   LINE      CODE     ---       #101
      01000056H   LINE      CODE     ---       #102
      01000056H   LINE      CODE     ---       #104
      01000059H   LINE      CODE     ---       #106
      0100005FH   LINE      CODE     ---       #109
      ---         BLOCKEND  ---      ---       LVL=0

      01001EAFH   BLOCK     CODE     ---       LVL=0
      01001EAFH   LINE      CODE     ---       #126
      01001EAFH   LINE      CODE     ---       #127
      01001EAFH   LINE      CODE     ---       #128
      01001EB5H   LINE      CODE     ---       #129
      ---         BLOCKEND  ---      ---       LVL=0

      01000DF3H   BLOCK     CODE     ---       LVL=0
      01000DF3H   BLOCK     CODE     NEAR LAB  LVL=1
      02000000H   SYMBOL    XDATA    BYTE      FlagPrechargeU
      02000001H   SYMBOL    XDATA    BYTE      FlagPrechargeV
      02000002H   SYMBOL    XDATA    BYTE      FlagPrechargeW
      ---         BLOCKEND  ---      ---       LVL=1
      01000DF3H   LINE      CODE     ---       #138
      01000DF3H   LINE      CODE     ---       #139
      01000DF3H   LINE      CODE     ---       #144
      01000DF9H   LINE      CODE     ---       #145
      01000DF9H   LINE      CODE     ---       #146
      01000DFBH   LINE      CODE     ---       #147
      01000E02H   LINE      CODE     ---       #148
      01000E06H   LINE      CODE     ---       #149
      01000E0AH   LINE      CODE     ---       #150
      01000E0EH   LINE      CODE     ---       #151
      01000E13H   LINE      CODE     ---       #152
      01000E17H   LINE      CODE     ---       #153
      01000E19H   LINE      CODE     ---       #154
      01000E1FH   LINE      CODE     ---       #155
      01000E1FH   LINE      CODE     ---       #158
      01000E39H   LINE      CODE     ---       #159
      01000E39H   LINE      CODE     ---       #161
      01000E42H   LINE      CODE     ---       #162
      01000E42H   LINE      CODE     ---       #163
      01000E48H   LINE      CODE     ---       #164
      01000E4FH   LINE      CODE     ---       #165
      01000E53H   LINE      CODE     ---       #166
      01000E56H   LINE      CODE     ---       #167
      01000E56H   LINE      CODE     ---       #168
      01000E58H   LINE      CODE     ---       #169
      01000E72H   LINE      CODE     ---       #170
      01000E72H   LINE      CODE     ---       #172
      01000E7BH   LINE      CODE     ---       #173
      01000E7BH   LINE      CODE     ---       #174
      01000E81H   LINE      CODE     ---       #175
      01000E88H   LINE      CODE     ---       #176
      01000E8CH   LINE      CODE     ---       #177
      01000E8FH   LINE      CODE     ---       #178
LX51 LINKER/LOCATER V4.66.1.0                                                         03/23/2017  15:15:44  PAGE 32


      01000E8FH   LINE      CODE     ---       #179
      01000E91H   LINE      CODE     ---       #180
      01000EABH   LINE      CODE     ---       #181
      01000EABH   LINE      CODE     ---       #183
      01000EB1H   LINE      CODE     ---       #184
      01000EB1H   LINE      CODE     ---       #185
      01000EB7H   LINE      CODE     ---       #186
      01000EBEH   LINE      CODE     ---       #187
      01000EC2H   LINE      CODE     ---       #188
      01000EC8H   LINE      CODE     ---       #189
      01000EC8H   LINE      CODE     ---       #190
      01000EC9H   LINE      CODE     ---       #192
      01000EC9H   LINE      CODE     ---       #193
      01000ECEH   LINE      CODE     ---       #194
      01000ECFH   LINE      CODE     ---       #195
      01000ED0H   LINE      CODE     ---       #196
      01000ED4H   LINE      CODE     ---       #197
      01000ED8H   LINE      CODE     ---       #198
      01000EDCH   LINE      CODE     ---       #199
      01000EE3H   LINE      CODE     ---       #200
      01000EE7H   LINE      CODE     ---       #201
      01000EEBH   LINE      CODE     ---       #202
      01000EEFH   LINE      CODE     ---       #203
      01000EF4H   LINE      CODE     ---       #204
      01000EF8H   LINE      CODE     ---       #205
      01000EFAH   LINE      CODE     ---       #207
      01000F00H   LINE      CODE     ---       #208
      01000F00H   LINE      CODE     ---       #209
      ---         BLOCKEND  ---      ---       LVL=0

      01001E65H   BLOCK     CODE     ---       LVL=0
      01001E65H   LINE      CODE     ---       #217
      01001E65H   LINE      CODE     ---       #218
      01001E65H   LINE      CODE     ---       #219
      01001E67H   LINE      CODE     ---       #220
      01001E71H   LINE      CODE     ---       #221
      01001E77H   LINE      CODE     ---       #222
      ---         BLOCKEND  ---      ---       LVL=0

      01001C76H   BLOCK     CODE     ---       LVL=0
      01001C76H   LINE      CODE     ---       #231
      01001C76H   LINE      CODE     ---       #232
      01001C76H   LINE      CODE     ---       #234
      01001C91H   LINE      CODE     ---       #235
      01001C91H   LINE      CODE     ---       #236
      01001C9BH   LINE      CODE     ---       #237
      01001CA0H   LINE      CODE     ---       #238
      01001CA0H   LINE      CODE     ---       #239
      ---         BLOCKEND  ---      ---       LVL=0

      01001CA1H   BLOCK     CODE     ---       LVL=0
      01001CA1H   LINE      CODE     ---       #248
      01001CA1H   LINE      CODE     ---       #249
      01001CA1H   LINE      CODE     ---       #250
      01001CBAH   LINE      CODE     ---       #251
      01001CBAH   LINE      CODE     ---       #252
      01001CBAH   LINE      CODE     ---       #253
      01001CBAH   LINE      CODE     ---       #254
      01001CBCH   LINE      CODE     ---       #255
      01001CBCH   LINE      CODE     ---       #256
      01001CBCH   LINE      CODE     ---       #257
      01001CBEH   LINE      CODE     ---       #258
      01001CBEH   LINE      CODE     ---       #259
      01001CBEH   LINE      CODE     ---       #260
      01001CC0H   LINE      CODE     ---       #261
LX51 LINKER/LOCATER V4.66.1.0                                                         03/23/2017  15:15:44  PAGE 33


      01001CC0H   LINE      CODE     ---       #262
      01001CC0H   LINE      CODE     ---       #263
      01001CC0H   LINE      CODE     ---       #264
      01001CC0H   LINE      CODE     ---       #265
      01001CC0H   LINE      CODE     ---       #266
      01001CC0H   LINE      CODE     ---       #267
      01001CC2H   LINE      CODE     ---       #268
      01001CC2H   LINE      CODE     ---       #269
      01001CC5H   LINE      CODE     ---       #270
      01001CC5H   LINE      CODE     ---       #271
      01001CC5H   LINE      CODE     ---       #274
      ---         BLOCKEND  ---      ---       LVL=0

      010011EAH   BLOCK     CODE     ---       LVL=0
      010011EAH   LINE      CODE     ---       #283
      010011EAH   LINE      CODE     ---       #284
      010011EAH   LINE      CODE     ---       #285
      010011EFH   LINE      CODE     ---       #286
      010011F1H   LINE      CODE     ---       #288
      010011F3H   LINE      CODE     ---       #289
      010011F5H   LINE      CODE     ---       #291
      010011F9H   LINE      CODE     ---       #292
      010011FDH   LINE      CODE     ---       #293
      01001201H   LINE      CODE     ---       #295
      01001207H   LINE      CODE     ---       #296
      0100120DH   LINE      CODE     ---       #297
      01001211H   LINE      CODE     ---       #298
      01001215H   LINE      CODE     ---       #299
      0100121BH   LINE      CODE     ---       #301
      01001221H   LINE      CODE     ---       #302
      01001225H   LINE      CODE     ---       #303
      01001229H   LINE      CODE     ---       #304
      0100122DH   LINE      CODE     ---       #305
      01001231H   LINE      CODE     ---       #307
      01001237H   LINE      CODE     ---       #308
      0100123BH   LINE      CODE     ---       #309
      0100123FH   LINE      CODE     ---       #310
      01001243H   LINE      CODE     ---       #311
      01001247H   LINE      CODE     ---       #313
      0100124BH   LINE      CODE     ---       #314
      0100124DH   LINE      CODE     ---       #315
      0100124FH   LINE      CODE     ---       #316
      01001251H   LINE      CODE     ---       #317
      01001253H   LINE      CODE     ---       #318
      01001255H   LINE      CODE     ---       #319
      01001257H   LINE      CODE     ---       #320
      01001259H   LINE      CODE     ---       #321
      01001261H   LINE      CODE     ---       #322
      0100126BH   LINE      CODE     ---       #323
      01001275H   LINE      CODE     ---       #324
      0100127FH   LINE      CODE     ---       #325
      01001289H   LINE      CODE     ---       #326
      01001293H   LINE      CODE     ---       #327
      0100129DH   LINE      CODE     ---       #328
      010012A7H   LINE      CODE     ---       #330
      010012ACH   LINE      CODE     ---       #331
      010012AEH   LINE      CODE     ---       #332
      010012B0H   LINE      CODE     ---       #333
      010012B2H   LINE      CODE     ---       #334
      010012B4H   LINE      CODE     ---       #335
      010012B6H   LINE      CODE     ---       #336
      010012B8H   LINE      CODE     ---       #337
      010012BAH   LINE      CODE     ---       #338
      010012C0H   LINE      CODE     ---       #339
      010012C4H   LINE      CODE     ---       #340
LX51 LINKER/LOCATER V4.66.1.0                                                         03/23/2017  15:15:44  PAGE 34


      010012C8H   LINE      CODE     ---       #342
      010012CEH   LINE      CODE     ---       #344
      ---         BLOCKEND  ---      ---       LVL=0

      01000571H   BLOCK     CODE     ---       LVL=0
      01000571H   LINE      CODE     ---       #357
      01000571H   LINE      CODE     ---       #358
      01000571H   LINE      CODE     ---       #360
      01000581H   LINE      CODE     ---       #361
      01000581H   LINE      CODE     ---       #362
      0100058FH   LINE      CODE     ---       #363
      010005A3H   LINE      CODE     ---       #364
      010005A3H   LINE      CODE     ---       #365
      010005A9H   LINE      CODE     ---       #366
      010005AFH   LINE      CODE     ---       #367
      010005B3H   LINE      CODE     ---       #368
      010005BAH   LINE      CODE     ---       #369
      010005BEH   LINE      CODE     ---       #370
      010005BEH   LINE      CODE     ---       #371
      010005C1H   LINE      CODE     ---       #372
      010005CAH   LINE      CODE     ---       #373
      010005CAH   LINE      CODE     ---       #374
      010005D8H   LINE      CODE     ---       #375
      010005ECH   LINE      CODE     ---       #376
      010005ECH   LINE      CODE     ---       #377
      010005F2H   LINE      CODE     ---       #378
      010005F8H   LINE      CODE     ---       #379
      010005FDH   LINE      CODE     ---       #380
      01000604H   LINE      CODE     ---       #381
      01000608H   LINE      CODE     ---       #382
      01000608H   LINE      CODE     ---       #383
      0100060BH   LINE      CODE     ---       #385
      0100060BH   LINE      CODE     ---       #386
      01000611H   LINE      CODE     ---       #387
      01000611H   LINE      CODE     ---       #388
      01000620H   LINE      CODE     ---       #389
      01000620H   LINE      CODE     ---       #390
      01000629H   LINE      CODE     ---       #391
      0100062FH   LINE      CODE     ---       #392
      01000633H   LINE      CODE     ---       #393
      01000635H   LINE      CODE     ---       #395
      01000635H   LINE      CODE     ---       #396
      01000643H   LINE      CODE     ---       #397
      0100064BH   LINE      CODE     ---       #398
      0100064BH   LINE      CODE     ---       #399
      0100064FH   LINE      CODE     ---       #400
      01000653H   LINE      CODE     ---       #401
      01000658H   LINE      CODE     ---       #402
      01000658H   LINE      CODE     ---       #403
      01000658H   LINE      CODE     ---       #404
      0100065AH   LINE      CODE     ---       #406
      0100065AH   LINE      CODE     ---       #407
      01000668H   LINE      CODE     ---       #408
      01000677H   LINE      CODE     ---       #409
      01000677H   LINE      CODE     ---       #410
      0100067BH   LINE      CODE     ---       #411
      0100067BH   LINE      CODE     ---       #412
      0100067BH   LINE      CODE     ---       #413
      01000681H   LINE      CODE     ---       #414
      01000681H   LINE      CODE     ---       #415
      01000690H   LINE      CODE     ---       #416
      01000690H   LINE      CODE     ---       #417
      01000699H   LINE      CODE     ---       #418
      0100069FH   LINE      CODE     ---       #419
      010006A4H   LINE      CODE     ---       #420
LX51 LINKER/LOCATER V4.66.1.0                                                         03/23/2017  15:15:44  PAGE 35


      010006A6H   LINE      CODE     ---       #422
      010006A6H   LINE      CODE     ---       #423
      010006B4H   LINE      CODE     ---       #424
      010006BCH   LINE      CODE     ---       #425
      010006BCH   LINE      CODE     ---       #426
      010006C0H   LINE      CODE     ---       #427
      010006C4H   LINE      CODE     ---       #428
      010006C9H   LINE      CODE     ---       #429
      010006C9H   LINE      CODE     ---       #430
      010006C9H   LINE      CODE     ---       #431
      010006CBH   LINE      CODE     ---       #433
      010006CBH   LINE      CODE     ---       #434
      010006D9H   LINE      CODE     ---       #435
      010006E1H   LINE      CODE     ---       #436
      010006E1H   LINE      CODE     ---       #437
      010006E5H   LINE      CODE     ---       #438
      010006E5H   LINE      CODE     ---       #439
      010006E5H   LINE      CODE     ---       #440
      010006E5H   LINE      CODE     ---       #443
      010006F5H   LINE      CODE     ---       #444
      010006F5H   LINE      CODE     ---       #445
      01000703H   LINE      CODE     ---       #446
      01000714H   LINE      CODE     ---       #447
      01000714H   LINE      CODE     ---       #448
      0100071AH   LINE      CODE     ---       #449
      01000720H   LINE      CODE     ---       #450
      01000726H   LINE      CODE     ---       #451
      01000726H   LINE      CODE     ---       #452
      01000728H   LINE      CODE     ---       #453
      01000731H   LINE      CODE     ---       #454
      01000731H   LINE      CODE     ---       #455
      01000737H   LINE      CODE     ---       #456
      01000737H   LINE      CODE     ---       #457
      01000745H   LINE      CODE     ---       #458
      0100074DH   LINE      CODE     ---       #459
      0100074DH   LINE      CODE     ---       #460
      01000751H   LINE      CODE     ---       #461
      01000755H   LINE      CODE     ---       #462
      0100075EH   LINE      CODE     ---       #463
      0100075EH   LINE      CODE     ---       #464
      01000768H   LINE      CODE     ---       #465
      0100076EH   LINE      CODE     ---       #466
      0100076EH   LINE      CODE     ---       #467
      0100076EH   LINE      CODE     ---       #468
      01000770H   LINE      CODE     ---       #470
      01000770H   LINE      CODE     ---       #471
      0100077EH   LINE      CODE     ---       #472
      01000786H   LINE      CODE     ---       #473
      01000786H   LINE      CODE     ---       #474
      0100078AH   LINE      CODE     ---       #475
      0100078AH   LINE      CODE     ---       #476
      0100078AH   LINE      CODE     ---       #477
      0100078AH   LINE      CODE     ---       #479
      010007A0H   LINE      CODE     ---       #483
      010007A0H   LINE      CODE     ---       #484
      010007A6H   LINE      CODE     ---       #485
      010007AAH   LINE      CODE     ---       #486
      010007ACH   LINE      CODE     ---       #488
      010007ACH   LINE      CODE     ---       #489
      010007B1H   LINE      CODE     ---       #490
      010007B1H   LINE      CODE     ---       #492
      ---         BLOCKEND  ---      ---       LVL=0

      01001741H   BLOCK     CODE     ---       LVL=0
      01001741H   LINE      CODE     ---       #500
LX51 LINKER/LOCATER V4.66.1.0                                                         03/23/2017  15:15:44  PAGE 36


      01001741H   LINE      CODE     ---       #501
      01001741H   LINE      CODE     ---       #502
      01001747H   LINE      CODE     ---       #503
      01001747H   LINE      CODE     ---       #505
      0100174EH   LINE      CODE     ---       #506
      0100174EH   LINE      CODE     ---       #507
      01001754H   LINE      CODE     ---       #508
      01001759H   LINE      CODE     ---       #509
      01001759H   LINE      CODE     ---       #511
      01001760H   LINE      CODE     ---       #512
      01001760H   LINE      CODE     ---       #513
      01001766H   LINE      CODE     ---       #514
      0100176BH   LINE      CODE     ---       #515
      0100176BH   LINE      CODE     ---       #517
      01001772H   LINE      CODE     ---       #518
      01001772H   LINE      CODE     ---       #519
      0100178DH   LINE      CODE     ---       #520
      0100178DH   LINE      CODE     ---       #521
      01001793H   LINE      CODE     ---       #522
      01001799H   LINE      CODE     ---       #523
      0100179EH   LINE      CODE     ---       #524
      0100179EH   LINE      CODE     ---       #525
      0100179EH   LINE      CODE     ---       #526
      0100179EH   LINE      CODE     ---       #528
      ---         BLOCKEND  ---      ---       LVL=0

      01000995H   BLOCK     CODE     ---       LVL=0
      01000995H   BLOCK     CODE     NEAR LAB  LVL=1
      02000003H   SYMBOL    XDATA    WORD      SpeedCtlCnt
      02000005H   SYMBOL    XDATA    WORD      ThetaCtlCnt
      02000007H   SYMBOL    XDATA    FLOAT     TempSlope
      0200000BH   SYMBOL    XDATA    FLOAT     TempVSConstant
      ---         BLOCKEND  ---      ---       LVL=1
      01000995H   LINE      CODE     ---       #543
      01000995H   LINE      CODE     ---       #544
      01000995H   LINE      CODE     ---       #550
      010009A3H   LINE      CODE     ---       #551
      010009B5H   LINE      CODE     ---       #552
      010009B5H   LINE      CODE     ---       #553
      010009B9H   LINE      CODE     ---       #555
      010009B9H   LINE      CODE     ---       #580
      010009B9H   LINE      CODE     ---       #582
      010009C7H   LINE      CODE     ---       #583
      010009C7H   LINE      CODE     ---       #584
      010009CDH   LINE      CODE     ---       #585
      010009CDH   LINE      CODE     ---       #588
      010009CDH   LINE      CODE     ---       #589
      010009CDH   LINE      CODE     ---       #590
      010009DDH   LINE      CODE     ---       #591
      010009DDH   LINE      CODE     ---       #592
      010009E7H   LINE      CODE     ---       #593
      010009E9H   LINE      CODE     ---       #594
      010009F2H   LINE      CODE     ---       #595
      010009F2H   LINE      CODE     ---       #596
      010009F8H   LINE      CODE     ---       #598
      010009FAH   LINE      CODE     ---       #600
      010009FAH   LINE      CODE     ---       #601
      01000A04H   LINE      CODE     ---       #602
      01000A04H   LINE      CODE     ---       #603
      01000A0AH   LINE      CODE     ---       #606
      01000A19H   LINE      CODE     ---       #607
      01000A19H   LINE      CODE     ---       #617
      01000A19H   LINE      CODE     ---       #618
      01000A19H   LINE      CODE     ---       #622
      01000A19H   LINE      CODE     ---       #623
LX51 LINKER/LOCATER V4.66.1.0                                                         03/23/2017  15:15:44  PAGE 37


      01000A19H   LINE      CODE     ---       #624
      01000A19H   LINE      CODE     ---       #625
      01000A19H   LINE      CODE     ---       #626
      01000A19H   LINE      CODE     ---       #635
      01000A19H   LINE      CODE     ---       #636
      01000A19H   LINE      CODE     ---       #658
      01000A19H   LINE      CODE     ---       #659
      01000A19H   LINE      CODE     ---       #660
      01000A19H   LINE      CODE     ---       #661
      01000A19H   LINE      CODE     ---       #662
      01000A19H   LINE      CODE     ---       #663
      01000A19H   LINE      CODE     ---       #664
      01000A19H   LINE      CODE     ---       #666
      01000A19H   LINE      CODE     ---       #667
      01000A19H   LINE      CODE     ---       #671
      01000A19H   LINE      CODE     ---       #672
      01000A19H   LINE      CODE     ---       #681
      01000A19H   LINE      CODE     ---       #689
      01000A19H   LINE      CODE     ---       #840
      01000A27H   LINE      CODE     ---       #841
      01000A39H   LINE      CODE     ---       #842
      01000A39H   LINE      CODE     ---       #843
      01000A3DH   LINE      CODE     ---       #844
      01000A57H   LINE      CODE     ---       #845
      01000A57H   LINE      CODE     ---       #846
      01000A65H   LINE      CODE     ---       #847
      01000A67H   LINE      CODE     ---       #848
      01000A75H   LINE      CODE     ---       #849
      01000A75H   LINE      CODE     ---       #850
      01000A83H   LINE      CODE     ---       #851
      01000A85H   LINE      CODE     ---       #853
      01000A85H   LINE      CODE     ---       #854
      01000A95H   LINE      CODE     ---       #855
      01000ABAH   LINE      CODE     ---       #856
      01000ABAH   LINE      CODE     ---       #857
      01000ABAH   LINE      CODE     ---       #859
      01000AC9H   LINE      CODE     ---       #860
      01000AC9H   LINE      CODE     ---       #861
      01000AD0H   LINE      CODE     ---       #862
      01000AD0H   LINE      CODE     ---       #864
      01000AE6H   LINE      CODE     ---       #865
      01000AE6H   LINE      CODE     ---       #866
      01000AF6H   LINE      CODE     ---       #867
      01000AF6H   LINE      CODE     ---       #868
      01000B01H   LINE      CODE     ---       #869
      01000B03H   LINE      CODE     ---       #871
      01000B03H   LINE      CODE     ---       #872
      01000B0DH   LINE      CODE     ---       #873
      01000B0DH   LINE      CODE     ---       #874
      01000B0DH   LINE      CODE     ---       #875
      01000B23H   LINE      CODE     ---       #876
      01000B23H   LINE      CODE     ---       #877
      01000B2BH   LINE      CODE     ---       #878
      01000B2BH   LINE      CODE     ---       #879
      01000B36H   LINE      CODE     ---       #880
      01000B37H   LINE      CODE     ---       #882
      01000B37H   LINE      CODE     ---       #883
      01000B40H   LINE      CODE     ---       #884
      01000B40H   LINE      CODE     ---       #885
      01000B40H   LINE      CODE     ---       #886
      01000B40H   LINE      CODE     ---       #888
      ---         BLOCKEND  ---      ---       LVL=0
      0200000FH   SYMBOL    XDATA    BYTE      CurrentCtlCnt

      010019B9H   BLOCK     CODE     ---       LVL=0
LX51 LINKER/LOCATER V4.66.1.0                                                         03/23/2017  15:15:44  PAGE 38


      010019B9H   BLOCK     CODE     NEAR LAB  LVL=1
      02000127H   SYMBOL    XDATA    WORD      MC_MotorONOFFDuty
      ---         BLOCKEND  ---      ---       LVL=1
      010019B9H   LINE      CODE     ---       #929
      010019B9H   LINE      CODE     ---       #930
      010019B9H   LINE      CODE     ---       #932
      010019B9H   LINE      CODE     ---       #933
      010019C0H   LINE      CODE     ---       #937
      010019D0H   LINE      CODE     ---       #938
      010019D0H   LINE      CODE     ---       #947
      010019D8H   LINE      CODE     ---       #948
      010019D8H   LINE      CODE     ---       #949
      010019DEH   LINE      CODE     ---       #950
      010019DEH   LINE      CODE     ---       #951
      010019E0H   LINE      CODE     ---       #952
      010019E0H   LINE      CODE     ---       #953
      010019E1H   LINE      CODE     ---       #954
      010019F0H   LINE      CODE     ---       #955
      010019F0H   LINE      CODE     ---       #956
      010019F6H   LINE      CODE     ---       #957
      010019F6H   LINE      CODE     ---       #958
      010019F8H   LINE      CODE     ---       #959
      010019F8H   LINE      CODE     ---       #960
      010019F8H   LINE      CODE     ---       #961
      010019F8H   LINE      CODE     ---       #981
      ---         BLOCKEND  ---      ---       LVL=0

      01001006H   BLOCK     CODE     ---       LVL=0
      01001006H   LINE      CODE     ---       #989
      01001006H   LINE      CODE     ---       #990
      01001006H   LINE      CODE     ---       #991
      0100100CH   LINE      CODE     ---       #992
      0100100CH   LINE      CODE     ---       #993
      0100102BH   LINE      CODE     ---       #994
      0100102BH   LINE      CODE     ---       #996
      01001032H   LINE      CODE     ---       #997
      01001032H   LINE      CODE     ---       #998
      01001051H   LINE      CODE     ---       #999
      01001051H   LINE      CODE     ---       #1001
      01001058H   LINE      CODE     ---       #1002
      01001058H   LINE      CODE     ---       #1003
      01001077H   LINE      CODE     ---       #1004
      01001077H   LINE      CODE     ---       #1006
      0100107EH   LINE      CODE     ---       #1007
      0100107EH   LINE      CODE     ---       #1008
      0100109DH   LINE      CODE     ---       #1009
      0100109DH   LINE      CODE     ---       #1011
      010010A4H   LINE      CODE     ---       #1012
      010010A4H   LINE      CODE     ---       #1013
      010010C3H   LINE      CODE     ---       #1015
      010010C3H   LINE      CODE     ---       #1017
      010010CAH   LINE      CODE     ---       #1018
      010010CAH   LINE      CODE     ---       #1019
      010010E9H   LINE      CODE     ---       #1020
      010010E9H   LINE      CODE     ---       #1022
      010010F0H   LINE      CODE     ---       #1023
      010010F0H   LINE      CODE     ---       #1024
      010010FEH   LINE      CODE     ---       #1025
      010010FEH   LINE      CODE     ---       #1026
      ---         BLOCKEND  ---      ---       LVL=0

      ---         MODULE    ---      ---       SPWM
      010007B2H   PUBLIC    CODE     ---       SPWM
      000000E2H   SFRSYM    DATA     BYTE      SV_USL
      000000ABH   SFRSYM    DATA     BYTE      TIM2_CNTRH
LX51 LINKER/LOCATER V4.66.1.0                                                         03/23/2017  15:15:44  PAGE 39


      000000B0H.4 SFRSYM    DATA     BIT       GP34
      000000A0H.5 SFRSYM    DATA     BIT       GP25
      00000090H.6 SFRSYM    DATA     BIT       GP16
      00000080H.7 SFRSYM    DATA     BIT       GP07
      00000088H.1 SFRSYM    DATA     BIT       IT01
      00000088H.3 SFRSYM    DATA     BIT       IT10
      000000F6H   SFRSYM    DATA     WORD      PI_UKMIN
      000000C2H   SFRSYM    DATA     WORD      MD_MA
      000000A3H   SFRSYM    DATA     BYTE      TIM3_CNTRH
      000000B0H.5 SFRSYM    DATA     BIT       GP35
      000000A0H.6 SFRSYM    DATA     BIT       GP26
      00000090H.7 SFRSYM    DATA     BIT       GP17
      00000080H   SFRSYM    DATA     BYTE      P0
      00000088H.4 SFRSYM    DATA     BIT       IT11
      000000CAH   SFRSYM    DATA     WORD      MD_MB
      00000093H   SFRSYM    DATA     BYTE      TIM4_CNTRH
      000000B0H.6 SFRSYM    DATA     BIT       GP36
      000000A0H.7 SFRSYM    DATA     BIT       GP27
      00000090H   SFRSYM    DATA     BYTE      P1
      000000D9H   SFRSYM    DATA     BYTE      EVT_FILT
      000000F4H   SFRSYM    DATA     WORD      PI_UKMAX
      0000008BH   SFRSYM    DATA     BYTE      TIM5_CNTRH
      000000B2H   SFRSYM    DATA     BYTE      TIM2_CMTRL
      000000B0H.7 SFRSYM    DATA     BIT       GP37
      000000A0H   SFRSYM    DATA     BYTE      P2
      000000AAH   SFRSYM    DATA     BYTE      TIM2_CNTRL
      000000B0H   SFRSYM    DATA     BYTE      P3
      000000A2H   SFRSYM    DATA     BYTE      TIM3_CNTRL
      000000D0H.6 SFRSYM    DATA     BIT       AC
      00000092H   SFRSYM    DATA     BYTE      TIM4_CNTRL
      0000008AH   SFRSYM    DATA     BYTE      TIM5_CNTRL
      000000B6H   SFRSYM    DATA     WORD      TIM0_CCR1
      000000A8H.7 SFRSYM    DATA     BIT       EA
      000000D5H   SFRSYM    DATA     BYTE      CMP_CR0
      000000BAH   SFRSYM    DATA     WORD      TIM0_CCR2
      000000D6H   SFRSYM    DATA     BYTE      CMP_CR1
      000000BCH   SFRSYM    DATA     WORD      TIM0_CCR3
      00000085H   SFRSYM    DATA     BYTE      PSCTL
      000000DAH   SFRSYM    DATA     BYTE      CMP_CR2
      000000BEH   SFRSYM    DATA     WORD      TIM0_CCR4
      000000B8H.2 SFRSYM    DATA     BIT       PX00
      000000EAH   SFRSYM    DATA     WORD      PI_EK
      000000F8H   SFRSYM    DATA     BIT       OISUH
      000000B8H.3 SFRSYM    DATA     BIT       PX01
      000000B8H.4 SFRSYM    DATA     BIT       PX10
      000000F8H.2 SFRSYM    DATA     BIT       OISVH
      000000B8H.5 SFRSYM    DATA     BIT       PX11
      000000F8H.4 SFRSYM    DATA     BIT       OISWH
      000000DCH   SFRSYM    DATA     WORD      LPF_K
      000000F2H   SFRSYM    DATA     WORD      PI_KI
      000000F8H.1 SFRSYM    DATA     BIT       OISUL
      000000A8H   SFRSYM    DATA     BYTE      IE
      000000F8H.3 SFRSYM    DATA     BIT       OISVL
      000000F8H.5 SFRSYM    DATA     BIT       OISWL
      000000D1H   SFRSYM    DATA     BYTE      P1IE
      00000098H.6 SFRSYM    DATA     BIT       MOD0
      000000D3H   SFRSYM    DATA     BYTE      P2IE
      000000D2H   SFRSYM    DATA     BYTE      P1IF
      000000F9H   SFRSYM    DATA     BYTE      PL_CR
      00000098H.7 SFRSYM    DATA     BIT       MOD1
      000000D4H   SFRSYM    DATA     BYTE      P2IF
      000000ACH   SFRSYM    DATA     WORD      TIM2_DR
      00000082H   SFRSYM    DATA     WORD      DP
      000000EEH   SFRSYM    DATA     WORD      PI_KP
      000000A4H   SFRSYM    DATA     WORD      TIM3_DR
LX51 LINKER/LOCATER V4.66.1.0                                                         03/23/2017  15:15:44  PAGE 40


      00000094H   SFRSYM    DATA     WORD      TIM4_DR
      0000008CH   SFRSYM    DATA     WORD      TIM5_DR
      000000F1H   SFRSYM    DATA     BYTE      OSC_CFG
      000000C1H   SFRSYM    DATA     BYTE      MD_MODE
      000000ECH   SFRSYM    DATA     WORD      PI_UK
      000000DEH   SFRSYM    DATA     WORD      LPF_X
      00000098H   SFRSYM    DATA     BIT       RI
      000000E6H   SFRSYM    DATA     WORD      LPF_Y
      000000C0H   SFRSYM    DATA     BIT       PTIM00
      000000D0H.7 SFRSYM    DATA     BIT       CY
      00000098H.1 SFRSYM    DATA     BIT       TI
      000000C0H.1 SFRSYM    DATA     BIT       PTIM01
      000000C0H.2 SFRSYM    DATA     BIT       PTIM10
      000000C0H.3 SFRSYM    DATA     BIT       PTIM11
      000000E1H   SFRSYM    DATA     BYTE      SV_CR
      00000098H   SFRSYM    DATA     BYTE      UT_CR
      00000099H   SFRSYM    DATA     BYTE      UT_DR
      000000F8H.6 SFRSYM    DATA     BIT       OIS4
      00000081H   SFRSYM    DATA     BYTE      SP
      000000D0H.2 SFRSYM    DATA     BIT       OV
      000000C4H   SFRSYM    DATA     BYTE      MD_DA0
      0000009AH   SFRSYM    DATA     WORD      UT_BAUD
      000000CCH   SFRSYM    DATA     BYTE      MD_DB0
      000000C5H   SFRSYM    DATA     BYTE      MD_DA1
      000000CDH   SFRSYM    DATA     BYTE      MD_DB1
      000000C6H   SFRSYM    DATA     BYTE      MD_DA2
      000000CEH   SFRSYM    DATA     BYTE      MD_DB2
      000000C7H   SFRSYM    DATA     BYTE      MD_DA3
      000000B4H   SFRSYM    DATA     WORD      TIM2_ADTR
      000000CFH   SFRSYM    DATA     BYTE      MD_DB3
      000000AFH   SFRSYM    DATA     BYTE      TIM2_ARRH
      000000A7H   SFRSYM    DATA     BYTE      TIM3_ARRH
      00000097H   SFRSYM    DATA     BYTE      TIM4_ARRH
      0000008FH   SFRSYM    DATA     BYTE      TIM5_ARRH
      000000AEH   SFRSYM    DATA     BYTE      TIM2_ARRL
      000000A6H   SFRSYM    DATA     BYTE      TIM3_ARRL
      00000087H   SFRSYM    DATA     BYTE      PCON
      000000E2H   SFRSYM    DATA     WORD      SV_US
      00000096H   SFRSYM    DATA     BYTE      TIM4_ARRL
      0000008EH   SFRSYM    DATA     BYTE      TIM5_ARRL
      000000B2H   SFRSYM    DATA     WORD      TIM2_CMTR
      00000088H   SFRSYM    DATA     BYTE      TCON
      000000AAH   SFRSYM    DATA     WORD      TIM2_CNTR
      000000A2H   SFRSYM    DATA     WORD      TIM3_CNTR
      00000092H   SFRSYM    DATA     WORD      TIM4_CNTR
      0000008AH   SFRSYM    DATA     WORD      TIM5_CNTR
      000000E5H   SFRSYM    DATA     BYTE      SV_ANGLEH
      000000D8H   SFRSYM    DATA     BIT       PUART0
      000000E4H   SFRSYM    DATA     BYTE      SV_ANGLEL
      000000C6H   SFRSYM    DATA     WORD      MD_DAH
      000000D8H.1 SFRSYM    DATA     BIT       PUART1
      000000D8H.2 SFRSYM    DATA     BIT       PI2C0
      00000088H.2 SFRSYM    DATA     BIT       IF0
      000000CEH   SFRSYM    DATA     WORD      MD_DBH
      000000D8H.3 SFRSYM    DATA     BIT       PI2C1
      000000F0H   SFRSYM    DATA     BYTE      B
      000000C4H   SFRSYM    DATA     WORD      MD_DAL
      000000A1H   SFRSYM    DATA     BYTE      TIM2_CR0
      000000CCH   SFRSYM    DATA     WORD      MD_DBL
      0000009CH   SFRSYM    DATA     BYTE      TIM3_CR0
      000000A9H   SFRSYM    DATA     BYTE      TIM2_CR1
      0000009EH   SFRSYM    DATA     BYTE      TIM4_CR0
      0000009DH   SFRSYM    DATA     BYTE      TIM3_CR1
      00000089H   SFRSYM    DATA     BYTE      TIM5_CR0
      0000009FH   SFRSYM    DATA     BYTE      TIM4_CR1
LX51 LINKER/LOCATER V4.66.1.0                                                         03/23/2017  15:15:44  PAGE 41


      000000F8H   SFRSYM    DATA     BYTE      DRV_OUT
      00000091H   SFRSYM    DATA     BYTE      TIM5_CR1
      000000E0H   SFRSYM    DATA     BYTE      ACC
      000000F7H   SFRSYM    DATA     BYTE      PI_UKMINH
      000000C3H   SFRSYM    DATA     BYTE      MD_MAH
      000000A8H.4 SFRSYM    DATA     BIT       ES0
      000000DBH   SFRSYM    DATA     BYTE      LVSR
      000000CBH   SFRSYM    DATA     BYTE      MD_MBH
      000000C0H.4 SFRSYM    DATA     BIT       PADC0
      000000B8H   SFRSYM    DATA     BYTE      IP0
      000000F5H   SFRSYM    DATA     BYTE      PI_UKMAXH
      000000C0H.5 SFRSYM    DATA     BIT       PADC1
      000000C0H   SFRSYM    DATA     BYTE      IP1
      000000C8H   SFRSYM    DATA     BYTE      IP2
      000000F6H   SFRSYM    DATA     BYTE      PI_UKMINL
      000000C2H   SFRSYM    DATA     BYTE      MD_MAL
      00000098H.2 SFRSYM    DATA     BIT       RB8
      000000D8H   SFRSYM    DATA     BYTE      IP3
      000000CAH   SFRSYM    DATA     BYTE      MD_MBL
      000000A8H   SFRSYM    DATA     BIT       EX0
      000000F4H   SFRSYM    DATA     BYTE      PI_UKMAXL
      00000098H.3 SFRSYM    DATA     BIT       TB8
      000000B7H   SFRSYM    DATA     BYTE      TIM0_CCR1H
      000000A8H.2 SFRSYM    DATA     BIT       EX1
      000000BBH   SFRSYM    DATA     BYTE      TIM0_CCR2H
      000000D0H   SFRSYM    DATA     BIT       P
      000000BDH   SFRSYM    DATA     BYTE      TIM0_CCR3H
      000000BFH   SFRSYM    DATA     BYTE      TIM0_CCR4H
      000000C8H.2 SFRSYM    DATA     BIT       PTIM230
      000000EBH   SFRSYM    DATA     BYTE      PI_EKH
      00000098H.5 SFRSYM    DATA     BIT       SM2
      000000B6H   SFRSYM    DATA     BYTE      TIM0_CCR1L
      000000B1H   SFRSYM    DATA     BYTE      TIM0_SR1
      000000C8H.3 SFRSYM    DATA     BIT       PTIM231
      000000BAH   SFRSYM    DATA     BYTE      TIM0_CCR2L
      000000BCH   SFRSYM    DATA     BYTE      TIM0_CCR3L
      000000BEH   SFRSYM    DATA     BYTE      TIM0_CCR4L
      000000D8H.6 SFRSYM    DATA     BIT       PMCD0
      000000C8H.4 SFRSYM    DATA     BIT       PTIM450
      000000D0H.3 SFRSYM    DATA     BIT       RS0
      000000DDH   SFRSYM    DATA     BYTE      LPF_KH
      000000F3H   SFRSYM    DATA     BYTE      PI_KIH
      000000EAH   SFRSYM    DATA     BYTE      PI_EKL
      000000E8H   SFRSYM    DATA     BYTE      FOC_SET0
      000000D8H.7 SFRSYM    DATA     BIT       PMCD1
      000000C8H.5 SFRSYM    DATA     BIT       PTIM451
      000000D0H.4 SFRSYM    DATA     BIT       RS1
      000000E9H   SFRSYM    DATA     BYTE      FOC_SET1
      000000B8H.6 SFRSYM    DATA     BIT       PFOC0
      000000DCH   SFRSYM    DATA     BYTE      LPF_KL
      000000F2H   SFRSYM    DATA     BYTE      PI_KIL
      000000B8H.7 SFRSYM    DATA     BIT       PFOC1
      000000ADH   SFRSYM    DATA     BYTE      TIM2_DRH
      000000B9H   SFRSYM    DATA     BYTE      TIM0_IER
      00000083H   SFRSYM    DATA     BYTE      DPH
      000000EFH   SFRSYM    DATA     BYTE      PI_KPH
      000000A5H   SFRSYM    DATA     BYTE      TIM3_DRH
      00000095H   SFRSYM    DATA     BYTE      TIM4_DRH
      0000008DH   SFRSYM    DATA     BYTE      TIM5_DRH
      000000ACH   SFRSYM    DATA     BYTE      TIM2_DRL
      00000082H   SFRSYM    DATA     BYTE      DPL
      000000EEH   SFRSYM    DATA     BYTE      PI_KPL
      000000A4H   SFRSYM    DATA     BYTE      TIM3_DRL
      000000F8H.7 SFRSYM    DATA     BIT       MOE
      000000C0H.6 SFRSYM    DATA     BIT       PCMP0
LX51 LINKER/LOCATER V4.66.1.0                                                         03/23/2017  15:15:44  PAGE 42


      000000EDH   SFRSYM    DATA     BYTE      PI_UKH
      00000094H   SFRSYM    DATA     BYTE      TIM4_DRL
      000000C0H.7 SFRSYM    DATA     BIT       PCMP1
      000000DFH   SFRSYM    DATA     BYTE      LPF_XH
      0000008CH   SFRSYM    DATA     BYTE      TIM5_DRL
      000000AEH   SFRSYM    DATA     WORD      TIM2_ARR
      000000A8H.5 SFRSYM    DATA     BIT       MCDIE
      000000C9H   SFRSYM    DATA     BYTE      RSTSRC
      000000E7H   SFRSYM    DATA     BYTE      LPF_YH
      000000A6H   SFRSYM    DATA     WORD      TIM3_ARR
      00000088H.6 SFRSYM    DATA     BIT       MCDIF
      00000098H.4 SFRSYM    DATA     BIT       REN
      00000096H   SFRSYM    DATA     WORD      TIM4_ARR
      000000ECH   SFRSYM    DATA     BYTE      PI_UKL
      000000D7H   SFRSYM    DATA     BYTE      CMP_SR
      0000008EH   SFRSYM    DATA     WORD      TIM5_ARR
      000000DEH   SFRSYM    DATA     BYTE      LPF_XL
      000000E6H   SFRSYM    DATA     BYTE      LPF_YL
      000000C8H   SFRSYM    DATA     BIT       PRTC0
      000000C8H.1 SFRSYM    DATA     BIT       PRTC1
      000000E8H.7 SFRSYM    DATA     BIT       FOCEN
      000000C8H.6 SFRSYM    DATA     BIT       PTSD0
      000000D8H.4 SFRSYM    DATA     BIT       PSPI0
      000000C8H.7 SFRSYM    DATA     BIT       PTSD1
      000000D8H.5 SFRSYM    DATA     BIT       PSPI1
      0000009BH   SFRSYM    DATA     BYTE      UT_BAUDH
      000000E4H   SFRSYM    DATA     WORD      SV_ANGLE
      000000B5H   SFRSYM    DATA     BYTE      TIM2_ADTRH
      0000009AH   SFRSYM    DATA     BYTE      UT_BAUDL
      000000FCH   SFRSYM    DATA     BYTE      P0_OE
      000000FDH   SFRSYM    DATA     BYTE      P1_OE
      000000D0H.5 SFRSYM    DATA     BIT       F0
      000000B4H   SFRSYM    DATA     BYTE      TIM2_ADTRL
      000000FEH   SFRSYM    DATA     BYTE      P2_OE
      000000D0H.1 SFRSYM    DATA     BIT       F1
      00000080H   SFRSYM    DATA     BIT       GP00
      000000FFH   SFRSYM    DATA     BYTE      P3_OE
      00000090H   SFRSYM    DATA     BIT       GP10
      00000080H.1 SFRSYM    DATA     BIT       GP01
      000000A8H.6 SFRSYM    DATA     BIT       RTCIE
      000000A0H   SFRSYM    DATA     BIT       GP20
      00000090H.1 SFRSYM    DATA     BIT       GP11
      00000080H.2 SFRSYM    DATA     BIT       GP02
      000000E3H   SFRSYM    DATA     BYTE      SV_USH
      000000B0H   SFRSYM    DATA     BIT       GP30
      000000A0H.1 SFRSYM    DATA     BIT       GP21
      00000090H.2 SFRSYM    DATA     BIT       GP12
      00000080H.3 SFRSYM    DATA     BIT       GP03
      000000B8H   SFRSYM    DATA     BIT       PLVW0
      000000A8H.1 SFRSYM    DATA     BIT       TSDIE
      000000D0H   SFRSYM    DATA     BYTE      PSW
      000000B0H.1 SFRSYM    DATA     BIT       GP31
      000000A0H.2 SFRSYM    DATA     BIT       GP22
      00000090H.3 SFRSYM    DATA     BIT       GP13
      00000080H.4 SFRSYM    DATA     BIT       GP04
      000000B8H.1 SFRSYM    DATA     BIT       PLVW1
      000000A8H.3 SFRSYM    DATA     BIT       SPIIE
      00000088H.5 SFRSYM    DATA     BIT       TSDIF
      000000B0H.2 SFRSYM    DATA     BIT       GP32
      000000A0H.3 SFRSYM    DATA     BIT       GP23
      00000090H.4 SFRSYM    DATA     BIT       GP14
      00000080H.5 SFRSYM    DATA     BIT       GP05
      00000084H   SFRSYM    DATA     BYTE      FLKEY
      000000B3H   SFRSYM    DATA     BYTE      TIM2_CMTRH
      000000B0H.3 SFRSYM    DATA     BIT       GP33
LX51 LINKER/LOCATER V4.66.1.0                                                         03/23/2017  15:15:44  PAGE 43


      000000A0H.4 SFRSYM    DATA     BIT       GP24
      00000090H.5 SFRSYM    DATA     BIT       GP15
      00000080H.6 SFRSYM    DATA     BIT       GP06
      00000088H   SFRSYM    DATA     BIT       IT00

      010007B2H   BLOCK     CODE     ---       LVL=0
      010007B2H   BLOCK     CODE     NEAR LAB  LVL=1
      02000115H   SYMBOL    XDATA    INT       PWMDuty1
      02000117H   SYMBOL    XDATA    INT       PWMDuty2
      02000119H   SYMBOL    XDATA    INT       SinTheta
      0200011BH   SYMBOL    XDATA    INT       CosTheta
      0200011DH   SYMBOL    XDATA    INT       Temp16
      0200011FH   SYMBOL    XDATA    INT       Temp16_1
      02000121H   SYMBOL    XDATA    INT       Temp16_1_VS
      02000123H   SYMBOL    XDATA    FLOAT     PWMDuty2_PWMRR
      ---         BLOCKEND  ---      ---       LVL=1
      010007B2H   LINE      CODE     ---       #27
      010007B2H   LINE      CODE     ---       #28
      010007B2H   LINE      CODE     ---       #38
      010007C6H   LINE      CODE     ---       #39
      010007D3H   LINE      CODE     ---       #40
      010007D3H   LINE      CODE     ---       #41
      010007DFH   LINE      CODE     ---       #42
      010007DFH   LINE      CODE     ---       #44
      010007EAH   LINE      CODE     ---       #45
      010007F9H   LINE      CODE     ---       #46
      01000808H   LINE      CODE     ---       #58
      01000818H   LINE      CODE     ---       #59
      01000818H   LINE      CODE     ---       #60
      01000822H   LINE      CODE     ---       #61
      01000824H   LINE      CODE     ---       #62
      0100082DH   LINE      CODE     ---       #63
      0100082DH   LINE      CODE     ---       #64
      01000837H   LINE      CODE     ---       #65
      01000839H   LINE      CODE     ---       #66
      0100084BH   LINE      CODE     ---       #67
      0100084BH   LINE      CODE     ---       #68
      01000852H   LINE      CODE     ---       #69
      01000854H   LINE      CODE     ---       #71
      01000854H   LINE      CODE     ---       #72
      0100085BH   LINE      CODE     ---       #73
      0100085BH   LINE      CODE     ---       #75
      01000874H   LINE      CODE     ---       #76
      0100089EH   LINE      CODE     ---       #79
      010008BBH   LINE      CODE     ---       #80
      010008D8H   LINE      CODE     ---       #82
      010008F7H   LINE      CODE     ---       #83
      010008FFH   LINE      CODE     ---       #84
      010008FFH   LINE      CODE     ---       #85
      01000906H   LINE      CODE     ---       #86
      01000906H   LINE      CODE     ---       #88
      01000921H   LINE      CODE     ---       #89
      01000921H   LINE      CODE     ---       #90
      0100092BH   LINE      CODE     ---       #91
      0100092BH   LINE      CODE     ---       #93
      0100094AH   LINE      CODE     ---       #94
      01000952H   LINE      CODE     ---       #95
      01000952H   LINE      CODE     ---       #96
      01000959H   LINE      CODE     ---       #97
      01000959H   LINE      CODE     ---       #98
      01000974H   LINE      CODE     ---       #99
      01000974H   LINE      CODE     ---       #100
      0100097EH   LINE      CODE     ---       #101
      0100097EH   LINE      CODE     ---       #103
      0100098AH   LINE      CODE     ---       #104
LX51 LINKER/LOCATER V4.66.1.0                                                         03/23/2017  15:15:44  PAGE 44


      01000994H   LINE      CODE     ---       #105
      ---         BLOCKEND  ---      ---       LVL=0

      ---         MODULE    ---      ---       SINCOS
      020000FBH   PUBLIC    XDATA    ---       TanAngle
      01001E1FH   PUBLIC    CODE     ---       _SinCos
      01001E78H   PUBLIC    CODE     ---       SinCosInit
      000000E2H   SFRSYM    DATA     BYTE      SV_USL
      000000ABH   SFRSYM    DATA     BYTE      TIM2_CNTRH
      000000B0H.4 SFRSYM    DATA     BIT       GP34
      000000A0H.5 SFRSYM    DATA     BIT       GP25
      00000090H.6 SFRSYM    DATA     BIT       GP16
      00000080H.7 SFRSYM    DATA     BIT       GP07
      00000088H.1 SFRSYM    DATA     BIT       IT01
      00000088H.3 SFRSYM    DATA     BIT       IT10
      000000F6H   SFRSYM    DATA     WORD      PI_UKMIN
      000000C2H   SFRSYM    DATA     WORD      MD_MA
      000000A3H   SFRSYM    DATA     BYTE      TIM3_CNTRH
      000000B0H.5 SFRSYM    DATA     BIT       GP35
      000000A0H.6 SFRSYM    DATA     BIT       GP26
      00000090H.7 SFRSYM    DATA     BIT       GP17
      00000080H   SFRSYM    DATA     BYTE      P0
      00000088H.4 SFRSYM    DATA     BIT       IT11
      000000CAH   SFRSYM    DATA     WORD      MD_MB
      00000093H   SFRSYM    DATA     BYTE      TIM4_CNTRH
      000000B0H.6 SFRSYM    DATA     BIT       GP36
      000000A0H.7 SFRSYM    DATA     BIT       GP27
      00000090H   SFRSYM    DATA     BYTE      P1
      000000D9H   SFRSYM    DATA     BYTE      EVT_FILT
      000000F4H   SFRSYM    DATA     WORD      PI_UKMAX
      0000008BH   SFRSYM    DATA     BYTE      TIM5_CNTRH
      000000B2H   SFRSYM    DATA     BYTE      TIM2_CMTRL
      000000B0H.7 SFRSYM    DATA     BIT       GP37
      000000A0H   SFRSYM    DATA     BYTE      P2
      000000AAH   SFRSYM    DATA     BYTE      TIM2_CNTRL
      000000B0H   SFRSYM    DATA     BYTE      P3
      000000A2H   SFRSYM    DATA     BYTE      TIM3_CNTRL
      000000D0H.6 SFRSYM    DATA     BIT       AC
      00000092H   SFRSYM    DATA     BYTE      TIM4_CNTRL
      0000008AH   SFRSYM    DATA     BYTE      TIM5_CNTRL
      000000B6H   SFRSYM    DATA     WORD      TIM0_CCR1
      000000A8H.7 SFRSYM    DATA     BIT       EA
      000000D5H   SFRSYM    DATA     BYTE      CMP_CR0
      000000BAH   SFRSYM    DATA     WORD      TIM0_CCR2
      000000D6H   SFRSYM    DATA     BYTE      CMP_CR1
      000000BCH   SFRSYM    DATA     WORD      TIM0_CCR3
      00000085H   SFRSYM    DATA     BYTE      PSCTL
      000000DAH   SFRSYM    DATA     BYTE      CMP_CR2
      000000BEH   SFRSYM    DATA     WORD      TIM0_CCR4
      000000B8H.2 SFRSYM    DATA     BIT       PX00
      000000EAH   SFRSYM    DATA     WORD      PI_EK
      000000F8H   SFRSYM    DATA     BIT       OISUH
      000000B8H.3 SFRSYM    DATA     BIT       PX01
      000000B8H.4 SFRSYM    DATA     BIT       PX10
      000000F8H.2 SFRSYM    DATA     BIT       OISVH
      000000B8H.5 SFRSYM    DATA     BIT       PX11
      000000F8H.4 SFRSYM    DATA     BIT       OISWH
      000000DCH   SFRSYM    DATA     WORD      LPF_K
      000000F2H   SFRSYM    DATA     WORD      PI_KI
      000000F8H.1 SFRSYM    DATA     BIT       OISUL
      000000A8H   SFRSYM    DATA     BYTE      IE
      000000F8H.3 SFRSYM    DATA     BIT       OISVL
      000000F8H.5 SFRSYM    DATA     BIT       OISWL
      000000D1H   SFRSYM    DATA     BYTE      P1IE
      00000098H.6 SFRSYM    DATA     BIT       MOD0
LX51 LINKER/LOCATER V4.66.1.0                                                         03/23/2017  15:15:44  PAGE 45


      000000D3H   SFRSYM    DATA     BYTE      P2IE
      000000D2H   SFRSYM    DATA     BYTE      P1IF
      000000F9H   SFRSYM    DATA     BYTE      PL_CR
      00000098H.7 SFRSYM    DATA     BIT       MOD1
      000000D4H   SFRSYM    DATA     BYTE      P2IF
      000000ACH   SFRSYM    DATA     WORD      TIM2_DR
      00000082H   SFRSYM    DATA     WORD      DP
      000000EEH   SFRSYM    DATA     WORD      PI_KP
      000000A4H   SFRSYM    DATA     WORD      TIM3_DR
      00000094H   SFRSYM    DATA     WORD      TIM4_DR
      0000008CH   SFRSYM    DATA     WORD      TIM5_DR
      000000F1H   SFRSYM    DATA     BYTE      OSC_CFG
      000000C1H   SFRSYM    DATA     BYTE      MD_MODE
      000000ECH   SFRSYM    DATA     WORD      PI_UK
      000000DEH   SFRSYM    DATA     WORD      LPF_X
      00000098H   SFRSYM    DATA     BIT       RI
      000000E6H   SFRSYM    DATA     WORD      LPF_Y
      000000C0H   SFRSYM    DATA     BIT       PTIM00
      000000D0H.7 SFRSYM    DATA     BIT       CY
      00000098H.1 SFRSYM    DATA     BIT       TI
      000000C0H.1 SFRSYM    DATA     BIT       PTIM01
      000000C0H.2 SFRSYM    DATA     BIT       PTIM10
      000000C0H.3 SFRSYM    DATA     BIT       PTIM11
      000000E1H   SFRSYM    DATA     BYTE      SV_CR
      00000098H   SFRSYM    DATA     BYTE      UT_CR
      00000099H   SFRSYM    DATA     BYTE      UT_DR
      000000F8H.6 SFRSYM    DATA     BIT       OIS4
      00000081H   SFRSYM    DATA     BYTE      SP
      000000D0H.2 SFRSYM    DATA     BIT       OV
      000000C4H   SFRSYM    DATA     BYTE      MD_DA0
      0000009AH   SFRSYM    DATA     WORD      UT_BAUD
      000000CCH   SFRSYM    DATA     BYTE      MD_DB0
      000000C5H   SFRSYM    DATA     BYTE      MD_DA1
      000000CDH   SFRSYM    DATA     BYTE      MD_DB1
      000000C6H   SFRSYM    DATA     BYTE      MD_DA2
      000000CEH   SFRSYM    DATA     BYTE      MD_DB2
      000000C7H   SFRSYM    DATA     BYTE      MD_DA3
      000000B4H   SFRSYM    DATA     WORD      TIM2_ADTR
      000000CFH   SFRSYM    DATA     BYTE      MD_DB3
      000000AFH   SFRSYM    DATA     BYTE      TIM2_ARRH
      000000A7H   SFRSYM    DATA     BYTE      TIM3_ARRH
      00000097H   SFRSYM    DATA     BYTE      TIM4_ARRH
      0000008FH   SFRSYM    DATA     BYTE      TIM5_ARRH
      000000AEH   SFRSYM    DATA     BYTE      TIM2_ARRL
      000000A6H   SFRSYM    DATA     BYTE      TIM3_ARRL
      00000087H   SFRSYM    DATA     BYTE      PCON
      000000E2H   SFRSYM    DATA     WORD      SV_US
      00000096H   SFRSYM    DATA     BYTE      TIM4_ARRL
      0000008EH   SFRSYM    DATA     BYTE      TIM5_ARRL
      000000B2H   SFRSYM    DATA     WORD      TIM2_CMTR
      00000088H   SFRSYM    DATA     BYTE      TCON
      000000AAH   SFRSYM    DATA     WORD      TIM2_CNTR
      000000A2H   SFRSYM    DATA     WORD      TIM3_CNTR
      00000092H   SFRSYM    DATA     WORD      TIM4_CNTR
      0000008AH   SFRSYM    DATA     WORD      TIM5_CNTR
      000000E5H   SFRSYM    DATA     BYTE      SV_ANGLEH
      000000D8H   SFRSYM    DATA     BIT       PUART0
      000000E4H   SFRSYM    DATA     BYTE      SV_ANGLEL
      000000C6H   SFRSYM    DATA     WORD      MD_DAH
      000000D8H.1 SFRSYM    DATA     BIT       PUART1
      000000D8H.2 SFRSYM    DATA     BIT       PI2C0
      00000088H.2 SFRSYM    DATA     BIT       IF0
      000000CEH   SFRSYM    DATA     WORD      MD_DBH
      000000D8H.3 SFRSYM    DATA     BIT       PI2C1
      000000F0H   SFRSYM    DATA     BYTE      B
LX51 LINKER/LOCATER V4.66.1.0                                                         03/23/2017  15:15:44  PAGE 46


      000000C4H   SFRSYM    DATA     WORD      MD_DAL
      000000A1H   SFRSYM    DATA     BYTE      TIM2_CR0
      000000CCH   SFRSYM    DATA     WORD      MD_DBL
      0000009CH   SFRSYM    DATA     BYTE      TIM3_CR0
      000000A9H   SFRSYM    DATA     BYTE      TIM2_CR1
      0000009EH   SFRSYM    DATA     BYTE      TIM4_CR0
      0000009DH   SFRSYM    DATA     BYTE      TIM3_CR1
      00000089H   SFRSYM    DATA     BYTE      TIM5_CR0
      0000009FH   SFRSYM    DATA     BYTE      TIM4_CR1
      000000F8H   SFRSYM    DATA     BYTE      DRV_OUT
      00000091H   SFRSYM    DATA     BYTE      TIM5_CR1
      000000E0H   SFRSYM    DATA     BYTE      ACC
      000000F7H   SFRSYM    DATA     BYTE      PI_UKMINH
      000000C3H   SFRSYM    DATA     BYTE      MD_MAH
      000000A8H.4 SFRSYM    DATA     BIT       ES0
      000000DBH   SFRSYM    DATA     BYTE      LVSR
      000000CBH   SFRSYM    DATA     BYTE      MD_MBH
      000000C0H.4 SFRSYM    DATA     BIT       PADC0
      000000B8H   SFRSYM    DATA     BYTE      IP0
      000000F5H   SFRSYM    DATA     BYTE      PI_UKMAXH
      000000C0H.5 SFRSYM    DATA     BIT       PADC1
      000000C0H   SFRSYM    DATA     BYTE      IP1
      000000C8H   SFRSYM    DATA     BYTE      IP2
      000000F6H   SFRSYM    DATA     BYTE      PI_UKMINL
      000000C2H   SFRSYM    DATA     BYTE      MD_MAL
      00000098H.2 SFRSYM    DATA     BIT       RB8
      000000D8H   SFRSYM    DATA     BYTE      IP3
      000000CAH   SFRSYM    DATA     BYTE      MD_MBL
      000000A8H   SFRSYM    DATA     BIT       EX0
      000000F4H   SFRSYM    DATA     BYTE      PI_UKMAXL
      00000098H.3 SFRSYM    DATA     BIT       TB8
      000000B7H   SFRSYM    DATA     BYTE      TIM0_CCR1H
      000000A8H.2 SFRSYM    DATA     BIT       EX1
      000000BBH   SFRSYM    DATA     BYTE      TIM0_CCR2H
      000000D0H   SFRSYM    DATA     BIT       P
      000000BDH   SFRSYM    DATA     BYTE      TIM0_CCR3H
      000000BFH   SFRSYM    DATA     BYTE      TIM0_CCR4H
      000000C8H.2 SFRSYM    DATA     BIT       PTIM230
      000000EBH   SFRSYM    DATA     BYTE      PI_EKH
      00000098H.5 SFRSYM    DATA     BIT       SM2
      000000B6H   SFRSYM    DATA     BYTE      TIM0_CCR1L
      000000B1H   SFRSYM    DATA     BYTE      TIM0_SR1
      000000C8H.3 SFRSYM    DATA     BIT       PTIM231
      000000BAH   SFRSYM    DATA     BYTE      TIM0_CCR2L
      000000BCH   SFRSYM    DATA     BYTE      TIM0_CCR3L
      000000BEH   SFRSYM    DATA     BYTE      TIM0_CCR4L
      000000D8H.6 SFRSYM    DATA     BIT       PMCD0
      000000C8H.4 SFRSYM    DATA     BIT       PTIM450
      000000D0H.3 SFRSYM    DATA     BIT       RS0
      000000DDH   SFRSYM    DATA     BYTE      LPF_KH
      000000F3H   SFRSYM    DATA     BYTE      PI_KIH
      000000EAH   SFRSYM    DATA     BYTE      PI_EKL
      000000E8H   SFRSYM    DATA     BYTE      FOC_SET0
      000000D8H.7 SFRSYM    DATA     BIT       PMCD1
      000000C8H.5 SFRSYM    DATA     BIT       PTIM451
      000000D0H.4 SFRSYM    DATA     BIT       RS1
      000000E9H   SFRSYM    DATA     BYTE      FOC_SET1
      000000B8H.6 SFRSYM    DATA     BIT       PFOC0
      000000DCH   SFRSYM    DATA     BYTE      LPF_KL
      000000F2H   SFRSYM    DATA     BYTE      PI_KIL
      000000B8H.7 SFRSYM    DATA     BIT       PFOC1
      000000ADH   SFRSYM    DATA     BYTE      TIM2_DRH
      000000B9H   SFRSYM    DATA     BYTE      TIM0_IER
      00000083H   SFRSYM    DATA     BYTE      DPH
      000000EFH   SFRSYM    DATA     BYTE      PI_KPH
LX51 LINKER/LOCATER V4.66.1.0                                                         03/23/2017  15:15:44  PAGE 47


      000000A5H   SFRSYM    DATA     BYTE      TIM3_DRH
      00000095H   SFRSYM    DATA     BYTE      TIM4_DRH
      0000008DH   SFRSYM    DATA     BYTE      TIM5_DRH
      000000ACH   SFRSYM    DATA     BYTE      TIM2_DRL
      00000082H   SFRSYM    DATA     BYTE      DPL
      000000EEH   SFRSYM    DATA     BYTE      PI_KPL
      000000A4H   SFRSYM    DATA     BYTE      TIM3_DRL
      000000F8H.7 SFRSYM    DATA     BIT       MOE
      000000C0H.6 SFRSYM    DATA     BIT       PCMP0
      000000EDH   SFRSYM    DATA     BYTE      PI_UKH
      00000094H   SFRSYM    DATA     BYTE      TIM4_DRL
      000000C0H.7 SFRSYM    DATA     BIT       PCMP1
      000000DFH   SFRSYM    DATA     BYTE      LPF_XH
      0000008CH   SFRSYM    DATA     BYTE      TIM5_DRL
      000000AEH   SFRSYM    DATA     WORD      TIM2_ARR
      000000A8H.5 SFRSYM    DATA     BIT       MCDIE
      000000C9H   SFRSYM    DATA     BYTE      RSTSRC
      000000E7H   SFRSYM    DATA     BYTE      LPF_YH
      000000A6H   SFRSYM    DATA     WORD      TIM3_ARR
      00000088H.6 SFRSYM    DATA     BIT       MCDIF
      00000098H.4 SFRSYM    DATA     BIT       REN
      00000096H   SFRSYM    DATA     WORD      TIM4_ARR
      000000ECH   SFRSYM    DATA     BYTE      PI_UKL
      000000D7H   SFRSYM    DATA     BYTE      CMP_SR
      0000008EH   SFRSYM    DATA     WORD      TIM5_ARR
      000000DEH   SFRSYM    DATA     BYTE      LPF_XL
      000000E6H   SFRSYM    DATA     BYTE      LPF_YL
      000000C8H   SFRSYM    DATA     BIT       PRTC0
      000000C8H.1 SFRSYM    DATA     BIT       PRTC1
      000000E8H.7 SFRSYM    DATA     BIT       FOCEN
      000000C8H.6 SFRSYM    DATA     BIT       PTSD0
      000000D8H.4 SFRSYM    DATA     BIT       PSPI0
      000000C8H.7 SFRSYM    DATA     BIT       PTSD1
      000000D8H.5 SFRSYM    DATA     BIT       PSPI1
      0000009BH   SFRSYM    DATA     BYTE      UT_BAUDH
      000000E4H   SFRSYM    DATA     WORD      SV_ANGLE
      000000B5H   SFRSYM    DATA     BYTE      TIM2_ADTRH
      0000009AH   SFRSYM    DATA     BYTE      UT_BAUDL
      000000FCH   SFRSYM    DATA     BYTE      P0_OE
      000000FDH   SFRSYM    DATA     BYTE      P1_OE
      000000D0H.5 SFRSYM    DATA     BIT       F0
      000000B4H   SFRSYM    DATA     BYTE      TIM2_ADTRL
      000000FEH   SFRSYM    DATA     BYTE      P2_OE
      000000D0H.1 SFRSYM    DATA     BIT       F1
      00000080H   SFRSYM    DATA     BIT       GP00
      000000FFH   SFRSYM    DATA     BYTE      P3_OE
      00000090H   SFRSYM    DATA     BIT       GP10
      00000080H.1 SFRSYM    DATA     BIT       GP01
      000000A8H.6 SFRSYM    DATA     BIT       RTCIE
      000000A0H   SFRSYM    DATA     BIT       GP20
      00000090H.1 SFRSYM    DATA     BIT       GP11
      00000080H.2 SFRSYM    DATA     BIT       GP02
      000000E3H   SFRSYM    DATA     BYTE      SV_USH
      000000B0H   SFRSYM    DATA     BIT       GP30
      000000A0H.1 SFRSYM    DATA     BIT       GP21
      00000090H.2 SFRSYM    DATA     BIT       GP12
      00000080H.3 SFRSYM    DATA     BIT       GP03
      000000B8H   SFRSYM    DATA     BIT       PLVW0
      000000A8H.1 SFRSYM    DATA     BIT       TSDIE
      000000D0H   SFRSYM    DATA     BYTE      PSW
      000000B0H.1 SFRSYM    DATA     BIT       GP31
      000000A0H.2 SFRSYM    DATA     BIT       GP22
      00000090H.3 SFRSYM    DATA     BIT       GP13
      00000080H.4 SFRSYM    DATA     BIT       GP04
      000000B8H.1 SFRSYM    DATA     BIT       PLVW1
LX51 LINKER/LOCATER V4.66.1.0                                                         03/23/2017  15:15:44  PAGE 48


      000000A8H.3 SFRSYM    DATA     BIT       SPIIE
      00000088H.5 SFRSYM    DATA     BIT       TSDIF
      000000B0H.2 SFRSYM    DATA     BIT       GP32
      000000A0H.3 SFRSYM    DATA     BIT       GP23
      00000090H.4 SFRSYM    DATA     BIT       GP14
      00000080H.5 SFRSYM    DATA     BIT       GP05
      00000084H   SFRSYM    DATA     BYTE      FLKEY
      000000B3H   SFRSYM    DATA     BYTE      TIM2_CMTRH
      000000B0H.3 SFRSYM    DATA     BIT       GP33
      000000A0H.4 SFRSYM    DATA     BIT       GP24
      00000090H.5 SFRSYM    DATA     BIT       GP15
      00000080H.6 SFRSYM    DATA     BIT       GP06
      00000088H   SFRSYM    DATA     BIT       IT00
      00000005H   SYMBOL    DATA     BYTE      i

      01001E78H   BLOCK     CODE     ---       LVL=0
      01001E78H   LINE      CODE     ---       #184
      01001E78H   LINE      CODE     ---       #185
      01001E78H   LINE      CODE     ---       #186
      01001E7BH   LINE      CODE     ---       #187
      01001E7EH   LINE      CODE     ---       #188
      01001E84H   LINE      CODE     ---       #189
      01001E89H   LINE      CODE     ---       #190
      ---         BLOCKEND  ---      ---       LVL=0

      01001E1FH   BLOCK     CODE     ---       LVL=0
      00000006H   SYMBOL    DATA     WORD      Angle
      01001E1FH   BLOCK     CODE     NEAR LAB  LVL=1
      00000007H   SYMBOL    DATA     BYTE      i
      ---         BLOCKEND  ---      ---       LVL=1
      01001E1FH   LINE      CODE     ---       #198
      01001E1FH   LINE      CODE     ---       #199
      01001E1FH   LINE      CODE     ---       #202
      01001E23H   LINE      CODE     ---       #203
      01001E26H   LINE      CODE     ---       #205
      01001E28H   LINE      CODE     ---       #206
      01001E28H   LINE      CODE     ---       #207
      01001E29H   LINE      CODE     ---       #208
      01001E2EH   LINE      CODE     ---       #210
      01001E36H   LINE      CODE     ---       #211
      ---         BLOCKEND  ---      ---       LVL=0

      ---         MODULE    ---      ---       MDU
      02000167H   PUBLIC    XDATA    ---       MDUControl
      010010FFH   PUBLIC    CODE     ---       MDUAPP
      01001DECH   PUBLIC    CODE     ---       MDUControlInit
      01001AAEH   PUBLIC    CODE     ---       _MDU_MULA_S16
      01001A00H   PUBLIC    CODE     ---       _MDU_MULA_U16
      01001DD2H   PUBLIC    CODE     ---       _MDU_MUL_U16
      01000026H   PUBLIC    CODE     ---       MDUInit
      000000E2H   SFRSYM    DATA     BYTE      SV_USL
      000000ABH   SFRSYM    DATA     BYTE      TIM2_CNTRH
      000000B0H.4 SFRSYM    DATA     BIT       GP34
      000000A0H.5 SFRSYM    DATA     BIT       GP25
      00000090H.6 SFRSYM    DATA     BIT       GP16
      00000080H.7 SFRSYM    DATA     BIT       GP07
      00000088H.1 SFRSYM    DATA     BIT       IT01
      00000088H.3 SFRSYM    DATA     BIT       IT10
      000000F6H   SFRSYM    DATA     WORD      PI_UKMIN
      000000C2H   SFRSYM    DATA     WORD      MD_MA
      000000A3H   SFRSYM    DATA     BYTE      TIM3_CNTRH
      000000B0H.5 SFRSYM    DATA     BIT       GP35
      000000A0H.6 SFRSYM    DATA     BIT       GP26
      00000090H.7 SFRSYM    DATA     BIT       GP17
      00000080H   SFRSYM    DATA     BYTE      P0
LX51 LINKER/LOCATER V4.66.1.0                                                         03/23/2017  15:15:44  PAGE 49


      00000088H.4 SFRSYM    DATA     BIT       IT11
      000000CAH   SFRSYM    DATA     WORD      MD_MB
      00000093H   SFRSYM    DATA     BYTE      TIM4_CNTRH
      000000B0H.6 SFRSYM    DATA     BIT       GP36
      000000A0H.7 SFRSYM    DATA     BIT       GP27
      00000090H   SFRSYM    DATA     BYTE      P1
      000000D9H   SFRSYM    DATA     BYTE      EVT_FILT
      000000F4H   SFRSYM    DATA     WORD      PI_UKMAX
      0000008BH   SFRSYM    DATA     BYTE      TIM5_CNTRH
      000000B2H   SFRSYM    DATA     BYTE      TIM2_CMTRL
      000000B0H.7 SFRSYM    DATA     BIT       GP37
      000000A0H   SFRSYM    DATA     BYTE      P2
      000000AAH   SFRSYM    DATA     BYTE      TIM2_CNTRL
      000000B0H   SFRSYM    DATA     BYTE      P3
      000000A2H   SFRSYM    DATA     BYTE      TIM3_CNTRL
      000000D0H.6 SFRSYM    DATA     BIT       AC
      00000092H   SFRSYM    DATA     BYTE      TIM4_CNTRL
      0000008AH   SFRSYM    DATA     BYTE      TIM5_CNTRL
      000000B6H   SFRSYM    DATA     WORD      TIM0_CCR1
      000000A8H.7 SFRSYM    DATA     BIT       EA
      000000D5H   SFRSYM    DATA     BYTE      CMP_CR0
      000000BAH   SFRSYM    DATA     WORD      TIM0_CCR2
      000000D6H   SFRSYM    DATA     BYTE      CMP_CR1
      000000BCH   SFRSYM    DATA     WORD      TIM0_CCR3
      00000085H   SFRSYM    DATA     BYTE      PSCTL
      000000DAH   SFRSYM    DATA     BYTE      CMP_CR2
      000000BEH   SFRSYM    DATA     WORD      TIM0_CCR4
      000000B8H.2 SFRSYM    DATA     BIT       PX00
      000000EAH   SFRSYM    DATA     WORD      PI_EK
      000000F8H   SFRSYM    DATA     BIT       OISUH
      000000B8H.3 SFRSYM    DATA     BIT       PX01
      000000B8H.4 SFRSYM    DATA     BIT       PX10
      000000F8H.2 SFRSYM    DATA     BIT       OISVH
      000000B8H.5 SFRSYM    DATA     BIT       PX11
      000000F8H.4 SFRSYM    DATA     BIT       OISWH
      000000DCH   SFRSYM    DATA     WORD      LPF_K
      000000F2H   SFRSYM    DATA     WORD      PI_KI
      000000F8H.1 SFRSYM    DATA     BIT       OISUL
      000000A8H   SFRSYM    DATA     BYTE      IE
      000000F8H.3 SFRSYM    DATA     BIT       OISVL
      000000F8H.5 SFRSYM    DATA     BIT       OISWL
      000000D1H   SFRSYM    DATA     BYTE      P1IE
      00000098H.6 SFRSYM    DATA     BIT       MOD0
      000000D3H   SFRSYM    DATA     BYTE      P2IE
      000000D2H   SFRSYM    DATA     BYTE      P1IF
      000000F9H   SFRSYM    DATA     BYTE      PL_CR
      00000098H.7 SFRSYM    DATA     BIT       MOD1
      000000D4H   SFRSYM    DATA     BYTE      P2IF
      000000ACH   SFRSYM    DATA     WORD      TIM2_DR
      00000082H   SFRSYM    DATA     WORD      DP
      000000EEH   SFRSYM    DATA     WORD      PI_KP
      000000A4H   SFRSYM    DATA     WORD      TIM3_DR
      00000094H   SFRSYM    DATA     WORD      TIM4_DR
      0000008CH   SFRSYM    DATA     WORD      TIM5_DR
      000000F1H   SFRSYM    DATA     BYTE      OSC_CFG
      000000C1H   SFRSYM    DATA     BYTE      MD_MODE
      000000ECH   SFRSYM    DATA     WORD      PI_UK
      000000DEH   SFRSYM    DATA     WORD      LPF_X
      00000098H   SFRSYM    DATA     BIT       RI
      000000E6H   SFRSYM    DATA     WORD      LPF_Y
      000000C0H   SFRSYM    DATA     BIT       PTIM00
      000000D0H.7 SFRSYM    DATA     BIT       CY
      00000098H.1 SFRSYM    DATA     BIT       TI
      000000C0H.1 SFRSYM    DATA     BIT       PTIM01
      000000C0H.2 SFRSYM    DATA     BIT       PTIM10
LX51 LINKER/LOCATER V4.66.1.0                                                         03/23/2017  15:15:44  PAGE 50


      000000C0H.3 SFRSYM    DATA     BIT       PTIM11
      000000E1H   SFRSYM    DATA     BYTE      SV_CR
      00000098H   SFRSYM    DATA     BYTE      UT_CR
      00000099H   SFRSYM    DATA     BYTE      UT_DR
      000000F8H.6 SFRSYM    DATA     BIT       OIS4
      00000081H   SFRSYM    DATA     BYTE      SP
      000000D0H.2 SFRSYM    DATA     BIT       OV
      000000C4H   SFRSYM    DATA     BYTE      MD_DA0
      0000009AH   SFRSYM    DATA     WORD      UT_BAUD
      000000CCH   SFRSYM    DATA     BYTE      MD_DB0
      000000C5H   SFRSYM    DATA     BYTE      MD_DA1
      000000CDH   SFRSYM    DATA     BYTE      MD_DB1
      000000C6H   SFRSYM    DATA     BYTE      MD_DA2
      000000CEH   SFRSYM    DATA     BYTE      MD_DB2
      000000C7H   SFRSYM    DATA     BYTE      MD_DA3
      000000B4H   SFRSYM    DATA     WORD      TIM2_ADTR
      000000CFH   SFRSYM    DATA     BYTE      MD_DB3
      000000AFH   SFRSYM    DATA     BYTE      TIM2_ARRH
      000000A7H   SFRSYM    DATA     BYTE      TIM3_ARRH
      00000097H   SFRSYM    DATA     BYTE      TIM4_ARRH
      0000008FH   SFRSYM    DATA     BYTE      TIM5_ARRH
      000000AEH   SFRSYM    DATA     BYTE      TIM2_ARRL
      000000A6H   SFRSYM    DATA     BYTE      TIM3_ARRL
      00000087H   SFRSYM    DATA     BYTE      PCON
      000000E2H   SFRSYM    DATA     WORD      SV_US
      00000096H   SFRSYM    DATA     BYTE      TIM4_ARRL
      0000008EH   SFRSYM    DATA     BYTE      TIM5_ARRL
      000000B2H   SFRSYM    DATA     WORD      TIM2_CMTR
      00000088H   SFRSYM    DATA     BYTE      TCON
      000000AAH   SFRSYM    DATA     WORD      TIM2_CNTR
      000000A2H   SFRSYM    DATA     WORD      TIM3_CNTR
      00000092H   SFRSYM    DATA     WORD      TIM4_CNTR
      0000008AH   SFRSYM    DATA     WORD      TIM5_CNTR
      000000E5H   SFRSYM    DATA     BYTE      SV_ANGLEH
      000000D8H   SFRSYM    DATA     BIT       PUART0
      000000E4H   SFRSYM    DATA     BYTE      SV_ANGLEL
      000000C6H   SFRSYM    DATA     WORD      MD_DAH
      000000D8H.1 SFRSYM    DATA     BIT       PUART1
      000000D8H.2 SFRSYM    DATA     BIT       PI2C0
      00000088H.2 SFRSYM    DATA     BIT       IF0
      000000CEH   SFRSYM    DATA     WORD      MD_DBH
      000000D8H.3 SFRSYM    DATA     BIT       PI2C1
      000000F0H   SFRSYM    DATA     BYTE      B
      000000C4H   SFRSYM    DATA     WORD      MD_DAL
      000000A1H   SFRSYM    DATA     BYTE      TIM2_CR0
      000000CCH   SFRSYM    DATA     WORD      MD_DBL
      0000009CH   SFRSYM    DATA     BYTE      TIM3_CR0
      000000A9H   SFRSYM    DATA     BYTE      TIM2_CR1
      0000009EH   SFRSYM    DATA     BYTE      TIM4_CR0
      0000009DH   SFRSYM    DATA     BYTE      TIM3_CR1
      00000089H   SFRSYM    DATA     BYTE      TIM5_CR0
      0000009FH   SFRSYM    DATA     BYTE      TIM4_CR1
      000000F8H   SFRSYM    DATA     BYTE      DRV_OUT
      00000091H   SFRSYM    DATA     BYTE      TIM5_CR1
      000000E0H   SFRSYM    DATA     BYTE      ACC
      000000F7H   SFRSYM    DATA     BYTE      PI_UKMINH
      000000C3H   SFRSYM    DATA     BYTE      MD_MAH
      000000A8H.4 SFRSYM    DATA     BIT       ES0
      000000DBH   SFRSYM    DATA     BYTE      LVSR
      000000CBH   SFRSYM    DATA     BYTE      MD_MBH
      000000C0H.4 SFRSYM    DATA     BIT       PADC0
      000000B8H   SFRSYM    DATA     BYTE      IP0
      000000F5H   SFRSYM    DATA     BYTE      PI_UKMAXH
      000000C0H.5 SFRSYM    DATA     BIT       PADC1
      000000C0H   SFRSYM    DATA     BYTE      IP1
LX51 LINKER/LOCATER V4.66.1.0                                                         03/23/2017  15:15:44  PAGE 51


      000000C8H   SFRSYM    DATA     BYTE      IP2
      000000F6H   SFRSYM    DATA     BYTE      PI_UKMINL
      000000C2H   SFRSYM    DATA     BYTE      MD_MAL
      00000098H.2 SFRSYM    DATA     BIT       RB8
      000000D8H   SFRSYM    DATA     BYTE      IP3
      000000CAH   SFRSYM    DATA     BYTE      MD_MBL
      000000A8H   SFRSYM    DATA     BIT       EX0
      000000F4H   SFRSYM    DATA     BYTE      PI_UKMAXL
      00000098H.3 SFRSYM    DATA     BIT       TB8
      000000B7H   SFRSYM    DATA     BYTE      TIM0_CCR1H
      000000A8H.2 SFRSYM    DATA     BIT       EX1
      000000BBH   SFRSYM    DATA     BYTE      TIM0_CCR2H
      000000D0H   SFRSYM    DATA     BIT       P
      000000BDH   SFRSYM    DATA     BYTE      TIM0_CCR3H
      000000BFH   SFRSYM    DATA     BYTE      TIM0_CCR4H
      000000C8H.2 SFRSYM    DATA     BIT       PTIM230
      000000EBH   SFRSYM    DATA     BYTE      PI_EKH
      00000098H.5 SFRSYM    DATA     BIT       SM2
      000000B6H   SFRSYM    DATA     BYTE      TIM0_CCR1L
      000000B1H   SFRSYM    DATA     BYTE      TIM0_SR1
      000000C8H.3 SFRSYM    DATA     BIT       PTIM231
      000000BAH   SFRSYM    DATA     BYTE      TIM0_CCR2L
      000000BCH   SFRSYM    DATA     BYTE      TIM0_CCR3L
      000000BEH   SFRSYM    DATA     BYTE      TIM0_CCR4L
      000000D8H.6 SFRSYM    DATA     BIT       PMCD0
      000000C8H.4 SFRSYM    DATA     BIT       PTIM450
      000000D0H.3 SFRSYM    DATA     BIT       RS0
      000000DDH   SFRSYM    DATA     BYTE      LPF_KH
      000000F3H   SFRSYM    DATA     BYTE      PI_KIH
      000000EAH   SFRSYM    DATA     BYTE      PI_EKL
      000000E8H   SFRSYM    DATA     BYTE      FOC_SET0
      000000D8H.7 SFRSYM    DATA     BIT       PMCD1
      000000C8H.5 SFRSYM    DATA     BIT       PTIM451
      000000D0H.4 SFRSYM    DATA     BIT       RS1
      000000E9H   SFRSYM    DATA     BYTE      FOC_SET1
      000000B8H.6 SFRSYM    DATA     BIT       PFOC0
      000000DCH   SFRSYM    DATA     BYTE      LPF_KL
      000000F2H   SFRSYM    DATA     BYTE      PI_KIL
      000000B8H.7 SFRSYM    DATA     BIT       PFOC1
      000000ADH   SFRSYM    DATA     BYTE      TIM2_DRH
      000000B9H   SFRSYM    DATA     BYTE      TIM0_IER
      00000083H   SFRSYM    DATA     BYTE      DPH
      000000EFH   SFRSYM    DATA     BYTE      PI_KPH
      000000A5H   SFRSYM    DATA     BYTE      TIM3_DRH
      00000095H   SFRSYM    DATA     BYTE      TIM4_DRH
      0000008DH   SFRSYM    DATA     BYTE      TIM5_DRH
      000000ACH   SFRSYM    DATA     BYTE      TIM2_DRL
      00000082H   SFRSYM    DATA     BYTE      DPL
      000000EEH   SFRSYM    DATA     BYTE      PI_KPL
      000000A4H   SFRSYM    DATA     BYTE      TIM3_DRL
      000000F8H.7 SFRSYM    DATA     BIT       MOE
      000000C0H.6 SFRSYM    DATA     BIT       PCMP0
      000000EDH   SFRSYM    DATA     BYTE      PI_UKH
      00000094H   SFRSYM    DATA     BYTE      TIM4_DRL
      000000C0H.7 SFRSYM    DATA     BIT       PCMP1
      000000DFH   SFRSYM    DATA     BYTE      LPF_XH
      0000008CH   SFRSYM    DATA     BYTE      TIM5_DRL
      000000AEH   SFRSYM    DATA     WORD      TIM2_ARR
      000000A8H.5 SFRSYM    DATA     BIT       MCDIE
      000000C9H   SFRSYM    DATA     BYTE      RSTSRC
      000000E7H   SFRSYM    DATA     BYTE      LPF_YH
      000000A6H   SFRSYM    DATA     WORD      TIM3_ARR
      00000088H.6 SFRSYM    DATA     BIT       MCDIF
      00000098H.4 SFRSYM    DATA     BIT       REN
      00000096H   SFRSYM    DATA     WORD      TIM4_ARR
LX51 LINKER/LOCATER V4.66.1.0                                                         03/23/2017  15:15:44  PAGE 52


      000000ECH   SFRSYM    DATA     BYTE      PI_UKL
      000000D7H   SFRSYM    DATA     BYTE      CMP_SR
      0000008EH   SFRSYM    DATA     WORD      TIM5_ARR
      000000DEH   SFRSYM    DATA     BYTE      LPF_XL
      000000E6H   SFRSYM    DATA     BYTE      LPF_YL
      000000C8H   SFRSYM    DATA     BIT       PRTC0
      000000C8H.1 SFRSYM    DATA     BIT       PRTC1
      000000E8H.7 SFRSYM    DATA     BIT       FOCEN
      000000C8H.6 SFRSYM    DATA     BIT       PTSD0
      000000D8H.4 SFRSYM    DATA     BIT       PSPI0
      000000C8H.7 SFRSYM    DATA     BIT       PTSD1
      000000D8H.5 SFRSYM    DATA     BIT       PSPI1
      0000009BH   SFRSYM    DATA     BYTE      UT_BAUDH
      000000E4H   SFRSYM    DATA     WORD      SV_ANGLE
      000000B5H   SFRSYM    DATA     BYTE      TIM2_ADTRH
      0000009AH   SFRSYM    DATA     BYTE      UT_BAUDL
      000000FCH   SFRSYM    DATA     BYTE      P0_OE
      000000FDH   SFRSYM    DATA     BYTE      P1_OE
      000000D0H.5 SFRSYM    DATA     BIT       F0
      000000B4H   SFRSYM    DATA     BYTE      TIM2_ADTRL
      000000FEH   SFRSYM    DATA     BYTE      P2_OE
      000000D0H.1 SFRSYM    DATA     BIT       F1
      00000080H   SFRSYM    DATA     BIT       GP00
      000000FFH   SFRSYM    DATA     BYTE      P3_OE
      00000090H   SFRSYM    DATA     BIT       GP10
      00000080H.1 SFRSYM    DATA     BIT       GP01
      000000A8H.6 SFRSYM    DATA     BIT       RTCIE
      000000A0H   SFRSYM    DATA     BIT       GP20
      00000090H.1 SFRSYM    DATA     BIT       GP11
      00000080H.2 SFRSYM    DATA     BIT       GP02
      000000E3H   SFRSYM    DATA     BYTE      SV_USH
      000000B0H   SFRSYM    DATA     BIT       GP30
      000000A0H.1 SFRSYM    DATA     BIT       GP21
      00000090H.2 SFRSYM    DATA     BIT       GP12
      00000080H.3 SFRSYM    DATA     BIT       GP03
      000000B8H   SFRSYM    DATA     BIT       PLVW0
      000000A8H.1 SFRSYM    DATA     BIT       TSDIE
      000000D0H   SFRSYM    DATA     BYTE      PSW
      000000B0H.1 SFRSYM    DATA     BIT       GP31
      000000A0H.2 SFRSYM    DATA     BIT       GP22
      00000090H.3 SFRSYM    DATA     BIT       GP13
      00000080H.4 SFRSYM    DATA     BIT       GP04
      000000B8H.1 SFRSYM    DATA     BIT       PLVW1
      000000A8H.3 SFRSYM    DATA     BIT       SPIIE
      00000088H.5 SFRSYM    DATA     BIT       TSDIF
      000000B0H.2 SFRSYM    DATA     BIT       GP32
      000000A0H.3 SFRSYM    DATA     BIT       GP23
      00000090H.4 SFRSYM    DATA     BIT       GP14
      00000080H.5 SFRSYM    DATA     BIT       GP05
      00000084H   SFRSYM    DATA     BYTE      FLKEY
      000000B3H   SFRSYM    DATA     BYTE      TIM2_CMTRH
      000000B0H.3 SFRSYM    DATA     BIT       GP33
      000000A0H.4 SFRSYM    DATA     BIT       GP24
      00000090H.5 SFRSYM    DATA     BIT       GP15
      00000080H.6 SFRSYM    DATA     BIT       GP06
      00000088H   SFRSYM    DATA     BIT       IT00

      01000026H   BLOCK     CODE     ---       LVL=0
      01000026H   LINE      CODE     ---       #25
      01000026H   LINE      CODE     ---       #26
      01000026H   LINE      CODE     ---       #31
      01000029H   LINE      CODE     ---       #32
      0100002CH   LINE      CODE     ---       #34
      0100002FH   LINE      CODE     ---       #36
      ---         BLOCKEND  ---      ---       LVL=0
LX51 LINKER/LOCATER V4.66.1.0                                                         03/23/2017  15:15:44  PAGE 53



      01001DD2H   BLOCK     CODE     ---       LVL=0
      00000006H   SYMBOL    DATA     WORD      TData0
      00000004H   SYMBOL    DATA     WORD      TData1
      01001DD2H   LINE      CODE     ---       #47
      01001DD2H   LINE      CODE     ---       #48
      01001DD2H   LINE      CODE     ---       #49
      01001DD5H   LINE      CODE     ---       #50
      01001DD8H   LINE      CODE     ---       #51
      01001DDBH   LINE      CODE     ---       #53
      01001DDFH   LINE      CODE     ---       #54
      01001DE7H   LINE      CODE     ---       #56
      01001DEBH   LINE      CODE     ---       #58
      ---         BLOCKEND  ---      ---       LVL=0
      00000006H   SYMBOL    DATA     WORD      TData0
      00000004H   SYMBOL    DATA     WORD      TData1
      00000002H   SYMBOL    DATA     ---       Result32
      00000006H   SYMBOL    DATA     INT       TData0
      00000004H   SYMBOL    DATA     INT       TData1
      00000006H   SYMBOL    DATA     INT       TData0
      00000004H   SYMBOL    DATA     INT       TData1
      00000002H   SYMBOL    DATA     ---       Result32

      010019F9H   BLOCK     CODE     ---       LVL=0
      ---         BLOCKEND  ---      ---       LVL=0

      01001A00H   BLOCK     CODE     ---       LVL=0
      00000006H   SYMBOL    DATA     WORD      TData0
      00000004H   SYMBOL    DATA     WORD      TData1
      00000003H   SYMBOL    DATA     BYTE      ALIGN
      01001A00H   LINE      CODE     ---       #125
      01001A00H   LINE      CODE     ---       #126
      01001A00H   LINE      CODE     ---       #127
      01001A04H   LINE      CODE     ---       #128
      01001A04H   LINE      CODE     ---       #129
      01001A07H   LINE      CODE     ---       #130
      01001A07H   LINE      CODE     ---       #131
      01001A09H   LINE      CODE     ---       #132
      01001A0DH   LINE      CODE     ---       #133
      01001A0DH   LINE      CODE     ---       #134
      01001A10H   LINE      CODE     ---       #135
      01001A10H   LINE      CODE     ---       #136
      01001A12H   LINE      CODE     ---       #137
      01001A16H   LINE      CODE     ---       #138
      01001A16H   LINE      CODE     ---       #139
      01001A19H   LINE      CODE     ---       #140
      01001A1CH   LINE      CODE     ---       #141
      01001A1EH   LINE      CODE     ---       #143
      01001A1EH   LINE      CODE     ---       #144
      01001A21H   LINE      CODE     ---       #145
      01001A24H   LINE      CODE     ---       #146
      01001A24H   LINE      CODE     ---       #148
      01001A27H   LINE      CODE     ---       #150
      01001A2BH   LINE      CODE     ---       #151
      01001A33H   LINE      CODE     ---       #153
      01001A37H   LINE      CODE     ---       #155
      ---         BLOCKEND  ---      ---       LVL=0
      00000006H   SYMBOL    DATA     WORD      TData0
      00000004H   SYMBOL    DATA     WORD      TData1
      00000003H   SYMBOL    DATA     BYTE      ALIGN

      01001AAEH   BLOCK     CODE     ---       LVL=0
      00000006H   SYMBOL    DATA     INT       TData0
      00000004H   SYMBOL    DATA     INT       TData1
      00000003H   SYMBOL    DATA     BYTE      ALIGN
LX51 LINKER/LOCATER V4.66.1.0                                                         03/23/2017  15:15:44  PAGE 54


      01001AAEH   LINE      CODE     ---       #203
      01001AAEH   LINE      CODE     ---       #204
      01001AAEH   LINE      CODE     ---       #205
      01001AB2H   LINE      CODE     ---       #206
      01001AB2H   LINE      CODE     ---       #207
      01001AB5H   LINE      CODE     ---       #208
      01001AB5H   LINE      CODE     ---       #209
      01001AB7H   LINE      CODE     ---       #210
      01001ABBH   LINE      CODE     ---       #211
      01001ABBH   LINE      CODE     ---       #212
      01001ABEH   LINE      CODE     ---       #213
      01001ABEH   LINE      CODE     ---       #214
      01001AC0H   LINE      CODE     ---       #215
      01001AC4H   LINE      CODE     ---       #216
      01001AC4H   LINE      CODE     ---       #217
      01001AC7H   LINE      CODE     ---       #218
      01001ACAH   LINE      CODE     ---       #219
      01001ACCH   LINE      CODE     ---       #221
      01001ACCH   LINE      CODE     ---       #222
      01001ACFH   LINE      CODE     ---       #223
      01001AD2H   LINE      CODE     ---       #224
      01001AD2H   LINE      CODE     ---       #226
      01001AD5H   LINE      CODE     ---       #228
      01001AD9H   LINE      CODE     ---       #229
      01001AE1H   LINE      CODE     ---       #231
      01001AE5H   LINE      CODE     ---       #233
      ---         BLOCKEND  ---      ---       LVL=0
      00000006H   SYMBOL    DATA     INT       TData0
      00000004H   SYMBOL    DATA     INT       TData1
      00000003H   SYMBOL    DATA     BYTE      ALIGN
      00000006H   SYMBOL    DATA     ---       TData0
      00000004H   SYMBOL    DATA     ---       TData1
      00000004H   SYMBOL    DATA     ---       TData1
      00000002H   SYMBOL    DATA     ---       Result32

      01001DECH   BLOCK     CODE     ---       LVL=0
      01001DECH   LINE      CODE     ---       #328
      01001DECH   LINE      CODE     ---       #329
      01001DECH   LINE      CODE     ---       #330
      01001DF1H   LINE      CODE     ---       #331
      01001DF3H   LINE      CODE     ---       #332
      01001DF5H   LINE      CODE     ---       #333
      01001DF7H   LINE      CODE     ---       #335
      01001DF9H   LINE      CODE     ---       #336
      01001DFBH   LINE      CODE     ---       #337
      01001DFDH   LINE      CODE     ---       #339
      01001E01H   LINE      CODE     ---       #341
      01001E05H   LINE      CODE     ---       #343
      ---         BLOCKEND  ---      ---       LVL=0

      010010FFH   BLOCK     CODE     ---       LVL=0
      010010FFH   LINE      CODE     ---       #352
      010010FFH   LINE      CODE     ---       #353
      010010FFH   LINE      CODE     ---       #356
      01001105H   LINE      CODE     ---       #357
      01001105H   LINE      CODE     ---       #359
      01001105H   LINE      CODE     ---       #360
      0100112AH   LINE      CODE     ---       #363
      0100112AH   LINE      CODE     ---       #369
      0100112FH   LINE      CODE     ---       #370
      0100112FH   LINE      CODE     ---       #373
      01001135H   LINE      CODE     ---       #374
      01001135H   LINE      CODE     ---       #375
      01001145H   LINE      CODE     ---       #376
      01001145H   LINE      CODE     ---       #377
LX51 LINKER/LOCATER V4.66.1.0                                                         03/23/2017  15:15:44  PAGE 55


      0100114EH   LINE      CODE     ---       #378
      01001150H   LINE      CODE     ---       #380
      01001150H   LINE      CODE     ---       #381
      01001188H   LINE      CODE     ---       #382
      01001188H   LINE      CODE     ---       #383
      0100118DH   LINE      CODE     ---       #384
      0100118DH   LINE      CODE     ---       #388
      01001193H   LINE      CODE     ---       #389
      01001193H   LINE      CODE     ---       #390
      010011A5H   LINE      CODE     ---       #391
      010011AAH   LINE      CODE     ---       #392
      010011AAH   LINE      CODE     ---       #395
      010011B0H   LINE      CODE     ---       #396
      010011B0H   LINE      CODE     ---       #397
      010011C7H   LINE      CODE     ---       #398
      010011CCH   LINE      CODE     ---       #399
      010011CCH   LINE      CODE     ---       #402
      010011D2H   LINE      CODE     ---       #403
      010011D2H   LINE      CODE     ---       #404
      010011E4H   LINE      CODE     ---       #405
      010011E9H   LINE      CODE     ---       #406
      010011E9H   LINE      CODE     ---       #441
      ---         BLOCKEND  ---      ---       LVL=0

      ---         MODULE    ---      ---       LPF
      01001D11H   PUBLIC    CODE     ---       _LPF
      000000E2H   SFRSYM    DATA     BYTE      SV_USL
      000000ABH   SFRSYM    DATA     BYTE      TIM2_CNTRH
      000000B0H.4 SFRSYM    DATA     BIT       GP34
      000000A0H.5 SFRSYM    DATA     BIT       GP25
      00000090H.6 SFRSYM    DATA     BIT       GP16
      00000080H.7 SFRSYM    DATA     BIT       GP07
      00000088H.1 SFRSYM    DATA     BIT       IT01
      00000088H.3 SFRSYM    DATA     BIT       IT10
      000000F6H   SFRSYM    DATA     WORD      PI_UKMIN
      000000C2H   SFRSYM    DATA     WORD      MD_MA
      000000A3H   SFRSYM    DATA     BYTE      TIM3_CNTRH
      000000B0H.5 SFRSYM    DATA     BIT       GP35
      000000A0H.6 SFRSYM    DATA     BIT       GP26
      00000090H.7 SFRSYM    DATA     BIT       GP17
      00000080H   SFRSYM    DATA     BYTE      P0
      00000088H.4 SFRSYM    DATA     BIT       IT11
      000000CAH   SFRSYM    DATA     WORD      MD_MB
      00000093H   SFRSYM    DATA     BYTE      TIM4_CNTRH
      000000B0H.6 SFRSYM    DATA     BIT       GP36
      000000A0H.7 SFRSYM    DATA     BIT       GP27
      00000090H   SFRSYM    DATA     BYTE      P1
      000000D9H   SFRSYM    DATA     BYTE      EVT_FILT
      000000F4H   SFRSYM    DATA     WORD      PI_UKMAX
      0000008BH   SFRSYM    DATA     BYTE      TIM5_CNTRH
      000000B2H   SFRSYM    DATA     BYTE      TIM2_CMTRL
      000000B0H.7 SFRSYM    DATA     BIT       GP37
      000000A0H   SFRSYM    DATA     BYTE      P2
      000000AAH   SFRSYM    DATA     BYTE      TIM2_CNTRL
      000000B0H   SFRSYM    DATA     BYTE      P3
      000000A2H   SFRSYM    DATA     BYTE      TIM3_CNTRL
      000000D0H.6 SFRSYM    DATA     BIT       AC
      00000092H   SFRSYM    DATA     BYTE      TIM4_CNTRL
      0000008AH   SFRSYM    DATA     BYTE      TIM5_CNTRL
      000000B6H   SFRSYM    DATA     WORD      TIM0_CCR1
      000000A8H.7 SFRSYM    DATA     BIT       EA
      000000D5H   SFRSYM    DATA     BYTE      CMP_CR0
      000000BAH   SFRSYM    DATA     WORD      TIM0_CCR2
      000000D6H   SFRSYM    DATA     BYTE      CMP_CR1
      000000BCH   SFRSYM    DATA     WORD      TIM0_CCR3
LX51 LINKER/LOCATER V4.66.1.0                                                         03/23/2017  15:15:44  PAGE 56


      00000085H   SFRSYM    DATA     BYTE      PSCTL
      000000DAH   SFRSYM    DATA     BYTE      CMP_CR2
      000000BEH   SFRSYM    DATA     WORD      TIM0_CCR4
      000000B8H.2 SFRSYM    DATA     BIT       PX00
      000000EAH   SFRSYM    DATA     WORD      PI_EK
      000000F8H   SFRSYM    DATA     BIT       OISUH
      000000B8H.3 SFRSYM    DATA     BIT       PX01
      000000B8H.4 SFRSYM    DATA     BIT       PX10
      000000F8H.2 SFRSYM    DATA     BIT       OISVH
      000000B8H.5 SFRSYM    DATA     BIT       PX11
      000000F8H.4 SFRSYM    DATA     BIT       OISWH
      000000DCH   SFRSYM    DATA     WORD      LPF_K
      000000F2H   SFRSYM    DATA     WORD      PI_KI
      000000F8H.1 SFRSYM    DATA     BIT       OISUL
      000000A8H   SFRSYM    DATA     BYTE      IE
      000000F8H.3 SFRSYM    DATA     BIT       OISVL
      000000F8H.5 SFRSYM    DATA     BIT       OISWL
      000000D1H   SFRSYM    DATA     BYTE      P1IE
      00000098H.6 SFRSYM    DATA     BIT       MOD0
      000000D3H   SFRSYM    DATA     BYTE      P2IE
      000000D2H   SFRSYM    DATA     BYTE      P1IF
      000000F9H   SFRSYM    DATA     BYTE      PL_CR
      00000098H.7 SFRSYM    DATA     BIT       MOD1
      000000D4H   SFRSYM    DATA     BYTE      P2IF
      000000ACH   SFRSYM    DATA     WORD      TIM2_DR
      00000082H   SFRSYM    DATA     WORD      DP
      000000EEH   SFRSYM    DATA     WORD      PI_KP
      000000A4H   SFRSYM    DATA     WORD      TIM3_DR
      00000094H   SFRSYM    DATA     WORD      TIM4_DR
      0000008CH   SFRSYM    DATA     WORD      TIM5_DR
      000000F1H   SFRSYM    DATA     BYTE      OSC_CFG
      000000C1H   SFRSYM    DATA     BYTE      MD_MODE
      000000ECH   SFRSYM    DATA     WORD      PI_UK
      000000DEH   SFRSYM    DATA     WORD      LPF_X
      00000098H   SFRSYM    DATA     BIT       RI
      000000E6H   SFRSYM    DATA     WORD      LPF_Y
      000000C0H   SFRSYM    DATA     BIT       PTIM00
      000000D0H.7 SFRSYM    DATA     BIT       CY
      00000098H.1 SFRSYM    DATA     BIT       TI
      000000C0H.1 SFRSYM    DATA     BIT       PTIM01
      000000C0H.2 SFRSYM    DATA     BIT       PTIM10
      000000C0H.3 SFRSYM    DATA     BIT       PTIM11
      000000E1H   SFRSYM    DATA     BYTE      SV_CR
      00000098H   SFRSYM    DATA     BYTE      UT_CR
      00000099H   SFRSYM    DATA     BYTE      UT_DR
      000000F8H.6 SFRSYM    DATA     BIT       OIS4
      00000081H   SFRSYM    DATA     BYTE      SP
      000000D0H.2 SFRSYM    DATA     BIT       OV
      000000C4H   SFRSYM    DATA     BYTE      MD_DA0
      0000009AH   SFRSYM    DATA     WORD      UT_BAUD
      000000CCH   SFRSYM    DATA     BYTE      MD_DB0
      000000C5H   SFRSYM    DATA     BYTE      MD_DA1
      000000CDH   SFRSYM    DATA     BYTE      MD_DB1
      000000C6H   SFRSYM    DATA     BYTE      MD_DA2
      000000CEH   SFRSYM    DATA     BYTE      MD_DB2
      000000C7H   SFRSYM    DATA     BYTE      MD_DA3
      000000B4H   SFRSYM    DATA     WORD      TIM2_ADTR
      000000CFH   SFRSYM    DATA     BYTE      MD_DB3
      000000AFH   SFRSYM    DATA     BYTE      TIM2_ARRH
      000000A7H   SFRSYM    DATA     BYTE      TIM3_ARRH
      00000097H   SFRSYM    DATA     BYTE      TIM4_ARRH
      0000008FH   SFRSYM    DATA     BYTE      TIM5_ARRH
      000000AEH   SFRSYM    DATA     BYTE      TIM2_ARRL
      000000A6H   SFRSYM    DATA     BYTE      TIM3_ARRL
      00000087H   SFRSYM    DATA     BYTE      PCON
LX51 LINKER/LOCATER V4.66.1.0                                                         03/23/2017  15:15:44  PAGE 57


      000000E2H   SFRSYM    DATA     WORD      SV_US
      00000096H   SFRSYM    DATA     BYTE      TIM4_ARRL
      0000008EH   SFRSYM    DATA     BYTE      TIM5_ARRL
      000000B2H   SFRSYM    DATA     WORD      TIM2_CMTR
      00000088H   SFRSYM    DATA     BYTE      TCON
      000000AAH   SFRSYM    DATA     WORD      TIM2_CNTR
      000000A2H   SFRSYM    DATA     WORD      TIM3_CNTR
      00000092H   SFRSYM    DATA     WORD      TIM4_CNTR
      0000008AH   SFRSYM    DATA     WORD      TIM5_CNTR
      000000E5H   SFRSYM    DATA     BYTE      SV_ANGLEH
      000000D8H   SFRSYM    DATA     BIT       PUART0
      000000E4H   SFRSYM    DATA     BYTE      SV_ANGLEL
      000000C6H   SFRSYM    DATA     WORD      MD_DAH
      000000D8H.1 SFRSYM    DATA     BIT       PUART1
      000000D8H.2 SFRSYM    DATA     BIT       PI2C0
      00000088H.2 SFRSYM    DATA     BIT       IF0
      000000CEH   SFRSYM    DATA     WORD      MD_DBH
      000000D8H.3 SFRSYM    DATA     BIT       PI2C1
      000000F0H   SFRSYM    DATA     BYTE      B
      000000C4H   SFRSYM    DATA     WORD      MD_DAL
      000000A1H   SFRSYM    DATA     BYTE      TIM2_CR0
      000000CCH   SFRSYM    DATA     WORD      MD_DBL
      0000009CH   SFRSYM    DATA     BYTE      TIM3_CR0
      000000A9H   SFRSYM    DATA     BYTE      TIM2_CR1
      0000009EH   SFRSYM    DATA     BYTE      TIM4_CR0
      0000009DH   SFRSYM    DATA     BYTE      TIM3_CR1
      00000089H   SFRSYM    DATA     BYTE      TIM5_CR0
      0000009FH   SFRSYM    DATA     BYTE      TIM4_CR1
      000000F8H   SFRSYM    DATA     BYTE      DRV_OUT
      00000091H   SFRSYM    DATA     BYTE      TIM5_CR1
      000000E0H   SFRSYM    DATA     BYTE      ACC
      000000F7H   SFRSYM    DATA     BYTE      PI_UKMINH
      000000C3H   SFRSYM    DATA     BYTE      MD_MAH
      000000A8H.4 SFRSYM    DATA     BIT       ES0
      000000DBH   SFRSYM    DATA     BYTE      LVSR
      000000CBH   SFRSYM    DATA     BYTE      MD_MBH
      000000C0H.4 SFRSYM    DATA     BIT       PADC0
      000000B8H   SFRSYM    DATA     BYTE      IP0
      000000F5H   SFRSYM    DATA     BYTE      PI_UKMAXH
      000000C0H.5 SFRSYM    DATA     BIT       PADC1
      000000C0H   SFRSYM    DATA     BYTE      IP1
      000000C8H   SFRSYM    DATA     BYTE      IP2
      000000F6H   SFRSYM    DATA     BYTE      PI_UKMINL
      000000C2H   SFRSYM    DATA     BYTE      MD_MAL
      00000098H.2 SFRSYM    DATA     BIT       RB8
      000000D8H   SFRSYM    DATA     BYTE      IP3
      000000CAH   SFRSYM    DATA     BYTE      MD_MBL
      000000A8H   SFRSYM    DATA     BIT       EX0
      000000F4H   SFRSYM    DATA     BYTE      PI_UKMAXL
      00000098H.3 SFRSYM    DATA     BIT       TB8
      000000B7H   SFRSYM    DATA     BYTE      TIM0_CCR1H
      000000A8H.2 SFRSYM    DATA     BIT       EX1
      000000BBH   SFRSYM    DATA     BYTE      TIM0_CCR2H
      000000D0H   SFRSYM    DATA     BIT       P
      000000BDH   SFRSYM    DATA     BYTE      TIM0_CCR3H
      000000BFH   SFRSYM    DATA     BYTE      TIM0_CCR4H
      000000C8H.2 SFRSYM    DATA     BIT       PTIM230
      000000EBH   SFRSYM    DATA     BYTE      PI_EKH
      00000098H.5 SFRSYM    DATA     BIT       SM2
      000000B6H   SFRSYM    DATA     BYTE      TIM0_CCR1L
      000000B1H   SFRSYM    DATA     BYTE      TIM0_SR1
      000000C8H.3 SFRSYM    DATA     BIT       PTIM231
      000000BAH   SFRSYM    DATA     BYTE      TIM0_CCR2L
      000000BCH   SFRSYM    DATA     BYTE      TIM0_CCR3L
      000000BEH   SFRSYM    DATA     BYTE      TIM0_CCR4L
LX51 LINKER/LOCATER V4.66.1.0                                                         03/23/2017  15:15:44  PAGE 58


      000000D8H.6 SFRSYM    DATA     BIT       PMCD0
      000000C8H.4 SFRSYM    DATA     BIT       PTIM450
      000000D0H.3 SFRSYM    DATA     BIT       RS0
      000000DDH   SFRSYM    DATA     BYTE      LPF_KH
      000000F3H   SFRSYM    DATA     BYTE      PI_KIH
      000000EAH   SFRSYM    DATA     BYTE      PI_EKL
      000000E8H   SFRSYM    DATA     BYTE      FOC_SET0
      000000D8H.7 SFRSYM    DATA     BIT       PMCD1
      000000C8H.5 SFRSYM    DATA     BIT       PTIM451
      000000D0H.4 SFRSYM    DATA     BIT       RS1
      000000E9H   SFRSYM    DATA     BYTE      FOC_SET1
      000000B8H.6 SFRSYM    DATA     BIT       PFOC0
      000000DCH   SFRSYM    DATA     BYTE      LPF_KL
      000000F2H   SFRSYM    DATA     BYTE      PI_KIL
      000000B8H.7 SFRSYM    DATA     BIT       PFOC1
      000000ADH   SFRSYM    DATA     BYTE      TIM2_DRH
      000000B9H   SFRSYM    DATA     BYTE      TIM0_IER
      00000083H   SFRSYM    DATA     BYTE      DPH
      000000EFH   SFRSYM    DATA     BYTE      PI_KPH
      000000A5H   SFRSYM    DATA     BYTE      TIM3_DRH
      00000095H   SFRSYM    DATA     BYTE      TIM4_DRH
      0000008DH   SFRSYM    DATA     BYTE      TIM5_DRH
      000000ACH   SFRSYM    DATA     BYTE      TIM2_DRL
      00000082H   SFRSYM    DATA     BYTE      DPL
      000000EEH   SFRSYM    DATA     BYTE      PI_KPL
      000000A4H   SFRSYM    DATA     BYTE      TIM3_DRL
      000000F8H.7 SFRSYM    DATA     BIT       MOE
      000000C0H.6 SFRSYM    DATA     BIT       PCMP0
      000000EDH   SFRSYM    DATA     BYTE      PI_UKH
      00000094H   SFRSYM    DATA     BYTE      TIM4_DRL
      000000C0H.7 SFRSYM    DATA     BIT       PCMP1
      000000DFH   SFRSYM    DATA     BYTE      LPF_XH
      0000008CH   SFRSYM    DATA     BYTE      TIM5_DRL
      000000AEH   SFRSYM    DATA     WORD      TIM2_ARR
      000000A8H.5 SFRSYM    DATA     BIT       MCDIE
      000000C9H   SFRSYM    DATA     BYTE      RSTSRC
      000000E7H   SFRSYM    DATA     BYTE      LPF_YH
      000000A6H   SFRSYM    DATA     WORD      TIM3_ARR
      00000088H.6 SFRSYM    DATA     BIT       MCDIF
      00000098H.4 SFRSYM    DATA     BIT       REN
      00000096H   SFRSYM    DATA     WORD      TIM4_ARR
      000000ECH   SFRSYM    DATA     BYTE      PI_UKL
      000000D7H   SFRSYM    DATA     BYTE      CMP_SR
      0000008EH   SFRSYM    DATA     WORD      TIM5_ARR
      000000DEH   SFRSYM    DATA     BYTE      LPF_XL
      000000E6H   SFRSYM    DATA     BYTE      LPF_YL
      000000C8H   SFRSYM    DATA     BIT       PRTC0
      000000C8H.1 SFRSYM    DATA     BIT       PRTC1
      000000E8H.7 SFRSYM    DATA     BIT       FOCEN
      000000C8H.6 SFRSYM    DATA     BIT       PTSD0
      000000D8H.4 SFRSYM    DATA     BIT       PSPI0
      000000C8H.7 SFRSYM    DATA     BIT       PTSD1
      000000D8H.5 SFRSYM    DATA     BIT       PSPI1
      0000009BH   SFRSYM    DATA     BYTE      UT_BAUDH
      000000E4H   SFRSYM    DATA     WORD      SV_ANGLE
      000000B5H   SFRSYM    DATA     BYTE      TIM2_ADTRH
      0000009AH   SFRSYM    DATA     BYTE      UT_BAUDL
      000000FCH   SFRSYM    DATA     BYTE      P0_OE
      000000FDH   SFRSYM    DATA     BYTE      P1_OE
      000000D0H.5 SFRSYM    DATA     BIT       F0
      000000B4H   SFRSYM    DATA     BYTE      TIM2_ADTRL
      000000FEH   SFRSYM    DATA     BYTE      P2_OE
      000000D0H.1 SFRSYM    DATA     BIT       F1
      00000080H   SFRSYM    DATA     BIT       GP00
      000000FFH   SFRSYM    DATA     BYTE      P3_OE
LX51 LINKER/LOCATER V4.66.1.0                                                         03/23/2017  15:15:44  PAGE 59


      00000090H   SFRSYM    DATA     BIT       GP10
      00000080H.1 SFRSYM    DATA     BIT       GP01
      000000A8H.6 SFRSYM    DATA     BIT       RTCIE
      000000A0H   SFRSYM    DATA     BIT       GP20
      00000090H.1 SFRSYM    DATA     BIT       GP11
      00000080H.2 SFRSYM    DATA     BIT       GP02
      000000E3H   SFRSYM    DATA     BYTE      SV_USH
      000000B0H   SFRSYM    DATA     BIT       GP30
      000000A0H.1 SFRSYM    DATA     BIT       GP21
      00000090H.2 SFRSYM    DATA     BIT       GP12
      00000080H.3 SFRSYM    DATA     BIT       GP03
      000000B8H   SFRSYM    DATA     BIT       PLVW0
      000000A8H.1 SFRSYM    DATA     BIT       TSDIE
      000000D0H   SFRSYM    DATA     BYTE      PSW
      000000B0H.1 SFRSYM    DATA     BIT       GP31
      000000A0H.2 SFRSYM    DATA     BIT       GP22
      00000090H.3 SFRSYM    DATA     BIT       GP13
      00000080H.4 SFRSYM    DATA     BIT       GP04
      000000B8H.1 SFRSYM    DATA     BIT       PLVW1
      000000A8H.3 SFRSYM    DATA     BIT       SPIIE
      00000088H.5 SFRSYM    DATA     BIT       TSDIF
      000000B0H.2 SFRSYM    DATA     BIT       GP32
      000000A0H.3 SFRSYM    DATA     BIT       GP23
      00000090H.4 SFRSYM    DATA     BIT       GP14
      00000080H.5 SFRSYM    DATA     BIT       GP05
      00000084H   SFRSYM    DATA     BYTE      FLKEY
      000000B3H   SFRSYM    DATA     BYTE      TIM2_CMTRH
      000000B0H.3 SFRSYM    DATA     BIT       GP33
      000000A0H.4 SFRSYM    DATA     BIT       GP24
      00000090H.5 SFRSYM    DATA     BIT       GP15
      00000080H.6 SFRSYM    DATA     BIT       GP06
      00000088H   SFRSYM    DATA     BIT       IT00

      01001D11H   BLOCK     CODE     ---       LVL=0
      00000006H   SYMBOL    DATA     WORD      Xn1
      00000004H   SYMBOL    DATA     WORD      Xn0
      00000002H   SYMBOL    DATA     WORD      K
      01001D11H   LINE      CODE     ---       #26
      01001D11H   LINE      CODE     ---       #27
      01001D11H   LINE      CODE     ---       #28
      01001D15H   LINE      CODE     ---       #29
      01001D19H   LINE      CODE     ---       #30
      01001D21H   LINE      CODE     ---       #31
      01001D24H   LINE      CODE     ---       #32
      01001D29H   LINE      CODE     ---       #33
      01001D2EH   LINE      CODE     ---       #34
      01001D32H   LINE      CODE     ---       #35
      ---         BLOCKEND  ---      ---       LVL=0

      ---         MODULE    ---      ---       BUZZERSCAN
      0200018CH   PUBLIC    XDATA    ---       BZScan
      01001B54H   PUBLIC    CODE     ---       BuzzerScan
      0100003EH   PUBLIC    CODE     ---       BuzzerInit
      000000E2H   SFRSYM    DATA     BYTE      SV_USL
      000000ABH   SFRSYM    DATA     BYTE      TIM2_CNTRH
      000000B0H.4 SFRSYM    DATA     BIT       GP34
      000000A0H.5 SFRSYM    DATA     BIT       GP25
      00000090H.6 SFRSYM    DATA     BIT       GP16
      00000080H.7 SFRSYM    DATA     BIT       GP07
      00000088H.1 SFRSYM    DATA     BIT       IT01
      00000088H.3 SFRSYM    DATA     BIT       IT10
      000000F6H   SFRSYM    DATA     WORD      PI_UKMIN
      000000C2H   SFRSYM    DATA     WORD      MD_MA
      000000A3H   SFRSYM    DATA     BYTE      TIM3_CNTRH
      000000B0H.5 SFRSYM    DATA     BIT       GP35
LX51 LINKER/LOCATER V4.66.1.0                                                         03/23/2017  15:15:44  PAGE 60


      000000A0H.6 SFRSYM    DATA     BIT       GP26
      00000090H.7 SFRSYM    DATA     BIT       GP17
      00000080H   SFRSYM    DATA     BYTE      P0
      00000088H.4 SFRSYM    DATA     BIT       IT11
      000000CAH   SFRSYM    DATA     WORD      MD_MB
      00000093H   SFRSYM    DATA     BYTE      TIM4_CNTRH
      000000B0H.6 SFRSYM    DATA     BIT       GP36
      000000A0H.7 SFRSYM    DATA     BIT       GP27
      00000090H   SFRSYM    DATA     BYTE      P1
      000000D9H   SFRSYM    DATA     BYTE      EVT_FILT
      000000F4H   SFRSYM    DATA     WORD      PI_UKMAX
      0000008BH   SFRSYM    DATA     BYTE      TIM5_CNTRH
      000000B2H   SFRSYM    DATA     BYTE      TIM2_CMTRL
      000000B0H.7 SFRSYM    DATA     BIT       GP37
      000000A0H   SFRSYM    DATA     BYTE      P2
      000000AAH   SFRSYM    DATA     BYTE      TIM2_CNTRL
      000000B0H   SFRSYM    DATA     BYTE      P3
      000000A2H   SFRSYM    DATA     BYTE      TIM3_CNTRL
      000000D0H.6 SFRSYM    DATA     BIT       AC
      00000092H   SFRSYM    DATA     BYTE      TIM4_CNTRL
      0000008AH   SFRSYM    DATA     BYTE      TIM5_CNTRL
      000000B6H   SFRSYM    DATA     WORD      TIM0_CCR1
      000000A8H.7 SFRSYM    DATA     BIT       EA
      000000D5H   SFRSYM    DATA     BYTE      CMP_CR0
      000000BAH   SFRSYM    DATA     WORD      TIM0_CCR2
      000000D6H   SFRSYM    DATA     BYTE      CMP_CR1
      000000BCH   SFRSYM    DATA     WORD      TIM0_CCR3
      00000085H   SFRSYM    DATA     BYTE      PSCTL
      000000DAH   SFRSYM    DATA     BYTE      CMP_CR2
      000000BEH   SFRSYM    DATA     WORD      TIM0_CCR4
      000000B8H.2 SFRSYM    DATA     BIT       PX00
      000000EAH   SFRSYM    DATA     WORD      PI_EK
      000000F8H   SFRSYM    DATA     BIT       OISUH
      000000B8H.3 SFRSYM    DATA     BIT       PX01
      000000B8H.4 SFRSYM    DATA     BIT       PX10
      000000F8H.2 SFRSYM    DATA     BIT       OISVH
      000000B8H.5 SFRSYM    DATA     BIT       PX11
      000000F8H.4 SFRSYM    DATA     BIT       OISWH
      000000DCH   SFRSYM    DATA     WORD      LPF_K
      000000F2H   SFRSYM    DATA     WORD      PI_KI
      000000F8H.1 SFRSYM    DATA     BIT       OISUL
      000000A8H   SFRSYM    DATA     BYTE      IE
      000000F8H.3 SFRSYM    DATA     BIT       OISVL
      000000F8H.5 SFRSYM    DATA     BIT       OISWL
      000000D1H   SFRSYM    DATA     BYTE      P1IE
      00000098H.6 SFRSYM    DATA     BIT       MOD0
      000000D3H   SFRSYM    DATA     BYTE      P2IE
      000000D2H   SFRSYM    DATA     BYTE      P1IF
      000000F9H   SFRSYM    DATA     BYTE      PL_CR
      00000098H.7 SFRSYM    DATA     BIT       MOD1
      000000D4H   SFRSYM    DATA     BYTE      P2IF
      000000ACH   SFRSYM    DATA     WORD      TIM2_DR
      00000082H   SFRSYM    DATA     WORD      DP
      000000EEH   SFRSYM    DATA     WORD      PI_KP
      000000A4H   SFRSYM    DATA     WORD      TIM3_DR
      00000094H   SFRSYM    DATA     WORD      TIM4_DR
      0000008CH   SFRSYM    DATA     WORD      TIM5_DR
      000000F1H   SFRSYM    DATA     BYTE      OSC_CFG
      000000C1H   SFRSYM    DATA     BYTE      MD_MODE
      000000ECH   SFRSYM    DATA     WORD      PI_UK
      000000DEH   SFRSYM    DATA     WORD      LPF_X
      00000098H   SFRSYM    DATA     BIT       RI
      000000E6H   SFRSYM    DATA     WORD      LPF_Y
      000000C0H   SFRSYM    DATA     BIT       PTIM00
      000000D0H.7 SFRSYM    DATA     BIT       CY
LX51 LINKER/LOCATER V4.66.1.0                                                         03/23/2017  15:15:44  PAGE 61


      00000098H.1 SFRSYM    DATA     BIT       TI
      000000C0H.1 SFRSYM    DATA     BIT       PTIM01
      000000C0H.2 SFRSYM    DATA     BIT       PTIM10
      000000C0H.3 SFRSYM    DATA     BIT       PTIM11
      000000E1H   SFRSYM    DATA     BYTE      SV_CR
      00000098H   SFRSYM    DATA     BYTE      UT_CR
      00000099H   SFRSYM    DATA     BYTE      UT_DR
      000000F8H.6 SFRSYM    DATA     BIT       OIS4
      00000081H   SFRSYM    DATA     BYTE      SP
      000000D0H.2 SFRSYM    DATA     BIT       OV
      000000C4H   SFRSYM    DATA     BYTE      MD_DA0
      0000009AH   SFRSYM    DATA     WORD      UT_BAUD
      000000CCH   SFRSYM    DATA     BYTE      MD_DB0
      000000C5H   SFRSYM    DATA     BYTE      MD_DA1
      000000CDH   SFRSYM    DATA     BYTE      MD_DB1
      000000C6H   SFRSYM    DATA     BYTE      MD_DA2
      000000CEH   SFRSYM    DATA     BYTE      MD_DB2
      000000C7H   SFRSYM    DATA     BYTE      MD_DA3
      000000B4H   SFRSYM    DATA     WORD      TIM2_ADTR
      000000CFH   SFRSYM    DATA     BYTE      MD_DB3
      000000AFH   SFRSYM    DATA     BYTE      TIM2_ARRH
      000000A7H   SFRSYM    DATA     BYTE      TIM3_ARRH
      00000097H   SFRSYM    DATA     BYTE      TIM4_ARRH
      0000008FH   SFRSYM    DATA     BYTE      TIM5_ARRH
      000000AEH   SFRSYM    DATA     BYTE      TIM2_ARRL
      000000A6H   SFRSYM    DATA     BYTE      TIM3_ARRL
      00000087H   SFRSYM    DATA     BYTE      PCON
      000000E2H   SFRSYM    DATA     WORD      SV_US
      00000096H   SFRSYM    DATA     BYTE      TIM4_ARRL
      0000008EH   SFRSYM    DATA     BYTE      TIM5_ARRL
      000000B2H   SFRSYM    DATA     WORD      TIM2_CMTR
      00000088H   SFRSYM    DATA     BYTE      TCON
      000000AAH   SFRSYM    DATA     WORD      TIM2_CNTR
      000000A2H   SFRSYM    DATA     WORD      TIM3_CNTR
      00000092H   SFRSYM    DATA     WORD      TIM4_CNTR
      0000008AH   SFRSYM    DATA     WORD      TIM5_CNTR
      000000E5H   SFRSYM    DATA     BYTE      SV_ANGLEH
      000000D8H   SFRSYM    DATA     BIT       PUART0
      000000E4H   SFRSYM    DATA     BYTE      SV_ANGLEL
      000000C6H   SFRSYM    DATA     WORD      MD_DAH
      000000D8H.1 SFRSYM    DATA     BIT       PUART1
      000000D8H.2 SFRSYM    DATA     BIT       PI2C0
      00000088H.2 SFRSYM    DATA     BIT       IF0
      000000CEH   SFRSYM    DATA     WORD      MD_DBH
      000000D8H.3 SFRSYM    DATA     BIT       PI2C1
      000000F0H   SFRSYM    DATA     BYTE      B
      000000C4H   SFRSYM    DATA     WORD      MD_DAL
      000000A1H   SFRSYM    DATA     BYTE      TIM2_CR0
      000000CCH   SFRSYM    DATA     WORD      MD_DBL
      0000009CH   SFRSYM    DATA     BYTE      TIM3_CR0
      000000A9H   SFRSYM    DATA     BYTE      TIM2_CR1
      0000009EH   SFRSYM    DATA     BYTE      TIM4_CR0
      0000009DH   SFRSYM    DATA     BYTE      TIM3_CR1
      00000089H   SFRSYM    DATA     BYTE      TIM5_CR0
      0000009FH   SFRSYM    DATA     BYTE      TIM4_CR1
      000000F8H   SFRSYM    DATA     BYTE      DRV_OUT
      00000091H   SFRSYM    DATA     BYTE      TIM5_CR1
      000000E0H   SFRSYM    DATA     BYTE      ACC
      000000F7H   SFRSYM    DATA     BYTE      PI_UKMINH
      000000C3H   SFRSYM    DATA     BYTE      MD_MAH
      000000A8H.4 SFRSYM    DATA     BIT       ES0
      000000DBH   SFRSYM    DATA     BYTE      LVSR
      000000CBH   SFRSYM    DATA     BYTE      MD_MBH
      000000C0H.4 SFRSYM    DATA     BIT       PADC0
      000000B8H   SFRSYM    DATA     BYTE      IP0
LX51 LINKER/LOCATER V4.66.1.0                                                         03/23/2017  15:15:44  PAGE 62


      000000F5H   SFRSYM    DATA     BYTE      PI_UKMAXH
      000000C0H.5 SFRSYM    DATA     BIT       PADC1
      000000C0H   SFRSYM    DATA     BYTE      IP1
      000000C8H   SFRSYM    DATA     BYTE      IP2
      000000F6H   SFRSYM    DATA     BYTE      PI_UKMINL
      000000C2H   SFRSYM    DATA     BYTE      MD_MAL
      00000098H.2 SFRSYM    DATA     BIT       RB8
      000000D8H   SFRSYM    DATA     BYTE      IP3
      000000CAH   SFRSYM    DATA     BYTE      MD_MBL
      000000A8H   SFRSYM    DATA     BIT       EX0
      000000F4H   SFRSYM    DATA     BYTE      PI_UKMAXL
      00000098H.3 SFRSYM    DATA     BIT       TB8
      000000B7H   SFRSYM    DATA     BYTE      TIM0_CCR1H
      000000A8H.2 SFRSYM    DATA     BIT       EX1
      000000BBH   SFRSYM    DATA     BYTE      TIM0_CCR2H
      000000D0H   SFRSYM    DATA     BIT       P
      000000BDH   SFRSYM    DATA     BYTE      TIM0_CCR3H
      000000BFH   SFRSYM    DATA     BYTE      TIM0_CCR4H
      000000C8H.2 SFRSYM    DATA     BIT       PTIM230
      000000EBH   SFRSYM    DATA     BYTE      PI_EKH
      00000098H.5 SFRSYM    DATA     BIT       SM2
      000000B6H   SFRSYM    DATA     BYTE      TIM0_CCR1L
      000000B1H   SFRSYM    DATA     BYTE      TIM0_SR1
      000000C8H.3 SFRSYM    DATA     BIT       PTIM231
      000000BAH   SFRSYM    DATA     BYTE      TIM0_CCR2L
      000000BCH   SFRSYM    DATA     BYTE      TIM0_CCR3L
      000000BEH   SFRSYM    DATA     BYTE      TIM0_CCR4L
      000000D8H.6 SFRSYM    DATA     BIT       PMCD0
      000000C8H.4 SFRSYM    DATA     BIT       PTIM450
      000000D0H.3 SFRSYM    DATA     BIT       RS0
      000000DDH   SFRSYM    DATA     BYTE      LPF_KH
      000000F3H   SFRSYM    DATA     BYTE      PI_KIH
      000000EAH   SFRSYM    DATA     BYTE      PI_EKL
      000000E8H   SFRSYM    DATA     BYTE      FOC_SET0
      000000D8H.7 SFRSYM    DATA     BIT       PMCD1
      000000C8H.5 SFRSYM    DATA     BIT       PTIM451
      000000D0H.4 SFRSYM    DATA     BIT       RS1
      000000E9H   SFRSYM    DATA     BYTE      FOC_SET1
      000000B8H.6 SFRSYM    DATA     BIT       PFOC0
      000000DCH   SFRSYM    DATA     BYTE      LPF_KL
      000000F2H   SFRSYM    DATA     BYTE      PI_KIL
      000000B8H.7 SFRSYM    DATA     BIT       PFOC1
      000000ADH   SFRSYM    DATA     BYTE      TIM2_DRH
      000000B9H   SFRSYM    DATA     BYTE      TIM0_IER
      00000083H   SFRSYM    DATA     BYTE      DPH
      000000EFH   SFRSYM    DATA     BYTE      PI_KPH
      000000A5H   SFRSYM    DATA     BYTE      TIM3_DRH
      00000095H   SFRSYM    DATA     BYTE      TIM4_DRH
      0000008DH   SFRSYM    DATA     BYTE      TIM5_DRH
      000000ACH   SFRSYM    DATA     BYTE      TIM2_DRL
      00000082H   SFRSYM    DATA     BYTE      DPL
      000000EEH   SFRSYM    DATA     BYTE      PI_KPL
      000000A4H   SFRSYM    DATA     BYTE      TIM3_DRL
      000000F8H.7 SFRSYM    DATA     BIT       MOE
      000000C0H.6 SFRSYM    DATA     BIT       PCMP0
      000000EDH   SFRSYM    DATA     BYTE      PI_UKH
      00000094H   SFRSYM    DATA     BYTE      TIM4_DRL
      000000C0H.7 SFRSYM    DATA     BIT       PCMP1
      000000DFH   SFRSYM    DATA     BYTE      LPF_XH
      0000008CH   SFRSYM    DATA     BYTE      TIM5_DRL
      000000AEH   SFRSYM    DATA     WORD      TIM2_ARR
      000000A8H.5 SFRSYM    DATA     BIT       MCDIE
      000000C9H   SFRSYM    DATA     BYTE      RSTSRC
      000000E7H   SFRSYM    DATA     BYTE      LPF_YH
      000000A6H   SFRSYM    DATA     WORD      TIM3_ARR
LX51 LINKER/LOCATER V4.66.1.0                                                         03/23/2017  15:15:44  PAGE 63


      00000088H.6 SFRSYM    DATA     BIT       MCDIF
      00000098H.4 SFRSYM    DATA     BIT       REN
      00000096H   SFRSYM    DATA     WORD      TIM4_ARR
      000000ECH   SFRSYM    DATA     BYTE      PI_UKL
      000000D7H   SFRSYM    DATA     BYTE      CMP_SR
      0000008EH   SFRSYM    DATA     WORD      TIM5_ARR
      000000DEH   SFRSYM    DATA     BYTE      LPF_XL
      000000E6H   SFRSYM    DATA     BYTE      LPF_YL
      000000C8H   SFRSYM    DATA     BIT       PRTC0
      000000C8H.1 SFRSYM    DATA     BIT       PRTC1
      000000E8H.7 SFRSYM    DATA     BIT       FOCEN
      000000C8H.6 SFRSYM    DATA     BIT       PTSD0
      000000D8H.4 SFRSYM    DATA     BIT       PSPI0
      000000C8H.7 SFRSYM    DATA     BIT       PTSD1
      000000D8H.5 SFRSYM    DATA     BIT       PSPI1
      0000009BH   SFRSYM    DATA     BYTE      UT_BAUDH
      000000E4H   SFRSYM    DATA     WORD      SV_ANGLE
      000000B5H   SFRSYM    DATA     BYTE      TIM2_ADTRH
      0000009AH   SFRSYM    DATA     BYTE      UT_BAUDL
      000000FCH   SFRSYM    DATA     BYTE      P0_OE
      000000FDH   SFRSYM    DATA     BYTE      P1_OE
      000000D0H.5 SFRSYM    DATA     BIT       F0
      000000B4H   SFRSYM    DATA     BYTE      TIM2_ADTRL
      000000FEH   SFRSYM    DATA     BYTE      P2_OE
      000000D0H.1 SFRSYM    DATA     BIT       F1
      00000080H   SFRSYM    DATA     BIT       GP00
      000000FFH   SFRSYM    DATA     BYTE      P3_OE
      00000090H   SFRSYM    DATA     BIT       GP10
      00000080H.1 SFRSYM    DATA     BIT       GP01
      000000A8H.6 SFRSYM    DATA     BIT       RTCIE
      000000A0H   SFRSYM    DATA     BIT       GP20
      00000090H.1 SFRSYM    DATA     BIT       GP11
      00000080H.2 SFRSYM    DATA     BIT       GP02
      000000E3H   SFRSYM    DATA     BYTE      SV_USH
      000000B0H   SFRSYM    DATA     BIT       GP30
      000000A0H.1 SFRSYM    DATA     BIT       GP21
      00000090H.2 SFRSYM    DATA     BIT       GP12
      00000080H.3 SFRSYM    DATA     BIT       GP03
      000000B8H   SFRSYM    DATA     BIT       PLVW0
      000000A8H.1 SFRSYM    DATA     BIT       TSDIE
      000000D0H   SFRSYM    DATA     BYTE      PSW
      000000B0H.1 SFRSYM    DATA     BIT       GP31
      000000A0H.2 SFRSYM    DATA     BIT       GP22
      00000090H.3 SFRSYM    DATA     BIT       GP13
      00000080H.4 SFRSYM    DATA     BIT       GP04
      000000B8H.1 SFRSYM    DATA     BIT       PLVW1
      000000A8H.3 SFRSYM    DATA     BIT       SPIIE
      00000088H.5 SFRSYM    DATA     BIT       TSDIF
      000000B0H.2 SFRSYM    DATA     BIT       GP32
      000000A0H.3 SFRSYM    DATA     BIT       GP23
      00000090H.4 SFRSYM    DATA     BIT       GP14
      00000080H.5 SFRSYM    DATA     BIT       GP05
      00000084H   SFRSYM    DATA     BYTE      FLKEY
      000000B3H   SFRSYM    DATA     BYTE      TIM2_CMTRH
      000000B0H.3 SFRSYM    DATA     BIT       GP33
      000000A0H.4 SFRSYM    DATA     BIT       GP24
      00000090H.5 SFRSYM    DATA     BIT       GP15
      00000080H.6 SFRSYM    DATA     BIT       GP06
      00000088H   SFRSYM    DATA     BIT       IT00

      0100003EH   BLOCK     CODE     ---       LVL=0
      0100003EH   LINE      CODE     ---       #25
      0100003EH   LINE      CODE     ---       #26
      0100003EH   LINE      CODE     ---       #27
      01000043H   LINE      CODE     ---       #28
LX51 LINKER/LOCATER V4.66.1.0                                                         03/23/2017  15:15:44  PAGE 64


      01000045H   LINE      CODE     ---       #29
      01000049H   LINE      CODE     ---       #30
      ---         BLOCKEND  ---      ---       LVL=0

      01001B54H   BLOCK     CODE     ---       LVL=0
      01001B54H   LINE      CODE     ---       #39
      01001B54H   LINE      CODE     ---       #40
      01001B54H   LINE      CODE     ---       #41
      01001B5AH   LINE      CODE     ---       #42
      01001B5AH   LINE      CODE     ---       #43
      01001B5AH   LINE      CODE     ---       #44
      01001B60H   LINE      CODE     ---       #45
      01001B60H   LINE      CODE     ---       #46
      01001B62H   LINE      CODE     ---       #47
      01001B70H   LINE      CODE     ---       #48
      01001B7FH   LINE      CODE     ---       #49
      01001B7FH   LINE      CODE     ---       #50
      01001B83H   LINE      CODE     ---       #51
      01001B85H   LINE      CODE     ---       #52
      01001B89H   LINE      CODE     ---       #53
      01001B89H   LINE      CODE     ---       #54
      01001B89H   LINE      CODE     ---       #55
      01001B89H   LINE      CODE     ---       #56
      01001B89H   LINE      CODE     ---       #57
      01001B89H   LINE      CODE     ---       #58
      01001B89H   LINE      CODE     ---       #59
      01001B89H   LINE      CODE     ---       #60
      01001B89H   LINE      CODE     ---       #61
      01001B89H   LINE      CODE     ---       #62
      01001B89H   LINE      CODE     ---       #63
      01001B89H   LINE      CODE     ---       #64
      01001B89H   LINE      CODE     ---       #66
      ---         BLOCKEND  ---      ---       LVL=0

      ---         MODULE    ---      ---       IRSCAN
      02000136H   PUBLIC    XDATA    ---       IRScan
      0200012DH   PUBLIC    XDATA    ---       IRControl
      01000F01H   PUBLIC    CODE     ---       IRScanControl
      01001C1CH   PUBLIC    CODE     ---       IRInit
      000000E2H   SFRSYM    DATA     BYTE      SV_USL
      000000ABH   SFRSYM    DATA     BYTE      TIM2_CNTRH
      000000B0H.4 SFRSYM    DATA     BIT       GP34
      000000A0H.5 SFRSYM    DATA     BIT       GP25
      00000090H.6 SFRSYM    DATA     BIT       GP16
      00000080H.7 SFRSYM    DATA     BIT       GP07
      00000088H.1 SFRSYM    DATA     BIT       IT01
      00000088H.3 SFRSYM    DATA     BIT       IT10
      000000F6H   SFRSYM    DATA     WORD      PI_UKMIN
      000000C2H   SFRSYM    DATA     WORD      MD_MA
      000000A3H   SFRSYM    DATA     BYTE      TIM3_CNTRH
      000000B0H.5 SFRSYM    DATA     BIT       GP35
      000000A0H.6 SFRSYM    DATA     BIT       GP26
      00000090H.7 SFRSYM    DATA     BIT       GP17
      00000080H   SFRSYM    DATA     BYTE      P0
      00000088H.4 SFRSYM    DATA     BIT       IT11
      000000CAH   SFRSYM    DATA     WORD      MD_MB
      00000093H   SFRSYM    DATA     BYTE      TIM4_CNTRH
      000000B0H.6 SFRSYM    DATA     BIT       GP36
      000000A0H.7 SFRSYM    DATA     BIT       GP27
      00000090H   SFRSYM    DATA     BYTE      P1
      000000D9H   SFRSYM    DATA     BYTE      EVT_FILT
      000000F4H   SFRSYM    DATA     WORD      PI_UKMAX
      0000008BH   SFRSYM    DATA     BYTE      TIM5_CNTRH
      000000B2H   SFRSYM    DATA     BYTE      TIM2_CMTRL
      000000B0H.7 SFRSYM    DATA     BIT       GP37
LX51 LINKER/LOCATER V4.66.1.0                                                         03/23/2017  15:15:44  PAGE 65


      000000A0H   SFRSYM    DATA     BYTE      P2
      000000AAH   SFRSYM    DATA     BYTE      TIM2_CNTRL
      000000B0H   SFRSYM    DATA     BYTE      P3
      000000A2H   SFRSYM    DATA     BYTE      TIM3_CNTRL
      000000D0H.6 SFRSYM    DATA     BIT       AC
      00000092H   SFRSYM    DATA     BYTE      TIM4_CNTRL
      0000008AH   SFRSYM    DATA     BYTE      TIM5_CNTRL
      000000B6H   SFRSYM    DATA     WORD      TIM0_CCR1
      000000A8H.7 SFRSYM    DATA     BIT       EA
      000000D5H   SFRSYM    DATA     BYTE      CMP_CR0
      000000BAH   SFRSYM    DATA     WORD      TIM0_CCR2
      000000D6H   SFRSYM    DATA     BYTE      CMP_CR1
      000000BCH   SFRSYM    DATA     WORD      TIM0_CCR3
      00000085H   SFRSYM    DATA     BYTE      PSCTL
      000000DAH   SFRSYM    DATA     BYTE      CMP_CR2
      000000BEH   SFRSYM    DATA     WORD      TIM0_CCR4
      000000B8H.2 SFRSYM    DATA     BIT       PX00
      000000EAH   SFRSYM    DATA     WORD      PI_EK
      000000F8H   SFRSYM    DATA     BIT       OISUH
      000000B8H.3 SFRSYM    DATA     BIT       PX01
      000000B8H.4 SFRSYM    DATA     BIT       PX10
      000000F8H.2 SFRSYM    DATA     BIT       OISVH
      000000B8H.5 SFRSYM    DATA     BIT       PX11
      000000F8H.4 SFRSYM    DATA     BIT       OISWH
      000000DCH   SFRSYM    DATA     WORD      LPF_K
      000000F2H   SFRSYM    DATA     WORD      PI_KI
      000000F8H.1 SFRSYM    DATA     BIT       OISUL
      000000A8H   SFRSYM    DATA     BYTE      IE
      000000F8H.3 SFRSYM    DATA     BIT       OISVL
      000000F8H.5 SFRSYM    DATA     BIT       OISWL
      000000D1H   SFRSYM    DATA     BYTE      P1IE
      00000098H.6 SFRSYM    DATA     BIT       MOD0
      000000D3H   SFRSYM    DATA     BYTE      P2IE
      000000D2H   SFRSYM    DATA     BYTE      P1IF
      000000F9H   SFRSYM    DATA     BYTE      PL_CR
      00000098H.7 SFRSYM    DATA     BIT       MOD1
      000000D4H   SFRSYM    DATA     BYTE      P2IF
      000000ACH   SFRSYM    DATA     WORD      TIM2_DR
      00000082H   SFRSYM    DATA     WORD      DP
      000000EEH   SFRSYM    DATA     WORD      PI_KP
      000000A4H   SFRSYM    DATA     WORD      TIM3_DR
      00000094H   SFRSYM    DATA     WORD      TIM4_DR
      0000008CH   SFRSYM    DATA     WORD      TIM5_DR
      000000F1H   SFRSYM    DATA     BYTE      OSC_CFG
      000000C1H   SFRSYM    DATA     BYTE      MD_MODE
      000000ECH   SFRSYM    DATA     WORD      PI_UK
      000000DEH   SFRSYM    DATA     WORD      LPF_X
      00000098H   SFRSYM    DATA     BIT       RI
      000000E6H   SFRSYM    DATA     WORD      LPF_Y
      000000C0H   SFRSYM    DATA     BIT       PTIM00
      000000D0H.7 SFRSYM    DATA     BIT       CY
      00000098H.1 SFRSYM    DATA     BIT       TI
      000000C0H.1 SFRSYM    DATA     BIT       PTIM01
      000000C0H.2 SFRSYM    DATA     BIT       PTIM10
      000000C0H.3 SFRSYM    DATA     BIT       PTIM11
      000000E1H   SFRSYM    DATA     BYTE      SV_CR
      00000098H   SFRSYM    DATA     BYTE      UT_CR
      00000099H   SFRSYM    DATA     BYTE      UT_DR
      000000F8H.6 SFRSYM    DATA     BIT       OIS4
      00000081H   SFRSYM    DATA     BYTE      SP
      000000D0H.2 SFRSYM    DATA     BIT       OV
      000000C4H   SFRSYM    DATA     BYTE      MD_DA0
      0000009AH   SFRSYM    DATA     WORD      UT_BAUD
      000000CCH   SFRSYM    DATA     BYTE      MD_DB0
      000000C5H   SFRSYM    DATA     BYTE      MD_DA1
LX51 LINKER/LOCATER V4.66.1.0                                                         03/23/2017  15:15:44  PAGE 66


      000000CDH   SFRSYM    DATA     BYTE      MD_DB1
      000000C6H   SFRSYM    DATA     BYTE      MD_DA2
      000000CEH   SFRSYM    DATA     BYTE      MD_DB2
      000000C7H   SFRSYM    DATA     BYTE      MD_DA3
      000000B4H   SFRSYM    DATA     WORD      TIM2_ADTR
      000000CFH   SFRSYM    DATA     BYTE      MD_DB3
      000000AFH   SFRSYM    DATA     BYTE      TIM2_ARRH
      000000A7H   SFRSYM    DATA     BYTE      TIM3_ARRH
      00000097H   SFRSYM    DATA     BYTE      TIM4_ARRH
      0000008FH   SFRSYM    DATA     BYTE      TIM5_ARRH
      000000AEH   SFRSYM    DATA     BYTE      TIM2_ARRL
      000000A6H   SFRSYM    DATA     BYTE      TIM3_ARRL
      00000087H   SFRSYM    DATA     BYTE      PCON
      000000E2H   SFRSYM    DATA     WORD      SV_US
      00000096H   SFRSYM    DATA     BYTE      TIM4_ARRL
      0000008EH   SFRSYM    DATA     BYTE      TIM5_ARRL
      000000B2H   SFRSYM    DATA     WORD      TIM2_CMTR
      00000088H   SFRSYM    DATA     BYTE      TCON
      000000AAH   SFRSYM    DATA     WORD      TIM2_CNTR
      000000A2H   SFRSYM    DATA     WORD      TIM3_CNTR
      00000092H   SFRSYM    DATA     WORD      TIM4_CNTR
      0000008AH   SFRSYM    DATA     WORD      TIM5_CNTR
      000000E5H   SFRSYM    DATA     BYTE      SV_ANGLEH
      000000D8H   SFRSYM    DATA     BIT       PUART0
      000000E4H   SFRSYM    DATA     BYTE      SV_ANGLEL
      000000C6H   SFRSYM    DATA     WORD      MD_DAH
      000000D8H.1 SFRSYM    DATA     BIT       PUART1
      000000D8H.2 SFRSYM    DATA     BIT       PI2C0
      00000088H.2 SFRSYM    DATA     BIT       IF0
      000000CEH   SFRSYM    DATA     WORD      MD_DBH
      000000D8H.3 SFRSYM    DATA     BIT       PI2C1
      000000F0H   SFRSYM    DATA     BYTE      B
      000000C4H   SFRSYM    DATA     WORD      MD_DAL
      000000A1H   SFRSYM    DATA     BYTE      TIM2_CR0
      000000CCH   SFRSYM    DATA     WORD      MD_DBL
      0000009CH   SFRSYM    DATA     BYTE      TIM3_CR0
      000000A9H   SFRSYM    DATA     BYTE      TIM2_CR1
      0000009EH   SFRSYM    DATA     BYTE      TIM4_CR0
      0000009DH   SFRSYM    DATA     BYTE      TIM3_CR1
      00000089H   SFRSYM    DATA     BYTE      TIM5_CR0
      0000009FH   SFRSYM    DATA     BYTE      TIM4_CR1
      000000F8H   SFRSYM    DATA     BYTE      DRV_OUT
      00000091H   SFRSYM    DATA     BYTE      TIM5_CR1
      000000E0H   SFRSYM    DATA     BYTE      ACC
      000000F7H   SFRSYM    DATA     BYTE      PI_UKMINH
      000000C3H   SFRSYM    DATA     BYTE      MD_MAH
      000000A8H.4 SFRSYM    DATA     BIT       ES0
      000000DBH   SFRSYM    DATA     BYTE      LVSR
      000000CBH   SFRSYM    DATA     BYTE      MD_MBH
      000000C0H.4 SFRSYM    DATA     BIT       PADC0
      000000B8H   SFRSYM    DATA     BYTE      IP0
      000000F5H   SFRSYM    DATA     BYTE      PI_UKMAXH
      000000C0H.5 SFRSYM    DATA     BIT       PADC1
      000000C0H   SFRSYM    DATA     BYTE      IP1
      000000C8H   SFRSYM    DATA     BYTE      IP2
      000000F6H   SFRSYM    DATA     BYTE      PI_UKMINL
      000000C2H   SFRSYM    DATA     BYTE      MD_MAL
      00000098H.2 SFRSYM    DATA     BIT       RB8
      000000D8H   SFRSYM    DATA     BYTE      IP3
      000000CAH   SFRSYM    DATA     BYTE      MD_MBL
      000000A8H   SFRSYM    DATA     BIT       EX0
      000000F4H   SFRSYM    DATA     BYTE      PI_UKMAXL
      00000098H.3 SFRSYM    DATA     BIT       TB8
      000000B7H   SFRSYM    DATA     BYTE      TIM0_CCR1H
      000000A8H.2 SFRSYM    DATA     BIT       EX1
LX51 LINKER/LOCATER V4.66.1.0                                                         03/23/2017  15:15:44  PAGE 67


      000000BBH   SFRSYM    DATA     BYTE      TIM0_CCR2H
      000000D0H   SFRSYM    DATA     BIT       P
      000000BDH   SFRSYM    DATA     BYTE      TIM0_CCR3H
      000000BFH   SFRSYM    DATA     BYTE      TIM0_CCR4H
      000000C8H.2 SFRSYM    DATA     BIT       PTIM230
      000000EBH   SFRSYM    DATA     BYTE      PI_EKH
      00000098H.5 SFRSYM    DATA     BIT       SM2
      000000B6H   SFRSYM    DATA     BYTE      TIM0_CCR1L
      000000B1H   SFRSYM    DATA     BYTE      TIM0_SR1
      000000C8H.3 SFRSYM    DATA     BIT       PTIM231
      000000BAH   SFRSYM    DATA     BYTE      TIM0_CCR2L
      000000BCH   SFRSYM    DATA     BYTE      TIM0_CCR3L
      000000BEH   SFRSYM    DATA     BYTE      TIM0_CCR4L
      000000D8H.6 SFRSYM    DATA     BIT       PMCD0
      000000C8H.4 SFRSYM    DATA     BIT       PTIM450
      000000D0H.3 SFRSYM    DATA     BIT       RS0
      000000DDH   SFRSYM    DATA     BYTE      LPF_KH
      000000F3H   SFRSYM    DATA     BYTE      PI_KIH
      000000EAH   SFRSYM    DATA     BYTE      PI_EKL
      000000E8H   SFRSYM    DATA     BYTE      FOC_SET0
      000000D8H.7 SFRSYM    DATA     BIT       PMCD1
      000000C8H.5 SFRSYM    DATA     BIT       PTIM451
      000000D0H.4 SFRSYM    DATA     BIT       RS1
      000000E9H   SFRSYM    DATA     BYTE      FOC_SET1
      000000B8H.6 SFRSYM    DATA     BIT       PFOC0
      000000DCH   SFRSYM    DATA     BYTE      LPF_KL
      000000F2H   SFRSYM    DATA     BYTE      PI_KIL
      000000B8H.7 SFRSYM    DATA     BIT       PFOC1
      000000ADH   SFRSYM    DATA     BYTE      TIM2_DRH
      000000B9H   SFRSYM    DATA     BYTE      TIM0_IER
      00000083H   SFRSYM    DATA     BYTE      DPH
      000000EFH   SFRSYM    DATA     BYTE      PI_KPH
      000000A5H   SFRSYM    DATA     BYTE      TIM3_DRH
      00000095H   SFRSYM    DATA     BYTE      TIM4_DRH
      0000008DH   SFRSYM    DATA     BYTE      TIM5_DRH
      000000ACH   SFRSYM    DATA     BYTE      TIM2_DRL
      00000082H   SFRSYM    DATA     BYTE      DPL
      000000EEH   SFRSYM    DATA     BYTE      PI_KPL
      000000A4H   SFRSYM    DATA     BYTE      TIM3_DRL
      000000F8H.7 SFRSYM    DATA     BIT       MOE
      000000C0H.6 SFRSYM    DATA     BIT       PCMP0
      000000EDH   SFRSYM    DATA     BYTE      PI_UKH
      00000094H   SFRSYM    DATA     BYTE      TIM4_DRL
      000000C0H.7 SFRSYM    DATA     BIT       PCMP1
      000000DFH   SFRSYM    DATA     BYTE      LPF_XH
      0000008CH   SFRSYM    DATA     BYTE      TIM5_DRL
      000000AEH   SFRSYM    DATA     WORD      TIM2_ARR
      000000A8H.5 SFRSYM    DATA     BIT       MCDIE
      000000C9H   SFRSYM    DATA     BYTE      RSTSRC
      000000E7H   SFRSYM    DATA     BYTE      LPF_YH
      000000A6H   SFRSYM    DATA     WORD      TIM3_ARR
      00000088H.6 SFRSYM    DATA     BIT       MCDIF
      00000098H.4 SFRSYM    DATA     BIT       REN
      00000096H   SFRSYM    DATA     WORD      TIM4_ARR
      000000ECH   SFRSYM    DATA     BYTE      PI_UKL
      000000D7H   SFRSYM    DATA     BYTE      CMP_SR
      0000008EH   SFRSYM    DATA     WORD      TIM5_ARR
      000000DEH   SFRSYM    DATA     BYTE      LPF_XL
      000000E6H   SFRSYM    DATA     BYTE      LPF_YL
      000000C8H   SFRSYM    DATA     BIT       PRTC0
      000000C8H.1 SFRSYM    DATA     BIT       PRTC1
      000000E8H.7 SFRSYM    DATA     BIT       FOCEN
      000000C8H.6 SFRSYM    DATA     BIT       PTSD0
      000000D8H.4 SFRSYM    DATA     BIT       PSPI0
      000000C8H.7 SFRSYM    DATA     BIT       PTSD1
LX51 LINKER/LOCATER V4.66.1.0                                                         03/23/2017  15:15:44  PAGE 68


      000000D8H.5 SFRSYM    DATA     BIT       PSPI1
      0000009BH   SFRSYM    DATA     BYTE      UT_BAUDH
      000000E4H   SFRSYM    DATA     WORD      SV_ANGLE
      000000B5H   SFRSYM    DATA     BYTE      TIM2_ADTRH
      0000009AH   SFRSYM    DATA     BYTE      UT_BAUDL
      000000FCH   SFRSYM    DATA     BYTE      P0_OE
      000000FDH   SFRSYM    DATA     BYTE      P1_OE
      000000D0H.5 SFRSYM    DATA     BIT       F0
      000000B4H   SFRSYM    DATA     BYTE      TIM2_ADTRL
      000000FEH   SFRSYM    DATA     BYTE      P2_OE
      000000D0H.1 SFRSYM    DATA     BIT       F1
      00000080H   SFRSYM    DATA     BIT       GP00
      000000FFH   SFRSYM    DATA     BYTE      P3_OE
      00000090H   SFRSYM    DATA     BIT       GP10
      00000080H.1 SFRSYM    DATA     BIT       GP01
      000000A8H.6 SFRSYM    DATA     BIT       RTCIE
      000000A0H   SFRSYM    DATA     BIT       GP20
      00000090H.1 SFRSYM    DATA     BIT       GP11
      00000080H.2 SFRSYM    DATA     BIT       GP02
      000000E3H   SFRSYM    DATA     BYTE      SV_USH
      000000B0H   SFRSYM    DATA     BIT       GP30
      000000A0H.1 SFRSYM    DATA     BIT       GP21
      00000090H.2 SFRSYM    DATA     BIT       GP12
      00000080H.3 SFRSYM    DATA     BIT       GP03
      000000B8H   SFRSYM    DATA     BIT       PLVW0
      000000A8H.1 SFRSYM    DATA     BIT       TSDIE
      000000D0H   SFRSYM    DATA     BYTE      PSW
      000000B0H.1 SFRSYM    DATA     BIT       GP31
      000000A0H.2 SFRSYM    DATA     BIT       GP22
      00000090H.3 SFRSYM    DATA     BIT       GP13
      00000080H.4 SFRSYM    DATA     BIT       GP04
      000000B8H.1 SFRSYM    DATA     BIT       PLVW1
      000000A8H.3 SFRSYM    DATA     BIT       SPIIE
      00000088H.5 SFRSYM    DATA     BIT       TSDIF
      000000B0H.2 SFRSYM    DATA     BIT       GP32
      000000A0H.3 SFRSYM    DATA     BIT       GP23
      00000090H.4 SFRSYM    DATA     BIT       GP14
      00000080H.5 SFRSYM    DATA     BIT       GP05
      00000084H   SFRSYM    DATA     BYTE      FLKEY
      000000B3H   SFRSYM    DATA     BYTE      TIM2_CMTRH
      000000B0H.3 SFRSYM    DATA     BIT       GP33
      000000A0H.4 SFRSYM    DATA     BIT       GP24
      00000090H.5 SFRSYM    DATA     BIT       GP15
      00000080H.6 SFRSYM    DATA     BIT       GP06
      00000088H   SFRSYM    DATA     BIT       IT00

      01001C1CH   BLOCK     CODE     ---       LVL=0
      01001C1CH   LINE      CODE     ---       #33
      01001C1CH   LINE      CODE     ---       #34
      01001C1CH   LINE      CODE     ---       #35
      01001C21H   LINE      CODE     ---       #36
      01001C23H   LINE      CODE     ---       #37
      01001C27H   LINE      CODE     ---       #38
      01001C2BH   LINE      CODE     ---       #39
      01001C2FH   LINE      CODE     ---       #40
      01001C33H   LINE      CODE     ---       #42
      01001C37H   LINE      CODE     ---       #43
      01001C39H   LINE      CODE     ---       #44
      01001C3BH   LINE      CODE     ---       #45
      01001C3DH   LINE      CODE     ---       #46
      01001C3FH   LINE      CODE     ---       #47
      01001C41H   LINE      CODE     ---       #48
      01001C43H   LINE      CODE     ---       #49
      01001C49H   LINE      CODE     ---       #51
      ---         BLOCKEND  ---      ---       LVL=0
LX51 LINKER/LOCATER V4.66.1.0                                                         03/23/2017  15:15:44  PAGE 69



      01000F01H   BLOCK     CODE     ---       LVL=0
      01000F01H   LINE      CODE     ---       #101
      01000F01H   LINE      CODE     ---       #102
      01000F01H   LINE      CODE     ---       #103
      01000F2DH   LINE      CODE     ---       #104
      01000F2DH   LINE      CODE     ---       #105
      01000F2DH   LINE      CODE     ---       #106
      01000F36H   LINE      CODE     ---       #107
      01000F36H   LINE      CODE     ---       #113
      01000F3AH   LINE      CODE     ---       #114
      01000F3FH   LINE      CODE     ---       #115
      01000F43H   LINE      CODE     ---       #116
      01000F43H   LINE      CODE     ---       #117
      01000F44H   LINE      CODE     ---       #118
      01000F44H   LINE      CODE     ---       #119
      01000F4DH   LINE      CODE     ---       #120
      01000F4DH   LINE      CODE     ---       #125
      01000F51H   LINE      CODE     ---       #126
      01000F56H   LINE      CODE     ---       #127
      01000F5AH   LINE      CODE     ---       #128
      01000F5AH   LINE      CODE     ---       #129
      01000F5BH   LINE      CODE     ---       #130
      01000F5BH   LINE      CODE     ---       #131
      01000F64H   LINE      CODE     ---       #132
      01000F64H   LINE      CODE     ---       #133
      01000F6CH   LINE      CODE     ---       #134
      01000F71H   LINE      CODE     ---       #135
      01000F76H   LINE      CODE     ---       #136
      01000F7AH   LINE      CODE     ---       #137
      01000F7AH   LINE      CODE     ---       #138
      01000F7BH   LINE      CODE     ---       #139
      01000F7BH   LINE      CODE     ---       #140
      01000F84H   LINE      CODE     ---       #141
      01000F84H   LINE      CODE     ---       #142
      01000F8CH   LINE      CODE     ---       #143
      01000F91H   LINE      CODE     ---       #144
      01000F96H   LINE      CODE     ---       #145
      01000F9AH   LINE      CODE     ---       #146
      01000F9AH   LINE      CODE     ---       #147
      01000F9BH   LINE      CODE     ---       #148
      01000F9BH   LINE      CODE     ---       #149
      01000FA1H   LINE      CODE     ---       #150
      01000FA1H   LINE      CODE     ---       #151
      01000FA9H   LINE      CODE     ---       #152
      01000FAEH   LINE      CODE     ---       #153
      01000FB3H   LINE      CODE     ---       #154
      01000FB7H   LINE      CODE     ---       #155
      01000FB7H   LINE      CODE     ---       #156
      01000FB8H   LINE      CODE     ---       #157
      01000FB8H   LINE      CODE     ---       #158
      01000FBEH   LINE      CODE     ---       #159
      01000FBEH   LINE      CODE     ---       #160
      01000FC7H   LINE      CODE     ---       #161
      01000FCCH   LINE      CODE     ---       #162
      01000FD1H   LINE      CODE     ---       #163
      01000FD5H   LINE      CODE     ---       #164
      01000FD5H   LINE      CODE     ---       #165
      01000FD6H   LINE      CODE     ---       #166
      01000FD6H   LINE      CODE     ---       #167
      01000FDCH   LINE      CODE     ---       #168
      01000FDCH   LINE      CODE     ---       #169
      01000FE3H   LINE      CODE     ---       #170
      01000FE9H   LINE      CODE     ---       #171
      01000FEEH   LINE      CODE     ---       #172
LX51 LINKER/LOCATER V4.66.1.0                                                         03/23/2017  15:15:44  PAGE 70


      01000FF3H   LINE      CODE     ---       #173
      01000FF3H   LINE      CODE     ---       #174
      01000FF4H   LINE      CODE     ---       #175
      01000FF4H   LINE      CODE     ---       #176
      01000FF9H   LINE      CODE     ---       #177
      01000FFBH   LINE      CODE     ---       #178
      01000FFDH   LINE      CODE     ---       #179
      01000FFFH   LINE      CODE     ---       #180
      01001001H   LINE      CODE     ---       #181
      01001003H   LINE      CODE     ---       #182
      01001005H   LINE      CODE     ---       #183
      01001005H   LINE      CODE     ---       #184
      01001005H   LINE      CODE     ---       #187
      ---         BLOCKEND  ---      ---       LVL=0

      ---         MODULE    ---      ---       KEYSCAN
      02000179H   PUBLIC    XDATA    ---       KS
      01001D33H   PUBLIC    CODE     ---       KeyScan
      010014D1H   PUBLIC    CODE     ---       KeyValue
      0100192EH   PUBLIC    CODE     ---       KeyInit
      000000E2H   SFRSYM    DATA     BYTE      SV_USL
      000000ABH   SFRSYM    DATA     BYTE      TIM2_CNTRH
      000000B0H.4 SFRSYM    DATA     BIT       GP34
      000000A0H.5 SFRSYM    DATA     BIT       GP25
      00000090H.6 SFRSYM    DATA     BIT       GP16
      00000080H.7 SFRSYM    DATA     BIT       GP07
      00000088H.1 SFRSYM    DATA     BIT       IT01
      00000088H.3 SFRSYM    DATA     BIT       IT10
      000000F6H   SFRSYM    DATA     WORD      PI_UKMIN
      000000C2H   SFRSYM    DATA     WORD      MD_MA
      000000A3H   SFRSYM    DATA     BYTE      TIM3_CNTRH
      000000B0H.5 SFRSYM    DATA     BIT       GP35
      000000A0H.6 SFRSYM    DATA     BIT       GP26
      00000090H.7 SFRSYM    DATA     BIT       GP17
      00000080H   SFRSYM    DATA     BYTE      P0
      00000088H.4 SFRSYM    DATA     BIT       IT11
      000000CAH   SFRSYM    DATA     WORD      MD_MB
      00000093H   SFRSYM    DATA     BYTE      TIM4_CNTRH
      000000B0H.6 SFRSYM    DATA     BIT       GP36
      000000A0H.7 SFRSYM    DATA     BIT       GP27
      00000090H   SFRSYM    DATA     BYTE      P1
      000000D9H   SFRSYM    DATA     BYTE      EVT_FILT
      000000F4H   SFRSYM    DATA     WORD      PI_UKMAX
      0000008BH   SFRSYM    DATA     BYTE      TIM5_CNTRH
      000000B2H   SFRSYM    DATA     BYTE      TIM2_CMTRL
      000000B0H.7 SFRSYM    DATA     BIT       GP37
      000000A0H   SFRSYM    DATA     BYTE      P2
      000000AAH   SFRSYM    DATA     BYTE      TIM2_CNTRL
      000000B0H   SFRSYM    DATA     BYTE      P3
      000000A2H   SFRSYM    DATA     BYTE      TIM3_CNTRL
      000000D0H.6 SFRSYM    DATA     BIT       AC
      00000092H   SFRSYM    DATA     BYTE      TIM4_CNTRL
      0000008AH   SFRSYM    DATA     BYTE      TIM5_CNTRL
      000000B6H   SFRSYM    DATA     WORD      TIM0_CCR1
      000000A8H.7 SFRSYM    DATA     BIT       EA
      000000D5H   SFRSYM    DATA     BYTE      CMP_CR0
      000000BAH   SFRSYM    DATA     WORD      TIM0_CCR2
      000000D6H   SFRSYM    DATA     BYTE      CMP_CR1
      000000BCH   SFRSYM    DATA     WORD      TIM0_CCR3
      00000085H   SFRSYM    DATA     BYTE      PSCTL
      000000DAH   SFRSYM    DATA     BYTE      CMP_CR2
      000000BEH   SFRSYM    DATA     WORD      TIM0_CCR4
      000000B8H.2 SFRSYM    DATA     BIT       PX00
      000000EAH   SFRSYM    DATA     WORD      PI_EK
      000000F8H   SFRSYM    DATA     BIT       OISUH
LX51 LINKER/LOCATER V4.66.1.0                                                         03/23/2017  15:15:44  PAGE 71


      000000B8H.3 SFRSYM    DATA     BIT       PX01
      000000B8H.4 SFRSYM    DATA     BIT       PX10
      000000F8H.2 SFRSYM    DATA     BIT       OISVH
      000000B8H.5 SFRSYM    DATA     BIT       PX11
      000000F8H.4 SFRSYM    DATA     BIT       OISWH
      000000DCH   SFRSYM    DATA     WORD      LPF_K
      000000F2H   SFRSYM    DATA     WORD      PI_KI
      000000F8H.1 SFRSYM    DATA     BIT       OISUL
      000000A8H   SFRSYM    DATA     BYTE      IE
      000000F8H.3 SFRSYM    DATA     BIT       OISVL
      000000F8H.5 SFRSYM    DATA     BIT       OISWL
      000000D1H   SFRSYM    DATA     BYTE      P1IE
      00000098H.6 SFRSYM    DATA     BIT       MOD0
      000000D3H   SFRSYM    DATA     BYTE      P2IE
      000000D2H   SFRSYM    DATA     BYTE      P1IF
      000000F9H   SFRSYM    DATA     BYTE      PL_CR
      00000098H.7 SFRSYM    DATA     BIT       MOD1
      000000D4H   SFRSYM    DATA     BYTE      P2IF
      000000ACH   SFRSYM    DATA     WORD      TIM2_DR
      00000082H   SFRSYM    DATA     WORD      DP
      000000EEH   SFRSYM    DATA     WORD      PI_KP
      000000A4H   SFRSYM    DATA     WORD      TIM3_DR
      00000094H   SFRSYM    DATA     WORD      TIM4_DR
      0000008CH   SFRSYM    DATA     WORD      TIM5_DR
      000000F1H   SFRSYM    DATA     BYTE      OSC_CFG
      000000C1H   SFRSYM    DATA     BYTE      MD_MODE
      000000ECH   SFRSYM    DATA     WORD      PI_UK
      000000DEH   SFRSYM    DATA     WORD      LPF_X
      00000098H   SFRSYM    DATA     BIT       RI
      000000E6H   SFRSYM    DATA     WORD      LPF_Y
      000000C0H   SFRSYM    DATA     BIT       PTIM00
      000000D0H.7 SFRSYM    DATA     BIT       CY
      00000098H.1 SFRSYM    DATA     BIT       TI
      000000C0H.1 SFRSYM    DATA     BIT       PTIM01
      000000C0H.2 SFRSYM    DATA     BIT       PTIM10
      000000C0H.3 SFRSYM    DATA     BIT       PTIM11
      000000E1H   SFRSYM    DATA     BYTE      SV_CR
      00000098H   SFRSYM    DATA     BYTE      UT_CR
      00000099H   SFRSYM    DATA     BYTE      UT_DR
      000000F8H.6 SFRSYM    DATA     BIT       OIS4
      00000081H   SFRSYM    DATA     BYTE      SP
      000000D0H.2 SFRSYM    DATA     BIT       OV
      000000C4H   SFRSYM    DATA     BYTE      MD_DA0
      0000009AH   SFRSYM    DATA     WORD      UT_BAUD
      000000CCH   SFRSYM    DATA     BYTE      MD_DB0
      000000C5H   SFRSYM    DATA     BYTE      MD_DA1
      000000CDH   SFRSYM    DATA     BYTE      MD_DB1
      000000C6H   SFRSYM    DATA     BYTE      MD_DA2
      000000CEH   SFRSYM    DATA     BYTE      MD_DB2
      000000C7H   SFRSYM    DATA     BYTE      MD_DA3
      000000B4H   SFRSYM    DATA     WORD      TIM2_ADTR
      000000CFH   SFRSYM    DATA     BYTE      MD_DB3
      000000AFH   SFRSYM    DATA     BYTE      TIM2_ARRH
      000000A7H   SFRSYM    DATA     BYTE      TIM3_ARRH
      00000097H   SFRSYM    DATA     BYTE      TIM4_ARRH
      0000008FH   SFRSYM    DATA     BYTE      TIM5_ARRH
      000000AEH   SFRSYM    DATA     BYTE      TIM2_ARRL
      000000A6H   SFRSYM    DATA     BYTE      TIM3_ARRL
      00000087H   SFRSYM    DATA     BYTE      PCON
      000000E2H   SFRSYM    DATA     WORD      SV_US
      00000096H   SFRSYM    DATA     BYTE      TIM4_ARRL
      0000008EH   SFRSYM    DATA     BYTE      TIM5_ARRL
      000000B2H   SFRSYM    DATA     WORD      TIM2_CMTR
      00000088H   SFRSYM    DATA     BYTE      TCON
      000000AAH   SFRSYM    DATA     WORD      TIM2_CNTR
LX51 LINKER/LOCATER V4.66.1.0                                                         03/23/2017  15:15:44  PAGE 72


      000000A2H   SFRSYM    DATA     WORD      TIM3_CNTR
      00000092H   SFRSYM    DATA     WORD      TIM4_CNTR
      0000008AH   SFRSYM    DATA     WORD      TIM5_CNTR
      000000E5H   SFRSYM    DATA     BYTE      SV_ANGLEH
      000000D8H   SFRSYM    DATA     BIT       PUART0
      000000E4H   SFRSYM    DATA     BYTE      SV_ANGLEL
      000000C6H   SFRSYM    DATA     WORD      MD_DAH
      000000D8H.1 SFRSYM    DATA     BIT       PUART1
      000000D8H.2 SFRSYM    DATA     BIT       PI2C0
      00000088H.2 SFRSYM    DATA     BIT       IF0
      000000CEH   SFRSYM    DATA     WORD      MD_DBH
      000000D8H.3 SFRSYM    DATA     BIT       PI2C1
      000000F0H   SFRSYM    DATA     BYTE      B
      000000C4H   SFRSYM    DATA     WORD      MD_DAL
      000000A1H   SFRSYM    DATA     BYTE      TIM2_CR0
      000000CCH   SFRSYM    DATA     WORD      MD_DBL
      0000009CH   SFRSYM    DATA     BYTE      TIM3_CR0
      000000A9H   SFRSYM    DATA     BYTE      TIM2_CR1
      0000009EH   SFRSYM    DATA     BYTE      TIM4_CR0
      0000009DH   SFRSYM    DATA     BYTE      TIM3_CR1
      00000089H   SFRSYM    DATA     BYTE      TIM5_CR0
      0000009FH   SFRSYM    DATA     BYTE      TIM4_CR1
      000000F8H   SFRSYM    DATA     BYTE      DRV_OUT
      00000091H   SFRSYM    DATA     BYTE      TIM5_CR1
      000000E0H   SFRSYM    DATA     BYTE      ACC
      000000F7H   SFRSYM    DATA     BYTE      PI_UKMINH
      000000C3H   SFRSYM    DATA     BYTE      MD_MAH
      000000A8H.4 SFRSYM    DATA     BIT       ES0
      000000DBH   SFRSYM    DATA     BYTE      LVSR
      000000CBH   SFRSYM    DATA     BYTE      MD_MBH
      000000C0H.4 SFRSYM    DATA     BIT       PADC0
      000000B8H   SFRSYM    DATA     BYTE      IP0
      000000F5H   SFRSYM    DATA     BYTE      PI_UKMAXH
      000000C0H.5 SFRSYM    DATA     BIT       PADC1
      000000C0H   SFRSYM    DATA     BYTE      IP1
      000000C8H   SFRSYM    DATA     BYTE      IP2
      000000F6H   SFRSYM    DATA     BYTE      PI_UKMINL
      000000C2H   SFRSYM    DATA     BYTE      MD_MAL
      00000098H.2 SFRSYM    DATA     BIT       RB8
      000000D8H   SFRSYM    DATA     BYTE      IP3
      000000CAH   SFRSYM    DATA     BYTE      MD_MBL
      000000A8H   SFRSYM    DATA     BIT       EX0
      000000F4H   SFRSYM    DATA     BYTE      PI_UKMAXL
      00000098H.3 SFRSYM    DATA     BIT       TB8
      000000B7H   SFRSYM    DATA     BYTE      TIM0_CCR1H
      000000A8H.2 SFRSYM    DATA     BIT       EX1
      000000BBH   SFRSYM    DATA     BYTE      TIM0_CCR2H
      000000D0H   SFRSYM    DATA     BIT       P
      000000BDH   SFRSYM    DATA     BYTE      TIM0_CCR3H
      000000BFH   SFRSYM    DATA     BYTE      TIM0_CCR4H
      000000C8H.2 SFRSYM    DATA     BIT       PTIM230
      000000EBH   SFRSYM    DATA     BYTE      PI_EKH
      00000098H.5 SFRSYM    DATA     BIT       SM2
      000000B6H   SFRSYM    DATA     BYTE      TIM0_CCR1L
      000000B1H   SFRSYM    DATA     BYTE      TIM0_SR1
      000000C8H.3 SFRSYM    DATA     BIT       PTIM231
      000000BAH   SFRSYM    DATA     BYTE      TIM0_CCR2L
      000000BCH   SFRSYM    DATA     BYTE      TIM0_CCR3L
      000000BEH   SFRSYM    DATA     BYTE      TIM0_CCR4L
      000000D8H.6 SFRSYM    DATA     BIT       PMCD0
      000000C8H.4 SFRSYM    DATA     BIT       PTIM450
      000000D0H.3 SFRSYM    DATA     BIT       RS0
      000000DDH   SFRSYM    DATA     BYTE      LPF_KH
      000000F3H   SFRSYM    DATA     BYTE      PI_KIH
      000000EAH   SFRSYM    DATA     BYTE      PI_EKL
LX51 LINKER/LOCATER V4.66.1.0                                                         03/23/2017  15:15:44  PAGE 73


      000000E8H   SFRSYM    DATA     BYTE      FOC_SET0
      000000D8H.7 SFRSYM    DATA     BIT       PMCD1
      000000C8H.5 SFRSYM    DATA     BIT       PTIM451
      000000D0H.4 SFRSYM    DATA     BIT       RS1
      000000E9H   SFRSYM    DATA     BYTE      FOC_SET1
      000000B8H.6 SFRSYM    DATA     BIT       PFOC0
      000000DCH   SFRSYM    DATA     BYTE      LPF_KL
      000000F2H   SFRSYM    DATA     BYTE      PI_KIL
      000000B8H.7 SFRSYM    DATA     BIT       PFOC1
      000000ADH   SFRSYM    DATA     BYTE      TIM2_DRH
      000000B9H   SFRSYM    DATA     BYTE      TIM0_IER
      00000083H   SFRSYM    DATA     BYTE      DPH
      000000EFH   SFRSYM    DATA     BYTE      PI_KPH
      000000A5H   SFRSYM    DATA     BYTE      TIM3_DRH
      00000095H   SFRSYM    DATA     BYTE      TIM4_DRH
      0000008DH   SFRSYM    DATA     BYTE      TIM5_DRH
      000000ACH   SFRSYM    DATA     BYTE      TIM2_DRL
      00000082H   SFRSYM    DATA     BYTE      DPL
      000000EEH   SFRSYM    DATA     BYTE      PI_KPL
      000000A4H   SFRSYM    DATA     BYTE      TIM3_DRL
      000000F8H.7 SFRSYM    DATA     BIT       MOE
      000000C0H.6 SFRSYM    DATA     BIT       PCMP0
      000000EDH   SFRSYM    DATA     BYTE      PI_UKH
      00000094H   SFRSYM    DATA     BYTE      TIM4_DRL
      000000C0H.7 SFRSYM    DATA     BIT       PCMP1
      000000DFH   SFRSYM    DATA     BYTE      LPF_XH
      0000008CH   SFRSYM    DATA     BYTE      TIM5_DRL
      000000AEH   SFRSYM    DATA     WORD      TIM2_ARR
      000000A8H.5 SFRSYM    DATA     BIT       MCDIE
      000000C9H   SFRSYM    DATA     BYTE      RSTSRC
      000000E7H   SFRSYM    DATA     BYTE      LPF_YH
      000000A6H   SFRSYM    DATA     WORD      TIM3_ARR
      00000088H.6 SFRSYM    DATA     BIT       MCDIF
      00000098H.4 SFRSYM    DATA     BIT       REN
      00000096H   SFRSYM    DATA     WORD      TIM4_ARR
      000000ECH   SFRSYM    DATA     BYTE      PI_UKL
      000000D7H   SFRSYM    DATA     BYTE      CMP_SR
      0000008EH   SFRSYM    DATA     WORD      TIM5_ARR
      000000DEH   SFRSYM    DATA     BYTE      LPF_XL
      000000E6H   SFRSYM    DATA     BYTE      LPF_YL
      000000C8H   SFRSYM    DATA     BIT       PRTC0
      000000C8H.1 SFRSYM    DATA     BIT       PRTC1
      000000E8H.7 SFRSYM    DATA     BIT       FOCEN
      000000C8H.6 SFRSYM    DATA     BIT       PTSD0
      000000D8H.4 SFRSYM    DATA     BIT       PSPI0
      000000C8H.7 SFRSYM    DATA     BIT       PTSD1
      000000D8H.5 SFRSYM    DATA     BIT       PSPI1
      0000009BH   SFRSYM    DATA     BYTE      UT_BAUDH
      000000E4H   SFRSYM    DATA     WORD      SV_ANGLE
      000000B5H   SFRSYM    DATA     BYTE      TIM2_ADTRH
      0000009AH   SFRSYM    DATA     BYTE      UT_BAUDL
      000000FCH   SFRSYM    DATA     BYTE      P0_OE
      000000FDH   SFRSYM    DATA     BYTE      P1_OE
      000000D0H.5 SFRSYM    DATA     BIT       F0
      000000B4H   SFRSYM    DATA     BYTE      TIM2_ADTRL
      000000FEH   SFRSYM    DATA     BYTE      P2_OE
      000000D0H.1 SFRSYM    DATA     BIT       F1
      00000080H   SFRSYM    DATA     BIT       GP00
      000000FFH   SFRSYM    DATA     BYTE      P3_OE
      00000090H   SFRSYM    DATA     BIT       GP10
      00000080H.1 SFRSYM    DATA     BIT       GP01
      000000A8H.6 SFRSYM    DATA     BIT       RTCIE
      000000A0H   SFRSYM    DATA     BIT       GP20
      00000090H.1 SFRSYM    DATA     BIT       GP11
      00000080H.2 SFRSYM    DATA     BIT       GP02
LX51 LINKER/LOCATER V4.66.1.0                                                         03/23/2017  15:15:44  PAGE 74


      000000E3H   SFRSYM    DATA     BYTE      SV_USH
      000000B0H   SFRSYM    DATA     BIT       GP30
      000000A0H.1 SFRSYM    DATA     BIT       GP21
      00000090H.2 SFRSYM    DATA     BIT       GP12
      00000080H.3 SFRSYM    DATA     BIT       GP03
      000000B8H   SFRSYM    DATA     BIT       PLVW0
      000000A8H.1 SFRSYM    DATA     BIT       TSDIE
      000000D0H   SFRSYM    DATA     BYTE      PSW
      000000B0H.1 SFRSYM    DATA     BIT       GP31
      000000A0H.2 SFRSYM    DATA     BIT       GP22
      00000090H.3 SFRSYM    DATA     BIT       GP13
      00000080H.4 SFRSYM    DATA     BIT       GP04
      000000B8H.1 SFRSYM    DATA     BIT       PLVW1
      000000A8H.3 SFRSYM    DATA     BIT       SPIIE
      00000088H.5 SFRSYM    DATA     BIT       TSDIF
      000000B0H.2 SFRSYM    DATA     BIT       GP32
      000000A0H.3 SFRSYM    DATA     BIT       GP23
      00000090H.4 SFRSYM    DATA     BIT       GP14
      00000080H.5 SFRSYM    DATA     BIT       GP05
      00000084H   SFRSYM    DATA     BYTE      FLKEY
      000000B3H   SFRSYM    DATA     BYTE      TIM2_CMTRH
      000000B0H.3 SFRSYM    DATA     BIT       GP33
      000000A0H.4 SFRSYM    DATA     BIT       GP24
      00000090H.5 SFRSYM    DATA     BIT       GP15
      00000080H.6 SFRSYM    DATA     BIT       GP06
      00000088H   SFRSYM    DATA     BIT       IT00

      0100192EH   BLOCK     CODE     ---       LVL=0
      0100192EH   LINE      CODE     ---       #26
      0100192EH   LINE      CODE     ---       #27
      0100192EH   LINE      CODE     ---       #28
      01001933H   LINE      CODE     ---       #29
      01001935H   LINE      CODE     ---       #30
      01001939H   LINE      CODE     ---       #32
      0100193BH   LINE      CODE     ---       #33
      0100193DH   LINE      CODE     ---       #34
      01001941H   LINE      CODE     ---       #36
      01001957H   LINE      CODE     ---       #37
      01001957H   LINE      CODE     ---       #38
      0100195AH   LINE      CODE     ---       #39
      0100195CH   LINE      CODE     ---       #41
      01001962H   LINE      CODE     ---       #42
      01001962H   LINE      CODE     ---       #43
      01001968H   LINE      CODE     ---       #44
      01001968H   LINE      CODE     ---       #45
      0100196AH   LINE      CODE     ---       #46
      0100196AH   LINE      CODE     ---       #47
      0100196BH   LINE      CODE     ---       #49
      0100196BH   LINE      CODE     ---       #50
      01001971H   LINE      CODE     ---       #51
      01001971H   LINE      CODE     ---       #52
      01001973H   LINE      CODE     ---       #53
      01001973H   LINE      CODE     ---       #54
      01001973H   LINE      CODE     ---       #56
      ---         BLOCKEND  ---      ---       LVL=0

      010014D1H   BLOCK     CODE     ---       LVL=0
      010014D1H   LINE      CODE     ---       #64
      010014D1H   LINE      CODE     ---       #65
      010014D1H   LINE      CODE     ---       #67
      010014D4H   LINE      CODE     ---       #68
      010014D4H   LINE      CODE     ---       #69
      010014E2H   LINE      CODE     ---       #70
      010014F3H   LINE      CODE     ---       #71
      010014F3H   LINE      CODE     ---       #72
LX51 LINKER/LOCATER V4.66.1.0                                                         03/23/2017  15:15:44  PAGE 75


      010014F9H   LINE      CODE     ---       #73
      010014FFH   LINE      CODE     ---       #74
      01001504H   LINE      CODE     ---       #75
      01001504H   LINE      CODE     ---       #76
      01001506H   LINE      CODE     ---       #77
      01001508H   LINE      CODE     ---       #78
      01001508H   LINE      CODE     ---       #79
      01001508H   LINE      CODE     ---       #80
      01001508H   LINE      CODE     ---       #82
      01001508H   LINE      CODE     ---       #83
      01001516H   LINE      CODE     ---       #84
      01001525H   LINE      CODE     ---       #85
      01001525H   LINE      CODE     ---       #86
      0100152CH   LINE      CODE     ---       #87
      01001531H   LINE      CODE     ---       #88
      01001534H   LINE      CODE     ---       #89
      01001534H   LINE      CODE     ---       #90
      01001534H   LINE      CODE     ---       #94
      01001534H   LINE      CODE     ---       #95
      01001534H   LINE      CODE     ---       #96
      01001534H   LINE      CODE     ---       #97
      01001534H   LINE      CODE     ---       #98
      01001534H   LINE      CODE     ---       #99
      01001534H   LINE      CODE     ---       #100
      01001534H   LINE      CODE     ---       #101
      01001534H   LINE      CODE     ---       #102
      01001534H   LINE      CODE     ---       #103
      01001534H   LINE      CODE     ---       #104
      01001534H   LINE      CODE     ---       #105
      01001534H   LINE      CODE     ---       #106
      01001534H   LINE      CODE     ---       #107
      01001534H   LINE      CODE     ---       #109
      01001534H   LINE      CODE     ---       #110
      01001542H   LINE      CODE     ---       #111
      01001551H   LINE      CODE     ---       #112
      01001551H   LINE      CODE     ---       #113
      01001558H   LINE      CODE     ---       #114
      0100155DH   LINE      CODE     ---       #115
      01001560H   LINE      CODE     ---       #116
      01001560H   LINE      CODE     ---       #117
      01001560H   LINE      CODE     ---       #119
      01001562H   LINE      CODE     ---       #120
      ---         BLOCKEND  ---      ---       LVL=0

      01001D33H   BLOCK     CODE     ---       LVL=0
      01001D33H   LINE      CODE     ---       #128
      01001D33H   LINE      CODE     ---       #129
      01001D33H   LINE      CODE     ---       #130
      01001D36H   LINE      CODE     ---       #131
      01001D36H   LINE      CODE     ---       #132
      01001D36H   LINE      CODE     ---       #137
      01001D36H   LINE      CODE     ---       #138
      01001D36H   LINE      CODE     ---       #143
      01001D36H   LINE      CODE     ---       #144
      01001D36H   LINE      CODE     ---       #145
      01001D36H   LINE      CODE     ---       #146
      01001D36H   LINE      CODE     ---       #148
      01001D3CH   LINE      CODE     ---       #149
      01001D3CH   LINE      CODE     ---       #150
      01001D42H   LINE      CODE     ---       #151
      01001D42H   LINE      CODE     ---       #152
      01001D47H   LINE      CODE     ---       #153
      01001D47H   LINE      CODE     ---       #154
      01001D48H   LINE      CODE     ---       #156
      01001D48H   LINE      CODE     ---       #157
LX51 LINKER/LOCATER V4.66.1.0                                                         03/23/2017  15:15:44  PAGE 76


      01001D4EH   LINE      CODE     ---       #158
      01001D4EH   LINE      CODE     ---       #159
      01001D54H   LINE      CODE     ---       #160
      01001D54H   LINE      CODE     ---       #161
      01001D54H   LINE      CODE     ---       #162
      ---         BLOCKEND  ---      ---       LVL=0

      ---         MODULE    ---      ---       PWMSCAN
      02000170H   PUBLIC    XDATA    ---       PWMINCtl
      01001D55H   PUBLIC    CODE     ---       PWMScan
      01001E06H   PUBLIC    CODE     ---       PWMIN_Init
      000000E2H   SFRSYM    DATA     BYTE      SV_USL
      000000ABH   SFRSYM    DATA     BYTE      TIM2_CNTRH
      000000B0H.4 SFRSYM    DATA     BIT       GP34
      000000A0H.5 SFRSYM    DATA     BIT       GP25
      00000090H.6 SFRSYM    DATA     BIT       GP16
      00000080H.7 SFRSYM    DATA     BIT       GP07
      00000088H.1 SFRSYM    DATA     BIT       IT01
      00000088H.3 SFRSYM    DATA     BIT       IT10
      000000F6H   SFRSYM    DATA     WORD      PI_UKMIN
      000000C2H   SFRSYM    DATA     WORD      MD_MA
      000000A3H   SFRSYM    DATA     BYTE      TIM3_CNTRH
      000000B0H.5 SFRSYM    DATA     BIT       GP35
      000000A0H.6 SFRSYM    DATA     BIT       GP26
      00000090H.7 SFRSYM    DATA     BIT       GP17
      00000080H   SFRSYM    DATA     BYTE      P0
      00000088H.4 SFRSYM    DATA     BIT       IT11
      000000CAH   SFRSYM    DATA     WORD      MD_MB
      00000093H   SFRSYM    DATA     BYTE      TIM4_CNTRH
      000000B0H.6 SFRSYM    DATA     BIT       GP36
      000000A0H.7 SFRSYM    DATA     BIT       GP27
      00000090H   SFRSYM    DATA     BYTE      P1
      000000D9H   SFRSYM    DATA     BYTE      EVT_FILT
      000000F4H   SFRSYM    DATA     WORD      PI_UKMAX
      0000008BH   SFRSYM    DATA     BYTE      TIM5_CNTRH
      000000B2H   SFRSYM    DATA     BYTE      TIM2_CMTRL
      000000B0H.7 SFRSYM    DATA     BIT       GP37
      000000A0H   SFRSYM    DATA     BYTE      P2
      000000AAH   SFRSYM    DATA     BYTE      TIM2_CNTRL
      000000B0H   SFRSYM    DATA     BYTE      P3
      000000A2H   SFRSYM    DATA     BYTE      TIM3_CNTRL
      000000D0H.6 SFRSYM    DATA     BIT       AC
      00000092H   SFRSYM    DATA     BYTE      TIM4_CNTRL
      0000008AH   SFRSYM    DATA     BYTE      TIM5_CNTRL
      000000B6H   SFRSYM    DATA     WORD      TIM0_CCR1
      000000A8H.7 SFRSYM    DATA     BIT       EA
      000000D5H   SFRSYM    DATA     BYTE      CMP_CR0
      000000BAH   SFRSYM    DATA     WORD      TIM0_CCR2
      000000D6H   SFRSYM    DATA     BYTE      CMP_CR1
      000000BCH   SFRSYM    DATA     WORD      TIM0_CCR3
      00000085H   SFRSYM    DATA     BYTE      PSCTL
      000000DAH   SFRSYM    DATA     BYTE      CMP_CR2
      000000BEH   SFRSYM    DATA     WORD      TIM0_CCR4
      000000B8H.2 SFRSYM    DATA     BIT       PX00
      000000EAH   SFRSYM    DATA     WORD      PI_EK
      000000F8H   SFRSYM    DATA     BIT       OISUH
      000000B8H.3 SFRSYM    DATA     BIT       PX01
      000000B8H.4 SFRSYM    DATA     BIT       PX10
      000000F8H.2 SFRSYM    DATA     BIT       OISVH
      000000B8H.5 SFRSYM    DATA     BIT       PX11
      000000F8H.4 SFRSYM    DATA     BIT       OISWH
      000000DCH   SFRSYM    DATA     WORD      LPF_K
      000000F2H   SFRSYM    DATA     WORD      PI_KI
      000000F8H.1 SFRSYM    DATA     BIT       OISUL
      000000A8H   SFRSYM    DATA     BYTE      IE
LX51 LINKER/LOCATER V4.66.1.0                                                         03/23/2017  15:15:44  PAGE 77


      000000F8H.3 SFRSYM    DATA     BIT       OISVL
      000000F8H.5 SFRSYM    DATA     BIT       OISWL
      000000D1H   SFRSYM    DATA     BYTE      P1IE
      00000098H.6 SFRSYM    DATA     BIT       MOD0
      000000D3H   SFRSYM    DATA     BYTE      P2IE
      000000D2H   SFRSYM    DATA     BYTE      P1IF
      000000F9H   SFRSYM    DATA     BYTE      PL_CR
      00000098H.7 SFRSYM    DATA     BIT       MOD1
      000000D4H   SFRSYM    DATA     BYTE      P2IF
      000000ACH   SFRSYM    DATA     WORD      TIM2_DR
      00000082H   SFRSYM    DATA     WORD      DP
      000000EEH   SFRSYM    DATA     WORD      PI_KP
      000000A4H   SFRSYM    DATA     WORD      TIM3_DR
      00000094H   SFRSYM    DATA     WORD      TIM4_DR
      0000008CH   SFRSYM    DATA     WORD      TIM5_DR
      000000F1H   SFRSYM    DATA     BYTE      OSC_CFG
      000000C1H   SFRSYM    DATA     BYTE      MD_MODE
      000000ECH   SFRSYM    DATA     WORD      PI_UK
      000000DEH   SFRSYM    DATA     WORD      LPF_X
      00000098H   SFRSYM    DATA     BIT       RI
      000000E6H   SFRSYM    DATA     WORD      LPF_Y
      000000C0H   SFRSYM    DATA     BIT       PTIM00
      000000D0H.7 SFRSYM    DATA     BIT       CY
      00000098H.1 SFRSYM    DATA     BIT       TI
      000000C0H.1 SFRSYM    DATA     BIT       PTIM01
      000000C0H.2 SFRSYM    DATA     BIT       PTIM10
      000000C0H.3 SFRSYM    DATA     BIT       PTIM11
      000000E1H   SFRSYM    DATA     BYTE      SV_CR
      00000098H   SFRSYM    DATA     BYTE      UT_CR
      00000099H   SFRSYM    DATA     BYTE      UT_DR
      000000F8H.6 SFRSYM    DATA     BIT       OIS4
      00000081H   SFRSYM    DATA     BYTE      SP
      000000D0H.2 SFRSYM    DATA     BIT       OV
      000000C4H   SFRSYM    DATA     BYTE      MD_DA0
      0000009AH   SFRSYM    DATA     WORD      UT_BAUD
      000000CCH   SFRSYM    DATA     BYTE      MD_DB0
      000000C5H   SFRSYM    DATA     BYTE      MD_DA1
      000000CDH   SFRSYM    DATA     BYTE      MD_DB1
      000000C6H   SFRSYM    DATA     BYTE      MD_DA2
      000000CEH   SFRSYM    DATA     BYTE      MD_DB2
      000000C7H   SFRSYM    DATA     BYTE      MD_DA3
      000000B4H   SFRSYM    DATA     WORD      TIM2_ADTR
      000000CFH   SFRSYM    DATA     BYTE      MD_DB3
      000000AFH   SFRSYM    DATA     BYTE      TIM2_ARRH
      000000A7H   SFRSYM    DATA     BYTE      TIM3_ARRH
      00000097H   SFRSYM    DATA     BYTE      TIM4_ARRH
      0000008FH   SFRSYM    DATA     BYTE      TIM5_ARRH
      000000AEH   SFRSYM    DATA     BYTE      TIM2_ARRL
      000000A6H   SFRSYM    DATA     BYTE      TIM3_ARRL
      00000087H   SFRSYM    DATA     BYTE      PCON
      000000E2H   SFRSYM    DATA     WORD      SV_US
      00000096H   SFRSYM    DATA     BYTE      TIM4_ARRL
      0000008EH   SFRSYM    DATA     BYTE      TIM5_ARRL
      000000B2H   SFRSYM    DATA     WORD      TIM2_CMTR
      00000088H   SFRSYM    DATA     BYTE      TCON
      000000AAH   SFRSYM    DATA     WORD      TIM2_CNTR
      000000A2H   SFRSYM    DATA     WORD      TIM3_CNTR
      00000092H   SFRSYM    DATA     WORD      TIM4_CNTR
      0000008AH   SFRSYM    DATA     WORD      TIM5_CNTR
      000000E5H   SFRSYM    DATA     BYTE      SV_ANGLEH
      000000D8H   SFRSYM    DATA     BIT       PUART0
      000000E4H   SFRSYM    DATA     BYTE      SV_ANGLEL
      000000C6H   SFRSYM    DATA     WORD      MD_DAH
      000000D8H.1 SFRSYM    DATA     BIT       PUART1
      000000D8H.2 SFRSYM    DATA     BIT       PI2C0
LX51 LINKER/LOCATER V4.66.1.0                                                         03/23/2017  15:15:44  PAGE 78


      00000088H.2 SFRSYM    DATA     BIT       IF0
      000000CEH   SFRSYM    DATA     WORD      MD_DBH
      000000D8H.3 SFRSYM    DATA     BIT       PI2C1
      000000F0H   SFRSYM    DATA     BYTE      B
      000000C4H   SFRSYM    DATA     WORD      MD_DAL
      000000A1H   SFRSYM    DATA     BYTE      TIM2_CR0
      000000CCH   SFRSYM    DATA     WORD      MD_DBL
      0000009CH   SFRSYM    DATA     BYTE      TIM3_CR0
      000000A9H   SFRSYM    DATA     BYTE      TIM2_CR1
      0000009EH   SFRSYM    DATA     BYTE      TIM4_CR0
      0000009DH   SFRSYM    DATA     BYTE      TIM3_CR1
      00000089H   SFRSYM    DATA     BYTE      TIM5_CR0
      0000009FH   SFRSYM    DATA     BYTE      TIM4_CR1
      000000F8H   SFRSYM    DATA     BYTE      DRV_OUT
      00000091H   SFRSYM    DATA     BYTE      TIM5_CR1
      000000E0H   SFRSYM    DATA     BYTE      ACC
      000000F7H   SFRSYM    DATA     BYTE      PI_UKMINH
      000000C3H   SFRSYM    DATA     BYTE      MD_MAH
      000000A8H.4 SFRSYM    DATA     BIT       ES0
      000000DBH   SFRSYM    DATA     BYTE      LVSR
      000000CBH   SFRSYM    DATA     BYTE      MD_MBH
      000000C0H.4 SFRSYM    DATA     BIT       PADC0
      000000B8H   SFRSYM    DATA     BYTE      IP0
      000000F5H   SFRSYM    DATA     BYTE      PI_UKMAXH
      000000C0H.5 SFRSYM    DATA     BIT       PADC1
      000000C0H   SFRSYM    DATA     BYTE      IP1
      000000C8H   SFRSYM    DATA     BYTE      IP2
      000000F6H   SFRSYM    DATA     BYTE      PI_UKMINL
      000000C2H   SFRSYM    DATA     BYTE      MD_MAL
      00000098H.2 SFRSYM    DATA     BIT       RB8
      000000D8H   SFRSYM    DATA     BYTE      IP3
      000000CAH   SFRSYM    DATA     BYTE      MD_MBL
      000000A8H   SFRSYM    DATA     BIT       EX0
      000000F4H   SFRSYM    DATA     BYTE      PI_UKMAXL
      00000098H.3 SFRSYM    DATA     BIT       TB8
      000000B7H   SFRSYM    DATA     BYTE      TIM0_CCR1H
      000000A8H.2 SFRSYM    DATA     BIT       EX1
      000000BBH   SFRSYM    DATA     BYTE      TIM0_CCR2H
      000000D0H   SFRSYM    DATA     BIT       P
      000000BDH   SFRSYM    DATA     BYTE      TIM0_CCR3H
      000000BFH   SFRSYM    DATA     BYTE      TIM0_CCR4H
      000000C8H.2 SFRSYM    DATA     BIT       PTIM230
      000000EBH   SFRSYM    DATA     BYTE      PI_EKH
      00000098H.5 SFRSYM    DATA     BIT       SM2
      000000B6H   SFRSYM    DATA     BYTE      TIM0_CCR1L
      000000B1H   SFRSYM    DATA     BYTE      TIM0_SR1
      000000C8H.3 SFRSYM    DATA     BIT       PTIM231
      000000BAH   SFRSYM    DATA     BYTE      TIM0_CCR2L
      000000BCH   SFRSYM    DATA     BYTE      TIM0_CCR3L
      000000BEH   SFRSYM    DATA     BYTE      TIM0_CCR4L
      000000D8H.6 SFRSYM    DATA     BIT       PMCD0
      000000C8H.4 SFRSYM    DATA     BIT       PTIM450
      000000D0H.3 SFRSYM    DATA     BIT       RS0
      000000DDH   SFRSYM    DATA     BYTE      LPF_KH
      000000F3H   SFRSYM    DATA     BYTE      PI_KIH
      000000EAH   SFRSYM    DATA     BYTE      PI_EKL
      000000E8H   SFRSYM    DATA     BYTE      FOC_SET0
      000000D8H.7 SFRSYM    DATA     BIT       PMCD1
      000000C8H.5 SFRSYM    DATA     BIT       PTIM451
      000000D0H.4 SFRSYM    DATA     BIT       RS1
      000000E9H   SFRSYM    DATA     BYTE      FOC_SET1
      000000B8H.6 SFRSYM    DATA     BIT       PFOC0
      000000DCH   SFRSYM    DATA     BYTE      LPF_KL
      000000F2H   SFRSYM    DATA     BYTE      PI_KIL
      000000B8H.7 SFRSYM    DATA     BIT       PFOC1
LX51 LINKER/LOCATER V4.66.1.0                                                         03/23/2017  15:15:44  PAGE 79


      000000ADH   SFRSYM    DATA     BYTE      TIM2_DRH
      000000B9H   SFRSYM    DATA     BYTE      TIM0_IER
      00000083H   SFRSYM    DATA     BYTE      DPH
      000000EFH   SFRSYM    DATA     BYTE      PI_KPH
      000000A5H   SFRSYM    DATA     BYTE      TIM3_DRH
      00000095H   SFRSYM    DATA     BYTE      TIM4_DRH
      0000008DH   SFRSYM    DATA     BYTE      TIM5_DRH
      000000ACH   SFRSYM    DATA     BYTE      TIM2_DRL
      00000082H   SFRSYM    DATA     BYTE      DPL
      000000EEH   SFRSYM    DATA     BYTE      PI_KPL
      000000A4H   SFRSYM    DATA     BYTE      TIM3_DRL
      000000F8H.7 SFRSYM    DATA     BIT       MOE
      000000C0H.6 SFRSYM    DATA     BIT       PCMP0
      000000EDH   SFRSYM    DATA     BYTE      PI_UKH
      00000094H   SFRSYM    DATA     BYTE      TIM4_DRL
      000000C0H.7 SFRSYM    DATA     BIT       PCMP1
      000000DFH   SFRSYM    DATA     BYTE      LPF_XH
      0000008CH   SFRSYM    DATA     BYTE      TIM5_DRL
      000000AEH   SFRSYM    DATA     WORD      TIM2_ARR
      000000A8H.5 SFRSYM    DATA     BIT       MCDIE
      000000C9H   SFRSYM    DATA     BYTE      RSTSRC
      000000E7H   SFRSYM    DATA     BYTE      LPF_YH
      000000A6H   SFRSYM    DATA     WORD      TIM3_ARR
      00000088H.6 SFRSYM    DATA     BIT       MCDIF
      00000098H.4 SFRSYM    DATA     BIT       REN
      00000096H   SFRSYM    DATA     WORD      TIM4_ARR
      000000ECH   SFRSYM    DATA     BYTE      PI_UKL
      000000D7H   SFRSYM    DATA     BYTE      CMP_SR
      0000008EH   SFRSYM    DATA     WORD      TIM5_ARR
      000000DEH   SFRSYM    DATA     BYTE      LPF_XL
      000000E6H   SFRSYM    DATA     BYTE      LPF_YL
      000000C8H   SFRSYM    DATA     BIT       PRTC0
      000000C8H.1 SFRSYM    DATA     BIT       PRTC1
      000000E8H.7 SFRSYM    DATA     BIT       FOCEN
      000000C8H.6 SFRSYM    DATA     BIT       PTSD0
      000000D8H.4 SFRSYM    DATA     BIT       PSPI0
      000000C8H.7 SFRSYM    DATA     BIT       PTSD1
      000000D8H.5 SFRSYM    DATA     BIT       PSPI1
      0000009BH   SFRSYM    DATA     BYTE      UT_BAUDH
      000000E4H   SFRSYM    DATA     WORD      SV_ANGLE
      000000B5H   SFRSYM    DATA     BYTE      TIM2_ADTRH
      0000009AH   SFRSYM    DATA     BYTE      UT_BAUDL
      000000FCH   SFRSYM    DATA     BYTE      P0_OE
      000000FDH   SFRSYM    DATA     BYTE      P1_OE
      000000D0H.5 SFRSYM    DATA     BIT       F0
      000000B4H   SFRSYM    DATA     BYTE      TIM2_ADTRL
      000000FEH   SFRSYM    DATA     BYTE      P2_OE
      000000D0H.1 SFRSYM    DATA     BIT       F1
      00000080H   SFRSYM    DATA     BIT       GP00
      000000FFH   SFRSYM    DATA     BYTE      P3_OE
      00000090H   SFRSYM    DATA     BIT       GP10
      00000080H.1 SFRSYM    DATA     BIT       GP01
      000000A8H.6 SFRSYM    DATA     BIT       RTCIE
      000000A0H   SFRSYM    DATA     BIT       GP20
      00000090H.1 SFRSYM    DATA     BIT       GP11
      00000080H.2 SFRSYM    DATA     BIT       GP02
      000000E3H   SFRSYM    DATA     BYTE      SV_USH
      000000B0H   SFRSYM    DATA     BIT       GP30
      000000A0H.1 SFRSYM    DATA     BIT       GP21
      00000090H.2 SFRSYM    DATA     BIT       GP12
      00000080H.3 SFRSYM    DATA     BIT       GP03
      000000B8H   SFRSYM    DATA     BIT       PLVW0
      000000A8H.1 SFRSYM    DATA     BIT       TSDIE
      000000D0H   SFRSYM    DATA     BYTE      PSW
      000000B0H.1 SFRSYM    DATA     BIT       GP31
LX51 LINKER/LOCATER V4.66.1.0                                                         03/23/2017  15:15:44  PAGE 80


      000000A0H.2 SFRSYM    DATA     BIT       GP22
      00000090H.3 SFRSYM    DATA     BIT       GP13
      00000080H.4 SFRSYM    DATA     BIT       GP04
      000000B8H.1 SFRSYM    DATA     BIT       PLVW1
      000000A8H.3 SFRSYM    DATA     BIT       SPIIE
      00000088H.5 SFRSYM    DATA     BIT       TSDIF
      000000B0H.2 SFRSYM    DATA     BIT       GP32
      000000A0H.3 SFRSYM    DATA     BIT       GP23
      00000090H.4 SFRSYM    DATA     BIT       GP14
      00000080H.5 SFRSYM    DATA     BIT       GP05
      00000084H   SFRSYM    DATA     BYTE      FLKEY
      000000B3H   SFRSYM    DATA     BYTE      TIM2_CMTRH
      000000B0H.3 SFRSYM    DATA     BIT       GP33
      000000A0H.4 SFRSYM    DATA     BIT       GP24
      00000090H.5 SFRSYM    DATA     BIT       GP15
      00000080H.6 SFRSYM    DATA     BIT       GP06
      00000088H   SFRSYM    DATA     BIT       IT00

      01001E06H   BLOCK     CODE     ---       LVL=0
      01001E06H   LINE      CODE     ---       #32
      01001E06H   LINE      CODE     ---       #33
      01001E06H   LINE      CODE     ---       #34
      01001E0BH   LINE      CODE     ---       #35
      01001E0FH   LINE      CODE     ---       #36
      01001E17H   LINE      CODE     ---       #37
      01001E1EH   LINE      CODE     ---       #38
      ---         BLOCKEND  ---      ---       LVL=0

      01001D55H   BLOCK     CODE     ---       LVL=0
      01001D55H   LINE      CODE     ---       #46
      01001D55H   LINE      CODE     ---       #47
      01001D55H   LINE      CODE     ---       #48
      01001D5FH   LINE      CODE     ---       #49
      01001D6FH   LINE      CODE     ---       #50
      01001D75H   LINE      CODE     ---       #51
      ---         BLOCKEND  ---      ---       LVL=0

      ---         MODULE    ---      ---       UARTSCAN
      02000155H   PUBLIC    XDATA    ---       UARTScan
      02000142H   PUBLIC    XDATA    ---       UARTControl
      01001BBDH   PUBLIC    CODE     ---       UARTScanInit
      000000E2H   SFRSYM    DATA     BYTE      SV_USL
      000000ABH   SFRSYM    DATA     BYTE      TIM2_CNTRH
      000000B0H.4 SFRSYM    DATA     BIT       GP34
      000000A0H.5 SFRSYM    DATA     BIT       GP25
      00000090H.6 SFRSYM    DATA     BIT       GP16
      00000080H.7 SFRSYM    DATA     BIT       GP07
      00000088H.1 SFRSYM    DATA     BIT       IT01
      00000088H.3 SFRSYM    DATA     BIT       IT10
      000000F6H   SFRSYM    DATA     WORD      PI_UKMIN
      000000C2H   SFRSYM    DATA     WORD      MD_MA
      000000A3H   SFRSYM    DATA     BYTE      TIM3_CNTRH
      000000B0H.5 SFRSYM    DATA     BIT       GP35
      000000A0H.6 SFRSYM    DATA     BIT       GP26
      00000090H.7 SFRSYM    DATA     BIT       GP17
      00000080H   SFRSYM    DATA     BYTE      P0
      00000088H.4 SFRSYM    DATA     BIT       IT11
      000000CAH   SFRSYM    DATA     WORD      MD_MB
      00000093H   SFRSYM    DATA     BYTE      TIM4_CNTRH
      000000B0H.6 SFRSYM    DATA     BIT       GP36
      000000A0H.7 SFRSYM    DATA     BIT       GP27
      00000090H   SFRSYM    DATA     BYTE      P1
      000000D9H   SFRSYM    DATA     BYTE      EVT_FILT
      000000F4H   SFRSYM    DATA     WORD      PI_UKMAX
      0000008BH   SFRSYM    DATA     BYTE      TIM5_CNTRH
LX51 LINKER/LOCATER V4.66.1.0                                                         03/23/2017  15:15:44  PAGE 81


      000000B2H   SFRSYM    DATA     BYTE      TIM2_CMTRL
      000000B0H.7 SFRSYM    DATA     BIT       GP37
      000000A0H   SFRSYM    DATA     BYTE      P2
      000000AAH   SFRSYM    DATA     BYTE      TIM2_CNTRL
      000000B0H   SFRSYM    DATA     BYTE      P3
      000000A2H   SFRSYM    DATA     BYTE      TIM3_CNTRL
      000000D0H.6 SFRSYM    DATA     BIT       AC
      00000092H   SFRSYM    DATA     BYTE      TIM4_CNTRL
      0000008AH   SFRSYM    DATA     BYTE      TIM5_CNTRL
      000000B6H   SFRSYM    DATA     WORD      TIM0_CCR1
      000000A8H.7 SFRSYM    DATA     BIT       EA
      000000D5H   SFRSYM    DATA     BYTE      CMP_CR0
      000000BAH   SFRSYM    DATA     WORD      TIM0_CCR2
      000000D6H   SFRSYM    DATA     BYTE      CMP_CR1
      000000BCH   SFRSYM    DATA     WORD      TIM0_CCR3
      00000085H   SFRSYM    DATA     BYTE      PSCTL
      000000DAH   SFRSYM    DATA     BYTE      CMP_CR2
      000000BEH   SFRSYM    DATA     WORD      TIM0_CCR4
      000000B8H.2 SFRSYM    DATA     BIT       PX00
      000000EAH   SFRSYM    DATA     WORD      PI_EK
      000000F8H   SFRSYM    DATA     BIT       OISUH
      000000B8H.3 SFRSYM    DATA     BIT       PX01
      000000B8H.4 SFRSYM    DATA     BIT       PX10
      000000F8H.2 SFRSYM    DATA     BIT       OISVH
      000000B8H.5 SFRSYM    DATA     BIT       PX11
      000000F8H.4 SFRSYM    DATA     BIT       OISWH
      000000DCH   SFRSYM    DATA     WORD      LPF_K
      000000F2H   SFRSYM    DATA     WORD      PI_KI
      000000F8H.1 SFRSYM    DATA     BIT       OISUL
      000000A8H   SFRSYM    DATA     BYTE      IE
      000000F8H.3 SFRSYM    DATA     BIT       OISVL
      000000F8H.5 SFRSYM    DATA     BIT       OISWL
      000000D1H   SFRSYM    DATA     BYTE      P1IE
      00000098H.6 SFRSYM    DATA     BIT       MOD0
      000000D3H   SFRSYM    DATA     BYTE      P2IE
      000000D2H   SFRSYM    DATA     BYTE      P1IF
      000000F9H   SFRSYM    DATA     BYTE      PL_CR
      00000098H.7 SFRSYM    DATA     BIT       MOD1
      000000D4H   SFRSYM    DATA     BYTE      P2IF
      000000ACH   SFRSYM    DATA     WORD      TIM2_DR
      00000082H   SFRSYM    DATA     WORD      DP
      000000EEH   SFRSYM    DATA     WORD      PI_KP
      000000A4H   SFRSYM    DATA     WORD      TIM3_DR
      00000094H   SFRSYM    DATA     WORD      TIM4_DR
      0000008CH   SFRSYM    DATA     WORD      TIM5_DR
      000000F1H   SFRSYM    DATA     BYTE      OSC_CFG
      000000C1H   SFRSYM    DATA     BYTE      MD_MODE
      000000ECH   SFRSYM    DATA     WORD      PI_UK
      000000DEH   SFRSYM    DATA     WORD      LPF_X
      00000098H   SFRSYM    DATA     BIT       RI
      000000E6H   SFRSYM    DATA     WORD      LPF_Y
      000000C0H   SFRSYM    DATA     BIT       PTIM00
      000000D0H.7 SFRSYM    DATA     BIT       CY
      00000098H.1 SFRSYM    DATA     BIT       TI
      000000C0H.1 SFRSYM    DATA     BIT       PTIM01
      000000C0H.2 SFRSYM    DATA     BIT       PTIM10
      000000C0H.3 SFRSYM    DATA     BIT       PTIM11
      000000E1H   SFRSYM    DATA     BYTE      SV_CR
      00000098H   SFRSYM    DATA     BYTE      UT_CR
      00000099H   SFRSYM    DATA     BYTE      UT_DR
      000000F8H.6 SFRSYM    DATA     BIT       OIS4
      00000081H   SFRSYM    DATA     BYTE      SP
      000000D0H.2 SFRSYM    DATA     BIT       OV
      000000C4H   SFRSYM    DATA     BYTE      MD_DA0
      0000009AH   SFRSYM    DATA     WORD      UT_BAUD
LX51 LINKER/LOCATER V4.66.1.0                                                         03/23/2017  15:15:44  PAGE 82


      000000CCH   SFRSYM    DATA     BYTE      MD_DB0
      000000C5H   SFRSYM    DATA     BYTE      MD_DA1
      000000CDH   SFRSYM    DATA     BYTE      MD_DB1
      000000C6H   SFRSYM    DATA     BYTE      MD_DA2
      000000CEH   SFRSYM    DATA     BYTE      MD_DB2
      000000C7H   SFRSYM    DATA     BYTE      MD_DA3
      000000B4H   SFRSYM    DATA     WORD      TIM2_ADTR
      000000CFH   SFRSYM    DATA     BYTE      MD_DB3
      000000AFH   SFRSYM    DATA     BYTE      TIM2_ARRH
      000000A7H   SFRSYM    DATA     BYTE      TIM3_ARRH
      00000097H   SFRSYM    DATA     BYTE      TIM4_ARRH
      0000008FH   SFRSYM    DATA     BYTE      TIM5_ARRH
      000000AEH   SFRSYM    DATA     BYTE      TIM2_ARRL
      000000A6H   SFRSYM    DATA     BYTE      TIM3_ARRL
      00000087H   SFRSYM    DATA     BYTE      PCON
      000000E2H   SFRSYM    DATA     WORD      SV_US
      00000096H   SFRSYM    DATA     BYTE      TIM4_ARRL
      0000008EH   SFRSYM    DATA     BYTE      TIM5_ARRL
      000000B2H   SFRSYM    DATA     WORD      TIM2_CMTR
      00000088H   SFRSYM    DATA     BYTE      TCON
      000000AAH   SFRSYM    DATA     WORD      TIM2_CNTR
      000000A2H   SFRSYM    DATA     WORD      TIM3_CNTR
      00000092H   SFRSYM    DATA     WORD      TIM4_CNTR
      0000008AH   SFRSYM    DATA     WORD      TIM5_CNTR
      000000E5H   SFRSYM    DATA     BYTE      SV_ANGLEH
      000000D8H   SFRSYM    DATA     BIT       PUART0
      000000E4H   SFRSYM    DATA     BYTE      SV_ANGLEL
      000000C6H   SFRSYM    DATA     WORD      MD_DAH
      000000D8H.1 SFRSYM    DATA     BIT       PUART1
      000000D8H.2 SFRSYM    DATA     BIT       PI2C0
      00000088H.2 SFRSYM    DATA     BIT       IF0
      000000CEH   SFRSYM    DATA     WORD      MD_DBH
      000000D8H.3 SFRSYM    DATA     BIT       PI2C1
      000000F0H   SFRSYM    DATA     BYTE      B
      000000C4H   SFRSYM    DATA     WORD      MD_DAL
      000000A1H   SFRSYM    DATA     BYTE      TIM2_CR0
      000000CCH   SFRSYM    DATA     WORD      MD_DBL
      0000009CH   SFRSYM    DATA     BYTE      TIM3_CR0
      000000A9H   SFRSYM    DATA     BYTE      TIM2_CR1
      0000009EH   SFRSYM    DATA     BYTE      TIM4_CR0
      0000009DH   SFRSYM    DATA     BYTE      TIM3_CR1
      00000089H   SFRSYM    DATA     BYTE      TIM5_CR0
      0000009FH   SFRSYM    DATA     BYTE      TIM4_CR1
      000000F8H   SFRSYM    DATA     BYTE      DRV_OUT
      00000091H   SFRSYM    DATA     BYTE      TIM5_CR1
      000000E0H   SFRSYM    DATA     BYTE      ACC
      000000F7H   SFRSYM    DATA     BYTE      PI_UKMINH
      000000C3H   SFRSYM    DATA     BYTE      MD_MAH
      000000A8H.4 SFRSYM    DATA     BIT       ES0
      000000DBH   SFRSYM    DATA     BYTE      LVSR
      000000CBH   SFRSYM    DATA     BYTE      MD_MBH
      000000C0H.4 SFRSYM    DATA     BIT       PADC0
      000000B8H   SFRSYM    DATA     BYTE      IP0
      000000F5H   SFRSYM    DATA     BYTE      PI_UKMAXH
      000000C0H.5 SFRSYM    DATA     BIT       PADC1
      000000C0H   SFRSYM    DATA     BYTE      IP1
      000000C8H   SFRSYM    DATA     BYTE      IP2
      000000F6H   SFRSYM    DATA     BYTE      PI_UKMINL
      000000C2H   SFRSYM    DATA     BYTE      MD_MAL
      00000098H.2 SFRSYM    DATA     BIT       RB8
      000000D8H   SFRSYM    DATA     BYTE      IP3
      000000CAH   SFRSYM    DATA     BYTE      MD_MBL
      000000A8H   SFRSYM    DATA     BIT       EX0
      000000F4H   SFRSYM    DATA     BYTE      PI_UKMAXL
      00000098H.3 SFRSYM    DATA     BIT       TB8
LX51 LINKER/LOCATER V4.66.1.0                                                         03/23/2017  15:15:44  PAGE 83


      000000B7H   SFRSYM    DATA     BYTE      TIM0_CCR1H
      000000A8H.2 SFRSYM    DATA     BIT       EX1
      000000BBH   SFRSYM    DATA     BYTE      TIM0_CCR2H
      000000D0H   SFRSYM    DATA     BIT       P
      000000BDH   SFRSYM    DATA     BYTE      TIM0_CCR3H
      000000BFH   SFRSYM    DATA     BYTE      TIM0_CCR4H
      000000C8H.2 SFRSYM    DATA     BIT       PTIM230
      000000EBH   SFRSYM    DATA     BYTE      PI_EKH
      00000098H.5 SFRSYM    DATA     BIT       SM2
      000000B6H   SFRSYM    DATA     BYTE      TIM0_CCR1L
      000000B1H   SFRSYM    DATA     BYTE      TIM0_SR1
      000000C8H.3 SFRSYM    DATA     BIT       PTIM231
      000000BAH   SFRSYM    DATA     BYTE      TIM0_CCR2L
      000000BCH   SFRSYM    DATA     BYTE      TIM0_CCR3L
      000000BEH   SFRSYM    DATA     BYTE      TIM0_CCR4L
      000000D8H.6 SFRSYM    DATA     BIT       PMCD0
      000000C8H.4 SFRSYM    DATA     BIT       PTIM450
      000000D0H.3 SFRSYM    DATA     BIT       RS0
      000000DDH   SFRSYM    DATA     BYTE      LPF_KH
      000000F3H   SFRSYM    DATA     BYTE      PI_KIH
      000000EAH   SFRSYM    DATA     BYTE      PI_EKL
      000000E8H   SFRSYM    DATA     BYTE      FOC_SET0
      000000D8H.7 SFRSYM    DATA     BIT       PMCD1
      000000C8H.5 SFRSYM    DATA     BIT       PTIM451
      000000D0H.4 SFRSYM    DATA     BIT       RS1
      000000E9H   SFRSYM    DATA     BYTE      FOC_SET1
      000000B8H.6 SFRSYM    DATA     BIT       PFOC0
      000000DCH   SFRSYM    DATA     BYTE      LPF_KL
      000000F2H   SFRSYM    DATA     BYTE      PI_KIL
      000000B8H.7 SFRSYM    DATA     BIT       PFOC1
      000000ADH   SFRSYM    DATA     BYTE      TIM2_DRH
      000000B9H   SFRSYM    DATA     BYTE      TIM0_IER
      00000083H   SFRSYM    DATA     BYTE      DPH
      000000EFH   SFRSYM    DATA     BYTE      PI_KPH
      000000A5H   SFRSYM    DATA     BYTE      TIM3_DRH
      00000095H   SFRSYM    DATA     BYTE      TIM4_DRH
      0000008DH   SFRSYM    DATA     BYTE      TIM5_DRH
      000000ACH   SFRSYM    DATA     BYTE      TIM2_DRL
      00000082H   SFRSYM    DATA     BYTE      DPL
      000000EEH   SFRSYM    DATA     BYTE      PI_KPL
      000000A4H   SFRSYM    DATA     BYTE      TIM3_DRL
      000000F8H.7 SFRSYM    DATA     BIT       MOE
      000000C0H.6 SFRSYM    DATA     BIT       PCMP0
      000000EDH   SFRSYM    DATA     BYTE      PI_UKH
      00000094H   SFRSYM    DATA     BYTE      TIM4_DRL
      000000C0H.7 SFRSYM    DATA     BIT       PCMP1
      000000DFH   SFRSYM    DATA     BYTE      LPF_XH
      0000008CH   SFRSYM    DATA     BYTE      TIM5_DRL
      000000AEH   SFRSYM    DATA     WORD      TIM2_ARR
      000000A8H.5 SFRSYM    DATA     BIT       MCDIE
      000000C9H   SFRSYM    DATA     BYTE      RSTSRC
      000000E7H   SFRSYM    DATA     BYTE      LPF_YH
      000000A6H   SFRSYM    DATA     WORD      TIM3_ARR
      00000088H.6 SFRSYM    DATA     BIT       MCDIF
      00000098H.4 SFRSYM    DATA     BIT       REN
      00000096H   SFRSYM    DATA     WORD      TIM4_ARR
      000000ECH   SFRSYM    DATA     BYTE      PI_UKL
      000000D7H   SFRSYM    DATA     BYTE      CMP_SR
      0000008EH   SFRSYM    DATA     WORD      TIM5_ARR
      000000DEH   SFRSYM    DATA     BYTE      LPF_XL
      000000E6H   SFRSYM    DATA     BYTE      LPF_YL
      000000C8H   SFRSYM    DATA     BIT       PRTC0
      000000C8H.1 SFRSYM    DATA     BIT       PRTC1
      000000E8H.7 SFRSYM    DATA     BIT       FOCEN
      000000C8H.6 SFRSYM    DATA     BIT       PTSD0
LX51 LINKER/LOCATER V4.66.1.0                                                         03/23/2017  15:15:44  PAGE 84


      000000D8H.4 SFRSYM    DATA     BIT       PSPI0
      000000C8H.7 SFRSYM    DATA     BIT       PTSD1
      000000D8H.5 SFRSYM    DATA     BIT       PSPI1
      0000009BH   SFRSYM    DATA     BYTE      UT_BAUDH
      000000E4H   SFRSYM    DATA     WORD      SV_ANGLE
      000000B5H   SFRSYM    DATA     BYTE      TIM2_ADTRH
      0000009AH   SFRSYM    DATA     BYTE      UT_BAUDL
      000000FCH   SFRSYM    DATA     BYTE      P0_OE
      000000FDH   SFRSYM    DATA     BYTE      P1_OE
      000000D0H.5 SFRSYM    DATA     BIT       F0
      000000B4H   SFRSYM    DATA     BYTE      TIM2_ADTRL
      000000FEH   SFRSYM    DATA     BYTE      P2_OE
      000000D0H.1 SFRSYM    DATA     BIT       F1
      00000080H   SFRSYM    DATA     BIT       GP00
      000000FFH   SFRSYM    DATA     BYTE      P3_OE
      00000090H   SFRSYM    DATA     BIT       GP10
      00000080H.1 SFRSYM    DATA     BIT       GP01
      000000A8H.6 SFRSYM    DATA     BIT       RTCIE
      000000A0H   SFRSYM    DATA     BIT       GP20
      00000090H.1 SFRSYM    DATA     BIT       GP11
      00000080H.2 SFRSYM    DATA     BIT       GP02
      000000E3H   SFRSYM    DATA     BYTE      SV_USH
      000000B0H   SFRSYM    DATA     BIT       GP30
      000000A0H.1 SFRSYM    DATA     BIT       GP21
      00000090H.2 SFRSYM    DATA     BIT       GP12
      00000080H.3 SFRSYM    DATA     BIT       GP03
      000000B8H   SFRSYM    DATA     BIT       PLVW0
      000000A8H.1 SFRSYM    DATA     BIT       TSDIE
      000000D0H   SFRSYM    DATA     BYTE      PSW
      000000B0H.1 SFRSYM    DATA     BIT       GP31
      000000A0H.2 SFRSYM    DATA     BIT       GP22
      00000090H.3 SFRSYM    DATA     BIT       GP13
      00000080H.4 SFRSYM    DATA     BIT       GP04
      000000B8H.1 SFRSYM    DATA     BIT       PLVW1
      000000A8H.3 SFRSYM    DATA     BIT       SPIIE
      00000088H.5 SFRSYM    DATA     BIT       TSDIF
      000000B0H.2 SFRSYM    DATA     BIT       GP32
      000000A0H.3 SFRSYM    DATA     BIT       GP23
      00000090H.4 SFRSYM    DATA     BIT       GP14
      00000080H.5 SFRSYM    DATA     BIT       GP05
      00000084H   SFRSYM    DATA     BYTE      FLKEY
      000000B3H   SFRSYM    DATA     BYTE      TIM2_CMTRH
      000000B0H.3 SFRSYM    DATA     BIT       GP33
      000000A0H.4 SFRSYM    DATA     BIT       GP24
      00000090H.5 SFRSYM    DATA     BIT       GP15
      00000080H.6 SFRSYM    DATA     BIT       GP06
      00000088H   SFRSYM    DATA     BIT       IT00

      01001BBDH   BLOCK     CODE     ---       LVL=0
      01001BBDH   LINE      CODE     ---       #32
      01001BBDH   LINE      CODE     ---       #33
      01001BBDH   LINE      CODE     ---       #34
      01001BC4H   LINE      CODE     ---       #36
      01001BC8H   LINE      CODE     ---       #37
      01001BCAH   LINE      CODE     ---       #38
      01001BCCH   LINE      CODE     ---       #39
      01001BCEH   LINE      CODE     ---       #40
      01001BD0H   LINE      CODE     ---       #42
      01001BD2H   LINE      CODE     ---       #43
      01001BD4H   LINE      CODE     ---       #44
      01001BD6H   LINE      CODE     ---       #45
      01001BD8H   LINE      CODE     ---       #46
      01001BDAH   LINE      CODE     ---       #47
      01001BDCH   LINE      CODE     ---       #48
      01001BDEH   LINE      CODE     ---       #49
LX51 LINKER/LOCATER V4.66.1.0                                                         03/23/2017  15:15:44  PAGE 85


      01001BE0H   LINE      CODE     ---       #50
      01001BE2H   LINE      CODE     ---       #51
      01001BE4H   LINE      CODE     ---       #52
      01001BE6H   LINE      CODE     ---       #53
      01001BE8H   LINE      CODE     ---       #54
      01001BECH   LINE      CODE     ---       #56
      ---         BLOCKEND  ---      ---       LVL=0

      ---         MODULE    ---      ---       LED
      02000187H   PUBLIC    XDATA    ---       LEDCtl
      0100143CH   PUBLIC    CODE     ---       LEDControl
      01001E99H   PUBLIC    CODE     ---       LEDControlInit
      000000E2H   SFRSYM    DATA     BYTE      SV_USL
      000000ABH   SFRSYM    DATA     BYTE      TIM2_CNTRH
      000000B0H.4 SFRSYM    DATA     BIT       GP34
      000000A0H.5 SFRSYM    DATA     BIT       GP25
      00000090H.6 SFRSYM    DATA     BIT       GP16
      00000080H.7 SFRSYM    DATA     BIT       GP07
      00000088H.1 SFRSYM    DATA     BIT       IT01
      00000088H.3 SFRSYM    DATA     BIT       IT10
      000000F6H   SFRSYM    DATA     WORD      PI_UKMIN
      000000C2H   SFRSYM    DATA     WORD      MD_MA
      000000A3H   SFRSYM    DATA     BYTE      TIM3_CNTRH
      000000B0H.5 SFRSYM    DATA     BIT       GP35
      000000A0H.6 SFRSYM    DATA     BIT       GP26
      00000090H.7 SFRSYM    DATA     BIT       GP17
      00000080H   SFRSYM    DATA     BYTE      P0
      00000088H.4 SFRSYM    DATA     BIT       IT11
      000000CAH   SFRSYM    DATA     WORD      MD_MB
      00000093H   SFRSYM    DATA     BYTE      TIM4_CNTRH
      000000B0H.6 SFRSYM    DATA     BIT       GP36
      000000A0H.7 SFRSYM    DATA     BIT       GP27
      00000090H   SFRSYM    DATA     BYTE      P1
      000000D9H   SFRSYM    DATA     BYTE      EVT_FILT
      000000F4H   SFRSYM    DATA     WORD      PI_UKMAX
      0000008BH   SFRSYM    DATA     BYTE      TIM5_CNTRH
      000000B2H   SFRSYM    DATA     BYTE      TIM2_CMTRL
      000000B0H.7 SFRSYM    DATA     BIT       GP37
      000000A0H   SFRSYM    DATA     BYTE      P2
      000000AAH   SFRSYM    DATA     BYTE      TIM2_CNTRL
      000000B0H   SFRSYM    DATA     BYTE      P3
      000000A2H   SFRSYM    DATA     BYTE      TIM3_CNTRL
      000000D0H.6 SFRSYM    DATA     BIT       AC
      00000092H   SFRSYM    DATA     BYTE      TIM4_CNTRL
      0000008AH   SFRSYM    DATA     BYTE      TIM5_CNTRL
      000000B6H   SFRSYM    DATA     WORD      TIM0_CCR1
      000000A8H.7 SFRSYM    DATA     BIT       EA
      000000D5H   SFRSYM    DATA     BYTE      CMP_CR0
      000000BAH   SFRSYM    DATA     WORD      TIM0_CCR2
      000000D6H   SFRSYM    DATA     BYTE      CMP_CR1
      000000BCH   SFRSYM    DATA     WORD      TIM0_CCR3
      00000085H   SFRSYM    DATA     BYTE      PSCTL
      000000DAH   SFRSYM    DATA     BYTE      CMP_CR2
      000000BEH   SFRSYM    DATA     WORD      TIM0_CCR4
      000000B8H.2 SFRSYM    DATA     BIT       PX00
      000000EAH   SFRSYM    DATA     WORD      PI_EK
      000000F8H   SFRSYM    DATA     BIT       OISUH
      000000B8H.3 SFRSYM    DATA     BIT       PX01
      000000B8H.4 SFRSYM    DATA     BIT       PX10
      000000F8H.2 SFRSYM    DATA     BIT       OISVH
      000000B8H.5 SFRSYM    DATA     BIT       PX11
      000000F8H.4 SFRSYM    DATA     BIT       OISWH
      000000DCH   SFRSYM    DATA     WORD      LPF_K
      000000F2H   SFRSYM    DATA     WORD      PI_KI
      000000F8H.1 SFRSYM    DATA     BIT       OISUL
LX51 LINKER/LOCATER V4.66.1.0                                                         03/23/2017  15:15:44  PAGE 86


      000000A8H   SFRSYM    DATA     BYTE      IE
      000000F8H.3 SFRSYM    DATA     BIT       OISVL
      000000F8H.5 SFRSYM    DATA     BIT       OISWL
      000000D1H   SFRSYM    DATA     BYTE      P1IE
      00000098H.6 SFRSYM    DATA     BIT       MOD0
      000000D3H   SFRSYM    DATA     BYTE      P2IE
      000000D2H   SFRSYM    DATA     BYTE      P1IF
      000000F9H   SFRSYM    DATA     BYTE      PL_CR
      00000098H.7 SFRSYM    DATA     BIT       MOD1
      000000D4H   SFRSYM    DATA     BYTE      P2IF
      000000ACH   SFRSYM    DATA     WORD      TIM2_DR
      00000082H   SFRSYM    DATA     WORD      DP
      000000EEH   SFRSYM    DATA     WORD      PI_KP
      000000A4H   SFRSYM    DATA     WORD      TIM3_DR
      00000094H   SFRSYM    DATA     WORD      TIM4_DR
      0000008CH   SFRSYM    DATA     WORD      TIM5_DR
      000000F1H   SFRSYM    DATA     BYTE      OSC_CFG
      000000C1H   SFRSYM    DATA     BYTE      MD_MODE
      000000ECH   SFRSYM    DATA     WORD      PI_UK
      000000DEH   SFRSYM    DATA     WORD      LPF_X
      00000098H   SFRSYM    DATA     BIT       RI
      000000E6H   SFRSYM    DATA     WORD      LPF_Y
      000000C0H   SFRSYM    DATA     BIT       PTIM00
      000000D0H.7 SFRSYM    DATA     BIT       CY
      00000098H.1 SFRSYM    DATA     BIT       TI
      000000C0H.1 SFRSYM    DATA     BIT       PTIM01
      000000C0H.2 SFRSYM    DATA     BIT       PTIM10
      000000C0H.3 SFRSYM    DATA     BIT       PTIM11
      000000E1H   SFRSYM    DATA     BYTE      SV_CR
      00000098H   SFRSYM    DATA     BYTE      UT_CR
      00000099H   SFRSYM    DATA     BYTE      UT_DR
      000000F8H.6 SFRSYM    DATA     BIT       OIS4
      00000081H   SFRSYM    DATA     BYTE      SP
      000000D0H.2 SFRSYM    DATA     BIT       OV
      000000C4H   SFRSYM    DATA     BYTE      MD_DA0
      0000009AH   SFRSYM    DATA     WORD      UT_BAUD
      000000CCH   SFRSYM    DATA     BYTE      MD_DB0
      000000C5H   SFRSYM    DATA     BYTE      MD_DA1
      000000CDH   SFRSYM    DATA     BYTE      MD_DB1
      000000C6H   SFRSYM    DATA     BYTE      MD_DA2
      000000CEH   SFRSYM    DATA     BYTE      MD_DB2
      000000C7H   SFRSYM    DATA     BYTE      MD_DA3
      000000B4H   SFRSYM    DATA     WORD      TIM2_ADTR
      000000CFH   SFRSYM    DATA     BYTE      MD_DB3
      000000AFH   SFRSYM    DATA     BYTE      TIM2_ARRH
      000000A7H   SFRSYM    DATA     BYTE      TIM3_ARRH
      00000097H   SFRSYM    DATA     BYTE      TIM4_ARRH
      0000008FH   SFRSYM    DATA     BYTE      TIM5_ARRH
      000000AEH   SFRSYM    DATA     BYTE      TIM2_ARRL
      000000A6H   SFRSYM    DATA     BYTE      TIM3_ARRL
      00000087H   SFRSYM    DATA     BYTE      PCON
      000000E2H   SFRSYM    DATA     WORD      SV_US
      00000096H   SFRSYM    DATA     BYTE      TIM4_ARRL
      0000008EH   SFRSYM    DATA     BYTE      TIM5_ARRL
      000000B2H   SFRSYM    DATA     WORD      TIM2_CMTR
      00000088H   SFRSYM    DATA     BYTE      TCON
      000000AAH   SFRSYM    DATA     WORD      TIM2_CNTR
      000000A2H   SFRSYM    DATA     WORD      TIM3_CNTR
      00000092H   SFRSYM    DATA     WORD      TIM4_CNTR
      0000008AH   SFRSYM    DATA     WORD      TIM5_CNTR
      000000E5H   SFRSYM    DATA     BYTE      SV_ANGLEH
      000000D8H   SFRSYM    DATA     BIT       PUART0
      000000E4H   SFRSYM    DATA     BYTE      SV_ANGLEL
      000000C6H   SFRSYM    DATA     WORD      MD_DAH
      000000D8H.1 SFRSYM    DATA     BIT       PUART1
LX51 LINKER/LOCATER V4.66.1.0                                                         03/23/2017  15:15:44  PAGE 87


      000000D8H.2 SFRSYM    DATA     BIT       PI2C0
      00000088H.2 SFRSYM    DATA     BIT       IF0
      000000CEH   SFRSYM    DATA     WORD      MD_DBH
      000000D8H.3 SFRSYM    DATA     BIT       PI2C1
      000000F0H   SFRSYM    DATA     BYTE      B
      000000C4H   SFRSYM    DATA     WORD      MD_DAL
      000000A1H   SFRSYM    DATA     BYTE      TIM2_CR0
      000000CCH   SFRSYM    DATA     WORD      MD_DBL
      0000009CH   SFRSYM    DATA     BYTE      TIM3_CR0
      000000A9H   SFRSYM    DATA     BYTE      TIM2_CR1
      0000009EH   SFRSYM    DATA     BYTE      TIM4_CR0
      0000009DH   SFRSYM    DATA     BYTE      TIM3_CR1
      00000089H   SFRSYM    DATA     BYTE      TIM5_CR0
      0000009FH   SFRSYM    DATA     BYTE      TIM4_CR1
      000000F8H   SFRSYM    DATA     BYTE      DRV_OUT
      00000091H   SFRSYM    DATA     BYTE      TIM5_CR1
      000000E0H   SFRSYM    DATA     BYTE      ACC
      000000F7H   SFRSYM    DATA     BYTE      PI_UKMINH
      000000C3H   SFRSYM    DATA     BYTE      MD_MAH
      000000A8H.4 SFRSYM    DATA     BIT       ES0
      000000DBH   SFRSYM    DATA     BYTE      LVSR
      000000CBH   SFRSYM    DATA     BYTE      MD_MBH
      000000C0H.4 SFRSYM    DATA     BIT       PADC0
      000000B8H   SFRSYM    DATA     BYTE      IP0
      000000F5H   SFRSYM    DATA     BYTE      PI_UKMAXH
      000000C0H.5 SFRSYM    DATA     BIT       PADC1
      000000C0H   SFRSYM    DATA     BYTE      IP1
      000000C8H   SFRSYM    DATA     BYTE      IP2
      000000F6H   SFRSYM    DATA     BYTE      PI_UKMINL
      000000C2H   SFRSYM    DATA     BYTE      MD_MAL
      00000098H.2 SFRSYM    DATA     BIT       RB8
      000000D8H   SFRSYM    DATA     BYTE      IP3
      000000CAH   SFRSYM    DATA     BYTE      MD_MBL
      000000A8H   SFRSYM    DATA     BIT       EX0
      000000F4H   SFRSYM    DATA     BYTE      PI_UKMAXL
      00000098H.3 SFRSYM    DATA     BIT       TB8
      000000B7H   SFRSYM    DATA     BYTE      TIM0_CCR1H
      000000A8H.2 SFRSYM    DATA     BIT       EX1
      000000BBH   SFRSYM    DATA     BYTE      TIM0_CCR2H
      000000D0H   SFRSYM    DATA     BIT       P
      000000BDH   SFRSYM    DATA     BYTE      TIM0_CCR3H
      000000BFH   SFRSYM    DATA     BYTE      TIM0_CCR4H
      000000C8H.2 SFRSYM    DATA     BIT       PTIM230
      000000EBH   SFRSYM    DATA     BYTE      PI_EKH
      00000098H.5 SFRSYM    DATA     BIT       SM2
      000000B6H   SFRSYM    DATA     BYTE      TIM0_CCR1L
      000000B1H   SFRSYM    DATA     BYTE      TIM0_SR1
      000000C8H.3 SFRSYM    DATA     BIT       PTIM231
      000000BAH   SFRSYM    DATA     BYTE      TIM0_CCR2L
      000000BCH   SFRSYM    DATA     BYTE      TIM0_CCR3L
      000000BEH   SFRSYM    DATA     BYTE      TIM0_CCR4L
      000000D8H.6 SFRSYM    DATA     BIT       PMCD0
      000000C8H.4 SFRSYM    DATA     BIT       PTIM450
      000000D0H.3 SFRSYM    DATA     BIT       RS0
      000000DDH   SFRSYM    DATA     BYTE      LPF_KH
      000000F3H   SFRSYM    DATA     BYTE      PI_KIH
      000000EAH   SFRSYM    DATA     BYTE      PI_EKL
      000000E8H   SFRSYM    DATA     BYTE      FOC_SET0
      000000D8H.7 SFRSYM    DATA     BIT       PMCD1
      000000C8H.5 SFRSYM    DATA     BIT       PTIM451
      000000D0H.4 SFRSYM    DATA     BIT       RS1
      000000E9H   SFRSYM    DATA     BYTE      FOC_SET1
      000000B8H.6 SFRSYM    DATA     BIT       PFOC0
      000000DCH   SFRSYM    DATA     BYTE      LPF_KL
      000000F2H   SFRSYM    DATA     BYTE      PI_KIL
LX51 LINKER/LOCATER V4.66.1.0                                                         03/23/2017  15:15:44  PAGE 88


      000000B8H.7 SFRSYM    DATA     BIT       PFOC1
      000000ADH   SFRSYM    DATA     BYTE      TIM2_DRH
      000000B9H   SFRSYM    DATA     BYTE      TIM0_IER
      00000083H   SFRSYM    DATA     BYTE      DPH
      000000EFH   SFRSYM    DATA     BYTE      PI_KPH
      000000A5H   SFRSYM    DATA     BYTE      TIM3_DRH
      00000095H   SFRSYM    DATA     BYTE      TIM4_DRH
      0000008DH   SFRSYM    DATA     BYTE      TIM5_DRH
      000000ACH   SFRSYM    DATA     BYTE      TIM2_DRL
      00000082H   SFRSYM    DATA     BYTE      DPL
      000000EEH   SFRSYM    DATA     BYTE      PI_KPL
      000000A4H   SFRSYM    DATA     BYTE      TIM3_DRL
      000000F8H.7 SFRSYM    DATA     BIT       MOE
      000000C0H.6 SFRSYM    DATA     BIT       PCMP0
      000000EDH   SFRSYM    DATA     BYTE      PI_UKH
      00000094H   SFRSYM    DATA     BYTE      TIM4_DRL
      000000C0H.7 SFRSYM    DATA     BIT       PCMP1
      000000DFH   SFRSYM    DATA     BYTE      LPF_XH
      0000008CH   SFRSYM    DATA     BYTE      TIM5_DRL
      000000AEH   SFRSYM    DATA     WORD      TIM2_ARR
      000000A8H.5 SFRSYM    DATA     BIT       MCDIE
      000000C9H   SFRSYM    DATA     BYTE      RSTSRC
      000000E7H   SFRSYM    DATA     BYTE      LPF_YH
      000000A6H   SFRSYM    DATA     WORD      TIM3_ARR
      00000088H.6 SFRSYM    DATA     BIT       MCDIF
      00000098H.4 SFRSYM    DATA     BIT       REN
      00000096H   SFRSYM    DATA     WORD      TIM4_ARR
      000000ECH   SFRSYM    DATA     BYTE      PI_UKL
      000000D7H   SFRSYM    DATA     BYTE      CMP_SR
      0000008EH   SFRSYM    DATA     WORD      TIM5_ARR
      000000DEH   SFRSYM    DATA     BYTE      LPF_XL
      000000E6H   SFRSYM    DATA     BYTE      LPF_YL
      000000C8H   SFRSYM    DATA     BIT       PRTC0
      000000C8H.1 SFRSYM    DATA     BIT       PRTC1
      000000E8H.7 SFRSYM    DATA     BIT       FOCEN
      000000C8H.6 SFRSYM    DATA     BIT       PTSD0
      000000D8H.4 SFRSYM    DATA     BIT       PSPI0
      000000C8H.7 SFRSYM    DATA     BIT       PTSD1
      000000D8H.5 SFRSYM    DATA     BIT       PSPI1
      0000009BH   SFRSYM    DATA     BYTE      UT_BAUDH
      000000E4H   SFRSYM    DATA     WORD      SV_ANGLE
      000000B5H   SFRSYM    DATA     BYTE      TIM2_ADTRH
      0000009AH   SFRSYM    DATA     BYTE      UT_BAUDL
      000000FCH   SFRSYM    DATA     BYTE      P0_OE
      000000FDH   SFRSYM    DATA     BYTE      P1_OE
      000000D0H.5 SFRSYM    DATA     BIT       F0
      000000B4H   SFRSYM    DATA     BYTE      TIM2_ADTRL
      000000FEH   SFRSYM    DATA     BYTE      P2_OE
      000000D0H.1 SFRSYM    DATA     BIT       F1
      00000080H   SFRSYM    DATA     BIT       GP00
      000000FFH   SFRSYM    DATA     BYTE      P3_OE
      00000090H   SFRSYM    DATA     BIT       GP10
      00000080H.1 SFRSYM    DATA     BIT       GP01
      000000A8H.6 SFRSYM    DATA     BIT       RTCIE
      000000A0H   SFRSYM    DATA     BIT       GP20
      00000090H.1 SFRSYM    DATA     BIT       GP11
      00000080H.2 SFRSYM    DATA     BIT       GP02
      000000E3H   SFRSYM    DATA     BYTE      SV_USH
      000000B0H   SFRSYM    DATA     BIT       GP30
      000000A0H.1 SFRSYM    DATA     BIT       GP21
      00000090H.2 SFRSYM    DATA     BIT       GP12
      00000080H.3 SFRSYM    DATA     BIT       GP03
      000000B8H   SFRSYM    DATA     BIT       PLVW0
      000000A8H.1 SFRSYM    DATA     BIT       TSDIE
      000000D0H   SFRSYM    DATA     BYTE      PSW
LX51 LINKER/LOCATER V4.66.1.0                                                         03/23/2017  15:15:44  PAGE 89


      000000B0H.1 SFRSYM    DATA     BIT       GP31
      000000A0H.2 SFRSYM    DATA     BIT       GP22
      00000090H.3 SFRSYM    DATA     BIT       GP13
      00000080H.4 SFRSYM    DATA     BIT       GP04
      000000B8H.1 SFRSYM    DATA     BIT       PLVW1
      000000A8H.3 SFRSYM    DATA     BIT       SPIIE
      00000088H.5 SFRSYM    DATA     BIT       TSDIF
      000000B0H.2 SFRSYM    DATA     BIT       GP32
      000000A0H.3 SFRSYM    DATA     BIT       GP23
      00000090H.4 SFRSYM    DATA     BIT       GP14
      00000080H.5 SFRSYM    DATA     BIT       GP05
      00000084H   SFRSYM    DATA     BYTE      FLKEY
      000000B3H   SFRSYM    DATA     BYTE      TIM2_CMTRH
      000000B0H.3 SFRSYM    DATA     BIT       GP33
      000000A0H.4 SFRSYM    DATA     BIT       GP24
      00000090H.5 SFRSYM    DATA     BIT       GP15
      00000080H.6 SFRSYM    DATA     BIT       GP06
      00000088H   SFRSYM    DATA     BIT       IT00

      01001E99H   BLOCK     CODE     ---       LVL=0
      01001E99H   LINE      CODE     ---       #26
      01001E99H   LINE      CODE     ---       #27
      01001E99H   LINE      CODE     ---       #28
      01001E9EH   LINE      CODE     ---       #29
      01001EA0H   LINE      CODE     ---       #30
      01001EA2H   LINE      CODE     ---       #31
      01001EA6H   LINE      CODE     ---       #33
      ---         BLOCKEND  ---      ---       LVL=0

      0100143CH   BLOCK     CODE     ---       LVL=0
      0100143CH   LINE      CODE     ---       #44
      0100143CH   LINE      CODE     ---       #45
      0100143CH   LINE      CODE     ---       #47
      01001443H   LINE      CODE     ---       #48
      01001443H   LINE      CODE     ---       #49
      01001445H   LINE      CODE     ---       #50
      01001445H   LINE      CODE     ---       #52
      0100144EH   LINE      CODE     ---       #53
      0100144EH   LINE      CODE     ---       #54
      01001450H   LINE      CODE     ---       #55
      01001450H   LINE      CODE     ---       #57
      01001455H   LINE      CODE     ---       #58
      01001455H   LINE      CODE     ---       #59
      0100146EH   LINE      CODE     ---       #60
      0100146EH   LINE      CODE     ---       #61
      01001472H   LINE      CODE     ---       #62
      01001472H   LINE      CODE     ---       #63
      01001474H   LINE      CODE     ---       #64
      0100147AH   LINE      CODE     ---       #65
      0100147EH   LINE      CODE     ---       #66
      01001485H   LINE      CODE     ---       #67
      01001485H   LINE      CODE     ---       #68
      010014A3H   LINE      CODE     ---       #69
      010014A3H   LINE      CODE     ---       #70
      010014A8H   LINE      CODE     ---       #71
      010014A8H   LINE      CODE     ---       #73
      010014A9H   LINE      CODE     ---       #75
      010014A9H   LINE      CODE     ---       #76
      010014AFH   LINE      CODE     ---       #77
      010014AFH   LINE      CODE     ---       #78
      010014B1H   LINE      CODE     ---       #79
      010014B3H   LINE      CODE     ---       #80
      010014BAH   LINE      CODE     ---       #81
      010014BAH   LINE      CODE     ---       #82
      010014C9H   LINE      CODE     ---       #83
LX51 LINKER/LOCATER V4.66.1.0                                                         03/23/2017  15:15:44  PAGE 90


      010014C9H   LINE      CODE     ---       #84
      010014CEH   LINE      CODE     ---       #85
      010014D0H   LINE      CODE     ---       #86
      010014D0H   LINE      CODE     ---       #87
      010014D0H   LINE      CODE     ---       #88
      010014D0H   LINE      CODE     ---       #89
      ---         BLOCKEND  ---      ---       LVL=0

      ---         MODULE    ---      ---       PID
      00000049H   PUBLIC    IDATA    ---       PowerPID
      02000185H   PUBLIC    XDATA    WORD      TargetSpeed
      00000039H   PUBLIC    IDATA    ---       SpeedPID
      00000029H   PUBLIC    IDATA    ---       CurrentPID
      02000183H   PUBLIC    XDATA    WORD      Delta_Speed
      02000181H   PUBLIC    XDATA    WORD      Delta_Current
      00000020H.2 PUBLIC    BIT      BIT       FlagStartPI
      00000021H   PUBLIC    IDATA    ---       SpeedRamp
      000000E2H   SFRSYM    DATA     BYTE      SV_USL
      000000ABH   SFRSYM    DATA     BYTE      TIM2_CNTRH
      000000B0H.4 SFRSYM    DATA     BIT       GP34
      000000A0H.5 SFRSYM    DATA     BIT       GP25
      00000090H.6 SFRSYM    DATA     BIT       GP16
      00000080H.7 SFRSYM    DATA     BIT       GP07
      00000088H.1 SFRSYM    DATA     BIT       IT01
      00000088H.3 SFRSYM    DATA     BIT       IT10
      000000F6H   SFRSYM    DATA     WORD      PI_UKMIN
      000000C2H   SFRSYM    DATA     WORD      MD_MA
      000000A3H   SFRSYM    DATA     BYTE      TIM3_CNTRH
      000000B0H.5 SFRSYM    DATA     BIT       GP35
      000000A0H.6 SFRSYM    DATA     BIT       GP26
      00000090H.7 SFRSYM    DATA     BIT       GP17
      00000080H   SFRSYM    DATA     BYTE      P0
      00000088H.4 SFRSYM    DATA     BIT       IT11
      000000CAH   SFRSYM    DATA     WORD      MD_MB
      00000093H   SFRSYM    DATA     BYTE      TIM4_CNTRH
      000000B0H.6 SFRSYM    DATA     BIT       GP36
      000000A0H.7 SFRSYM    DATA     BIT       GP27
      00000090H   SFRSYM    DATA     BYTE      P1
      000000D9H   SFRSYM    DATA     BYTE      EVT_FILT
      000000F4H   SFRSYM    DATA     WORD      PI_UKMAX
      0000008BH   SFRSYM    DATA     BYTE      TIM5_CNTRH
      000000B2H   SFRSYM    DATA     BYTE      TIM2_CMTRL
      000000B0H.7 SFRSYM    DATA     BIT       GP37
      000000A0H   SFRSYM    DATA     BYTE      P2
      000000AAH   SFRSYM    DATA     BYTE      TIM2_CNTRL
      000000B0H   SFRSYM    DATA     BYTE      P3
      000000A2H   SFRSYM    DATA     BYTE      TIM3_CNTRL
      000000D0H.6 SFRSYM    DATA     BIT       AC
      00000092H   SFRSYM    DATA     BYTE      TIM4_CNTRL
      0000008AH   SFRSYM    DATA     BYTE      TIM5_CNTRL
      000000B6H   SFRSYM    DATA     WORD      TIM0_CCR1
      000000A8H.7 SFRSYM    DATA     BIT       EA
      000000D5H   SFRSYM    DATA     BYTE      CMP_CR0
      000000BAH   SFRSYM    DATA     WORD      TIM0_CCR2
      000000D6H   SFRSYM    DATA     BYTE      CMP_CR1
      000000BCH   SFRSYM    DATA     WORD      TIM0_CCR3
      00000085H   SFRSYM    DATA     BYTE      PSCTL
      000000DAH   SFRSYM    DATA     BYTE      CMP_CR2
      000000BEH   SFRSYM    DATA     WORD      TIM0_CCR4
      000000B8H.2 SFRSYM    DATA     BIT       PX00
      000000EAH   SFRSYM    DATA     WORD      PI_EK
      000000F8H   SFRSYM    DATA     BIT       OISUH
      000000B8H.3 SFRSYM    DATA     BIT       PX01
      000000B8H.4 SFRSYM    DATA     BIT       PX10
      000000F8H.2 SFRSYM    DATA     BIT       OISVH
LX51 LINKER/LOCATER V4.66.1.0                                                         03/23/2017  15:15:44  PAGE 91


      000000B8H.5 SFRSYM    DATA     BIT       PX11
      000000F8H.4 SFRSYM    DATA     BIT       OISWH
      000000DCH   SFRSYM    DATA     WORD      LPF_K
      000000F2H   SFRSYM    DATA     WORD      PI_KI
      000000F8H.1 SFRSYM    DATA     BIT       OISUL
      000000A8H   SFRSYM    DATA     BYTE      IE
      000000F8H.3 SFRSYM    DATA     BIT       OISVL
      000000F8H.5 SFRSYM    DATA     BIT       OISWL
      000000D1H   SFRSYM    DATA     BYTE      P1IE
      00000098H.6 SFRSYM    DATA     BIT       MOD0
      000000D3H   SFRSYM    DATA     BYTE      P2IE
      000000D2H   SFRSYM    DATA     BYTE      P1IF
      000000F9H   SFRSYM    DATA     BYTE      PL_CR
      00000098H.7 SFRSYM    DATA     BIT       MOD1
      000000D4H   SFRSYM    DATA     BYTE      P2IF
      000000ACH   SFRSYM    DATA     WORD      TIM2_DR
      00000082H   SFRSYM    DATA     WORD      DP
      000000EEH   SFRSYM    DATA     WORD      PI_KP
      000000A4H   SFRSYM    DATA     WORD      TIM3_DR
      00000094H   SFRSYM    DATA     WORD      TIM4_DR
      0000008CH   SFRSYM    DATA     WORD      TIM5_DR
      000000F1H   SFRSYM    DATA     BYTE      OSC_CFG
      000000C1H   SFRSYM    DATA     BYTE      MD_MODE
      000000ECH   SFRSYM    DATA     WORD      PI_UK
      000000DEH   SFRSYM    DATA     WORD      LPF_X
      00000098H   SFRSYM    DATA     BIT       RI
      000000E6H   SFRSYM    DATA     WORD      LPF_Y
      000000C0H   SFRSYM    DATA     BIT       PTIM00
      000000D0H.7 SFRSYM    DATA     BIT       CY
      00000098H.1 SFRSYM    DATA     BIT       TI
      000000C0H.1 SFRSYM    DATA     BIT       PTIM01
      000000C0H.2 SFRSYM    DATA     BIT       PTIM10
      000000C0H.3 SFRSYM    DATA     BIT       PTIM11
      000000E1H   SFRSYM    DATA     BYTE      SV_CR
      00000098H   SFRSYM    DATA     BYTE      UT_CR
      00000099H   SFRSYM    DATA     BYTE      UT_DR
      000000F8H.6 SFRSYM    DATA     BIT       OIS4
      00000081H   SFRSYM    DATA     BYTE      SP
      000000D0H.2 SFRSYM    DATA     BIT       OV
      000000C4H   SFRSYM    DATA     BYTE      MD_DA0
      0000009AH   SFRSYM    DATA     WORD      UT_BAUD
      000000CCH   SFRSYM    DATA     BYTE      MD_DB0
      000000C5H   SFRSYM    DATA     BYTE      MD_DA1
      000000CDH   SFRSYM    DATA     BYTE      MD_DB1
      000000C6H   SFRSYM    DATA     BYTE      MD_DA2
      000000CEH   SFRSYM    DATA     BYTE      MD_DB2
      000000C7H   SFRSYM    DATA     BYTE      MD_DA3
      000000B4H   SFRSYM    DATA     WORD      TIM2_ADTR
      000000CFH   SFRSYM    DATA     BYTE      MD_DB3
      000000AFH   SFRSYM    DATA     BYTE      TIM2_ARRH
      000000A7H   SFRSYM    DATA     BYTE      TIM3_ARRH
      00000097H   SFRSYM    DATA     BYTE      TIM4_ARRH
      0000008FH   SFRSYM    DATA     BYTE      TIM5_ARRH
      000000AEH   SFRSYM    DATA     BYTE      TIM2_ARRL
      000000A6H   SFRSYM    DATA     BYTE      TIM3_ARRL
      00000087H   SFRSYM    DATA     BYTE      PCON
      000000E2H   SFRSYM    DATA     WORD      SV_US
      00000096H   SFRSYM    DATA     BYTE      TIM4_ARRL
      0000008EH   SFRSYM    DATA     BYTE      TIM5_ARRL
      000000B2H   SFRSYM    DATA     WORD      TIM2_CMTR
      00000088H   SFRSYM    DATA     BYTE      TCON
      000000AAH   SFRSYM    DATA     WORD      TIM2_CNTR
      000000A2H   SFRSYM    DATA     WORD      TIM3_CNTR
      00000092H   SFRSYM    DATA     WORD      TIM4_CNTR
      0000008AH   SFRSYM    DATA     WORD      TIM5_CNTR
LX51 LINKER/LOCATER V4.66.1.0                                                         03/23/2017  15:15:44  PAGE 92


      000000E5H   SFRSYM    DATA     BYTE      SV_ANGLEH
      000000D8H   SFRSYM    DATA     BIT       PUART0
      000000E4H   SFRSYM    DATA     BYTE      SV_ANGLEL
      000000C6H   SFRSYM    DATA     WORD      MD_DAH
      000000D8H.1 SFRSYM    DATA     BIT       PUART1
      000000D8H.2 SFRSYM    DATA     BIT       PI2C0
      00000088H.2 SFRSYM    DATA     BIT       IF0
      000000CEH   SFRSYM    DATA     WORD      MD_DBH
      000000D8H.3 SFRSYM    DATA     BIT       PI2C1
      000000F0H   SFRSYM    DATA     BYTE      B
      000000C4H   SFRSYM    DATA     WORD      MD_DAL
      000000A1H   SFRSYM    DATA     BYTE      TIM2_CR0
      000000CCH   SFRSYM    DATA     WORD      MD_DBL
      0000009CH   SFRSYM    DATA     BYTE      TIM3_CR0
      000000A9H   SFRSYM    DATA     BYTE      TIM2_CR1
      0000009EH   SFRSYM    DATA     BYTE      TIM4_CR0
      0000009DH   SFRSYM    DATA     BYTE      TIM3_CR1
      00000089H   SFRSYM    DATA     BYTE      TIM5_CR0
      0000009FH   SFRSYM    DATA     BYTE      TIM4_CR1
      000000F8H   SFRSYM    DATA     BYTE      DRV_OUT
      00000091H   SFRSYM    DATA     BYTE      TIM5_CR1
      000000E0H   SFRSYM    DATA     BYTE      ACC
      000000F7H   SFRSYM    DATA     BYTE      PI_UKMINH
      000000C3H   SFRSYM    DATA     BYTE      MD_MAH
      000000A8H.4 SFRSYM    DATA     BIT       ES0
      000000DBH   SFRSYM    DATA     BYTE      LVSR
      000000CBH   SFRSYM    DATA     BYTE      MD_MBH
      000000C0H.4 SFRSYM    DATA     BIT       PADC0
      000000B8H   SFRSYM    DATA     BYTE      IP0
      000000F5H   SFRSYM    DATA     BYTE      PI_UKMAXH
      000000C0H.5 SFRSYM    DATA     BIT       PADC1
      000000C0H   SFRSYM    DATA     BYTE      IP1
      000000C8H   SFRSYM    DATA     BYTE      IP2
      000000F6H   SFRSYM    DATA     BYTE      PI_UKMINL
      000000C2H   SFRSYM    DATA     BYTE      MD_MAL
      00000098H.2 SFRSYM    DATA     BIT       RB8
      000000D8H   SFRSYM    DATA     BYTE      IP3
      000000CAH   SFRSYM    DATA     BYTE      MD_MBL
      000000A8H   SFRSYM    DATA     BIT       EX0
      000000F4H   SFRSYM    DATA     BYTE      PI_UKMAXL
      00000098H.3 SFRSYM    DATA     BIT       TB8
      000000B7H   SFRSYM    DATA     BYTE      TIM0_CCR1H
      000000A8H.2 SFRSYM    DATA     BIT       EX1
      000000BBH   SFRSYM    DATA     BYTE      TIM0_CCR2H
      000000D0H   SFRSYM    DATA     BIT       P
      000000BDH   SFRSYM    DATA     BYTE      TIM0_CCR3H
      000000BFH   SFRSYM    DATA     BYTE      TIM0_CCR4H
      000000C8H.2 SFRSYM    DATA     BIT       PTIM230
      000000EBH   SFRSYM    DATA     BYTE      PI_EKH
      00000098H.5 SFRSYM    DATA     BIT       SM2
      000000B6H   SFRSYM    DATA     BYTE      TIM0_CCR1L
      000000B1H   SFRSYM    DATA     BYTE      TIM0_SR1
      000000C8H.3 SFRSYM    DATA     BIT       PTIM231
      000000BAH   SFRSYM    DATA     BYTE      TIM0_CCR2L
      000000BCH   SFRSYM    DATA     BYTE      TIM0_CCR3L
      000000BEH   SFRSYM    DATA     BYTE      TIM0_CCR4L
      000000D8H.6 SFRSYM    DATA     BIT       PMCD0
      000000C8H.4 SFRSYM    DATA     BIT       PTIM450
      000000D0H.3 SFRSYM    DATA     BIT       RS0
      000000DDH   SFRSYM    DATA     BYTE      LPF_KH
      000000F3H   SFRSYM    DATA     BYTE      PI_KIH
      000000EAH   SFRSYM    DATA     BYTE      PI_EKL
      000000E8H   SFRSYM    DATA     BYTE      FOC_SET0
      000000D8H.7 SFRSYM    DATA     BIT       PMCD1
      000000C8H.5 SFRSYM    DATA     BIT       PTIM451
LX51 LINKER/LOCATER V4.66.1.0                                                         03/23/2017  15:15:44  PAGE 93


      000000D0H.4 SFRSYM    DATA     BIT       RS1
      000000E9H   SFRSYM    DATA     BYTE      FOC_SET1
      000000B8H.6 SFRSYM    DATA     BIT       PFOC0
      000000DCH   SFRSYM    DATA     BYTE      LPF_KL
      000000F2H   SFRSYM    DATA     BYTE      PI_KIL
      000000B8H.7 SFRSYM    DATA     BIT       PFOC1
      000000ADH   SFRSYM    DATA     BYTE      TIM2_DRH
      000000B9H   SFRSYM    DATA     BYTE      TIM0_IER
      00000083H   SFRSYM    DATA     BYTE      DPH
      000000EFH   SFRSYM    DATA     BYTE      PI_KPH
      000000A5H   SFRSYM    DATA     BYTE      TIM3_DRH
      00000095H   SFRSYM    DATA     BYTE      TIM4_DRH
      0000008DH   SFRSYM    DATA     BYTE      TIM5_DRH
      000000ACH   SFRSYM    DATA     BYTE      TIM2_DRL
      00000082H   SFRSYM    DATA     BYTE      DPL
      000000EEH   SFRSYM    DATA     BYTE      PI_KPL
      000000A4H   SFRSYM    DATA     BYTE      TIM3_DRL
      000000F8H.7 SFRSYM    DATA     BIT       MOE
      000000C0H.6 SFRSYM    DATA     BIT       PCMP0
      000000EDH   SFRSYM    DATA     BYTE      PI_UKH
      00000094H   SFRSYM    DATA     BYTE      TIM4_DRL
      000000C0H.7 SFRSYM    DATA     BIT       PCMP1
      000000DFH   SFRSYM    DATA     BYTE      LPF_XH
      0000008CH   SFRSYM    DATA     BYTE      TIM5_DRL
      000000AEH   SFRSYM    DATA     WORD      TIM2_ARR
      000000A8H.5 SFRSYM    DATA     BIT       MCDIE
      000000C9H   SFRSYM    DATA     BYTE      RSTSRC
      000000E7H   SFRSYM    DATA     BYTE      LPF_YH
      000000A6H   SFRSYM    DATA     WORD      TIM3_ARR
      00000088H.6 SFRSYM    DATA     BIT       MCDIF
      00000098H.4 SFRSYM    DATA     BIT       REN
      00000096H   SFRSYM    DATA     WORD      TIM4_ARR
      000000ECH   SFRSYM    DATA     BYTE      PI_UKL
      000000D7H   SFRSYM    DATA     BYTE      CMP_SR
      0000008EH   SFRSYM    DATA     WORD      TIM5_ARR
      000000DEH   SFRSYM    DATA     BYTE      LPF_XL
      000000E6H   SFRSYM    DATA     BYTE      LPF_YL
      000000C8H   SFRSYM    DATA     BIT       PRTC0
      000000C8H.1 SFRSYM    DATA     BIT       PRTC1
      000000E8H.7 SFRSYM    DATA     BIT       FOCEN
      000000C8H.6 SFRSYM    DATA     BIT       PTSD0
      000000D8H.4 SFRSYM    DATA     BIT       PSPI0
      000000C8H.7 SFRSYM    DATA     BIT       PTSD1
      000000D8H.5 SFRSYM    DATA     BIT       PSPI1
      0000009BH   SFRSYM    DATA     BYTE      UT_BAUDH
      000000E4H   SFRSYM    DATA     WORD      SV_ANGLE
      000000B5H   SFRSYM    DATA     BYTE      TIM2_ADTRH
      0000009AH   SFRSYM    DATA     BYTE      UT_BAUDL
      000000FCH   SFRSYM    DATA     BYTE      P0_OE
      000000FDH   SFRSYM    DATA     BYTE      P1_OE
      000000D0H.5 SFRSYM    DATA     BIT       F0
      000000B4H   SFRSYM    DATA     BYTE      TIM2_ADTRL
      000000FEH   SFRSYM    DATA     BYTE      P2_OE
      000000D0H.1 SFRSYM    DATA     BIT       F1
      00000080H   SFRSYM    DATA     BIT       GP00
      000000FFH   SFRSYM    DATA     BYTE      P3_OE
      00000090H   SFRSYM    DATA     BIT       GP10
      00000080H.1 SFRSYM    DATA     BIT       GP01
      000000A8H.6 SFRSYM    DATA     BIT       RTCIE
      000000A0H   SFRSYM    DATA     BIT       GP20
      00000090H.1 SFRSYM    DATA     BIT       GP11
      00000080H.2 SFRSYM    DATA     BIT       GP02
      000000E3H   SFRSYM    DATA     BYTE      SV_USH
      000000B0H   SFRSYM    DATA     BIT       GP30
      000000A0H.1 SFRSYM    DATA     BIT       GP21
LX51 LINKER/LOCATER V4.66.1.0                                                         03/23/2017  15:15:44  PAGE 94


      00000090H.2 SFRSYM    DATA     BIT       GP12
      00000080H.3 SFRSYM    DATA     BIT       GP03
      000000B8H   SFRSYM    DATA     BIT       PLVW0
      000000A8H.1 SFRSYM    DATA     BIT       TSDIE
      000000D0H   SFRSYM    DATA     BYTE      PSW
      000000B0H.1 SFRSYM    DATA     BIT       GP31
      000000A0H.2 SFRSYM    DATA     BIT       GP22
      00000090H.3 SFRSYM    DATA     BIT       GP13
      00000080H.4 SFRSYM    DATA     BIT       GP04
      000000B8H.1 SFRSYM    DATA     BIT       PLVW1
      000000A8H.3 SFRSYM    DATA     BIT       SPIIE
      00000088H.5 SFRSYM    DATA     BIT       TSDIF
      000000B0H.2 SFRSYM    DATA     BIT       GP32
      000000A0H.3 SFRSYM    DATA     BIT       GP23
      00000090H.4 SFRSYM    DATA     BIT       GP14
      00000080H.5 SFRSYM    DATA     BIT       GP05
      00000084H   SFRSYM    DATA     BYTE      FLKEY
      000000B3H   SFRSYM    DATA     BYTE      TIM2_CMTRH
      000000B0H.3 SFRSYM    DATA     BIT       GP33
      000000A0H.4 SFRSYM    DATA     BIT       GP24
      00000090H.5 SFRSYM    DATA     BIT       GP15
      00000080H.6 SFRSYM    DATA     BIT       GP06
      00000088H   SFRSYM    DATA     BIT       IT00
      00000006H   SYMBOL    DATA     WORD      TargetCurrent

      ---         MODULE    ---      ---       UARTINIT
      000000E2H   SFRSYM    DATA     BYTE      SV_USL
      000000ABH   SFRSYM    DATA     BYTE      TIM2_CNTRH
      000000B0H.4 SFRSYM    DATA     BIT       GP34
      000000A0H.5 SFRSYM    DATA     BIT       GP25
      00000090H.6 SFRSYM    DATA     BIT       GP16
      00000080H.7 SFRSYM    DATA     BIT       GP07
      00000088H.1 SFRSYM    DATA     BIT       IT01
      00000088H.3 SFRSYM    DATA     BIT       IT10
      000000F6H   SFRSYM    DATA     WORD      PI_UKMIN
      000000C2H   SFRSYM    DATA     WORD      MD_MA
      000000A3H   SFRSYM    DATA     BYTE      TIM3_CNTRH
      000000B0H.5 SFRSYM    DATA     BIT       GP35
      000000A0H.6 SFRSYM    DATA     BIT       GP26
      00000090H.7 SFRSYM    DATA     BIT       GP17
      00000080H   SFRSYM    DATA     BYTE      P0
      00000088H.4 SFRSYM    DATA     BIT       IT11
      000000CAH   SFRSYM    DATA     WORD      MD_MB
      00000093H   SFRSYM    DATA     BYTE      TIM4_CNTRH
      000000B0H.6 SFRSYM    DATA     BIT       GP36
      000000A0H.7 SFRSYM    DATA     BIT       GP27
      00000090H   SFRSYM    DATA     BYTE      P1
      000000D9H   SFRSYM    DATA     BYTE      EVT_FILT
      000000F4H   SFRSYM    DATA     WORD      PI_UKMAX
      0000008BH   SFRSYM    DATA     BYTE      TIM5_CNTRH
      000000B2H   SFRSYM    DATA     BYTE      TIM2_CMTRL
      000000B0H.7 SFRSYM    DATA     BIT       GP37
      000000A0H   SFRSYM    DATA     BYTE      P2
      000000AAH   SFRSYM    DATA     BYTE      TIM2_CNTRL
      000000B0H   SFRSYM    DATA     BYTE      P3
      000000A2H   SFRSYM    DATA     BYTE      TIM3_CNTRL
      000000D0H.6 SFRSYM    DATA     BIT       AC
      00000092H   SFRSYM    DATA     BYTE      TIM4_CNTRL
      0000008AH   SFRSYM    DATA     BYTE      TIM5_CNTRL
      000000B6H   SFRSYM    DATA     WORD      TIM0_CCR1
      000000A8H.7 SFRSYM    DATA     BIT       EA
      000000D5H   SFRSYM    DATA     BYTE      CMP_CR0
      000000BAH   SFRSYM    DATA     WORD      TIM0_CCR2
      000000D6H   SFRSYM    DATA     BYTE      CMP_CR1
      000000BCH   SFRSYM    DATA     WORD      TIM0_CCR3
LX51 LINKER/LOCATER V4.66.1.0                                                         03/23/2017  15:15:44  PAGE 95


      00000085H   SFRSYM    DATA     BYTE      PSCTL
      000000DAH   SFRSYM    DATA     BYTE      CMP_CR2
      000000BEH   SFRSYM    DATA     WORD      TIM0_CCR4
      000000B8H.2 SFRSYM    DATA     BIT       PX00
      000000EAH   SFRSYM    DATA     WORD      PI_EK
      000000F8H   SFRSYM    DATA     BIT       OISUH
      000000B8H.3 SFRSYM    DATA     BIT       PX01
      000000B8H.4 SFRSYM    DATA     BIT       PX10
      000000F8H.2 SFRSYM    DATA     BIT       OISVH
      000000B8H.5 SFRSYM    DATA     BIT       PX11
      000000F8H.4 SFRSYM    DATA     BIT       OISWH
      000000DCH   SFRSYM    DATA     WORD      LPF_K
      000000F2H   SFRSYM    DATA     WORD      PI_KI
      000000F8H.1 SFRSYM    DATA     BIT       OISUL
      000000A8H   SFRSYM    DATA     BYTE      IE
      000000F8H.3 SFRSYM    DATA     BIT       OISVL
      000000F8H.5 SFRSYM    DATA     BIT       OISWL
      000000D1H   SFRSYM    DATA     BYTE      P1IE
      00000098H.6 SFRSYM    DATA     BIT       MOD0
      000000D3H   SFRSYM    DATA     BYTE      P2IE
      000000D2H   SFRSYM    DATA     BYTE      P1IF
      000000F9H   SFRSYM    DATA     BYTE      PL_CR
      00000098H.7 SFRSYM    DATA     BIT       MOD1
      000000D4H   SFRSYM    DATA     BYTE      P2IF
      000000ACH   SFRSYM    DATA     WORD      TIM2_DR
      00000082H   SFRSYM    DATA     WORD      DP
      000000EEH   SFRSYM    DATA     WORD      PI_KP
      000000A4H   SFRSYM    DATA     WORD      TIM3_DR
      00000094H   SFRSYM    DATA     WORD      TIM4_DR
      0000008CH   SFRSYM    DATA     WORD      TIM5_DR
      000000F1H   SFRSYM    DATA     BYTE      OSC_CFG
      000000C1H   SFRSYM    DATA     BYTE      MD_MODE
      000000ECH   SFRSYM    DATA     WORD      PI_UK
      000000DEH   SFRSYM    DATA     WORD      LPF_X
      00000098H   SFRSYM    DATA     BIT       RI
      000000E6H   SFRSYM    DATA     WORD      LPF_Y
      000000C0H   SFRSYM    DATA     BIT       PTIM00
      000000D0H.7 SFRSYM    DATA     BIT       CY
      00000098H.1 SFRSYM    DATA     BIT       TI
      000000C0H.1 SFRSYM    DATA     BIT       PTIM01
      000000C0H.2 SFRSYM    DATA     BIT       PTIM10
      000000C0H.3 SFRSYM    DATA     BIT       PTIM11
      000000E1H   SFRSYM    DATA     BYTE      SV_CR
      00000098H   SFRSYM    DATA     BYTE      UT_CR
      00000099H   SFRSYM    DATA     BYTE      UT_DR
      000000F8H.6 SFRSYM    DATA     BIT       OIS4
      00000081H   SFRSYM    DATA     BYTE      SP
      000000D0H.2 SFRSYM    DATA     BIT       OV
      000000C4H   SFRSYM    DATA     BYTE      MD_DA0
      0000009AH   SFRSYM    DATA     WORD      UT_BAUD
      000000CCH   SFRSYM    DATA     BYTE      MD_DB0
      000000C5H   SFRSYM    DATA     BYTE      MD_DA1
      000000CDH   SFRSYM    DATA     BYTE      MD_DB1
      000000C6H   SFRSYM    DATA     BYTE      MD_DA2
      000000CEH   SFRSYM    DATA     BYTE      MD_DB2
      000000C7H   SFRSYM    DATA     BYTE      MD_DA3
      000000B4H   SFRSYM    DATA     WORD      TIM2_ADTR
      000000CFH   SFRSYM    DATA     BYTE      MD_DB3
      000000AFH   SFRSYM    DATA     BYTE      TIM2_ARRH
      000000A7H   SFRSYM    DATA     BYTE      TIM3_ARRH
      00000097H   SFRSYM    DATA     BYTE      TIM4_ARRH
      0000008FH   SFRSYM    DATA     BYTE      TIM5_ARRH
      000000AEH   SFRSYM    DATA     BYTE      TIM2_ARRL
      000000A6H   SFRSYM    DATA     BYTE      TIM3_ARRL
      00000087H   SFRSYM    DATA     BYTE      PCON
LX51 LINKER/LOCATER V4.66.1.0                                                         03/23/2017  15:15:44  PAGE 96


      000000E2H   SFRSYM    DATA     WORD      SV_US
      00000096H   SFRSYM    DATA     BYTE      TIM4_ARRL
      0000008EH   SFRSYM    DATA     BYTE      TIM5_ARRL
      000000B2H   SFRSYM    DATA     WORD      TIM2_CMTR
      00000088H   SFRSYM    DATA     BYTE      TCON
      000000AAH   SFRSYM    DATA     WORD      TIM2_CNTR
      000000A2H   SFRSYM    DATA     WORD      TIM3_CNTR
      00000092H   SFRSYM    DATA     WORD      TIM4_CNTR
      0000008AH   SFRSYM    DATA     WORD      TIM5_CNTR
      000000E5H   SFRSYM    DATA     BYTE      SV_ANGLEH
      000000D8H   SFRSYM    DATA     BIT       PUART0
      000000E4H   SFRSYM    DATA     BYTE      SV_ANGLEL
      000000C6H   SFRSYM    DATA     WORD      MD_DAH
      000000D8H.1 SFRSYM    DATA     BIT       PUART1
      000000D8H.2 SFRSYM    DATA     BIT       PI2C0
      00000088H.2 SFRSYM    DATA     BIT       IF0
      000000CEH   SFRSYM    DATA     WORD      MD_DBH
      000000D8H.3 SFRSYM    DATA     BIT       PI2C1
      000000F0H   SFRSYM    DATA     BYTE      B
      000000C4H   SFRSYM    DATA     WORD      MD_DAL
      000000A1H   SFRSYM    DATA     BYTE      TIM2_CR0
      000000CCH   SFRSYM    DATA     WORD      MD_DBL
      0000009CH   SFRSYM    DATA     BYTE      TIM3_CR0
      000000A9H   SFRSYM    DATA     BYTE      TIM2_CR1
      0000009EH   SFRSYM    DATA     BYTE      TIM4_CR0
      0000009DH   SFRSYM    DATA     BYTE      TIM3_CR1
      00000089H   SFRSYM    DATA     BYTE      TIM5_CR0
      0000009FH   SFRSYM    DATA     BYTE      TIM4_CR1
      000000F8H   SFRSYM    DATA     BYTE      DRV_OUT
      00000091H   SFRSYM    DATA     BYTE      TIM5_CR1
      000000E0H   SFRSYM    DATA     BYTE      ACC
      000000F7H   SFRSYM    DATA     BYTE      PI_UKMINH
      000000C3H   SFRSYM    DATA     BYTE      MD_MAH
      000000A8H.4 SFRSYM    DATA     BIT       ES0
      000000DBH   SFRSYM    DATA     BYTE      LVSR
      000000CBH   SFRSYM    DATA     BYTE      MD_MBH
      000000C0H.4 SFRSYM    DATA     BIT       PADC0
      000000B8H   SFRSYM    DATA     BYTE      IP0
      000000F5H   SFRSYM    DATA     BYTE      PI_UKMAXH
      000000C0H.5 SFRSYM    DATA     BIT       PADC1
      000000C0H   SFRSYM    DATA     BYTE      IP1
      000000C8H   SFRSYM    DATA     BYTE      IP2
      000000F6H   SFRSYM    DATA     BYTE      PI_UKMINL
      000000C2H   SFRSYM    DATA     BYTE      MD_MAL
      00000098H.2 SFRSYM    DATA     BIT       RB8
      000000D8H   SFRSYM    DATA     BYTE      IP3
      000000CAH   SFRSYM    DATA     BYTE      MD_MBL
      000000A8H   SFRSYM    DATA     BIT       EX0
      000000F4H   SFRSYM    DATA     BYTE      PI_UKMAXL
      00000098H.3 SFRSYM    DATA     BIT       TB8
      000000B7H   SFRSYM    DATA     BYTE      TIM0_CCR1H
      000000A8H.2 SFRSYM    DATA     BIT       EX1
      000000BBH   SFRSYM    DATA     BYTE      TIM0_CCR2H
      000000D0H   SFRSYM    DATA     BIT       P
      000000BDH   SFRSYM    DATA     BYTE      TIM0_CCR3H
      000000BFH   SFRSYM    DATA     BYTE      TIM0_CCR4H
      000000C8H.2 SFRSYM    DATA     BIT       PTIM230
      000000EBH   SFRSYM    DATA     BYTE      PI_EKH
      00000098H.5 SFRSYM    DATA     BIT       SM2
      000000B6H   SFRSYM    DATA     BYTE      TIM0_CCR1L
      000000B1H   SFRSYM    DATA     BYTE      TIM0_SR1
      000000C8H.3 SFRSYM    DATA     BIT       PTIM231
      000000BAH   SFRSYM    DATA     BYTE      TIM0_CCR2L
      000000BCH   SFRSYM    DATA     BYTE      TIM0_CCR3L
      000000BEH   SFRSYM    DATA     BYTE      TIM0_CCR4L
LX51 LINKER/LOCATER V4.66.1.0                                                         03/23/2017  15:15:44  PAGE 97


      000000D8H.6 SFRSYM    DATA     BIT       PMCD0
      000000C8H.4 SFRSYM    DATA     BIT       PTIM450
      000000D0H.3 SFRSYM    DATA     BIT       RS0
      000000DDH   SFRSYM    DATA     BYTE      LPF_KH
      000000F3H   SFRSYM    DATA     BYTE      PI_KIH
      000000EAH   SFRSYM    DATA     BYTE      PI_EKL
      000000E8H   SFRSYM    DATA     BYTE      FOC_SET0
      000000D8H.7 SFRSYM    DATA     BIT       PMCD1
      000000C8H.5 SFRSYM    DATA     BIT       PTIM451
      000000D0H.4 SFRSYM    DATA     BIT       RS1
      000000E9H   SFRSYM    DATA     BYTE      FOC_SET1
      000000B8H.6 SFRSYM    DATA     BIT       PFOC0
      000000DCH   SFRSYM    DATA     BYTE      LPF_KL
      000000F2H   SFRSYM    DATA     BYTE      PI_KIL
      000000B8H.7 SFRSYM    DATA     BIT       PFOC1
      000000ADH   SFRSYM    DATA     BYTE      TIM2_DRH
      000000B9H   SFRSYM    DATA     BYTE      TIM0_IER
      00000083H   SFRSYM    DATA     BYTE      DPH
      000000EFH   SFRSYM    DATA     BYTE      PI_KPH
      000000A5H   SFRSYM    DATA     BYTE      TIM3_DRH
      00000095H   SFRSYM    DATA     BYTE      TIM4_DRH
      0000008DH   SFRSYM    DATA     BYTE      TIM5_DRH
      000000ACH   SFRSYM    DATA     BYTE      TIM2_DRL
      00000082H   SFRSYM    DATA     BYTE      DPL
      000000EEH   SFRSYM    DATA     BYTE      PI_KPL
      000000A4H   SFRSYM    DATA     BYTE      TIM3_DRL
      000000F8H.7 SFRSYM    DATA     BIT       MOE
      000000C0H.6 SFRSYM    DATA     BIT       PCMP0
      000000EDH   SFRSYM    DATA     BYTE      PI_UKH
      00000094H   SFRSYM    DATA     BYTE      TIM4_DRL
      000000C0H.7 SFRSYM    DATA     BIT       PCMP1
      000000DFH   SFRSYM    DATA     BYTE      LPF_XH
      0000008CH   SFRSYM    DATA     BYTE      TIM5_DRL
      000000AEH   SFRSYM    DATA     WORD      TIM2_ARR
      000000A8H.5 SFRSYM    DATA     BIT       MCDIE
      000000C9H   SFRSYM    DATA     BYTE      RSTSRC
      000000E7H   SFRSYM    DATA     BYTE      LPF_YH
      000000A6H   SFRSYM    DATA     WORD      TIM3_ARR
      00000088H.6 SFRSYM    DATA     BIT       MCDIF
      00000098H.4 SFRSYM    DATA     BIT       REN
      00000096H   SFRSYM    DATA     WORD      TIM4_ARR
      000000ECH   SFRSYM    DATA     BYTE      PI_UKL
      000000D7H   SFRSYM    DATA     BYTE      CMP_SR
      0000008EH   SFRSYM    DATA     WORD      TIM5_ARR
      000000DEH   SFRSYM    DATA     BYTE      LPF_XL
      000000E6H   SFRSYM    DATA     BYTE      LPF_YL
      000000C8H   SFRSYM    DATA     BIT       PRTC0
      000000C8H.1 SFRSYM    DATA     BIT       PRTC1
      000000E8H.7 SFRSYM    DATA     BIT       FOCEN
      000000C8H.6 SFRSYM    DATA     BIT       PTSD0
      000000D8H.4 SFRSYM    DATA     BIT       PSPI0
      000000C8H.7 SFRSYM    DATA     BIT       PTSD1
      000000D8H.5 SFRSYM    DATA     BIT       PSPI1
      0000009BH   SFRSYM    DATA     BYTE      UT_BAUDH
      000000E4H   SFRSYM    DATA     WORD      SV_ANGLE
      000000B5H   SFRSYM    DATA     BYTE      TIM2_ADTRH
      0000009AH   SFRSYM    DATA     BYTE      UT_BAUDL
      000000FCH   SFRSYM    DATA     BYTE      P0_OE
      000000FDH   SFRSYM    DATA     BYTE      P1_OE
      000000D0H.5 SFRSYM    DATA     BIT       F0
      000000B4H   SFRSYM    DATA     BYTE      TIM2_ADTRL
      000000FEH   SFRSYM    DATA     BYTE      P2_OE
      000000D0H.1 SFRSYM    DATA     BIT       F1
      00000080H   SFRSYM    DATA     BIT       GP00
      000000FFH   SFRSYM    DATA     BYTE      P3_OE
LX51 LINKER/LOCATER V4.66.1.0                                                         03/23/2017  15:15:44  PAGE 98


      00000090H   SFRSYM    DATA     BIT       GP10
      00000080H.1 SFRSYM    DATA     BIT       GP01
      000000A8H.6 SFRSYM    DATA     BIT       RTCIE
      000000A0H   SFRSYM    DATA     BIT       GP20
      00000090H.1 SFRSYM    DATA     BIT       GP11
      00000080H.2 SFRSYM    DATA     BIT       GP02
      000000E3H   SFRSYM    DATA     BYTE      SV_USH
      000000B0H   SFRSYM    DATA     BIT       GP30
      000000A0H.1 SFRSYM    DATA     BIT       GP21
      00000090H.2 SFRSYM    DATA     BIT       GP12
      00000080H.3 SFRSYM    DATA     BIT       GP03
      000000B8H   SFRSYM    DATA     BIT       PLVW0
      000000A8H.1 SFRSYM    DATA     BIT       TSDIE
      000000D0H   SFRSYM    DATA     BYTE      PSW
      000000B0H.1 SFRSYM    DATA     BIT       GP31
      000000A0H.2 SFRSYM    DATA     BIT       GP22
      00000090H.3 SFRSYM    DATA     BIT       GP13
      00000080H.4 SFRSYM    DATA     BIT       GP04
      000000B8H.1 SFRSYM    DATA     BIT       PLVW1
      000000A8H.3 SFRSYM    DATA     BIT       SPIIE
      00000088H.5 SFRSYM    DATA     BIT       TSDIF
      000000B0H.2 SFRSYM    DATA     BIT       GP32
      000000A0H.3 SFRSYM    DATA     BIT       GP23
      00000090H.4 SFRSYM    DATA     BIT       GP14
      00000080H.5 SFRSYM    DATA     BIT       GP05
      00000084H   SFRSYM    DATA     BYTE      FLKEY
      000000B3H   SFRSYM    DATA     BYTE      TIM2_CMTRH
      000000B0H.3 SFRSYM    DATA     BIT       GP33
      000000A0H.4 SFRSYM    DATA     BIT       GP24
      00000090H.5 SFRSYM    DATA     BIT       GP15
      00000080H.6 SFRSYM    DATA     BIT       GP06
      00000088H   SFRSYM    DATA     BIT       IT00
      00000004H   SYMBOL    DATA     WORD      Data

      ---         MODULE    ---      ---       TIMERINIT
      0100184DH   PUBLIC    CODE     ---       TIM4Init
      01001AE6H   PUBLIC    CODE     ---       TIM3Init
      01000CADH   PUBLIC    CODE     ---       TIM0Init
      000000E2H   SFRSYM    DATA     BYTE      SV_USL
      000000ABH   SFRSYM    DATA     BYTE      TIM2_CNTRH
      000000B0H.4 SFRSYM    DATA     BIT       GP34
      000000A0H.5 SFRSYM    DATA     BIT       GP25
      00000090H.6 SFRSYM    DATA     BIT       GP16
      00000080H.7 SFRSYM    DATA     BIT       GP07
      00000088H.1 SFRSYM    DATA     BIT       IT01
      00000088H.3 SFRSYM    DATA     BIT       IT10
      000000F6H   SFRSYM    DATA     WORD      PI_UKMIN
      000000C2H   SFRSYM    DATA     WORD      MD_MA
      000000A3H   SFRSYM    DATA     BYTE      TIM3_CNTRH
      000000B0H.5 SFRSYM    DATA     BIT       GP35
      000000A0H.6 SFRSYM    DATA     BIT       GP26
      00000090H.7 SFRSYM    DATA     BIT       GP17
      00000080H   SFRSYM    DATA     BYTE      P0
      00000088H.4 SFRSYM    DATA     BIT       IT11
      000000CAH   SFRSYM    DATA     WORD      MD_MB
      00000093H   SFRSYM    DATA     BYTE      TIM4_CNTRH
      000000B0H.6 SFRSYM    DATA     BIT       GP36
      000000A0H.7 SFRSYM    DATA     BIT       GP27
      00000090H   SFRSYM    DATA     BYTE      P1
      000000D9H   SFRSYM    DATA     BYTE      EVT_FILT
      000000F4H   SFRSYM    DATA     WORD      PI_UKMAX
      0000008BH   SFRSYM    DATA     BYTE      TIM5_CNTRH
      000000B2H   SFRSYM    DATA     BYTE      TIM2_CMTRL
      000000B0H.7 SFRSYM    DATA     BIT       GP37
      000000A0H   SFRSYM    DATA     BYTE      P2
LX51 LINKER/LOCATER V4.66.1.0                                                         03/23/2017  15:15:44  PAGE 99


      000000AAH   SFRSYM    DATA     BYTE      TIM2_CNTRL
      000000B0H   SFRSYM    DATA     BYTE      P3
      000000A2H   SFRSYM    DATA     BYTE      TIM3_CNTRL
      000000D0H.6 SFRSYM    DATA     BIT       AC
      00000092H   SFRSYM    DATA     BYTE      TIM4_CNTRL
      0000008AH   SFRSYM    DATA     BYTE      TIM5_CNTRL
      000000B6H   SFRSYM    DATA     WORD      TIM0_CCR1
      000000A8H.7 SFRSYM    DATA     BIT       EA
      000000D5H   SFRSYM    DATA     BYTE      CMP_CR0
      000000BAH   SFRSYM    DATA     WORD      TIM0_CCR2
      000000D6H   SFRSYM    DATA     BYTE      CMP_CR1
      000000BCH   SFRSYM    DATA     WORD      TIM0_CCR3
      00000085H   SFRSYM    DATA     BYTE      PSCTL
      000000DAH   SFRSYM    DATA     BYTE      CMP_CR2
      000000BEH   SFRSYM    DATA     WORD      TIM0_CCR4
      000000B8H.2 SFRSYM    DATA     BIT       PX00
      000000EAH   SFRSYM    DATA     WORD      PI_EK
      000000F8H   SFRSYM    DATA     BIT       OISUH
      000000B8H.3 SFRSYM    DATA     BIT       PX01
      000000B8H.4 SFRSYM    DATA     BIT       PX10
      000000F8H.2 SFRSYM    DATA     BIT       OISVH
      000000B8H.5 SFRSYM    DATA     BIT       PX11
      000000F8H.4 SFRSYM    DATA     BIT       OISWH
      000000DCH   SFRSYM    DATA     WORD      LPF_K
      000000F2H   SFRSYM    DATA     WORD      PI_KI
      000000F8H.1 SFRSYM    DATA     BIT       OISUL
      000000A8H   SFRSYM    DATA     BYTE      IE
      000000F8H.3 SFRSYM    DATA     BIT       OISVL
      000000F8H.5 SFRSYM    DATA     BIT       OISWL
      000000D1H   SFRSYM    DATA     BYTE      P1IE
      00000098H.6 SFRSYM    DATA     BIT       MOD0
      000000D3H   SFRSYM    DATA     BYTE      P2IE
      000000D2H   SFRSYM    DATA     BYTE      P1IF
      000000F9H   SFRSYM    DATA     BYTE      PL_CR
      00000098H.7 SFRSYM    DATA     BIT       MOD1
      000000D4H   SFRSYM    DATA     BYTE      P2IF
      000000ACH   SFRSYM    DATA     WORD      TIM2_DR
      00000082H   SFRSYM    DATA     WORD      DP
      000000EEH   SFRSYM    DATA     WORD      PI_KP
      000000A4H   SFRSYM    DATA     WORD      TIM3_DR
      00000094H   SFRSYM    DATA     WORD      TIM4_DR
      0000008CH   SFRSYM    DATA     WORD      TIM5_DR
      000000F1H   SFRSYM    DATA     BYTE      OSC_CFG
      000000C1H   SFRSYM    DATA     BYTE      MD_MODE
      000000ECH   SFRSYM    DATA     WORD      PI_UK
      000000DEH   SFRSYM    DATA     WORD      LPF_X
      00000098H   SFRSYM    DATA     BIT       RI
      000000E6H   SFRSYM    DATA     WORD      LPF_Y
      000000C0H   SFRSYM    DATA     BIT       PTIM00
      000000D0H.7 SFRSYM    DATA     BIT       CY
      00000098H.1 SFRSYM    DATA     BIT       TI
      000000C0H.1 SFRSYM    DATA     BIT       PTIM01
      000000C0H.2 SFRSYM    DATA     BIT       PTIM10
      000000C0H.3 SFRSYM    DATA     BIT       PTIM11
      000000E1H   SFRSYM    DATA     BYTE      SV_CR
      00000098H   SFRSYM    DATA     BYTE      UT_CR
      00000099H   SFRSYM    DATA     BYTE      UT_DR
      000000F8H.6 SFRSYM    DATA     BIT       OIS4
      00000081H   SFRSYM    DATA     BYTE      SP
      000000D0H.2 SFRSYM    DATA     BIT       OV
      000000C4H   SFRSYM    DATA     BYTE      MD_DA0
      0000009AH   SFRSYM    DATA     WORD      UT_BAUD
      000000CCH   SFRSYM    DATA     BYTE      MD_DB0
      000000C5H   SFRSYM    DATA     BYTE      MD_DA1
      000000CDH   SFRSYM    DATA     BYTE      MD_DB1
LX51 LINKER/LOCATER V4.66.1.0                                                         03/23/2017  15:15:44  PAGE 100


      000000C6H   SFRSYM    DATA     BYTE      MD_DA2
      000000CEH   SFRSYM    DATA     BYTE      MD_DB2
      000000C7H   SFRSYM    DATA     BYTE      MD_DA3
      000000B4H   SFRSYM    DATA     WORD      TIM2_ADTR
      000000CFH   SFRSYM    DATA     BYTE      MD_DB3
      000000AFH   SFRSYM    DATA     BYTE      TIM2_ARRH
      000000A7H   SFRSYM    DATA     BYTE      TIM3_ARRH
      00000097H   SFRSYM    DATA     BYTE      TIM4_ARRH
      0000008FH   SFRSYM    DATA     BYTE      TIM5_ARRH
      000000AEH   SFRSYM    DATA     BYTE      TIM2_ARRL
      000000A6H   SFRSYM    DATA     BYTE      TIM3_ARRL
      00000087H   SFRSYM    DATA     BYTE      PCON
      000000E2H   SFRSYM    DATA     WORD      SV_US
      00000096H   SFRSYM    DATA     BYTE      TIM4_ARRL
      0000008EH   SFRSYM    DATA     BYTE      TIM5_ARRL
      000000B2H   SFRSYM    DATA     WORD      TIM2_CMTR
      00000088H   SFRSYM    DATA     BYTE      TCON
      000000AAH   SFRSYM    DATA     WORD      TIM2_CNTR
      000000A2H   SFRSYM    DATA     WORD      TIM3_CNTR
      00000092H   SFRSYM    DATA     WORD      TIM4_CNTR
      0000008AH   SFRSYM    DATA     WORD      TIM5_CNTR
      000000E5H   SFRSYM    DATA     BYTE      SV_ANGLEH
      000000D8H   SFRSYM    DATA     BIT       PUART0
      000000E4H   SFRSYM    DATA     BYTE      SV_ANGLEL
      000000C6H   SFRSYM    DATA     WORD      MD_DAH
      000000D8H.1 SFRSYM    DATA     BIT       PUART1
      000000D8H.2 SFRSYM    DATA     BIT       PI2C0
      00000088H.2 SFRSYM    DATA     BIT       IF0
      000000CEH   SFRSYM    DATA     WORD      MD_DBH
      000000D8H.3 SFRSYM    DATA     BIT       PI2C1
      000000F0H   SFRSYM    DATA     BYTE      B
      000000C4H   SFRSYM    DATA     WORD      MD_DAL
      000000A1H   SFRSYM    DATA     BYTE      TIM2_CR0
      000000CCH   SFRSYM    DATA     WORD      MD_DBL
      0000009CH   SFRSYM    DATA     BYTE      TIM3_CR0
      000000A9H   SFRSYM    DATA     BYTE      TIM2_CR1
      0000009EH   SFRSYM    DATA     BYTE      TIM4_CR0
      0000009DH   SFRSYM    DATA     BYTE      TIM3_CR1
      00000089H   SFRSYM    DATA     BYTE      TIM5_CR0
      0000009FH   SFRSYM    DATA     BYTE      TIM4_CR1
      000000F8H   SFRSYM    DATA     BYTE      DRV_OUT
      00000091H   SFRSYM    DATA     BYTE      TIM5_CR1
      000000E0H   SFRSYM    DATA     BYTE      ACC
      000000F7H   SFRSYM    DATA     BYTE      PI_UKMINH
      000000C3H   SFRSYM    DATA     BYTE      MD_MAH
      000000A8H.4 SFRSYM    DATA     BIT       ES0
      000000DBH   SFRSYM    DATA     BYTE      LVSR
      000000CBH   SFRSYM    DATA     BYTE      MD_MBH
      000000C0H.4 SFRSYM    DATA     BIT       PADC0
      000000B8H   SFRSYM    DATA     BYTE      IP0
      000000F5H   SFRSYM    DATA     BYTE      PI_UKMAXH
      000000C0H.5 SFRSYM    DATA     BIT       PADC1
      000000C0H   SFRSYM    DATA     BYTE      IP1
      000000C8H   SFRSYM    DATA     BYTE      IP2
      000000F6H   SFRSYM    DATA     BYTE      PI_UKMINL
      000000C2H   SFRSYM    DATA     BYTE      MD_MAL
      00000098H.2 SFRSYM    DATA     BIT       RB8
      000000D8H   SFRSYM    DATA     BYTE      IP3
      000000CAH   SFRSYM    DATA     BYTE      MD_MBL
      000000A8H   SFRSYM    DATA     BIT       EX0
      000000F4H   SFRSYM    DATA     BYTE      PI_UKMAXL
      00000098H.3 SFRSYM    DATA     BIT       TB8
      000000B7H   SFRSYM    DATA     BYTE      TIM0_CCR1H
      000000A8H.2 SFRSYM    DATA     BIT       EX1
      000000BBH   SFRSYM    DATA     BYTE      TIM0_CCR2H
LX51 LINKER/LOCATER V4.66.1.0                                                         03/23/2017  15:15:44  PAGE 101


      000000D0H   SFRSYM    DATA     BIT       P
      000000BDH   SFRSYM    DATA     BYTE      TIM0_CCR3H
      000000BFH   SFRSYM    DATA     BYTE      TIM0_CCR4H
      000000C8H.2 SFRSYM    DATA     BIT       PTIM230
      000000EBH   SFRSYM    DATA     BYTE      PI_EKH
      00000098H.5 SFRSYM    DATA     BIT       SM2
      000000B6H   SFRSYM    DATA     BYTE      TIM0_CCR1L
      000000B1H   SFRSYM    DATA     BYTE      TIM0_SR1
      000000C8H.3 SFRSYM    DATA     BIT       PTIM231
      000000BAH   SFRSYM    DATA     BYTE      TIM0_CCR2L
      000000BCH   SFRSYM    DATA     BYTE      TIM0_CCR3L
      000000BEH   SFRSYM    DATA     BYTE      TIM0_CCR4L
      000000D8H.6 SFRSYM    DATA     BIT       PMCD0
      000000C8H.4 SFRSYM    DATA     BIT       PTIM450
      000000D0H.3 SFRSYM    DATA     BIT       RS0
      000000DDH   SFRSYM    DATA     BYTE      LPF_KH
      000000F3H   SFRSYM    DATA     BYTE      PI_KIH
      000000EAH   SFRSYM    DATA     BYTE      PI_EKL
      000000E8H   SFRSYM    DATA     BYTE      FOC_SET0
      000000D8H.7 SFRSYM    DATA     BIT       PMCD1
      000000C8H.5 SFRSYM    DATA     BIT       PTIM451
      000000D0H.4 SFRSYM    DATA     BIT       RS1
      000000E9H   SFRSYM    DATA     BYTE      FOC_SET1
      000000B8H.6 SFRSYM    DATA     BIT       PFOC0
      000000DCH   SFRSYM    DATA     BYTE      LPF_KL
      000000F2H   SFRSYM    DATA     BYTE      PI_KIL
      000000B8H.7 SFRSYM    DATA     BIT       PFOC1
      000000ADH   SFRSYM    DATA     BYTE      TIM2_DRH
      000000B9H   SFRSYM    DATA     BYTE      TIM0_IER
      00000083H   SFRSYM    DATA     BYTE      DPH
      000000EFH   SFRSYM    DATA     BYTE      PI_KPH
      000000A5H   SFRSYM    DATA     BYTE      TIM3_DRH
      00000095H   SFRSYM    DATA     BYTE      TIM4_DRH
      0000008DH   SFRSYM    DATA     BYTE      TIM5_DRH
      000000ACH   SFRSYM    DATA     BYTE      TIM2_DRL
      00000082H   SFRSYM    DATA     BYTE      DPL
      000000EEH   SFRSYM    DATA     BYTE      PI_KPL
      000000A4H   SFRSYM    DATA     BYTE      TIM3_DRL
      000000F8H.7 SFRSYM    DATA     BIT       MOE
      000000C0H.6 SFRSYM    DATA     BIT       PCMP0
      000000EDH   SFRSYM    DATA     BYTE      PI_UKH
      00000094H   SFRSYM    DATA     BYTE      TIM4_DRL
      000000C0H.7 SFRSYM    DATA     BIT       PCMP1
      000000DFH   SFRSYM    DATA     BYTE      LPF_XH
      0000008CH   SFRSYM    DATA     BYTE      TIM5_DRL
      000000AEH   SFRSYM    DATA     WORD      TIM2_ARR
      000000A8H.5 SFRSYM    DATA     BIT       MCDIE
      000000C9H   SFRSYM    DATA     BYTE      RSTSRC
      000000E7H   SFRSYM    DATA     BYTE      LPF_YH
      000000A6H   SFRSYM    DATA     WORD      TIM3_ARR
      00000088H.6 SFRSYM    DATA     BIT       MCDIF
      00000098H.4 SFRSYM    DATA     BIT       REN
      00000096H   SFRSYM    DATA     WORD      TIM4_ARR
      000000ECH   SFRSYM    DATA     BYTE      PI_UKL
      000000D7H   SFRSYM    DATA     BYTE      CMP_SR
      0000008EH   SFRSYM    DATA     WORD      TIM5_ARR
      000000DEH   SFRSYM    DATA     BYTE      LPF_XL
      000000E6H   SFRSYM    DATA     BYTE      LPF_YL
      000000C8H   SFRSYM    DATA     BIT       PRTC0
      000000C8H.1 SFRSYM    DATA     BIT       PRTC1
      000000E8H.7 SFRSYM    DATA     BIT       FOCEN
      000000C8H.6 SFRSYM    DATA     BIT       PTSD0
      000000D8H.4 SFRSYM    DATA     BIT       PSPI0
      000000C8H.7 SFRSYM    DATA     BIT       PTSD1
      000000D8H.5 SFRSYM    DATA     BIT       PSPI1
LX51 LINKER/LOCATER V4.66.1.0                                                         03/23/2017  15:15:44  PAGE 102


      0000009BH   SFRSYM    DATA     BYTE      UT_BAUDH
      000000E4H   SFRSYM    DATA     WORD      SV_ANGLE
      000000B5H   SFRSYM    DATA     BYTE      TIM2_ADTRH
      0000009AH   SFRSYM    DATA     BYTE      UT_BAUDL
      000000FCH   SFRSYM    DATA     BYTE      P0_OE
      000000FDH   SFRSYM    DATA     BYTE      P1_OE
      000000D0H.5 SFRSYM    DATA     BIT       F0
      000000B4H   SFRSYM    DATA     BYTE      TIM2_ADTRL
      000000FEH   SFRSYM    DATA     BYTE      P2_OE
      000000D0H.1 SFRSYM    DATA     BIT       F1
      00000080H   SFRSYM    DATA     BIT       GP00
      000000FFH   SFRSYM    DATA     BYTE      P3_OE
      00000090H   SFRSYM    DATA     BIT       GP10
      00000080H.1 SFRSYM    DATA     BIT       GP01
      000000A8H.6 SFRSYM    DATA     BIT       RTCIE
      000000A0H   SFRSYM    DATA     BIT       GP20
      00000090H.1 SFRSYM    DATA     BIT       GP11
      00000080H.2 SFRSYM    DATA     BIT       GP02
      000000E3H   SFRSYM    DATA     BYTE      SV_USH
      000000B0H   SFRSYM    DATA     BIT       GP30
      000000A0H.1 SFRSYM    DATA     BIT       GP21
      00000090H.2 SFRSYM    DATA     BIT       GP12
      00000080H.3 SFRSYM    DATA     BIT       GP03
      000000B8H   SFRSYM    DATA     BIT       PLVW0
      000000A8H.1 SFRSYM    DATA     BIT       TSDIE
      000000D0H   SFRSYM    DATA     BYTE      PSW
      000000B0H.1 SFRSYM    DATA     BIT       GP31
      000000A0H.2 SFRSYM    DATA     BIT       GP22
      00000090H.3 SFRSYM    DATA     BIT       GP13
      00000080H.4 SFRSYM    DATA     BIT       GP04
      000000B8H.1 SFRSYM    DATA     BIT       PLVW1
      000000A8H.3 SFRSYM    DATA     BIT       SPIIE
      00000088H.5 SFRSYM    DATA     BIT       TSDIF
      000000B0H.2 SFRSYM    DATA     BIT       GP32
      000000A0H.3 SFRSYM    DATA     BIT       GP23
      00000090H.4 SFRSYM    DATA     BIT       GP14
      00000080H.5 SFRSYM    DATA     BIT       GP05
      00000084H   SFRSYM    DATA     BYTE      FLKEY
      000000B3H   SFRSYM    DATA     BYTE      TIM2_CMTRH
      000000B0H.3 SFRSYM    DATA     BIT       GP33
      000000A0H.4 SFRSYM    DATA     BIT       GP24
      00000090H.5 SFRSYM    DATA     BIT       GP15
      00000080H.6 SFRSYM    DATA     BIT       GP06
      00000088H   SFRSYM    DATA     BIT       IT00

      01000CADH   BLOCK     CODE     ---       LVL=0
      01000CADH   LINE      CODE     ---       #22
      01000CADH   LINE      CODE     ---       #23
      01000CADH   LINE      CODE     ---       #24
      01000CB4H   LINE      CODE     ---       #34
      01000CB8H   LINE      CODE     ---       #35
      01000CBCH   LINE      CODE     ---       #36
      01000CC0H   LINE      CODE     ---       #39
      01000CC4H   LINE      CODE     ---       #42
      01000CC8H   LINE      CODE     ---       #45
      01000CCEH   LINE      CODE     ---       #46
      01000CD3H   LINE      CODE     ---       #47
      01000CDDH   LINE      CODE     ---       #48
      01000CE5H   LINE      CODE     ---       #62
      01000CECH   LINE      CODE     ---       #65
      01000CF3H   LINE      CODE     ---       #66
      01000CF7H   LINE      CODE     ---       #67
      01000CFBH   LINE      CODE     ---       #68
      01000CFFH   LINE      CODE     ---       #69
      01000D06H   LINE      CODE     ---       #70
LX51 LINKER/LOCATER V4.66.1.0                                                         03/23/2017  15:15:44  PAGE 103


      01000D0AH   LINE      CODE     ---       #71
      01000D0EH   LINE      CODE     ---       #72
      01000D12H   LINE      CODE     ---       #75
      01000D19H   LINE      CODE     ---       #76
      01000D1DH   LINE      CODE     ---       #77
      01000D21H   LINE      CODE     ---       #78
      01000D25H   LINE      CODE     ---       #79
      01000D2CH   LINE      CODE     ---       #80
      01000D30H   LINE      CODE     ---       #81
      01000D34H   LINE      CODE     ---       #82
      01000D38H   LINE      CODE     ---       #85
      01000D3FH   LINE      CODE     ---       #86
      01000D43H   LINE      CODE     ---       #87
      01000D47H   LINE      CODE     ---       #88
      01000D4BH   LINE      CODE     ---       #89
      01000D52H   LINE      CODE     ---       #90
      01000D56H   LINE      CODE     ---       #91
      01000D5AH   LINE      CODE     ---       #92
      01000D5EH   LINE      CODE     ---       #95
      01000D65H   LINE      CODE     ---       #96
      01000D69H   LINE      CODE     ---       #97
      01000D6DH   LINE      CODE     ---       #98
      01000D71H   LINE      CODE     ---       #99
      01000D78H   LINE      CODE     ---       #100
      01000D7CH   LINE      CODE     ---       #104
      01000D82H   LINE      CODE     ---       #107
      01000D88H   LINE      CODE     ---       #108
      01000D8DH   LINE      CODE     ---       #109
      01000D91H   LINE      CODE     ---       #110
      01000D95H   LINE      CODE     ---       #113
      01000D9CH   LINE      CODE     ---       #114
      01000DA0H   LINE      CODE     ---       #115
      01000DA3H   LINE      CODE     ---       #123
      01000DAAH   LINE      CODE     ---       #124
      01000DAEH   LINE      CODE     ---       #127
      01000DB1H   LINE      CODE     ---       #128
      01000DB4H   LINE      CODE     ---       #129
      01000DB7H   LINE      CODE     ---       #130
      01000DBAH   LINE      CODE     ---       #131
      01000DBDH   LINE      CODE     ---       #132
      01000DC0H   LINE      CODE     ---       #135
      01000DC3H   LINE      CODE     ---       #136
      01000DC6H   LINE      CODE     ---       #137
      01000DC9H   LINE      CODE     ---       #138
      01000DCCH   LINE      CODE     ---       #139
      01000DCFH   LINE      CODE     ---       #140
      01000DD2H   LINE      CODE     ---       #143
      01000DD7H   LINE      CODE     ---       #144
      01000DDBH   LINE      CODE     ---       #145
      01000DDFH   LINE      CODE     ---       #146
      01000DE3H   LINE      CODE     ---       #147
      01000DE7H   LINE      CODE     ---       #148
      01000DEBH   LINE      CODE     ---       #150
      01000DF2H   LINE      CODE     ---       #152
      ---         BLOCKEND  ---      ---       LVL=0

      01001AE6H   BLOCK     CODE     ---       LVL=0
      01001AE6H   LINE      CODE     ---       #325
      01001AE6H   LINE      CODE     ---       #326
      01001AE6H   LINE      CODE     ---       #327
      01001AE9H   LINE      CODE     ---       #334
      01001AECH   LINE      CODE     ---       #335
      01001AEFH   LINE      CODE     ---       #336
      01001AF2H   LINE      CODE     ---       #345
      01001AF5H   LINE      CODE     ---       #346
LX51 LINKER/LOCATER V4.66.1.0                                                         03/23/2017  15:15:44  PAGE 104


      01001AF8H   LINE      CODE     ---       #347
      01001AFBH   LINE      CODE     ---       #349
      01001B03H   LINE      CODE     ---       #350
      01001B0BH   LINE      CODE     ---       #351
      01001B13H   LINE      CODE     ---       #352
      01001B16H   LINE      CODE     ---       #353
      01001B19H   LINE      CODE     ---       #384
      01001B1CH   LINE      CODE     ---       #386
      ---         BLOCKEND  ---      ---       LVL=0

      0100184DH   BLOCK     CODE     ---       LVL=0
      0100184DH   LINE      CODE     ---       #394
      0100184DH   LINE      CODE     ---       #395
      0100184DH   LINE      CODE     ---       #396
      01001850H   LINE      CODE     ---       #403
      01001853H   LINE      CODE     ---       #404
      01001856H   LINE      CODE     ---       #405
      01001859H   LINE      CODE     ---       #414
      0100185CH   LINE      CODE     ---       #415
      0100185FH   LINE      CODE     ---       #416
      01001862H   LINE      CODE     ---       #418
      0100186AH   LINE      CODE     ---       #419
      01001872H   LINE      CODE     ---       #420
      0100187AH   LINE      CODE     ---       #421
      0100187DH   LINE      CODE     ---       #422
      01001880H   LINE      CODE     ---       #424
      01001886H   LINE      CODE     ---       #425
      01001892H   LINE      CODE     ---       #426
      01001898H   LINE      CODE     ---       #428
      0100189BH   LINE      CODE     ---       #430
      ---         BLOCKEND  ---      ---       LVL=0
      00000006H   SYMBOL    DATA     WORD      DR
      00000082H   SYMBOL    DATA     WORD      ARR

      ---         MODULE    ---      ---       SPIINIT
      0100189CH   PUBLIC    CODE     ---       SPIInit
      000000E2H   SFRSYM    DATA     BYTE      SV_USL
      000000ABH   SFRSYM    DATA     BYTE      TIM2_CNTRH
      000000B0H.4 SFRSYM    DATA     BIT       GP34
      000000A0H.5 SFRSYM    DATA     BIT       GP25
      00000090H.6 SFRSYM    DATA     BIT       GP16
      00000080H.7 SFRSYM    DATA     BIT       GP07
      00000088H.1 SFRSYM    DATA     BIT       IT01
      00000088H.3 SFRSYM    DATA     BIT       IT10
      000000F6H   SFRSYM    DATA     WORD      PI_UKMIN
      000000C2H   SFRSYM    DATA     WORD      MD_MA
      000000A3H   SFRSYM    DATA     BYTE      TIM3_CNTRH
      000000B0H.5 SFRSYM    DATA     BIT       GP35
      000000A0H.6 SFRSYM    DATA     BIT       GP26
      00000090H.7 SFRSYM    DATA     BIT       GP17
      00000080H   SFRSYM    DATA     BYTE      P0
      00000088H.4 SFRSYM    DATA     BIT       IT11
      000000CAH   SFRSYM    DATA     WORD      MD_MB
      00000093H   SFRSYM    DATA     BYTE      TIM4_CNTRH
      000000B0H.6 SFRSYM    DATA     BIT       GP36
      000000A0H.7 SFRSYM    DATA     BIT       GP27
      00000090H   SFRSYM    DATA     BYTE      P1
      000000D9H   SFRSYM    DATA     BYTE      EVT_FILT
      000000F4H   SFRSYM    DATA     WORD      PI_UKMAX
      0000008BH   SFRSYM    DATA     BYTE      TIM5_CNTRH
      000000B2H   SFRSYM    DATA     BYTE      TIM2_CMTRL
      000000B0H.7 SFRSYM    DATA     BIT       GP37
      000000A0H   SFRSYM    DATA     BYTE      P2
      000000AAH   SFRSYM    DATA     BYTE      TIM2_CNTRL
      000000B0H   SFRSYM    DATA     BYTE      P3
LX51 LINKER/LOCATER V4.66.1.0                                                         03/23/2017  15:15:44  PAGE 105


      000000A2H   SFRSYM    DATA     BYTE      TIM3_CNTRL
      000000D0H.6 SFRSYM    DATA     BIT       AC
      00000092H   SFRSYM    DATA     BYTE      TIM4_CNTRL
      0000008AH   SFRSYM    DATA     BYTE      TIM5_CNTRL
      000000B6H   SFRSYM    DATA     WORD      TIM0_CCR1
      000000A8H.7 SFRSYM    DATA     BIT       EA
      000000D5H   SFRSYM    DATA     BYTE      CMP_CR0
      000000BAH   SFRSYM    DATA     WORD      TIM0_CCR2
      000000D6H   SFRSYM    DATA     BYTE      CMP_CR1
      000000BCH   SFRSYM    DATA     WORD      TIM0_CCR3
      00000085H   SFRSYM    DATA     BYTE      PSCTL
      000000DAH   SFRSYM    DATA     BYTE      CMP_CR2
      000000BEH   SFRSYM    DATA     WORD      TIM0_CCR4
      000000B8H.2 SFRSYM    DATA     BIT       PX00
      000000EAH   SFRSYM    DATA     WORD      PI_EK
      000000F8H   SFRSYM    DATA     BIT       OISUH
      000000B8H.3 SFRSYM    DATA     BIT       PX01
      000000B8H.4 SFRSYM    DATA     BIT       PX10
      000000F8H.2 SFRSYM    DATA     BIT       OISVH
      000000B8H.5 SFRSYM    DATA     BIT       PX11
      000000F8H.4 SFRSYM    DATA     BIT       OISWH
      000000DCH   SFRSYM    DATA     WORD      LPF_K
      000000F2H   SFRSYM    DATA     WORD      PI_KI
      000000F8H.1 SFRSYM    DATA     BIT       OISUL
      000000A8H   SFRSYM    DATA     BYTE      IE
      000000F8H.3 SFRSYM    DATA     BIT       OISVL
      000000F8H.5 SFRSYM    DATA     BIT       OISWL
      000000D1H   SFRSYM    DATA     BYTE      P1IE
      00000098H.6 SFRSYM    DATA     BIT       MOD0
      000000D3H   SFRSYM    DATA     BYTE      P2IE
      000000D2H   SFRSYM    DATA     BYTE      P1IF
      000000F9H   SFRSYM    DATA     BYTE      PL_CR
      00000098H.7 SFRSYM    DATA     BIT       MOD1
      000000D4H   SFRSYM    DATA     BYTE      P2IF
      000000ACH   SFRSYM    DATA     WORD      TIM2_DR
      00000082H   SFRSYM    DATA     WORD      DP
      000000EEH   SFRSYM    DATA     WORD      PI_KP
      000000A4H   SFRSYM    DATA     WORD      TIM3_DR
      00000094H   SFRSYM    DATA     WORD      TIM4_DR
      0000008CH   SFRSYM    DATA     WORD      TIM5_DR
      000000F1H   SFRSYM    DATA     BYTE      OSC_CFG
      000000C1H   SFRSYM    DATA     BYTE      MD_MODE
      000000ECH   SFRSYM    DATA     WORD      PI_UK
      000000DEH   SFRSYM    DATA     WORD      LPF_X
      00000098H   SFRSYM    DATA     BIT       RI
      000000E6H   SFRSYM    DATA     WORD      LPF_Y
      000000C0H   SFRSYM    DATA     BIT       PTIM00
      000000D0H.7 SFRSYM    DATA     BIT       CY
      00000098H.1 SFRSYM    DATA     BIT       TI
      000000C0H.1 SFRSYM    DATA     BIT       PTIM01
      000000C0H.2 SFRSYM    DATA     BIT       PTIM10
      000000C0H.3 SFRSYM    DATA     BIT       PTIM11
      000000E1H   SFRSYM    DATA     BYTE      SV_CR
      00000098H   SFRSYM    DATA     BYTE      UT_CR
      00000099H   SFRSYM    DATA     BYTE      UT_DR
      000000F8H.6 SFRSYM    DATA     BIT       OIS4
      00000081H   SFRSYM    DATA     BYTE      SP
      000000D0H.2 SFRSYM    DATA     BIT       OV
      000000C4H   SFRSYM    DATA     BYTE      MD_DA0
      0000009AH   SFRSYM    DATA     WORD      UT_BAUD
      000000CCH   SFRSYM    DATA     BYTE      MD_DB0
      000000C5H   SFRSYM    DATA     BYTE      MD_DA1
      000000CDH   SFRSYM    DATA     BYTE      MD_DB1
      000000C6H   SFRSYM    DATA     BYTE      MD_DA2
      000000CEH   SFRSYM    DATA     BYTE      MD_DB2
LX51 LINKER/LOCATER V4.66.1.0                                                         03/23/2017  15:15:44  PAGE 106


      000000C7H   SFRSYM    DATA     BYTE      MD_DA3
      000000B4H   SFRSYM    DATA     WORD      TIM2_ADTR
      000000CFH   SFRSYM    DATA     BYTE      MD_DB3
      000000AFH   SFRSYM    DATA     BYTE      TIM2_ARRH
      000000A7H   SFRSYM    DATA     BYTE      TIM3_ARRH
      00000097H   SFRSYM    DATA     BYTE      TIM4_ARRH
      0000008FH   SFRSYM    DATA     BYTE      TIM5_ARRH
      000000AEH   SFRSYM    DATA     BYTE      TIM2_ARRL
      000000A6H   SFRSYM    DATA     BYTE      TIM3_ARRL
      00000087H   SFRSYM    DATA     BYTE      PCON
      000000E2H   SFRSYM    DATA     WORD      SV_US
      00000096H   SFRSYM    DATA     BYTE      TIM4_ARRL
      0000008EH   SFRSYM    DATA     BYTE      TIM5_ARRL
      000000B2H   SFRSYM    DATA     WORD      TIM2_CMTR
      00000088H   SFRSYM    DATA     BYTE      TCON
      000000AAH   SFRSYM    DATA     WORD      TIM2_CNTR
      000000A2H   SFRSYM    DATA     WORD      TIM3_CNTR
      00000092H   SFRSYM    DATA     WORD      TIM4_CNTR
      0000008AH   SFRSYM    DATA     WORD      TIM5_CNTR
      000000E5H   SFRSYM    DATA     BYTE      SV_ANGLEH
      000000D8H   SFRSYM    DATA     BIT       PUART0
      000000E4H   SFRSYM    DATA     BYTE      SV_ANGLEL
      000000C6H   SFRSYM    DATA     WORD      MD_DAH
      000000D8H.1 SFRSYM    DATA     BIT       PUART1
      000000D8H.2 SFRSYM    DATA     BIT       PI2C0
      00000088H.2 SFRSYM    DATA     BIT       IF0
      000000CEH   SFRSYM    DATA     WORD      MD_DBH
      000000D8H.3 SFRSYM    DATA     BIT       PI2C1
      000000F0H   SFRSYM    DATA     BYTE      B
      000000C4H   SFRSYM    DATA     WORD      MD_DAL
      000000A1H   SFRSYM    DATA     BYTE      TIM2_CR0
      000000CCH   SFRSYM    DATA     WORD      MD_DBL
      0000009CH   SFRSYM    DATA     BYTE      TIM3_CR0
      000000A9H   SFRSYM    DATA     BYTE      TIM2_CR1
      0000009EH   SFRSYM    DATA     BYTE      TIM4_CR0
      0000009DH   SFRSYM    DATA     BYTE      TIM3_CR1
      00000089H   SFRSYM    DATA     BYTE      TIM5_CR0
      0000009FH   SFRSYM    DATA     BYTE      TIM4_CR1
      000000F8H   SFRSYM    DATA     BYTE      DRV_OUT
      00000091H   SFRSYM    DATA     BYTE      TIM5_CR1
      000000E0H   SFRSYM    DATA     BYTE      ACC
      000000F7H   SFRSYM    DATA     BYTE      PI_UKMINH
      000000C3H   SFRSYM    DATA     BYTE      MD_MAH
      000000A8H.4 SFRSYM    DATA     BIT       ES0
      000000DBH   SFRSYM    DATA     BYTE      LVSR
      000000CBH   SFRSYM    DATA     BYTE      MD_MBH
      000000C0H.4 SFRSYM    DATA     BIT       PADC0
      000000B8H   SFRSYM    DATA     BYTE      IP0
      000000F5H   SFRSYM    DATA     BYTE      PI_UKMAXH
      000000C0H.5 SFRSYM    DATA     BIT       PADC1
      000000C0H   SFRSYM    DATA     BYTE      IP1
      000000C8H   SFRSYM    DATA     BYTE      IP2
      000000F6H   SFRSYM    DATA     BYTE      PI_UKMINL
      000000C2H   SFRSYM    DATA     BYTE      MD_MAL
      00000098H.2 SFRSYM    DATA     BIT       RB8
      000000D8H   SFRSYM    DATA     BYTE      IP3
      000000CAH   SFRSYM    DATA     BYTE      MD_MBL
      000000A8H   SFRSYM    DATA     BIT       EX0
      000000F4H   SFRSYM    DATA     BYTE      PI_UKMAXL
      00000098H.3 SFRSYM    DATA     BIT       TB8
      000000B7H   SFRSYM    DATA     BYTE      TIM0_CCR1H
      000000A8H.2 SFRSYM    DATA     BIT       EX1
      000000BBH   SFRSYM    DATA     BYTE      TIM0_CCR2H
      000000D0H   SFRSYM    DATA     BIT       P
      000000BDH   SFRSYM    DATA     BYTE      TIM0_CCR3H
LX51 LINKER/LOCATER V4.66.1.0                                                         03/23/2017  15:15:44  PAGE 107


      000000BFH   SFRSYM    DATA     BYTE      TIM0_CCR4H
      000000C8H.2 SFRSYM    DATA     BIT       PTIM230
      000000EBH   SFRSYM    DATA     BYTE      PI_EKH
      00000098H.5 SFRSYM    DATA     BIT       SM2
      000000B6H   SFRSYM    DATA     BYTE      TIM0_CCR1L
      000000B1H   SFRSYM    DATA     BYTE      TIM0_SR1
      000000C8H.3 SFRSYM    DATA     BIT       PTIM231
      000000BAH   SFRSYM    DATA     BYTE      TIM0_CCR2L
      000000BCH   SFRSYM    DATA     BYTE      TIM0_CCR3L
      000000BEH   SFRSYM    DATA     BYTE      TIM0_CCR4L
      000000D8H.6 SFRSYM    DATA     BIT       PMCD0
      000000C8H.4 SFRSYM    DATA     BIT       PTIM450
      000000D0H.3 SFRSYM    DATA     BIT       RS0
      000000DDH   SFRSYM    DATA     BYTE      LPF_KH
      000000F3H   SFRSYM    DATA     BYTE      PI_KIH
      000000EAH   SFRSYM    DATA     BYTE      PI_EKL
      000000E8H   SFRSYM    DATA     BYTE      FOC_SET0
      000000D8H.7 SFRSYM    DATA     BIT       PMCD1
      000000C8H.5 SFRSYM    DATA     BIT       PTIM451
      000000D0H.4 SFRSYM    DATA     BIT       RS1
      000000E9H   SFRSYM    DATA     BYTE      FOC_SET1
      000000B8H.6 SFRSYM    DATA     BIT       PFOC0
      000000DCH   SFRSYM    DATA     BYTE      LPF_KL
      000000F2H   SFRSYM    DATA     BYTE      PI_KIL
      000000B8H.7 SFRSYM    DATA     BIT       PFOC1
      000000ADH   SFRSYM    DATA     BYTE      TIM2_DRH
      000000B9H   SFRSYM    DATA     BYTE      TIM0_IER
      00000083H   SFRSYM    DATA     BYTE      DPH
      000000EFH   SFRSYM    DATA     BYTE      PI_KPH
      000000A5H   SFRSYM    DATA     BYTE      TIM3_DRH
      00000095H   SFRSYM    DATA     BYTE      TIM4_DRH
      0000008DH   SFRSYM    DATA     BYTE      TIM5_DRH
      000000ACH   SFRSYM    DATA     BYTE      TIM2_DRL
      00000082H   SFRSYM    DATA     BYTE      DPL
      000000EEH   SFRSYM    DATA     BYTE      PI_KPL
      000000A4H   SFRSYM    DATA     BYTE      TIM3_DRL
      000000F8H.7 SFRSYM    DATA     BIT       MOE
      000000C0H.6 SFRSYM    DATA     BIT       PCMP0
      000000EDH   SFRSYM    DATA     BYTE      PI_UKH
      00000094H   SFRSYM    DATA     BYTE      TIM4_DRL
      000000C0H.7 SFRSYM    DATA     BIT       PCMP1
      000000DFH   SFRSYM    DATA     BYTE      LPF_XH
      0000008CH   SFRSYM    DATA     BYTE      TIM5_DRL
      000000AEH   SFRSYM    DATA     WORD      TIM2_ARR
      000000A8H.5 SFRSYM    DATA     BIT       MCDIE
      000000C9H   SFRSYM    DATA     BYTE      RSTSRC
      000000E7H   SFRSYM    DATA     BYTE      LPF_YH
      000000A6H   SFRSYM    DATA     WORD      TIM3_ARR
      00000088H.6 SFRSYM    DATA     BIT       MCDIF
      00000098H.4 SFRSYM    DATA     BIT       REN
      00000096H   SFRSYM    DATA     WORD      TIM4_ARR
      000000ECH   SFRSYM    DATA     BYTE      PI_UKL
      000000D7H   SFRSYM    DATA     BYTE      CMP_SR
      0000008EH   SFRSYM    DATA     WORD      TIM5_ARR
      000000DEH   SFRSYM    DATA     BYTE      LPF_XL
      000000E6H   SFRSYM    DATA     BYTE      LPF_YL
      000000C8H   SFRSYM    DATA     BIT       PRTC0
      000000C8H.1 SFRSYM    DATA     BIT       PRTC1
      000000E8H.7 SFRSYM    DATA     BIT       FOCEN
      000000C8H.6 SFRSYM    DATA     BIT       PTSD0
      000000D8H.4 SFRSYM    DATA     BIT       PSPI0
      000000C8H.7 SFRSYM    DATA     BIT       PTSD1
      000000D8H.5 SFRSYM    DATA     BIT       PSPI1
      0000009BH   SFRSYM    DATA     BYTE      UT_BAUDH
      000000E4H   SFRSYM    DATA     WORD      SV_ANGLE
LX51 LINKER/LOCATER V4.66.1.0                                                         03/23/2017  15:15:44  PAGE 108


      000000B5H   SFRSYM    DATA     BYTE      TIM2_ADTRH
      0000009AH   SFRSYM    DATA     BYTE      UT_BAUDL
      000000FCH   SFRSYM    DATA     BYTE      P0_OE
      000000FDH   SFRSYM    DATA     BYTE      P1_OE
      000000D0H.5 SFRSYM    DATA     BIT       F0
      000000B4H   SFRSYM    DATA     BYTE      TIM2_ADTRL
      000000FEH   SFRSYM    DATA     BYTE      P2_OE
      000000D0H.1 SFRSYM    DATA     BIT       F1
      00000080H   SFRSYM    DATA     BIT       GP00
      000000FFH   SFRSYM    DATA     BYTE      P3_OE
      00000090H   SFRSYM    DATA     BIT       GP10
      00000080H.1 SFRSYM    DATA     BIT       GP01
      000000A8H.6 SFRSYM    DATA     BIT       RTCIE
      000000A0H   SFRSYM    DATA     BIT       GP20
      00000090H.1 SFRSYM    DATA     BIT       GP11
      00000080H.2 SFRSYM    DATA     BIT       GP02
      000000E3H   SFRSYM    DATA     BYTE      SV_USH
      000000B0H   SFRSYM    DATA     BIT       GP30
      000000A0H.1 SFRSYM    DATA     BIT       GP21
      00000090H.2 SFRSYM    DATA     BIT       GP12
      00000080H.3 SFRSYM    DATA     BIT       GP03
      000000B8H   SFRSYM    DATA     BIT       PLVW0
      000000A8H.1 SFRSYM    DATA     BIT       TSDIE
      000000D0H   SFRSYM    DATA     BYTE      PSW
      000000B0H.1 SFRSYM    DATA     BIT       GP31
      000000A0H.2 SFRSYM    DATA     BIT       GP22
      00000090H.3 SFRSYM    DATA     BIT       GP13
      00000080H.4 SFRSYM    DATA     BIT       GP04
      000000B8H.1 SFRSYM    DATA     BIT       PLVW1
      000000A8H.3 SFRSYM    DATA     BIT       SPIIE
      00000088H.5 SFRSYM    DATA     BIT       TSDIF
      000000B0H.2 SFRSYM    DATA     BIT       GP32
      000000A0H.3 SFRSYM    DATA     BIT       GP23
      00000090H.4 SFRSYM    DATA     BIT       GP14
      00000080H.5 SFRSYM    DATA     BIT       GP05
      00000084H   SFRSYM    DATA     BYTE      FLKEY
      000000B3H   SFRSYM    DATA     BYTE      TIM2_CMTRH
      000000B0H.3 SFRSYM    DATA     BIT       GP33
      000000A0H.4 SFRSYM    DATA     BIT       GP24
      00000090H.5 SFRSYM    DATA     BIT       GP15
      00000080H.6 SFRSYM    DATA     BIT       GP06
      00000088H   SFRSYM    DATA     BIT       IT00

      0100189CH   BLOCK     CODE     ---       LVL=0
      0100189CH   LINE      CODE     ---       #23
      0100189CH   LINE      CODE     ---       #24
      0100189CH   LINE      CODE     ---       #25
      010018A3H   LINE      CODE     ---       #32
      010018AAH   LINE      CODE     ---       #33
      010018ADH   LINE      CODE     ---       #42
      010018B4H   LINE      CODE     ---       #43
      010018B8H   LINE      CODE     ---       #51
      010018BDH   LINE      CODE     ---       #52
      010018C1H   LINE      CODE     ---       #54
      010018C8H   LINE      CODE     ---       #63
      010018CDH   LINE      CODE     ---       #64
      010018D1H   LINE      CODE     ---       #65
      010018D5H   LINE      CODE     ---       #66
      010018D9H   LINE      CODE     ---       #67
      010018DBH   LINE      CODE     ---       #69
      010018DFH   LINE      CODE     ---       #71
      010018E6H   LINE      CODE     ---       #73
      ---         BLOCKEND  ---      ---       LVL=0
      00000002H   SYMBOL    DATA     WORD      Data
      00000005H   SYMBOL    DATA     BYTE      Channel
LX51 LINKER/LOCATER V4.66.1.0                                                         03/23/2017  15:15:44  PAGE 109



      ---         MODULE    ---      ---       GPIOINIT
      010017F7H   PUBLIC    CODE     ---       GPIOInit
      000000E2H   SFRSYM    DATA     BYTE      SV_USL
      000000ABH   SFRSYM    DATA     BYTE      TIM2_CNTRH
      000000B0H.4 SFRSYM    DATA     BIT       GP34
      000000A0H.5 SFRSYM    DATA     BIT       GP25
      00000090H.6 SFRSYM    DATA     BIT       GP16
      00000080H.7 SFRSYM    DATA     BIT       GP07
      00000088H.1 SFRSYM    DATA     BIT       IT01
      00000088H.3 SFRSYM    DATA     BIT       IT10
      000000F6H   SFRSYM    DATA     WORD      PI_UKMIN
      000000C2H   SFRSYM    DATA     WORD      MD_MA
      000000A3H   SFRSYM    DATA     BYTE      TIM3_CNTRH
      000000B0H.5 SFRSYM    DATA     BIT       GP35
      000000A0H.6 SFRSYM    DATA     BIT       GP26
      00000090H.7 SFRSYM    DATA     BIT       GP17
      00000080H   SFRSYM    DATA     BYTE      P0
      00000088H.4 SFRSYM    DATA     BIT       IT11
      000000CAH   SFRSYM    DATA     WORD      MD_MB
      00000093H   SFRSYM    DATA     BYTE      TIM4_CNTRH
      000000B0H.6 SFRSYM    DATA     BIT       GP36
      000000A0H.7 SFRSYM    DATA     BIT       GP27
      00000090H   SFRSYM    DATA     BYTE      P1
      000000D9H   SFRSYM    DATA     BYTE      EVT_FILT
      000000F4H   SFRSYM    DATA     WORD      PI_UKMAX
      0000008BH   SFRSYM    DATA     BYTE      TIM5_CNTRH
      000000B2H   SFRSYM    DATA     BYTE      TIM2_CMTRL
      000000B0H.7 SFRSYM    DATA     BIT       GP37
      000000A0H   SFRSYM    DATA     BYTE      P2
      000000AAH   SFRSYM    DATA     BYTE      TIM2_CNTRL
      000000B0H   SFRSYM    DATA     BYTE      P3
      000000A2H   SFRSYM    DATA     BYTE      TIM3_CNTRL
      000000D0H.6 SFRSYM    DATA     BIT       AC
      00000092H   SFRSYM    DATA     BYTE      TIM4_CNTRL
      0000008AH   SFRSYM    DATA     BYTE      TIM5_CNTRL
      000000B6H   SFRSYM    DATA     WORD      TIM0_CCR1
      000000A8H.7 SFRSYM    DATA     BIT       EA
      000000D5H   SFRSYM    DATA     BYTE      CMP_CR0
      000000BAH   SFRSYM    DATA     WORD      TIM0_CCR2
      000000D6H   SFRSYM    DATA     BYTE      CMP_CR1
      000000BCH   SFRSYM    DATA     WORD      TIM0_CCR3
      00000085H   SFRSYM    DATA     BYTE      PSCTL
      000000DAH   SFRSYM    DATA     BYTE      CMP_CR2
      000000BEH   SFRSYM    DATA     WORD      TIM0_CCR4
      000000B8H.2 SFRSYM    DATA     BIT       PX00
      000000EAH   SFRSYM    DATA     WORD      PI_EK
      000000F8H   SFRSYM    DATA     BIT       OISUH
      000000B8H.3 SFRSYM    DATA     BIT       PX01
      000000B8H.4 SFRSYM    DATA     BIT       PX10
      000000F8H.2 SFRSYM    DATA     BIT       OISVH
      000000B8H.5 SFRSYM    DATA     BIT       PX11
      000000F8H.4 SFRSYM    DATA     BIT       OISWH
      000000DCH   SFRSYM    DATA     WORD      LPF_K
      000000F2H   SFRSYM    DATA     WORD      PI_KI
      000000F8H.1 SFRSYM    DATA     BIT       OISUL
      000000A8H   SFRSYM    DATA     BYTE      IE
      000000F8H.3 SFRSYM    DATA     BIT       OISVL
      000000F8H.5 SFRSYM    DATA     BIT       OISWL
      000000D1H   SFRSYM    DATA     BYTE      P1IE
      00000098H.6 SFRSYM    DATA     BIT       MOD0
      000000D3H   SFRSYM    DATA     BYTE      P2IE
      000000D2H   SFRSYM    DATA     BYTE      P1IF
      000000F9H   SFRSYM    DATA     BYTE      PL_CR
      00000098H.7 SFRSYM    DATA     BIT       MOD1
LX51 LINKER/LOCATER V4.66.1.0                                                         03/23/2017  15:15:44  PAGE 110


      000000D4H   SFRSYM    DATA     BYTE      P2IF
      000000ACH   SFRSYM    DATA     WORD      TIM2_DR
      00000082H   SFRSYM    DATA     WORD      DP
      000000EEH   SFRSYM    DATA     WORD      PI_KP
      000000A4H   SFRSYM    DATA     WORD      TIM3_DR
      00000094H   SFRSYM    DATA     WORD      TIM4_DR
      0000008CH   SFRSYM    DATA     WORD      TIM5_DR
      000000F1H   SFRSYM    DATA     BYTE      OSC_CFG
      000000C1H   SFRSYM    DATA     BYTE      MD_MODE
      000000ECH   SFRSYM    DATA     WORD      PI_UK
      000000DEH   SFRSYM    DATA     WORD      LPF_X
      00000098H   SFRSYM    DATA     BIT       RI
      000000E6H   SFRSYM    DATA     WORD      LPF_Y
      000000C0H   SFRSYM    DATA     BIT       PTIM00
      000000D0H.7 SFRSYM    DATA     BIT       CY
      00000098H.1 SFRSYM    DATA     BIT       TI
      000000C0H.1 SFRSYM    DATA     BIT       PTIM01
      000000C0H.2 SFRSYM    DATA     BIT       PTIM10
      000000C0H.3 SFRSYM    DATA     BIT       PTIM11
      000000E1H   SFRSYM    DATA     BYTE      SV_CR
      00000098H   SFRSYM    DATA     BYTE      UT_CR
      00000099H   SFRSYM    DATA     BYTE      UT_DR
      000000F8H.6 SFRSYM    DATA     BIT       OIS4
      00000081H   SFRSYM    DATA     BYTE      SP
      000000D0H.2 SFRSYM    DATA     BIT       OV
      000000C4H   SFRSYM    DATA     BYTE      MD_DA0
      0000009AH   SFRSYM    DATA     WORD      UT_BAUD
      000000CCH   SFRSYM    DATA     BYTE      MD_DB0
      000000C5H   SFRSYM    DATA     BYTE      MD_DA1
      000000CDH   SFRSYM    DATA     BYTE      MD_DB1
      000000C6H   SFRSYM    DATA     BYTE      MD_DA2
      000000CEH   SFRSYM    DATA     BYTE      MD_DB2
      000000C7H   SFRSYM    DATA     BYTE      MD_DA3
      000000B4H   SFRSYM    DATA     WORD      TIM2_ADTR
      000000CFH   SFRSYM    DATA     BYTE      MD_DB3
      000000AFH   SFRSYM    DATA     BYTE      TIM2_ARRH
      000000A7H   SFRSYM    DATA     BYTE      TIM3_ARRH
      00000097H   SFRSYM    DATA     BYTE      TIM4_ARRH
      0000008FH   SFRSYM    DATA     BYTE      TIM5_ARRH
      000000AEH   SFRSYM    DATA     BYTE      TIM2_ARRL
      000000A6H   SFRSYM    DATA     BYTE      TIM3_ARRL
      00000087H   SFRSYM    DATA     BYTE      PCON
      000000E2H   SFRSYM    DATA     WORD      SV_US
      00000096H   SFRSYM    DATA     BYTE      TIM4_ARRL
      0000008EH   SFRSYM    DATA     BYTE      TIM5_ARRL
      000000B2H   SFRSYM    DATA     WORD      TIM2_CMTR
      00000088H   SFRSYM    DATA     BYTE      TCON
      000000AAH   SFRSYM    DATA     WORD      TIM2_CNTR
      000000A2H   SFRSYM    DATA     WORD      TIM3_CNTR
      00000092H   SFRSYM    DATA     WORD      TIM4_CNTR
      0000008AH   SFRSYM    DATA     WORD      TIM5_CNTR
      000000E5H   SFRSYM    DATA     BYTE      SV_ANGLEH
      000000D8H   SFRSYM    DATA     BIT       PUART0
      000000E4H   SFRSYM    DATA     BYTE      SV_ANGLEL
      000000C6H   SFRSYM    DATA     WORD      MD_DAH
      000000D8H.1 SFRSYM    DATA     BIT       PUART1
      000000D8H.2 SFRSYM    DATA     BIT       PI2C0
      00000088H.2 SFRSYM    DATA     BIT       IF0
      000000CEH   SFRSYM    DATA     WORD      MD_DBH
      000000D8H.3 SFRSYM    DATA     BIT       PI2C1
      000000F0H   SFRSYM    DATA     BYTE      B
      000000C4H   SFRSYM    DATA     WORD      MD_DAL
      000000A1H   SFRSYM    DATA     BYTE      TIM2_CR0
      000000CCH   SFRSYM    DATA     WORD      MD_DBL
      0000009CH   SFRSYM    DATA     BYTE      TIM3_CR0
LX51 LINKER/LOCATER V4.66.1.0                                                         03/23/2017  15:15:44  PAGE 111


      000000A9H   SFRSYM    DATA     BYTE      TIM2_CR1
      0000009EH   SFRSYM    DATA     BYTE      TIM4_CR0
      0000009DH   SFRSYM    DATA     BYTE      TIM3_CR1
      00000089H   SFRSYM    DATA     BYTE      TIM5_CR0
      0000009FH   SFRSYM    DATA     BYTE      TIM4_CR1
      000000F8H   SFRSYM    DATA     BYTE      DRV_OUT
      00000091H   SFRSYM    DATA     BYTE      TIM5_CR1
      000000E0H   SFRSYM    DATA     BYTE      ACC
      000000F7H   SFRSYM    DATA     BYTE      PI_UKMINH
      000000C3H   SFRSYM    DATA     BYTE      MD_MAH
      000000A8H.4 SFRSYM    DATA     BIT       ES0
      000000DBH   SFRSYM    DATA     BYTE      LVSR
      000000CBH   SFRSYM    DATA     BYTE      MD_MBH
      000000C0H.4 SFRSYM    DATA     BIT       PADC0
      000000B8H   SFRSYM    DATA     BYTE      IP0
      000000F5H   SFRSYM    DATA     BYTE      PI_UKMAXH
      000000C0H.5 SFRSYM    DATA     BIT       PADC1
      000000C0H   SFRSYM    DATA     BYTE      IP1
      000000C8H   SFRSYM    DATA     BYTE      IP2
      000000F6H   SFRSYM    DATA     BYTE      PI_UKMINL
      000000C2H   SFRSYM    DATA     BYTE      MD_MAL
      00000098H.2 SFRSYM    DATA     BIT       RB8
      000000D8H   SFRSYM    DATA     BYTE      IP3
      000000CAH   SFRSYM    DATA     BYTE      MD_MBL
      000000A8H   SFRSYM    DATA     BIT       EX0
      000000F4H   SFRSYM    DATA     BYTE      PI_UKMAXL
      00000098H.3 SFRSYM    DATA     BIT       TB8
      000000B7H   SFRSYM    DATA     BYTE      TIM0_CCR1H
      000000A8H.2 SFRSYM    DATA     BIT       EX1
      000000BBH   SFRSYM    DATA     BYTE      TIM0_CCR2H
      000000D0H   SFRSYM    DATA     BIT       P
      000000BDH   SFRSYM    DATA     BYTE      TIM0_CCR3H
      000000BFH   SFRSYM    DATA     BYTE      TIM0_CCR4H
      000000C8H.2 SFRSYM    DATA     BIT       PTIM230
      000000EBH   SFRSYM    DATA     BYTE      PI_EKH
      00000098H.5 SFRSYM    DATA     BIT       SM2
      000000B6H   SFRSYM    DATA     BYTE      TIM0_CCR1L
      000000B1H   SFRSYM    DATA     BYTE      TIM0_SR1
      000000C8H.3 SFRSYM    DATA     BIT       PTIM231
      000000BAH   SFRSYM    DATA     BYTE      TIM0_CCR2L
      000000BCH   SFRSYM    DATA     BYTE      TIM0_CCR3L
      000000BEH   SFRSYM    DATA     BYTE      TIM0_CCR4L
      000000D8H.6 SFRSYM    DATA     BIT       PMCD0
      000000C8H.4 SFRSYM    DATA     BIT       PTIM450
      000000D0H.3 SFRSYM    DATA     BIT       RS0
      000000DDH   SFRSYM    DATA     BYTE      LPF_KH
      000000F3H   SFRSYM    DATA     BYTE      PI_KIH
      000000EAH   SFRSYM    DATA     BYTE      PI_EKL
      000000E8H   SFRSYM    DATA     BYTE      FOC_SET0
      000000D8H.7 SFRSYM    DATA     BIT       PMCD1
      000000C8H.5 SFRSYM    DATA     BIT       PTIM451
      000000D0H.4 SFRSYM    DATA     BIT       RS1
      000000E9H   SFRSYM    DATA     BYTE      FOC_SET1
      000000B8H.6 SFRSYM    DATA     BIT       PFOC0
      000000DCH   SFRSYM    DATA     BYTE      LPF_KL
      000000F2H   SFRSYM    DATA     BYTE      PI_KIL
      000000B8H.7 SFRSYM    DATA     BIT       PFOC1
      000000ADH   SFRSYM    DATA     BYTE      TIM2_DRH
      000000B9H   SFRSYM    DATA     BYTE      TIM0_IER
      00000083H   SFRSYM    DATA     BYTE      DPH
      000000EFH   SFRSYM    DATA     BYTE      PI_KPH
      000000A5H   SFRSYM    DATA     BYTE      TIM3_DRH
      00000095H   SFRSYM    DATA     BYTE      TIM4_DRH
      0000008DH   SFRSYM    DATA     BYTE      TIM5_DRH
      000000ACH   SFRSYM    DATA     BYTE      TIM2_DRL
LX51 LINKER/LOCATER V4.66.1.0                                                         03/23/2017  15:15:44  PAGE 112


      00000082H   SFRSYM    DATA     BYTE      DPL
      000000EEH   SFRSYM    DATA     BYTE      PI_KPL
      000000A4H   SFRSYM    DATA     BYTE      TIM3_DRL
      000000F8H.7 SFRSYM    DATA     BIT       MOE
      000000C0H.6 SFRSYM    DATA     BIT       PCMP0
      000000EDH   SFRSYM    DATA     BYTE      PI_UKH
      00000094H   SFRSYM    DATA     BYTE      TIM4_DRL
      000000C0H.7 SFRSYM    DATA     BIT       PCMP1
      000000DFH   SFRSYM    DATA     BYTE      LPF_XH
      0000008CH   SFRSYM    DATA     BYTE      TIM5_DRL
      000000AEH   SFRSYM    DATA     WORD      TIM2_ARR
      000000A8H.5 SFRSYM    DATA     BIT       MCDIE
      000000C9H   SFRSYM    DATA     BYTE      RSTSRC
      000000E7H   SFRSYM    DATA     BYTE      LPF_YH
      000000A6H   SFRSYM    DATA     WORD      TIM3_ARR
      00000088H.6 SFRSYM    DATA     BIT       MCDIF
      00000098H.4 SFRSYM    DATA     BIT       REN
      00000096H   SFRSYM    DATA     WORD      TIM4_ARR
      000000ECH   SFRSYM    DATA     BYTE      PI_UKL
      000000D7H   SFRSYM    DATA     BYTE      CMP_SR
      0000008EH   SFRSYM    DATA     WORD      TIM5_ARR
      000000DEH   SFRSYM    DATA     BYTE      LPF_XL
      000000E6H   SFRSYM    DATA     BYTE      LPF_YL
      000000C8H   SFRSYM    DATA     BIT       PRTC0
      000000C8H.1 SFRSYM    DATA     BIT       PRTC1
      000000E8H.7 SFRSYM    DATA     BIT       FOCEN
      000000C8H.6 SFRSYM    DATA     BIT       PTSD0
      000000D8H.4 SFRSYM    DATA     BIT       PSPI0
      000000C8H.7 SFRSYM    DATA     BIT       PTSD1
      000000D8H.5 SFRSYM    DATA     BIT       PSPI1
      0000009BH   SFRSYM    DATA     BYTE      UT_BAUDH
      000000E4H   SFRSYM    DATA     WORD      SV_ANGLE
      000000B5H   SFRSYM    DATA     BYTE      TIM2_ADTRH
      0000009AH   SFRSYM    DATA     BYTE      UT_BAUDL
      000000FCH   SFRSYM    DATA     BYTE      P0_OE
      000000FDH   SFRSYM    DATA     BYTE      P1_OE
      000000D0H.5 SFRSYM    DATA     BIT       F0
      000000B4H   SFRSYM    DATA     BYTE      TIM2_ADTRL
      000000FEH   SFRSYM    DATA     BYTE      P2_OE
      000000D0H.1 SFRSYM    DATA     BIT       F1
      00000080H   SFRSYM    DATA     BIT       GP00
      000000FFH   SFRSYM    DATA     BYTE      P3_OE
      00000090H   SFRSYM    DATA     BIT       GP10
      00000080H.1 SFRSYM    DATA     BIT       GP01
      000000A8H.6 SFRSYM    DATA     BIT       RTCIE
      000000A0H   SFRSYM    DATA     BIT       GP20
      00000090H.1 SFRSYM    DATA     BIT       GP11
      00000080H.2 SFRSYM    DATA     BIT       GP02
      000000E3H   SFRSYM    DATA     BYTE      SV_USH
      000000B0H   SFRSYM    DATA     BIT       GP30
      000000A0H.1 SFRSYM    DATA     BIT       GP21
      00000090H.2 SFRSYM    DATA     BIT       GP12
      00000080H.3 SFRSYM    DATA     BIT       GP03
      000000B8H   SFRSYM    DATA     BIT       PLVW0
      000000A8H.1 SFRSYM    DATA     BIT       TSDIE
      000000D0H   SFRSYM    DATA     BYTE      PSW
      000000B0H.1 SFRSYM    DATA     BIT       GP31
      000000A0H.2 SFRSYM    DATA     BIT       GP22
      00000090H.3 SFRSYM    DATA     BIT       GP13
      00000080H.4 SFRSYM    DATA     BIT       GP04
      000000B8H.1 SFRSYM    DATA     BIT       PLVW1
      000000A8H.3 SFRSYM    DATA     BIT       SPIIE
      00000088H.5 SFRSYM    DATA     BIT       TSDIF
      000000B0H.2 SFRSYM    DATA     BIT       GP32
      000000A0H.3 SFRSYM    DATA     BIT       GP23
LX51 LINKER/LOCATER V4.66.1.0                                                         03/23/2017  15:15:44  PAGE 113


      00000090H.4 SFRSYM    DATA     BIT       GP14
      00000080H.5 SFRSYM    DATA     BIT       GP05
      00000084H   SFRSYM    DATA     BYTE      FLKEY
      000000B3H   SFRSYM    DATA     BYTE      TIM2_CMTRH
      000000B0H.3 SFRSYM    DATA     BIT       GP33
      000000A0H.4 SFRSYM    DATA     BIT       GP24
      00000090H.5 SFRSYM    DATA     BIT       GP15
      00000080H.6 SFRSYM    DATA     BIT       GP06
      00000088H   SFRSYM    DATA     BIT       IT00

      010017F7H   BLOCK     CODE     ---       LVL=0
      010017F7H   LINE      CODE     ---       #22
      010017F7H   LINE      CODE     ---       #23
      010017F7H   LINE      CODE     ---       #24
      010017FAH   LINE      CODE     ---       #25
      01001801H   LINE      CODE     ---       #27
      01001804H   LINE      CODE     ---       #28
      01001808H   LINE      CODE     ---       #30
      0100180BH   LINE      CODE     ---       #31
      0100180FH   LINE      CODE     ---       #33
      01001812H   LINE      CODE     ---       #34
      01001816H   LINE      CODE     ---       #36
      01001819H   LINE      CODE     ---       #37
      0100181EH   LINE      CODE     ---       #38
      01001820H   LINE      CODE     ---       #40
      01001823H   LINE      CODE     ---       #41
      01001827H   LINE      CODE     ---       #43
      0100182AH   LINE      CODE     ---       #44
      01001831H   LINE      CODE     ---       #46
      01001834H   LINE      CODE     ---       #47
      0100183BH   LINE      CODE     ---       #48
      01001842H   LINE      CODE     ---       #50
      01001845H   LINE      CODE     ---       #51
      0100184CH   LINE      CODE     ---       #54
      ---         BLOCKEND  ---      ---       LVL=0

      ---         MODULE    ---      ---       ADCINIT
      020000B7H   PUBLIC    XDATA    ---       ADCData
      0100139CH   PUBLIC    CODE     ---       ADCDataInit
      010015EFH   PUBLIC    CODE     ---       ADCInit
      000000E2H   SFRSYM    DATA     BYTE      SV_USL
      000000ABH   SFRSYM    DATA     BYTE      TIM2_CNTRH
      000000B0H.4 SFRSYM    DATA     BIT       GP34
      000000A0H.5 SFRSYM    DATA     BIT       GP25
      00000090H.6 SFRSYM    DATA     BIT       GP16
      00000080H.7 SFRSYM    DATA     BIT       GP07
      00000088H.1 SFRSYM    DATA     BIT       IT01
      00000088H.3 SFRSYM    DATA     BIT       IT10
      000000F6H   SFRSYM    DATA     WORD      PI_UKMIN
      000000C2H   SFRSYM    DATA     WORD      MD_MA
      000000A3H   SFRSYM    DATA     BYTE      TIM3_CNTRH
      000000B0H.5 SFRSYM    DATA     BIT       GP35
      000000A0H.6 SFRSYM    DATA     BIT       GP26
      00000090H.7 SFRSYM    DATA     BIT       GP17
      00000080H   SFRSYM    DATA     BYTE      P0
      00000088H.4 SFRSYM    DATA     BIT       IT11
      000000CAH   SFRSYM    DATA     WORD      MD_MB
      00000093H   SFRSYM    DATA     BYTE      TIM4_CNTRH
      000000B0H.6 SFRSYM    DATA     BIT       GP36
      000000A0H.7 SFRSYM    DATA     BIT       GP27
      00000090H   SFRSYM    DATA     BYTE      P1
      000000D9H   SFRSYM    DATA     BYTE      EVT_FILT
      000000F4H   SFRSYM    DATA     WORD      PI_UKMAX
      0000008BH   SFRSYM    DATA     BYTE      TIM5_CNTRH
      000000B2H   SFRSYM    DATA     BYTE      TIM2_CMTRL
LX51 LINKER/LOCATER V4.66.1.0                                                         03/23/2017  15:15:44  PAGE 114


      000000B0H.7 SFRSYM    DATA     BIT       GP37
      000000A0H   SFRSYM    DATA     BYTE      P2
      000000AAH   SFRSYM    DATA     BYTE      TIM2_CNTRL
      000000B0H   SFRSYM    DATA     BYTE      P3
      000000A2H   SFRSYM    DATA     BYTE      TIM3_CNTRL
      000000D0H.6 SFRSYM    DATA     BIT       AC
      00000092H   SFRSYM    DATA     BYTE      TIM4_CNTRL
      0000008AH   SFRSYM    DATA     BYTE      TIM5_CNTRL
      000000B6H   SFRSYM    DATA     WORD      TIM0_CCR1
      000000A8H.7 SFRSYM    DATA     BIT       EA
      000000D5H   SFRSYM    DATA     BYTE      CMP_CR0
      000000BAH   SFRSYM    DATA     WORD      TIM0_CCR2
      000000D6H   SFRSYM    DATA     BYTE      CMP_CR1
      000000BCH   SFRSYM    DATA     WORD      TIM0_CCR3
      00000085H   SFRSYM    DATA     BYTE      PSCTL
      000000DAH   SFRSYM    DATA     BYTE      CMP_CR2
      000000BEH   SFRSYM    DATA     WORD      TIM0_CCR4
      000000B8H.2 SFRSYM    DATA     BIT       PX00
      000000EAH   SFRSYM    DATA     WORD      PI_EK
      000000F8H   SFRSYM    DATA     BIT       OISUH
      000000B8H.3 SFRSYM    DATA     BIT       PX01
      000000B8H.4 SFRSYM    DATA     BIT       PX10
      000000F8H.2 SFRSYM    DATA     BIT       OISVH
      000000B8H.5 SFRSYM    DATA     BIT       PX11
      000000F8H.4 SFRSYM    DATA     BIT       OISWH
      000000DCH   SFRSYM    DATA     WORD      LPF_K
      000000F2H   SFRSYM    DATA     WORD      PI_KI
      000000F8H.1 SFRSYM    DATA     BIT       OISUL
      000000A8H   SFRSYM    DATA     BYTE      IE
      000000F8H.3 SFRSYM    DATA     BIT       OISVL
      000000F8H.5 SFRSYM    DATA     BIT       OISWL
      000000D1H   SFRSYM    DATA     BYTE      P1IE
      00000098H.6 SFRSYM    DATA     BIT       MOD0
      000000D3H   SFRSYM    DATA     BYTE      P2IE
      000000D2H   SFRSYM    DATA     BYTE      P1IF
      000000F9H   SFRSYM    DATA     BYTE      PL_CR
      00000098H.7 SFRSYM    DATA     BIT       MOD1
      000000D4H   SFRSYM    DATA     BYTE      P2IF
      000000ACH   SFRSYM    DATA     WORD      TIM2_DR
      00000082H   SFRSYM    DATA     WORD      DP
      000000EEH   SFRSYM    DATA     WORD      PI_KP
      000000A4H   SFRSYM    DATA     WORD      TIM3_DR
      00000094H   SFRSYM    DATA     WORD      TIM4_DR
      0000008CH   SFRSYM    DATA     WORD      TIM5_DR
      000000F1H   SFRSYM    DATA     BYTE      OSC_CFG
      000000C1H   SFRSYM    DATA     BYTE      MD_MODE
      000000ECH   SFRSYM    DATA     WORD      PI_UK
      000000DEH   SFRSYM    DATA     WORD      LPF_X
      00000098H   SFRSYM    DATA     BIT       RI
      000000E6H   SFRSYM    DATA     WORD      LPF_Y
      000000C0H   SFRSYM    DATA     BIT       PTIM00
      000000D0H.7 SFRSYM    DATA     BIT       CY
      00000098H.1 SFRSYM    DATA     BIT       TI
      000000C0H.1 SFRSYM    DATA     BIT       PTIM01
      000000C0H.2 SFRSYM    DATA     BIT       PTIM10
      000000C0H.3 SFRSYM    DATA     BIT       PTIM11
      000000E1H   SFRSYM    DATA     BYTE      SV_CR
      00000098H   SFRSYM    DATA     BYTE      UT_CR
      00000099H   SFRSYM    DATA     BYTE      UT_DR
      000000F8H.6 SFRSYM    DATA     BIT       OIS4
      00000081H   SFRSYM    DATA     BYTE      SP
      000000D0H.2 SFRSYM    DATA     BIT       OV
      000000C4H   SFRSYM    DATA     BYTE      MD_DA0
      0000009AH   SFRSYM    DATA     WORD      UT_BAUD
      000000CCH   SFRSYM    DATA     BYTE      MD_DB0
LX51 LINKER/LOCATER V4.66.1.0                                                         03/23/2017  15:15:44  PAGE 115


      000000C5H   SFRSYM    DATA     BYTE      MD_DA1
      000000CDH   SFRSYM    DATA     BYTE      MD_DB1
      000000C6H   SFRSYM    DATA     BYTE      MD_DA2
      000000CEH   SFRSYM    DATA     BYTE      MD_DB2
      000000C7H   SFRSYM    DATA     BYTE      MD_DA3
      000000B4H   SFRSYM    DATA     WORD      TIM2_ADTR
      000000CFH   SFRSYM    DATA     BYTE      MD_DB3
      000000AFH   SFRSYM    DATA     BYTE      TIM2_ARRH
      000000A7H   SFRSYM    DATA     BYTE      TIM3_ARRH
      00000097H   SFRSYM    DATA     BYTE      TIM4_ARRH
      0000008FH   SFRSYM    DATA     BYTE      TIM5_ARRH
      000000AEH   SFRSYM    DATA     BYTE      TIM2_ARRL
      000000A6H   SFRSYM    DATA     BYTE      TIM3_ARRL
      00000087H   SFRSYM    DATA     BYTE      PCON
      000000E2H   SFRSYM    DATA     WORD      SV_US
      00000096H   SFRSYM    DATA     BYTE      TIM4_ARRL
      0000008EH   SFRSYM    DATA     BYTE      TIM5_ARRL
      000000B2H   SFRSYM    DATA     WORD      TIM2_CMTR
      00000088H   SFRSYM    DATA     BYTE      TCON
      000000AAH   SFRSYM    DATA     WORD      TIM2_CNTR
      000000A2H   SFRSYM    DATA     WORD      TIM3_CNTR
      00000092H   SFRSYM    DATA     WORD      TIM4_CNTR
      0000008AH   SFRSYM    DATA     WORD      TIM5_CNTR
      000000E5H   SFRSYM    DATA     BYTE      SV_ANGLEH
      000000D8H   SFRSYM    DATA     BIT       PUART0
      000000E4H   SFRSYM    DATA     BYTE      SV_ANGLEL
      000000C6H   SFRSYM    DATA     WORD      MD_DAH
      000000D8H.1 SFRSYM    DATA     BIT       PUART1
      000000D8H.2 SFRSYM    DATA     BIT       PI2C0
      00000088H.2 SFRSYM    DATA     BIT       IF0
      000000CEH   SFRSYM    DATA     WORD      MD_DBH
      000000D8H.3 SFRSYM    DATA     BIT       PI2C1
      000000F0H   SFRSYM    DATA     BYTE      B
      000000C4H   SFRSYM    DATA     WORD      MD_DAL
      000000A1H   SFRSYM    DATA     BYTE      TIM2_CR0
      000000CCH   SFRSYM    DATA     WORD      MD_DBL
      0000009CH   SFRSYM    DATA     BYTE      TIM3_CR0
      000000A9H   SFRSYM    DATA     BYTE      TIM2_CR1
      0000009EH   SFRSYM    DATA     BYTE      TIM4_CR0
      0000009DH   SFRSYM    DATA     BYTE      TIM3_CR1
      00000089H   SFRSYM    DATA     BYTE      TIM5_CR0
      0000009FH   SFRSYM    DATA     BYTE      TIM4_CR1
      000000F8H   SFRSYM    DATA     BYTE      DRV_OUT
      00000091H   SFRSYM    DATA     BYTE      TIM5_CR1
      000000E0H   SFRSYM    DATA     BYTE      ACC
      000000F7H   SFRSYM    DATA     BYTE      PI_UKMINH
      000000C3H   SFRSYM    DATA     BYTE      MD_MAH
      000000A8H.4 SFRSYM    DATA     BIT       ES0
      000000DBH   SFRSYM    DATA     BYTE      LVSR
      000000CBH   SFRSYM    DATA     BYTE      MD_MBH
      000000C0H.4 SFRSYM    DATA     BIT       PADC0
      000000B8H   SFRSYM    DATA     BYTE      IP0
      000000F5H   SFRSYM    DATA     BYTE      PI_UKMAXH
      000000C0H.5 SFRSYM    DATA     BIT       PADC1
      000000C0H   SFRSYM    DATA     BYTE      IP1
      000000C8H   SFRSYM    DATA     BYTE      IP2
      000000F6H   SFRSYM    DATA     BYTE      PI_UKMINL
      000000C2H   SFRSYM    DATA     BYTE      MD_MAL
      00000098H.2 SFRSYM    DATA     BIT       RB8
      000000D8H   SFRSYM    DATA     BYTE      IP3
      000000CAH   SFRSYM    DATA     BYTE      MD_MBL
      000000A8H   SFRSYM    DATA     BIT       EX0
      000000F4H   SFRSYM    DATA     BYTE      PI_UKMAXL
      00000098H.3 SFRSYM    DATA     BIT       TB8
      000000B7H   SFRSYM    DATA     BYTE      TIM0_CCR1H
LX51 LINKER/LOCATER V4.66.1.0                                                         03/23/2017  15:15:44  PAGE 116


      000000A8H.2 SFRSYM    DATA     BIT       EX1
      000000BBH   SFRSYM    DATA     BYTE      TIM0_CCR2H
      000000D0H   SFRSYM    DATA     BIT       P
      000000BDH   SFRSYM    DATA     BYTE      TIM0_CCR3H
      000000BFH   SFRSYM    DATA     BYTE      TIM0_CCR4H
      000000C8H.2 SFRSYM    DATA     BIT       PTIM230
      000000EBH   SFRSYM    DATA     BYTE      PI_EKH
      00000098H.5 SFRSYM    DATA     BIT       SM2
      000000B6H   SFRSYM    DATA     BYTE      TIM0_CCR1L
      000000B1H   SFRSYM    DATA     BYTE      TIM0_SR1
      000000C8H.3 SFRSYM    DATA     BIT       PTIM231
      000000BAH   SFRSYM    DATA     BYTE      TIM0_CCR2L
      000000BCH   SFRSYM    DATA     BYTE      TIM0_CCR3L
      000000BEH   SFRSYM    DATA     BYTE      TIM0_CCR4L
      000000D8H.6 SFRSYM    DATA     BIT       PMCD0
      000000C8H.4 SFRSYM    DATA     BIT       PTIM450
      000000D0H.3 SFRSYM    DATA     BIT       RS0
      000000DDH   SFRSYM    DATA     BYTE      LPF_KH
      000000F3H   SFRSYM    DATA     BYTE      PI_KIH
      000000EAH   SFRSYM    DATA     BYTE      PI_EKL
      000000E8H   SFRSYM    DATA     BYTE      FOC_SET0
      000000D8H.7 SFRSYM    DATA     BIT       PMCD1
      000000C8H.5 SFRSYM    DATA     BIT       PTIM451
      000000D0H.4 SFRSYM    DATA     BIT       RS1
      000000E9H   SFRSYM    DATA     BYTE      FOC_SET1
      000000B8H.6 SFRSYM    DATA     BIT       PFOC0
      000000DCH   SFRSYM    DATA     BYTE      LPF_KL
      000000F2H   SFRSYM    DATA     BYTE      PI_KIL
      000000B8H.7 SFRSYM    DATA     BIT       PFOC1
      000000ADH   SFRSYM    DATA     BYTE      TIM2_DRH
      000000B9H   SFRSYM    DATA     BYTE      TIM0_IER
      00000083H   SFRSYM    DATA     BYTE      DPH
      000000EFH   SFRSYM    DATA     BYTE      PI_KPH
      000000A5H   SFRSYM    DATA     BYTE      TIM3_DRH
      00000095H   SFRSYM    DATA     BYTE      TIM4_DRH
      0000008DH   SFRSYM    DATA     BYTE      TIM5_DRH
      000000ACH   SFRSYM    DATA     BYTE      TIM2_DRL
      00000082H   SFRSYM    DATA     BYTE      DPL
      000000EEH   SFRSYM    DATA     BYTE      PI_KPL
      000000A4H   SFRSYM    DATA     BYTE      TIM3_DRL
      000000F8H.7 SFRSYM    DATA     BIT       MOE
      000000C0H.6 SFRSYM    DATA     BIT       PCMP0
      000000EDH   SFRSYM    DATA     BYTE      PI_UKH
      00000094H   SFRSYM    DATA     BYTE      TIM4_DRL
      000000C0H.7 SFRSYM    DATA     BIT       PCMP1
      000000DFH   SFRSYM    DATA     BYTE      LPF_XH
      0000008CH   SFRSYM    DATA     BYTE      TIM5_DRL
      000000AEH   SFRSYM    DATA     WORD      TIM2_ARR
      000000A8H.5 SFRSYM    DATA     BIT       MCDIE
      000000C9H   SFRSYM    DATA     BYTE      RSTSRC
      000000E7H   SFRSYM    DATA     BYTE      LPF_YH
      000000A6H   SFRSYM    DATA     WORD      TIM3_ARR
      00000088H.6 SFRSYM    DATA     BIT       MCDIF
      00000098H.4 SFRSYM    DATA     BIT       REN
      00000096H   SFRSYM    DATA     WORD      TIM4_ARR
      000000ECH   SFRSYM    DATA     BYTE      PI_UKL
      000000D7H   SFRSYM    DATA     BYTE      CMP_SR
      0000008EH   SFRSYM    DATA     WORD      TIM5_ARR
      000000DEH   SFRSYM    DATA     BYTE      LPF_XL
      000000E6H   SFRSYM    DATA     BYTE      LPF_YL
      000000C8H   SFRSYM    DATA     BIT       PRTC0
      000000C8H.1 SFRSYM    DATA     BIT       PRTC1
      000000E8H.7 SFRSYM    DATA     BIT       FOCEN
      000000C8H.6 SFRSYM    DATA     BIT       PTSD0
      000000D8H.4 SFRSYM    DATA     BIT       PSPI0
LX51 LINKER/LOCATER V4.66.1.0                                                         03/23/2017  15:15:44  PAGE 117


      000000C8H.7 SFRSYM    DATA     BIT       PTSD1
      000000D8H.5 SFRSYM    DATA     BIT       PSPI1
      0000009BH   SFRSYM    DATA     BYTE      UT_BAUDH
      000000E4H   SFRSYM    DATA     WORD      SV_ANGLE
      000000B5H   SFRSYM    DATA     BYTE      TIM2_ADTRH
      0000009AH   SFRSYM    DATA     BYTE      UT_BAUDL
      000000FCH   SFRSYM    DATA     BYTE      P0_OE
      000000FDH   SFRSYM    DATA     BYTE      P1_OE
      000000D0H.5 SFRSYM    DATA     BIT       F0
      000000B4H   SFRSYM    DATA     BYTE      TIM2_ADTRL
      000000FEH   SFRSYM    DATA     BYTE      P2_OE
      000000D0H.1 SFRSYM    DATA     BIT       F1
      00000080H   SFRSYM    DATA     BIT       GP00
      000000FFH   SFRSYM    DATA     BYTE      P3_OE
      00000090H   SFRSYM    DATA     BIT       GP10
      00000080H.1 SFRSYM    DATA     BIT       GP01
      000000A8H.6 SFRSYM    DATA     BIT       RTCIE
      000000A0H   SFRSYM    DATA     BIT       GP20
      00000090H.1 SFRSYM    DATA     BIT       GP11
      00000080H.2 SFRSYM    DATA     BIT       GP02
      000000E3H   SFRSYM    DATA     BYTE      SV_USH
      000000B0H   SFRSYM    DATA     BIT       GP30
      000000A0H.1 SFRSYM    DATA     BIT       GP21
      00000090H.2 SFRSYM    DATA     BIT       GP12
      00000080H.3 SFRSYM    DATA     BIT       GP03
      000000B8H   SFRSYM    DATA     BIT       PLVW0
      000000A8H.1 SFRSYM    DATA     BIT       TSDIE
      000000D0H   SFRSYM    DATA     BYTE      PSW
      000000B0H.1 SFRSYM    DATA     BIT       GP31
      000000A0H.2 SFRSYM    DATA     BIT       GP22
      00000090H.3 SFRSYM    DATA     BIT       GP13
      00000080H.4 SFRSYM    DATA     BIT       GP04
      000000B8H.1 SFRSYM    DATA     BIT       PLVW1
      000000A8H.3 SFRSYM    DATA     BIT       SPIIE
      00000088H.5 SFRSYM    DATA     BIT       TSDIF
      000000B0H.2 SFRSYM    DATA     BIT       GP32
      000000A0H.3 SFRSYM    DATA     BIT       GP23
      00000090H.4 SFRSYM    DATA     BIT       GP14
      00000080H.5 SFRSYM    DATA     BIT       GP05
      00000084H   SFRSYM    DATA     BYTE      FLKEY
      000000B3H   SFRSYM    DATA     BYTE      TIM2_CMTRH
      000000B0H.3 SFRSYM    DATA     BIT       GP33
      000000A0H.4 SFRSYM    DATA     BIT       GP24
      00000090H.5 SFRSYM    DATA     BIT       GP15
      00000080H.6 SFRSYM    DATA     BIT       GP06
      00000088H   SFRSYM    DATA     BIT       IT00

      010015EFH   BLOCK     CODE     ---       LVL=0
      010015EFH   LINE      CODE     ---       #26
      010015EFH   LINE      CODE     ---       #27
      010015EFH   LINE      CODE     ---       #34
      010015F6H   LINE      CODE     ---       #35
      010015FAH   LINE      CODE     ---       #36
      01001601H   LINE      CODE     ---       #46
      01001605H   LINE      CODE     ---       #47
      01001609H   LINE      CODE     ---       #54
      01001610H   LINE      CODE     ---       #55
      01001617H   LINE      CODE     ---       #56
      0100161EH   LINE      CODE     ---       #57
      01001625H   LINE      CODE     ---       #60
      0100162CH   LINE      CODE     ---       #61
      01001633H   LINE      CODE     ---       #62
      0100163AH   LINE      CODE     ---       #63
      01001641H   LINE      CODE     ---       #64
      01001648H   LINE      CODE     ---       #65
LX51 LINKER/LOCATER V4.66.1.0                                                         03/23/2017  15:15:44  PAGE 118


      0100164FH   LINE      CODE     ---       #72
      01001655H   LINE      CODE     ---       #73
      01001659H   LINE      CODE     ---       #81
      01001660H   LINE      CODE     ---       #82
      01001664H   LINE      CODE     ---       #83
      0100166BH   LINE      CODE     ---       #84
      0100166FH   LINE      CODE     ---       #86
      ---         BLOCKEND  ---      ---       LVL=0

      0100139CH   BLOCK     CODE     ---       LVL=0
      0100139CH   LINE      CODE     ---       #95
      0100139CH   LINE      CODE     ---       #96
      0100139CH   LINE      CODE     ---       #98
      010013A3H   LINE      CODE     ---       #99
      010013A7H   LINE      CODE     ---       #100
      010013ABH   LINE      CODE     ---       #101
      010013AFH   LINE      CODE     ---       #102
      010013B3H   LINE      CODE     ---       #103
      010013B7H   LINE      CODE     ---       #104
      010013BBH   LINE      CODE     ---       #105
      010013BFH   LINE      CODE     ---       #106
      010013C3H   LINE      CODE     ---       #107
      010013C7H   LINE      CODE     ---       #108
      010013CBH   LINE      CODE     ---       #109
      010013CFH   LINE      CODE     ---       #110
      010013D7H   LINE      CODE     ---       #111
      010013E1H   LINE      CODE     ---       #112
      010013EBH   LINE      CODE     ---       #113
      010013F5H   LINE      CODE     ---       #114
      010013FFH   LINE      CODE     ---       #115
      01001409H   LINE      CODE     ---       #116
      01001413H   LINE      CODE     ---       #117
      0100141DH   LINE      CODE     ---       #118
      01001427H   LINE      CODE     ---       #119
      01001431H   LINE      CODE     ---       #120
      0100143BH   LINE      CODE     ---       #122
      ---         BLOCKEND  ---      ---       LVL=0

      ---         MODULE    ---      ---       CMPINIT
      01001B8AH   PUBLIC    CODE     ---       CMPIint
      000000E2H   SFRSYM    DATA     BYTE      SV_USL
      000000ABH   SFRSYM    DATA     BYTE      TIM2_CNTRH
      000000B0H.4 SFRSYM    DATA     BIT       GP34
      000000A0H.5 SFRSYM    DATA     BIT       GP25
      00000090H.6 SFRSYM    DATA     BIT       GP16
      00000080H.7 SFRSYM    DATA     BIT       GP07
      00000088H.1 SFRSYM    DATA     BIT       IT01
      00000088H.3 SFRSYM    DATA     BIT       IT10
      000000F6H   SFRSYM    DATA     WORD      PI_UKMIN
      000000C2H   SFRSYM    DATA     WORD      MD_MA
      000000A3H   SFRSYM    DATA     BYTE      TIM3_CNTRH
      000000B0H.5 SFRSYM    DATA     BIT       GP35
      000000A0H.6 SFRSYM    DATA     BIT       GP26
      00000090H.7 SFRSYM    DATA     BIT       GP17
      00000080H   SFRSYM    DATA     BYTE      P0
      00000088H.4 SFRSYM    DATA     BIT       IT11
      000000CAH   SFRSYM    DATA     WORD      MD_MB
      00000093H   SFRSYM    DATA     BYTE      TIM4_CNTRH
      000000B0H.6 SFRSYM    DATA     BIT       GP36
      000000A0H.7 SFRSYM    DATA     BIT       GP27
      00000090H   SFRSYM    DATA     BYTE      P1
      000000D9H   SFRSYM    DATA     BYTE      EVT_FILT
      000000F4H   SFRSYM    DATA     WORD      PI_UKMAX
      0000008BH   SFRSYM    DATA     BYTE      TIM5_CNTRH
      000000B2H   SFRSYM    DATA     BYTE      TIM2_CMTRL
LX51 LINKER/LOCATER V4.66.1.0                                                         03/23/2017  15:15:44  PAGE 119


      000000B0H.7 SFRSYM    DATA     BIT       GP37
      000000A0H   SFRSYM    DATA     BYTE      P2
      000000AAH   SFRSYM    DATA     BYTE      TIM2_CNTRL
      000000B0H   SFRSYM    DATA     BYTE      P3
      000000A2H   SFRSYM    DATA     BYTE      TIM3_CNTRL
      000000D0H.6 SFRSYM    DATA     BIT       AC
      00000092H   SFRSYM    DATA     BYTE      TIM4_CNTRL
      0000008AH   SFRSYM    DATA     BYTE      TIM5_CNTRL
      000000B6H   SFRSYM    DATA     WORD      TIM0_CCR1
      000000A8H.7 SFRSYM    DATA     BIT       EA
      000000D5H   SFRSYM    DATA     BYTE      CMP_CR0
      000000BAH   SFRSYM    DATA     WORD      TIM0_CCR2
      000000D6H   SFRSYM    DATA     BYTE      CMP_CR1
      000000BCH   SFRSYM    DATA     WORD      TIM0_CCR3
      00000085H   SFRSYM    DATA     BYTE      PSCTL
      000000DAH   SFRSYM    DATA     BYTE      CMP_CR2
      000000BEH   SFRSYM    DATA     WORD      TIM0_CCR4
      000000B8H.2 SFRSYM    DATA     BIT       PX00
      000000EAH   SFRSYM    DATA     WORD      PI_EK
      000000F8H   SFRSYM    DATA     BIT       OISUH
      000000B8H.3 SFRSYM    DATA     BIT       PX01
      000000B8H.4 SFRSYM    DATA     BIT       PX10
      000000F8H.2 SFRSYM    DATA     BIT       OISVH
      000000B8H.5 SFRSYM    DATA     BIT       PX11
      000000F8H.4 SFRSYM    DATA     BIT       OISWH
      000000DCH   SFRSYM    DATA     WORD      LPF_K
      000000F2H   SFRSYM    DATA     WORD      PI_KI
      000000F8H.1 SFRSYM    DATA     BIT       OISUL
      000000A8H   SFRSYM    DATA     BYTE      IE
      000000F8H.3 SFRSYM    DATA     BIT       OISVL
      000000F8H.5 SFRSYM    DATA     BIT       OISWL
      000000D1H   SFRSYM    DATA     BYTE      P1IE
      00000098H.6 SFRSYM    DATA     BIT       MOD0
      000000D3H   SFRSYM    DATA     BYTE      P2IE
      000000D2H   SFRSYM    DATA     BYTE      P1IF
      000000F9H   SFRSYM    DATA     BYTE      PL_CR
      00000098H.7 SFRSYM    DATA     BIT       MOD1
      000000D4H   SFRSYM    DATA     BYTE      P2IF
      000000ACH   SFRSYM    DATA     WORD      TIM2_DR
      00000082H   SFRSYM    DATA     WORD      DP
      000000EEH   SFRSYM    DATA     WORD      PI_KP
      000000A4H   SFRSYM    DATA     WORD      TIM3_DR
      00000094H   SFRSYM    DATA     WORD      TIM4_DR
      0000008CH   SFRSYM    DATA     WORD      TIM5_DR
      000000F1H   SFRSYM    DATA     BYTE      OSC_CFG
      000000C1H   SFRSYM    DATA     BYTE      MD_MODE
      000000ECH   SFRSYM    DATA     WORD      PI_UK
      000000DEH   SFRSYM    DATA     WORD      LPF_X
      00000098H   SFRSYM    DATA     BIT       RI
      000000E6H   SFRSYM    DATA     WORD      LPF_Y
      000000C0H   SFRSYM    DATA     BIT       PTIM00
      000000D0H.7 SFRSYM    DATA     BIT       CY
      00000098H.1 SFRSYM    DATA     BIT       TI
      000000C0H.1 SFRSYM    DATA     BIT       PTIM01
      000000C0H.2 SFRSYM    DATA     BIT       PTIM10
      000000C0H.3 SFRSYM    DATA     BIT       PTIM11
      000000E1H   SFRSYM    DATA     BYTE      SV_CR
      00000098H   SFRSYM    DATA     BYTE      UT_CR
      00000099H   SFRSYM    DATA     BYTE      UT_DR
      000000F8H.6 SFRSYM    DATA     BIT       OIS4
      00000081H   SFRSYM    DATA     BYTE      SP
      000000D0H.2 SFRSYM    DATA     BIT       OV
      000000C4H   SFRSYM    DATA     BYTE      MD_DA0
      0000009AH   SFRSYM    DATA     WORD      UT_BAUD
      000000CCH   SFRSYM    DATA     BYTE      MD_DB0
LX51 LINKER/LOCATER V4.66.1.0                                                         03/23/2017  15:15:44  PAGE 120


      000000C5H   SFRSYM    DATA     BYTE      MD_DA1
      000000CDH   SFRSYM    DATA     BYTE      MD_DB1
      000000C6H   SFRSYM    DATA     BYTE      MD_DA2
      000000CEH   SFRSYM    DATA     BYTE      MD_DB2
      000000C7H   SFRSYM    DATA     BYTE      MD_DA3
      000000B4H   SFRSYM    DATA     WORD      TIM2_ADTR
      000000CFH   SFRSYM    DATA     BYTE      MD_DB3
      000000AFH   SFRSYM    DATA     BYTE      TIM2_ARRH
      000000A7H   SFRSYM    DATA     BYTE      TIM3_ARRH
      00000097H   SFRSYM    DATA     BYTE      TIM4_ARRH
      0000008FH   SFRSYM    DATA     BYTE      TIM5_ARRH
      000000AEH   SFRSYM    DATA     BYTE      TIM2_ARRL
      000000A6H   SFRSYM    DATA     BYTE      TIM3_ARRL
      00000087H   SFRSYM    DATA     BYTE      PCON
      000000E2H   SFRSYM    DATA     WORD      SV_US
      00000096H   SFRSYM    DATA     BYTE      TIM4_ARRL
      0000008EH   SFRSYM    DATA     BYTE      TIM5_ARRL
      000000B2H   SFRSYM    DATA     WORD      TIM2_CMTR
      00000088H   SFRSYM    DATA     BYTE      TCON
      000000AAH   SFRSYM    DATA     WORD      TIM2_CNTR
      000000A2H   SFRSYM    DATA     WORD      TIM3_CNTR
      00000092H   SFRSYM    DATA     WORD      TIM4_CNTR
      0000008AH   SFRSYM    DATA     WORD      TIM5_CNTR
      000000E5H   SFRSYM    DATA     BYTE      SV_ANGLEH
      000000D8H   SFRSYM    DATA     BIT       PUART0
      000000E4H   SFRSYM    DATA     BYTE      SV_ANGLEL
      000000C6H   SFRSYM    DATA     WORD      MD_DAH
      000000D8H.1 SFRSYM    DATA     BIT       PUART1
      000000D8H.2 SFRSYM    DATA     BIT       PI2C0
      00000088H.2 SFRSYM    DATA     BIT       IF0
      000000CEH   SFRSYM    DATA     WORD      MD_DBH
      000000D8H.3 SFRSYM    DATA     BIT       PI2C1
      000000F0H   SFRSYM    DATA     BYTE      B
      000000C4H   SFRSYM    DATA     WORD      MD_DAL
      000000A1H   SFRSYM    DATA     BYTE      TIM2_CR0
      000000CCH   SFRSYM    DATA     WORD      MD_DBL
      0000009CH   SFRSYM    DATA     BYTE      TIM3_CR0
      000000A9H   SFRSYM    DATA     BYTE      TIM2_CR1
      0000009EH   SFRSYM    DATA     BYTE      TIM4_CR0
      0000009DH   SFRSYM    DATA     BYTE      TIM3_CR1
      00000089H   SFRSYM    DATA     BYTE      TIM5_CR0
      0000009FH   SFRSYM    DATA     BYTE      TIM4_CR1
      000000F8H   SFRSYM    DATA     BYTE      DRV_OUT
      00000091H   SFRSYM    DATA     BYTE      TIM5_CR1
      000000E0H   SFRSYM    DATA     BYTE      ACC
      000000F7H   SFRSYM    DATA     BYTE      PI_UKMINH
      000000C3H   SFRSYM    DATA     BYTE      MD_MAH
      000000A8H.4 SFRSYM    DATA     BIT       ES0
      000000DBH   SFRSYM    DATA     BYTE      LVSR
      000000CBH   SFRSYM    DATA     BYTE      MD_MBH
      000000C0H.4 SFRSYM    DATA     BIT       PADC0
      000000B8H   SFRSYM    DATA     BYTE      IP0
      000000F5H   SFRSYM    DATA     BYTE      PI_UKMAXH
      000000C0H.5 SFRSYM    DATA     BIT       PADC1
      000000C0H   SFRSYM    DATA     BYTE      IP1
      000000C8H   SFRSYM    DATA     BYTE      IP2
      000000F6H   SFRSYM    DATA     BYTE      PI_UKMINL
      000000C2H   SFRSYM    DATA     BYTE      MD_MAL
      00000098H.2 SFRSYM    DATA     BIT       RB8
      000000D8H   SFRSYM    DATA     BYTE      IP3
      000000CAH   SFRSYM    DATA     BYTE      MD_MBL
      000000A8H   SFRSYM    DATA     BIT       EX0
      000000F4H   SFRSYM    DATA     BYTE      PI_UKMAXL
      00000098H.3 SFRSYM    DATA     BIT       TB8
      000000B7H   SFRSYM    DATA     BYTE      TIM0_CCR1H
LX51 LINKER/LOCATER V4.66.1.0                                                         03/23/2017  15:15:44  PAGE 121


      000000A8H.2 SFRSYM    DATA     BIT       EX1
      000000BBH   SFRSYM    DATA     BYTE      TIM0_CCR2H
      000000D0H   SFRSYM    DATA     BIT       P
      000000BDH   SFRSYM    DATA     BYTE      TIM0_CCR3H
      000000BFH   SFRSYM    DATA     BYTE      TIM0_CCR4H
      000000C8H.2 SFRSYM    DATA     BIT       PTIM230
      000000EBH   SFRSYM    DATA     BYTE      PI_EKH
      00000098H.5 SFRSYM    DATA     BIT       SM2
      000000B6H   SFRSYM    DATA     BYTE      TIM0_CCR1L
      000000B1H   SFRSYM    DATA     BYTE      TIM0_SR1
      000000C8H.3 SFRSYM    DATA     BIT       PTIM231
      000000BAH   SFRSYM    DATA     BYTE      TIM0_CCR2L
      000000BCH   SFRSYM    DATA     BYTE      TIM0_CCR3L
      000000BEH   SFRSYM    DATA     BYTE      TIM0_CCR4L
      000000D8H.6 SFRSYM    DATA     BIT       PMCD0
      000000C8H.4 SFRSYM    DATA     BIT       PTIM450
      000000D0H.3 SFRSYM    DATA     BIT       RS0
      000000DDH   SFRSYM    DATA     BYTE      LPF_KH
      000000F3H   SFRSYM    DATA     BYTE      PI_KIH
      000000EAH   SFRSYM    DATA     BYTE      PI_EKL
      000000E8H   SFRSYM    DATA     BYTE      FOC_SET0
      000000D8H.7 SFRSYM    DATA     BIT       PMCD1
      000000C8H.5 SFRSYM    DATA     BIT       PTIM451
      000000D0H.4 SFRSYM    DATA     BIT       RS1
      000000E9H   SFRSYM    DATA     BYTE      FOC_SET1
      000000B8H.6 SFRSYM    DATA     BIT       PFOC0
      000000DCH   SFRSYM    DATA     BYTE      LPF_KL
      000000F2H   SFRSYM    DATA     BYTE      PI_KIL
      000000B8H.7 SFRSYM    DATA     BIT       PFOC1
      000000ADH   SFRSYM    DATA     BYTE      TIM2_DRH
      000000B9H   SFRSYM    DATA     BYTE      TIM0_IER
      00000083H   SFRSYM    DATA     BYTE      DPH
      000000EFH   SFRSYM    DATA     BYTE      PI_KPH
      000000A5H   SFRSYM    DATA     BYTE      TIM3_DRH
      00000095H   SFRSYM    DATA     BYTE      TIM4_DRH
      0000008DH   SFRSYM    DATA     BYTE      TIM5_DRH
      000000ACH   SFRSYM    DATA     BYTE      TIM2_DRL
      00000082H   SFRSYM    DATA     BYTE      DPL
      000000EEH   SFRSYM    DATA     BYTE      PI_KPL
      000000A4H   SFRSYM    DATA     BYTE      TIM3_DRL
      000000F8H.7 SFRSYM    DATA     BIT       MOE
      000000C0H.6 SFRSYM    DATA     BIT       PCMP0
      000000EDH   SFRSYM    DATA     BYTE      PI_UKH
      00000094H   SFRSYM    DATA     BYTE      TIM4_DRL
      000000C0H.7 SFRSYM    DATA     BIT       PCMP1
      000000DFH   SFRSYM    DATA     BYTE      LPF_XH
      0000008CH   SFRSYM    DATA     BYTE      TIM5_DRL
      000000AEH   SFRSYM    DATA     WORD      TIM2_ARR
      000000A8H.5 SFRSYM    DATA     BIT       MCDIE
      000000C9H   SFRSYM    DATA     BYTE      RSTSRC
      000000E7H   SFRSYM    DATA     BYTE      LPF_YH
      000000A6H   SFRSYM    DATA     WORD      TIM3_ARR
      00000088H.6 SFRSYM    DATA     BIT       MCDIF
      00000098H.4 SFRSYM    DATA     BIT       REN
      00000096H   SFRSYM    DATA     WORD      TIM4_ARR
      000000ECH   SFRSYM    DATA     BYTE      PI_UKL
      000000D7H   SFRSYM    DATA     BYTE      CMP_SR
      0000008EH   SFRSYM    DATA     WORD      TIM5_ARR
      000000DEH   SFRSYM    DATA     BYTE      LPF_XL
      000000E6H   SFRSYM    DATA     BYTE      LPF_YL
      000000C8H   SFRSYM    DATA     BIT       PRTC0
      000000C8H.1 SFRSYM    DATA     BIT       PRTC1
      000000E8H.7 SFRSYM    DATA     BIT       FOCEN
      000000C8H.6 SFRSYM    DATA     BIT       PTSD0
      000000D8H.4 SFRSYM    DATA     BIT       PSPI0
LX51 LINKER/LOCATER V4.66.1.0                                                         03/23/2017  15:15:44  PAGE 122


      000000C8H.7 SFRSYM    DATA     BIT       PTSD1
      000000D8H.5 SFRSYM    DATA     BIT       PSPI1
      0000009BH   SFRSYM    DATA     BYTE      UT_BAUDH
      000000E4H   SFRSYM    DATA     WORD      SV_ANGLE
      000000B5H   SFRSYM    DATA     BYTE      TIM2_ADTRH
      0000009AH   SFRSYM    DATA     BYTE      UT_BAUDL
      000000FCH   SFRSYM    DATA     BYTE      P0_OE
      000000FDH   SFRSYM    DATA     BYTE      P1_OE
      000000D0H.5 SFRSYM    DATA     BIT       F0
      000000B4H   SFRSYM    DATA     BYTE      TIM2_ADTRL
      000000FEH   SFRSYM    DATA     BYTE      P2_OE
      000000D0H.1 SFRSYM    DATA     BIT       F1
      00000080H   SFRSYM    DATA     BIT       GP00
      000000FFH   SFRSYM    DATA     BYTE      P3_OE
      00000090H   SFRSYM    DATA     BIT       GP10
      00000080H.1 SFRSYM    DATA     BIT       GP01
      000000A8H.6 SFRSYM    DATA     BIT       RTCIE
      000000A0H   SFRSYM    DATA     BIT       GP20
      00000090H.1 SFRSYM    DATA     BIT       GP11
      00000080H.2 SFRSYM    DATA     BIT       GP02
      000000E3H   SFRSYM    DATA     BYTE      SV_USH
      000000B0H   SFRSYM    DATA     BIT       GP30
      000000A0H.1 SFRSYM    DATA     BIT       GP21
      00000090H.2 SFRSYM    DATA     BIT       GP12
      00000080H.3 SFRSYM    DATA     BIT       GP03
      000000B8H   SFRSYM    DATA     BIT       PLVW0
      000000A8H.1 SFRSYM    DATA     BIT       TSDIE
      000000D0H   SFRSYM    DATA     BYTE      PSW
      000000B0H.1 SFRSYM    DATA     BIT       GP31
      000000A0H.2 SFRSYM    DATA     BIT       GP22
      00000090H.3 SFRSYM    DATA     BIT       GP13
      00000080H.4 SFRSYM    DATA     BIT       GP04
      000000B8H.1 SFRSYM    DATA     BIT       PLVW1
      000000A8H.3 SFRSYM    DATA     BIT       SPIIE
      00000088H.5 SFRSYM    DATA     BIT       TSDIF
      000000B0H.2 SFRSYM    DATA     BIT       GP32
      000000A0H.3 SFRSYM    DATA     BIT       GP23
      00000090H.4 SFRSYM    DATA     BIT       GP14
      00000080H.5 SFRSYM    DATA     BIT       GP05
      00000084H   SFRSYM    DATA     BYTE      FLKEY
      000000B3H   SFRSYM    DATA     BYTE      TIM2_CMTRH
      000000B0H.3 SFRSYM    DATA     BIT       GP33
      000000A0H.4 SFRSYM    DATA     BIT       GP24
      00000090H.5 SFRSYM    DATA     BIT       GP15
      00000080H.6 SFRSYM    DATA     BIT       GP06
      00000088H   SFRSYM    DATA     BIT       IT00

      01001B8AH   BLOCK     CODE     ---       LVL=0
      01001B8AH   LINE      CODE     ---       #23
      01001B8AH   LINE      CODE     ---       #24
      01001B8AH   LINE      CODE     ---       #39
      01001B91H   LINE      CODE     ---       #40
      01001B95H   LINE      CODE     ---       #41
      01001B98H   LINE      CODE     ---       #48
      01001B9BH   LINE      CODE     ---       #49
      01001B9EH   LINE      CODE     ---       #50
      01001BA1H   LINE      CODE     ---       #51
      01001BA4H   LINE      CODE     ---       #52
      01001BA7H   LINE      CODE     ---       #53
      01001BAAH   LINE      CODE     ---       #56
      01001BADH   LINE      CODE     ---       #59
      01001BB0H   LINE      CODE     ---       #60
      01001BB3H   LINE      CODE     ---       #68
      01001BB6H   LINE      CODE     ---       #69
      01001BB9H   LINE      CODE     ---       #70
LX51 LINKER/LOCATER V4.66.1.0                                                         03/23/2017  15:15:44  PAGE 123


      01001BBCH   LINE      CODE     ---       #98
      ---         BLOCKEND  ---      ---       LVL=0

      ---         MODULE    ---      ---       AMPINIT
      01001E37H   PUBLIC    CODE     ---       AMPIint
      000000E2H   SFRSYM    DATA     BYTE      SV_USL
      000000ABH   SFRSYM    DATA     BYTE      TIM2_CNTRH
      000000B0H.4 SFRSYM    DATA     BIT       GP34
      000000A0H.5 SFRSYM    DATA     BIT       GP25
      00000090H.6 SFRSYM    DATA     BIT       GP16
      00000080H.7 SFRSYM    DATA     BIT       GP07
      00000088H.1 SFRSYM    DATA     BIT       IT01
      00000088H.3 SFRSYM    DATA     BIT       IT10
      000000F6H   SFRSYM    DATA     WORD      PI_UKMIN
      000000C2H   SFRSYM    DATA     WORD      MD_MA
      000000A3H   SFRSYM    DATA     BYTE      TIM3_CNTRH
      000000B0H.5 SFRSYM    DATA     BIT       GP35
      000000A0H.6 SFRSYM    DATA     BIT       GP26
      00000090H.7 SFRSYM    DATA     BIT       GP17
      00000080H   SFRSYM    DATA     BYTE      P0
      00000088H.4 SFRSYM    DATA     BIT       IT11
      000000CAH   SFRSYM    DATA     WORD      MD_MB
      00000093H   SFRSYM    DATA     BYTE      TIM4_CNTRH
      000000B0H.6 SFRSYM    DATA     BIT       GP36
      000000A0H.7 SFRSYM    DATA     BIT       GP27
      00000090H   SFRSYM    DATA     BYTE      P1
      000000D9H   SFRSYM    DATA     BYTE      EVT_FILT
      000000F4H   SFRSYM    DATA     WORD      PI_UKMAX
      0000008BH   SFRSYM    DATA     BYTE      TIM5_CNTRH
      000000B2H   SFRSYM    DATA     BYTE      TIM2_CMTRL
      000000B0H.7 SFRSYM    DATA     BIT       GP37
      000000A0H   SFRSYM    DATA     BYTE      P2
      000000AAH   SFRSYM    DATA     BYTE      TIM2_CNTRL
      000000B0H   SFRSYM    DATA     BYTE      P3
      000000A2H   SFRSYM    DATA     BYTE      TIM3_CNTRL
      000000D0H.6 SFRSYM    DATA     BIT       AC
      00000092H   SFRSYM    DATA     BYTE      TIM4_CNTRL
      0000008AH   SFRSYM    DATA     BYTE      TIM5_CNTRL
      000000B6H   SFRSYM    DATA     WORD      TIM0_CCR1
      000000A8H.7 SFRSYM    DATA     BIT       EA
      000000D5H   SFRSYM    DATA     BYTE      CMP_CR0
      000000BAH   SFRSYM    DATA     WORD      TIM0_CCR2
      000000D6H   SFRSYM    DATA     BYTE      CMP_CR1
      000000BCH   SFRSYM    DATA     WORD      TIM0_CCR3
      00000085H   SFRSYM    DATA     BYTE      PSCTL
      000000DAH   SFRSYM    DATA     BYTE      CMP_CR2
      000000BEH   SFRSYM    DATA     WORD      TIM0_CCR4
      000000B8H.2 SFRSYM    DATA     BIT       PX00
      000000EAH   SFRSYM    DATA     WORD      PI_EK
      000000F8H   SFRSYM    DATA     BIT       OISUH
      000000B8H.3 SFRSYM    DATA     BIT       PX01
      000000B8H.4 SFRSYM    DATA     BIT       PX10
      000000F8H.2 SFRSYM    DATA     BIT       OISVH
      000000B8H.5 SFRSYM    DATA     BIT       PX11
      000000F8H.4 SFRSYM    DATA     BIT       OISWH
      000000DCH   SFRSYM    DATA     WORD      LPF_K
      000000F2H   SFRSYM    DATA     WORD      PI_KI
      000000F8H.1 SFRSYM    DATA     BIT       OISUL
      000000A8H   SFRSYM    DATA     BYTE      IE
      000000F8H.3 SFRSYM    DATA     BIT       OISVL
      000000F8H.5 SFRSYM    DATA     BIT       OISWL
      000000D1H   SFRSYM    DATA     BYTE      P1IE
      00000098H.6 SFRSYM    DATA     BIT       MOD0
      000000D3H   SFRSYM    DATA     BYTE      P2IE
      000000D2H   SFRSYM    DATA     BYTE      P1IF
LX51 LINKER/LOCATER V4.66.1.0                                                         03/23/2017  15:15:44  PAGE 124


      000000F9H   SFRSYM    DATA     BYTE      PL_CR
      00000098H.7 SFRSYM    DATA     BIT       MOD1
      000000D4H   SFRSYM    DATA     BYTE      P2IF
      000000ACH   SFRSYM    DATA     WORD      TIM2_DR
      00000082H   SFRSYM    DATA     WORD      DP
      000000EEH   SFRSYM    DATA     WORD      PI_KP
      000000A4H   SFRSYM    DATA     WORD      TIM3_DR
      00000094H   SFRSYM    DATA     WORD      TIM4_DR
      0000008CH   SFRSYM    DATA     WORD      TIM5_DR
      000000F1H   SFRSYM    DATA     BYTE      OSC_CFG
      000000C1H   SFRSYM    DATA     BYTE      MD_MODE
      000000ECH   SFRSYM    DATA     WORD      PI_UK
      000000DEH   SFRSYM    DATA     WORD      LPF_X
      00000098H   SFRSYM    DATA     BIT       RI
      000000E6H   SFRSYM    DATA     WORD      LPF_Y
      000000C0H   SFRSYM    DATA     BIT       PTIM00
      000000D0H.7 SFRSYM    DATA     BIT       CY
      00000098H.1 SFRSYM    DATA     BIT       TI
      000000C0H.1 SFRSYM    DATA     BIT       PTIM01
      000000C0H.2 SFRSYM    DATA     BIT       PTIM10
      000000C0H.3 SFRSYM    DATA     BIT       PTIM11
      000000E1H   SFRSYM    DATA     BYTE      SV_CR
      00000098H   SFRSYM    DATA     BYTE      UT_CR
      00000099H   SFRSYM    DATA     BYTE      UT_DR
      000000F8H.6 SFRSYM    DATA     BIT       OIS4
      00000081H   SFRSYM    DATA     BYTE      SP
      000000D0H.2 SFRSYM    DATA     BIT       OV
      000000C4H   SFRSYM    DATA     BYTE      MD_DA0
      0000009AH   SFRSYM    DATA     WORD      UT_BAUD
      000000CCH   SFRSYM    DATA     BYTE      MD_DB0
      000000C5H   SFRSYM    DATA     BYTE      MD_DA1
      000000CDH   SFRSYM    DATA     BYTE      MD_DB1
      000000C6H   SFRSYM    DATA     BYTE      MD_DA2
      000000CEH   SFRSYM    DATA     BYTE      MD_DB2
      000000C7H   SFRSYM    DATA     BYTE      MD_DA3
      000000B4H   SFRSYM    DATA     WORD      TIM2_ADTR
      000000CFH   SFRSYM    DATA     BYTE      MD_DB3
      000000AFH   SFRSYM    DATA     BYTE      TIM2_ARRH
      000000A7H   SFRSYM    DATA     BYTE      TIM3_ARRH
      00000097H   SFRSYM    DATA     BYTE      TIM4_ARRH
      0000008FH   SFRSYM    DATA     BYTE      TIM5_ARRH
      000000AEH   SFRSYM    DATA     BYTE      TIM2_ARRL
      000000A6H   SFRSYM    DATA     BYTE      TIM3_ARRL
      00000087H   SFRSYM    DATA     BYTE      PCON
      000000E2H   SFRSYM    DATA     WORD      SV_US
      00000096H   SFRSYM    DATA     BYTE      TIM4_ARRL
      0000008EH   SFRSYM    DATA     BYTE      TIM5_ARRL
      000000B2H   SFRSYM    DATA     WORD      TIM2_CMTR
      00000088H   SFRSYM    DATA     BYTE      TCON
      000000AAH   SFRSYM    DATA     WORD      TIM2_CNTR
      000000A2H   SFRSYM    DATA     WORD      TIM3_CNTR
      00000092H   SFRSYM    DATA     WORD      TIM4_CNTR
      0000008AH   SFRSYM    DATA     WORD      TIM5_CNTR
      000000E5H   SFRSYM    DATA     BYTE      SV_ANGLEH
      000000D8H   SFRSYM    DATA     BIT       PUART0
      000000E4H   SFRSYM    DATA     BYTE      SV_ANGLEL
      000000C6H   SFRSYM    DATA     WORD      MD_DAH
      000000D8H.1 SFRSYM    DATA     BIT       PUART1
      000000D8H.2 SFRSYM    DATA     BIT       PI2C0
      00000088H.2 SFRSYM    DATA     BIT       IF0
      000000CEH   SFRSYM    DATA     WORD      MD_DBH
      000000D8H.3 SFRSYM    DATA     BIT       PI2C1
      000000F0H   SFRSYM    DATA     BYTE      B
      000000C4H   SFRSYM    DATA     WORD      MD_DAL
      000000A1H   SFRSYM    DATA     BYTE      TIM2_CR0
LX51 LINKER/LOCATER V4.66.1.0                                                         03/23/2017  15:15:44  PAGE 125


      000000CCH   SFRSYM    DATA     WORD      MD_DBL
      0000009CH   SFRSYM    DATA     BYTE      TIM3_CR0
      000000A9H   SFRSYM    DATA     BYTE      TIM2_CR1
      0000009EH   SFRSYM    DATA     BYTE      TIM4_CR0
      0000009DH   SFRSYM    DATA     BYTE      TIM3_CR1
      00000089H   SFRSYM    DATA     BYTE      TIM5_CR0
      0000009FH   SFRSYM    DATA     BYTE      TIM4_CR1
      000000F8H   SFRSYM    DATA     BYTE      DRV_OUT
      00000091H   SFRSYM    DATA     BYTE      TIM5_CR1
      000000E0H   SFRSYM    DATA     BYTE      ACC
      000000F7H   SFRSYM    DATA     BYTE      PI_UKMINH
      000000C3H   SFRSYM    DATA     BYTE      MD_MAH
      000000A8H.4 SFRSYM    DATA     BIT       ES0
      000000DBH   SFRSYM    DATA     BYTE      LVSR
      000000CBH   SFRSYM    DATA     BYTE      MD_MBH
      000000C0H.4 SFRSYM    DATA     BIT       PADC0
      000000B8H   SFRSYM    DATA     BYTE      IP0
      000000F5H   SFRSYM    DATA     BYTE      PI_UKMAXH
      000000C0H.5 SFRSYM    DATA     BIT       PADC1
      000000C0H   SFRSYM    DATA     BYTE      IP1
      000000C8H   SFRSYM    DATA     BYTE      IP2
      000000F6H   SFRSYM    DATA     BYTE      PI_UKMINL
      000000C2H   SFRSYM    DATA     BYTE      MD_MAL
      00000098H.2 SFRSYM    DATA     BIT       RB8
      000000D8H   SFRSYM    DATA     BYTE      IP3
      000000CAH   SFRSYM    DATA     BYTE      MD_MBL
      000000A8H   SFRSYM    DATA     BIT       EX0
      000000F4H   SFRSYM    DATA     BYTE      PI_UKMAXL
      00000098H.3 SFRSYM    DATA     BIT       TB8
      000000B7H   SFRSYM    DATA     BYTE      TIM0_CCR1H
      000000A8H.2 SFRSYM    DATA     BIT       EX1
      000000BBH   SFRSYM    DATA     BYTE      TIM0_CCR2H
      000000D0H   SFRSYM    DATA     BIT       P
      000000BDH   SFRSYM    DATA     BYTE      TIM0_CCR3H
      000000BFH   SFRSYM    DATA     BYTE      TIM0_CCR4H
      000000C8H.2 SFRSYM    DATA     BIT       PTIM230
      000000EBH   SFRSYM    DATA     BYTE      PI_EKH
      00000098H.5 SFRSYM    DATA     BIT       SM2
      000000B6H   SFRSYM    DATA     BYTE      TIM0_CCR1L
      000000B1H   SFRSYM    DATA     BYTE      TIM0_SR1
      000000C8H.3 SFRSYM    DATA     BIT       PTIM231
      000000BAH   SFRSYM    DATA     BYTE      TIM0_CCR2L
      000000BCH   SFRSYM    DATA     BYTE      TIM0_CCR3L
      000000BEH   SFRSYM    DATA     BYTE      TIM0_CCR4L
      000000D8H.6 SFRSYM    DATA     BIT       PMCD0
      000000C8H.4 SFRSYM    DATA     BIT       PTIM450
      000000D0H.3 SFRSYM    DATA     BIT       RS0
      000000DDH   SFRSYM    DATA     BYTE      LPF_KH
      000000F3H   SFRSYM    DATA     BYTE      PI_KIH
      000000EAH   SFRSYM    DATA     BYTE      PI_EKL
      000000E8H   SFRSYM    DATA     BYTE      FOC_SET0
      000000D8H.7 SFRSYM    DATA     BIT       PMCD1
      000000C8H.5 SFRSYM    DATA     BIT       PTIM451
      000000D0H.4 SFRSYM    DATA     BIT       RS1
      000000E9H   SFRSYM    DATA     BYTE      FOC_SET1
      000000B8H.6 SFRSYM    DATA     BIT       PFOC0
      000000DCH   SFRSYM    DATA     BYTE      LPF_KL
      000000F2H   SFRSYM    DATA     BYTE      PI_KIL
      000000B8H.7 SFRSYM    DATA     BIT       PFOC1
      000000ADH   SFRSYM    DATA     BYTE      TIM2_DRH
      000000B9H   SFRSYM    DATA     BYTE      TIM0_IER
      00000083H   SFRSYM    DATA     BYTE      DPH
      000000EFH   SFRSYM    DATA     BYTE      PI_KPH
      000000A5H   SFRSYM    DATA     BYTE      TIM3_DRH
      00000095H   SFRSYM    DATA     BYTE      TIM4_DRH
LX51 LINKER/LOCATER V4.66.1.0                                                         03/23/2017  15:15:44  PAGE 126


      0000008DH   SFRSYM    DATA     BYTE      TIM5_DRH
      000000ACH   SFRSYM    DATA     BYTE      TIM2_DRL
      00000082H   SFRSYM    DATA     BYTE      DPL
      000000EEH   SFRSYM    DATA     BYTE      PI_KPL
      000000A4H   SFRSYM    DATA     BYTE      TIM3_DRL
      000000F8H.7 SFRSYM    DATA     BIT       MOE
      000000C0H.6 SFRSYM    DATA     BIT       PCMP0
      000000EDH   SFRSYM    DATA     BYTE      PI_UKH
      00000094H   SFRSYM    DATA     BYTE      TIM4_DRL
      000000C0H.7 SFRSYM    DATA     BIT       PCMP1
      000000DFH   SFRSYM    DATA     BYTE      LPF_XH
      0000008CH   SFRSYM    DATA     BYTE      TIM5_DRL
      000000AEH   SFRSYM    DATA     WORD      TIM2_ARR
      000000A8H.5 SFRSYM    DATA     BIT       MCDIE
      000000C9H   SFRSYM    DATA     BYTE      RSTSRC
      000000E7H   SFRSYM    DATA     BYTE      LPF_YH
      000000A6H   SFRSYM    DATA     WORD      TIM3_ARR
      00000088H.6 SFRSYM    DATA     BIT       MCDIF
      00000098H.4 SFRSYM    DATA     BIT       REN
      00000096H   SFRSYM    DATA     WORD      TIM4_ARR
      000000ECH   SFRSYM    DATA     BYTE      PI_UKL
      000000D7H   SFRSYM    DATA     BYTE      CMP_SR
      0000008EH   SFRSYM    DATA     WORD      TIM5_ARR
      000000DEH   SFRSYM    DATA     BYTE      LPF_XL
      000000E6H   SFRSYM    DATA     BYTE      LPF_YL
      000000C8H   SFRSYM    DATA     BIT       PRTC0
      000000C8H.1 SFRSYM    DATA     BIT       PRTC1
      000000E8H.7 SFRSYM    DATA     BIT       FOCEN
      000000C8H.6 SFRSYM    DATA     BIT       PTSD0
      000000D8H.4 SFRSYM    DATA     BIT       PSPI0
      000000C8H.7 SFRSYM    DATA     BIT       PTSD1
      000000D8H.5 SFRSYM    DATA     BIT       PSPI1
      0000009BH   SFRSYM    DATA     BYTE      UT_BAUDH
      000000E4H   SFRSYM    DATA     WORD      SV_ANGLE
      000000B5H   SFRSYM    DATA     BYTE      TIM2_ADTRH
      0000009AH   SFRSYM    DATA     BYTE      UT_BAUDL
      000000FCH   SFRSYM    DATA     BYTE      P0_OE
      000000FDH   SFRSYM    DATA     BYTE      P1_OE
      000000D0H.5 SFRSYM    DATA     BIT       F0
      000000B4H   SFRSYM    DATA     BYTE      TIM2_ADTRL
      000000FEH   SFRSYM    DATA     BYTE      P2_OE
      000000D0H.1 SFRSYM    DATA     BIT       F1
      00000080H   SFRSYM    DATA     BIT       GP00
      000000FFH   SFRSYM    DATA     BYTE      P3_OE
      00000090H   SFRSYM    DATA     BIT       GP10
      00000080H.1 SFRSYM    DATA     BIT       GP01
      000000A8H.6 SFRSYM    DATA     BIT       RTCIE
      000000A0H   SFRSYM    DATA     BIT       GP20
      00000090H.1 SFRSYM    DATA     BIT       GP11
      00000080H.2 SFRSYM    DATA     BIT       GP02
      000000E3H   SFRSYM    DATA     BYTE      SV_USH
      000000B0H   SFRSYM    DATA     BIT       GP30
      000000A0H.1 SFRSYM    DATA     BIT       GP21
      00000090H.2 SFRSYM    DATA     BIT       GP12
      00000080H.3 SFRSYM    DATA     BIT       GP03
      000000B8H   SFRSYM    DATA     BIT       PLVW0
      000000A8H.1 SFRSYM    DATA     BIT       TSDIE
      000000D0H   SFRSYM    DATA     BYTE      PSW
      000000B0H.1 SFRSYM    DATA     BIT       GP31
      000000A0H.2 SFRSYM    DATA     BIT       GP22
      00000090H.3 SFRSYM    DATA     BIT       GP13
      00000080H.4 SFRSYM    DATA     BIT       GP04
      000000B8H.1 SFRSYM    DATA     BIT       PLVW1
      000000A8H.3 SFRSYM    DATA     BIT       SPIIE
      00000088H.5 SFRSYM    DATA     BIT       TSDIF
LX51 LINKER/LOCATER V4.66.1.0                                                         03/23/2017  15:15:44  PAGE 127


      000000B0H.2 SFRSYM    DATA     BIT       GP32
      000000A0H.3 SFRSYM    DATA     BIT       GP23
      00000090H.4 SFRSYM    DATA     BIT       GP14
      00000080H.5 SFRSYM    DATA     BIT       GP05
      00000084H   SFRSYM    DATA     BYTE      FLKEY
      000000B3H   SFRSYM    DATA     BYTE      TIM2_CMTRH
      000000B0H.3 SFRSYM    DATA     BIT       GP33
      000000A0H.4 SFRSYM    DATA     BIT       GP24
      00000090H.5 SFRSYM    DATA     BIT       GP15
      00000080H.6 SFRSYM    DATA     BIT       GP06
      00000088H   SFRSYM    DATA     BIT       IT00

      01001E37H   BLOCK     CODE     ---       LVL=0
      01001E37H   LINE      CODE     ---       #23
      01001E37H   LINE      CODE     ---       #24
      01001E37H   LINE      CODE     ---       #26
      01001E3EH   LINE      CODE     ---       #27
      01001E43H   LINE      CODE     ---       #28
      01001E47H   LINE      CODE     ---       #39
      01001E4EH   LINE      CODE     ---       #45
      ---         BLOCKEND  ---      ---       LVL=0

      ---         MODULE    ---      ---       DRIVERINIT
      01001DB5H   PUBLIC    CODE     ---       DriverInit
      000000E2H   SFRSYM    DATA     BYTE      SV_USL
      000000ABH   SFRSYM    DATA     BYTE      TIM2_CNTRH
      000000B0H.4 SFRSYM    DATA     BIT       GP34
      000000A0H.5 SFRSYM    DATA     BIT       GP25
      00000090H.6 SFRSYM    DATA     BIT       GP16
      00000080H.7 SFRSYM    DATA     BIT       GP07
      00000088H.1 SFRSYM    DATA     BIT       IT01
      00000088H.3 SFRSYM    DATA     BIT       IT10
      000000F6H   SFRSYM    DATA     WORD      PI_UKMIN
      000000C2H   SFRSYM    DATA     WORD      MD_MA
      000000A3H   SFRSYM    DATA     BYTE      TIM3_CNTRH
      000000B0H.5 SFRSYM    DATA     BIT       GP35
      000000A0H.6 SFRSYM    DATA     BIT       GP26
      00000090H.7 SFRSYM    DATA     BIT       GP17
      00000080H   SFRSYM    DATA     BYTE      P0
      00000088H.4 SFRSYM    DATA     BIT       IT11
      000000CAH   SFRSYM    DATA     WORD      MD_MB
      00000093H   SFRSYM    DATA     BYTE      TIM4_CNTRH
      000000B0H.6 SFRSYM    DATA     BIT       GP36
      000000A0H.7 SFRSYM    DATA     BIT       GP27
      00000090H   SFRSYM    DATA     BYTE      P1
      000000D9H   SFRSYM    DATA     BYTE      EVT_FILT
      000000F4H   SFRSYM    DATA     WORD      PI_UKMAX
      0000008BH   SFRSYM    DATA     BYTE      TIM5_CNTRH
      000000B2H   SFRSYM    DATA     BYTE      TIM2_CMTRL
      000000B0H.7 SFRSYM    DATA     BIT       GP37
      000000A0H   SFRSYM    DATA     BYTE      P2
      000000AAH   SFRSYM    DATA     BYTE      TIM2_CNTRL
      000000B0H   SFRSYM    DATA     BYTE      P3
      000000A2H   SFRSYM    DATA     BYTE      TIM3_CNTRL
      000000D0H.6 SFRSYM    DATA     BIT       AC
      00000092H   SFRSYM    DATA     BYTE      TIM4_CNTRL
      0000008AH   SFRSYM    DATA     BYTE      TIM5_CNTRL
      000000B6H   SFRSYM    DATA     WORD      TIM0_CCR1
      000000A8H.7 SFRSYM    DATA     BIT       EA
      000000D5H   SFRSYM    DATA     BYTE      CMP_CR0
      000000BAH   SFRSYM    DATA     WORD      TIM0_CCR2
      000000D6H   SFRSYM    DATA     BYTE      CMP_CR1
      000000BCH   SFRSYM    DATA     WORD      TIM0_CCR3
      00000085H   SFRSYM    DATA     BYTE      PSCTL
      000000DAH   SFRSYM    DATA     BYTE      CMP_CR2
LX51 LINKER/LOCATER V4.66.1.0                                                         03/23/2017  15:15:44  PAGE 128


      000000BEH   SFRSYM    DATA     WORD      TIM0_CCR4
      000000B8H.2 SFRSYM    DATA     BIT       PX00
      000000EAH   SFRSYM    DATA     WORD      PI_EK
      000000F8H   SFRSYM    DATA     BIT       OISUH
      000000B8H.3 SFRSYM    DATA     BIT       PX01
      000000B8H.4 SFRSYM    DATA     BIT       PX10
      000000F8H.2 SFRSYM    DATA     BIT       OISVH
      000000B8H.5 SFRSYM    DATA     BIT       PX11
      000000F8H.4 SFRSYM    DATA     BIT       OISWH
      000000DCH   SFRSYM    DATA     WORD      LPF_K
      000000F2H   SFRSYM    DATA     WORD      PI_KI
      000000F8H.1 SFRSYM    DATA     BIT       OISUL
      000000A8H   SFRSYM    DATA     BYTE      IE
      000000F8H.3 SFRSYM    DATA     BIT       OISVL
      000000F8H.5 SFRSYM    DATA     BIT       OISWL
      000000D1H   SFRSYM    DATA     BYTE      P1IE
      00000098H.6 SFRSYM    DATA     BIT       MOD0
      000000D3H   SFRSYM    DATA     BYTE      P2IE
      000000D2H   SFRSYM    DATA     BYTE      P1IF
      000000F9H   SFRSYM    DATA     BYTE      PL_CR
      00000098H.7 SFRSYM    DATA     BIT       MOD1
      000000D4H   SFRSYM    DATA     BYTE      P2IF
      000000ACH   SFRSYM    DATA     WORD      TIM2_DR
      00000082H   SFRSYM    DATA     WORD      DP
      000000EEH   SFRSYM    DATA     WORD      PI_KP
      000000A4H   SFRSYM    DATA     WORD      TIM3_DR
      00000094H   SFRSYM    DATA     WORD      TIM4_DR
      0000008CH   SFRSYM    DATA     WORD      TIM5_DR
      000000F1H   SFRSYM    DATA     BYTE      OSC_CFG
      000000C1H   SFRSYM    DATA     BYTE      MD_MODE
      000000ECH   SFRSYM    DATA     WORD      PI_UK
      000000DEH   SFRSYM    DATA     WORD      LPF_X
      00000098H   SFRSYM    DATA     BIT       RI
      000000E6H   SFRSYM    DATA     WORD      LPF_Y
      000000C0H   SFRSYM    DATA     BIT       PTIM00
      000000D0H.7 SFRSYM    DATA     BIT       CY
      00000098H.1 SFRSYM    DATA     BIT       TI
      000000C0H.1 SFRSYM    DATA     BIT       PTIM01
      000000C0H.2 SFRSYM    DATA     BIT       PTIM10
      000000C0H.3 SFRSYM    DATA     BIT       PTIM11
      000000E1H   SFRSYM    DATA     BYTE      SV_CR
      00000098H   SFRSYM    DATA     BYTE      UT_CR
      00000099H   SFRSYM    DATA     BYTE      UT_DR
      000000F8H.6 SFRSYM    DATA     BIT       OIS4
      00000081H   SFRSYM    DATA     BYTE      SP
      000000D0H.2 SFRSYM    DATA     BIT       OV
      000000C4H   SFRSYM    DATA     BYTE      MD_DA0
      0000009AH   SFRSYM    DATA     WORD      UT_BAUD
      000000CCH   SFRSYM    DATA     BYTE      MD_DB0
      000000C5H   SFRSYM    DATA     BYTE      MD_DA1
      000000CDH   SFRSYM    DATA     BYTE      MD_DB1
      000000C6H   SFRSYM    DATA     BYTE      MD_DA2
      000000CEH   SFRSYM    DATA     BYTE      MD_DB2
      000000C7H   SFRSYM    DATA     BYTE      MD_DA3
      000000B4H   SFRSYM    DATA     WORD      TIM2_ADTR
      000000CFH   SFRSYM    DATA     BYTE      MD_DB3
      000000AFH   SFRSYM    DATA     BYTE      TIM2_ARRH
      000000A7H   SFRSYM    DATA     BYTE      TIM3_ARRH
      00000097H   SFRSYM    DATA     BYTE      TIM4_ARRH
      0000008FH   SFRSYM    DATA     BYTE      TIM5_ARRH
      000000AEH   SFRSYM    DATA     BYTE      TIM2_ARRL
      000000A6H   SFRSYM    DATA     BYTE      TIM3_ARRL
      00000087H   SFRSYM    DATA     BYTE      PCON
      000000E2H   SFRSYM    DATA     WORD      SV_US
      00000096H   SFRSYM    DATA     BYTE      TIM4_ARRL
LX51 LINKER/LOCATER V4.66.1.0                                                         03/23/2017  15:15:44  PAGE 129


      0000008EH   SFRSYM    DATA     BYTE      TIM5_ARRL
      000000B2H   SFRSYM    DATA     WORD      TIM2_CMTR
      00000088H   SFRSYM    DATA     BYTE      TCON
      000000AAH   SFRSYM    DATA     WORD      TIM2_CNTR
      000000A2H   SFRSYM    DATA     WORD      TIM3_CNTR
      00000092H   SFRSYM    DATA     WORD      TIM4_CNTR
      0000008AH   SFRSYM    DATA     WORD      TIM5_CNTR
      000000E5H   SFRSYM    DATA     BYTE      SV_ANGLEH
      000000D8H   SFRSYM    DATA     BIT       PUART0
      000000E4H   SFRSYM    DATA     BYTE      SV_ANGLEL
      000000C6H   SFRSYM    DATA     WORD      MD_DAH
      000000D8H.1 SFRSYM    DATA     BIT       PUART1
      000000D8H.2 SFRSYM    DATA     BIT       PI2C0
      00000088H.2 SFRSYM    DATA     BIT       IF0
      000000CEH   SFRSYM    DATA     WORD      MD_DBH
      000000D8H.3 SFRSYM    DATA     BIT       PI2C1
      000000F0H   SFRSYM    DATA     BYTE      B
      000000C4H   SFRSYM    DATA     WORD      MD_DAL
      000000A1H   SFRSYM    DATA     BYTE      TIM2_CR0
      000000CCH   SFRSYM    DATA     WORD      MD_DBL
      0000009CH   SFRSYM    DATA     BYTE      TIM3_CR0
      000000A9H   SFRSYM    DATA     BYTE      TIM2_CR1
      0000009EH   SFRSYM    DATA     BYTE      TIM4_CR0
      0000009DH   SFRSYM    DATA     BYTE      TIM3_CR1
      00000089H   SFRSYM    DATA     BYTE      TIM5_CR0
      0000009FH   SFRSYM    DATA     BYTE      TIM4_CR1
      000000F8H   SFRSYM    DATA     BYTE      DRV_OUT
      00000091H   SFRSYM    DATA     BYTE      TIM5_CR1
      000000E0H   SFRSYM    DATA     BYTE      ACC
      000000F7H   SFRSYM    DATA     BYTE      PI_UKMINH
      000000C3H   SFRSYM    DATA     BYTE      MD_MAH
      000000A8H.4 SFRSYM    DATA     BIT       ES0
      000000DBH   SFRSYM    DATA     BYTE      LVSR
      000000CBH   SFRSYM    DATA     BYTE      MD_MBH
      000000C0H.4 SFRSYM    DATA     BIT       PADC0
      000000B8H   SFRSYM    DATA     BYTE      IP0
      000000F5H   SFRSYM    DATA     BYTE      PI_UKMAXH
      000000C0H.5 SFRSYM    DATA     BIT       PADC1
      000000C0H   SFRSYM    DATA     BYTE      IP1
      000000C8H   SFRSYM    DATA     BYTE      IP2
      000000F6H   SFRSYM    DATA     BYTE      PI_UKMINL
      000000C2H   SFRSYM    DATA     BYTE      MD_MAL
      00000098H.2 SFRSYM    DATA     BIT       RB8
      000000D8H   SFRSYM    DATA     BYTE      IP3
      000000CAH   SFRSYM    DATA     BYTE      MD_MBL
      000000A8H   SFRSYM    DATA     BIT       EX0
      000000F4H   SFRSYM    DATA     BYTE      PI_UKMAXL
      00000098H.3 SFRSYM    DATA     BIT       TB8
      000000B7H   SFRSYM    DATA     BYTE      TIM0_CCR1H
      000000A8H.2 SFRSYM    DATA     BIT       EX1
      000000BBH   SFRSYM    DATA     BYTE      TIM0_CCR2H
      000000D0H   SFRSYM    DATA     BIT       P
      000000BDH   SFRSYM    DATA     BYTE      TIM0_CCR3H
      000000BFH   SFRSYM    DATA     BYTE      TIM0_CCR4H
      000000C8H.2 SFRSYM    DATA     BIT       PTIM230
      000000EBH   SFRSYM    DATA     BYTE      PI_EKH
      00000098H.5 SFRSYM    DATA     BIT       SM2
      000000B6H   SFRSYM    DATA     BYTE      TIM0_CCR1L
      000000B1H   SFRSYM    DATA     BYTE      TIM0_SR1
      000000C8H.3 SFRSYM    DATA     BIT       PTIM231
      000000BAH   SFRSYM    DATA     BYTE      TIM0_CCR2L
      000000BCH   SFRSYM    DATA     BYTE      TIM0_CCR3L
      000000BEH   SFRSYM    DATA     BYTE      TIM0_CCR4L
      000000D8H.6 SFRSYM    DATA     BIT       PMCD0
      000000C8H.4 SFRSYM    DATA     BIT       PTIM450
LX51 LINKER/LOCATER V4.66.1.0                                                         03/23/2017  15:15:44  PAGE 130


      000000D0H.3 SFRSYM    DATA     BIT       RS0
      000000DDH   SFRSYM    DATA     BYTE      LPF_KH
      000000F3H   SFRSYM    DATA     BYTE      PI_KIH
      000000EAH   SFRSYM    DATA     BYTE      PI_EKL
      000000E8H   SFRSYM    DATA     BYTE      FOC_SET0
      000000D8H.7 SFRSYM    DATA     BIT       PMCD1
      000000C8H.5 SFRSYM    DATA     BIT       PTIM451
      000000D0H.4 SFRSYM    DATA     BIT       RS1
      000000E9H   SFRSYM    DATA     BYTE      FOC_SET1
      000000B8H.6 SFRSYM    DATA     BIT       PFOC0
      000000DCH   SFRSYM    DATA     BYTE      LPF_KL
      000000F2H   SFRSYM    DATA     BYTE      PI_KIL
      000000B8H.7 SFRSYM    DATA     BIT       PFOC1
      000000ADH   SFRSYM    DATA     BYTE      TIM2_DRH
      000000B9H   SFRSYM    DATA     BYTE      TIM0_IER
      00000083H   SFRSYM    DATA     BYTE      DPH
      000000EFH   SFRSYM    DATA     BYTE      PI_KPH
      000000A5H   SFRSYM    DATA     BYTE      TIM3_DRH
      00000095H   SFRSYM    DATA     BYTE      TIM4_DRH
      0000008DH   SFRSYM    DATA     BYTE      TIM5_DRH
      000000ACH   SFRSYM    DATA     BYTE      TIM2_DRL
      00000082H   SFRSYM    DATA     BYTE      DPL
      000000EEH   SFRSYM    DATA     BYTE      PI_KPL
      000000A4H   SFRSYM    DATA     BYTE      TIM3_DRL
      000000F8H.7 SFRSYM    DATA     BIT       MOE
      000000C0H.6 SFRSYM    DATA     BIT       PCMP0
      000000EDH   SFRSYM    DATA     BYTE      PI_UKH
      00000094H   SFRSYM    DATA     BYTE      TIM4_DRL
      000000C0H.7 SFRSYM    DATA     BIT       PCMP1
      000000DFH   SFRSYM    DATA     BYTE      LPF_XH
      0000008CH   SFRSYM    DATA     BYTE      TIM5_DRL
      000000AEH   SFRSYM    DATA     WORD      TIM2_ARR
      000000A8H.5 SFRSYM    DATA     BIT       MCDIE
      000000C9H   SFRSYM    DATA     BYTE      RSTSRC
      000000E7H   SFRSYM    DATA     BYTE      LPF_YH
      000000A6H   SFRSYM    DATA     WORD      TIM3_ARR
      00000088H.6 SFRSYM    DATA     BIT       MCDIF
      00000098H.4 SFRSYM    DATA     BIT       REN
      00000096H   SFRSYM    DATA     WORD      TIM4_ARR
      000000ECH   SFRSYM    DATA     BYTE      PI_UKL
      000000D7H   SFRSYM    DATA     BYTE      CMP_SR
      0000008EH   SFRSYM    DATA     WORD      TIM5_ARR
      000000DEH   SFRSYM    DATA     BYTE      LPF_XL
      000000E6H   SFRSYM    DATA     BYTE      LPF_YL
      000000C8H   SFRSYM    DATA     BIT       PRTC0
      000000C8H.1 SFRSYM    DATA     BIT       PRTC1
      000000E8H.7 SFRSYM    DATA     BIT       FOCEN
      000000C8H.6 SFRSYM    DATA     BIT       PTSD0
      000000D8H.4 SFRSYM    DATA     BIT       PSPI0
      000000C8H.7 SFRSYM    DATA     BIT       PTSD1
      000000D8H.5 SFRSYM    DATA     BIT       PSPI1
      0000009BH   SFRSYM    DATA     BYTE      UT_BAUDH
      000000E4H   SFRSYM    DATA     WORD      SV_ANGLE
      000000B5H   SFRSYM    DATA     BYTE      TIM2_ADTRH
      0000009AH   SFRSYM    DATA     BYTE      UT_BAUDL
      000000FCH   SFRSYM    DATA     BYTE      P0_OE
      000000FDH   SFRSYM    DATA     BYTE      P1_OE
      000000D0H.5 SFRSYM    DATA     BIT       F0
      000000B4H   SFRSYM    DATA     BYTE      TIM2_ADTRL
      000000FEH   SFRSYM    DATA     BYTE      P2_OE
      000000D0H.1 SFRSYM    DATA     BIT       F1
      00000080H   SFRSYM    DATA     BIT       GP00
      000000FFH   SFRSYM    DATA     BYTE      P3_OE
      00000090H   SFRSYM    DATA     BIT       GP10
      00000080H.1 SFRSYM    DATA     BIT       GP01
LX51 LINKER/LOCATER V4.66.1.0                                                         03/23/2017  15:15:44  PAGE 131


      000000A8H.6 SFRSYM    DATA     BIT       RTCIE
      000000A0H   SFRSYM    DATA     BIT       GP20
      00000090H.1 SFRSYM    DATA     BIT       GP11
      00000080H.2 SFRSYM    DATA     BIT       GP02
      000000E3H   SFRSYM    DATA     BYTE      SV_USH
      000000B0H   SFRSYM    DATA     BIT       GP30
      000000A0H.1 SFRSYM    DATA     BIT       GP21
      00000090H.2 SFRSYM    DATA     BIT       GP12
      00000080H.3 SFRSYM    DATA     BIT       GP03
      000000B8H   SFRSYM    DATA     BIT       PLVW0
      000000A8H.1 SFRSYM    DATA     BIT       TSDIE
      000000D0H   SFRSYM    DATA     BYTE      PSW
      000000B0H.1 SFRSYM    DATA     BIT       GP31
      000000A0H.2 SFRSYM    DATA     BIT       GP22
      00000090H.3 SFRSYM    DATA     BIT       GP13
      00000080H.4 SFRSYM    DATA     BIT       GP04
      000000B8H.1 SFRSYM    DATA     BIT       PLVW1
      000000A8H.3 SFRSYM    DATA     BIT       SPIIE
      00000088H.5 SFRSYM    DATA     BIT       TSDIF
      000000B0H.2 SFRSYM    DATA     BIT       GP32
      000000A0H.3 SFRSYM    DATA     BIT       GP23
      00000090H.4 SFRSYM    DATA     BIT       GP14
      00000080H.5 SFRSYM    DATA     BIT       GP05
      00000084H   SFRSYM    DATA     BYTE      FLKEY
      000000B3H   SFRSYM    DATA     BYTE      TIM2_CMTRH
      000000B0H.3 SFRSYM    DATA     BIT       GP33
      000000A0H.4 SFRSYM    DATA     BIT       GP24
      00000090H.5 SFRSYM    DATA     BIT       GP15
      00000080H.6 SFRSYM    DATA     BIT       GP06
      00000088H   SFRSYM    DATA     BIT       IT00

      01001DB5H   BLOCK     CODE     ---       LVL=0
      01001DB5H   BLOCK     CODE     NEAR LAB  LVL=1
      00000006H   SYMBOL    DATA     WORD      PRDRVCnt
      ---         BLOCKEND  ---      ---       LVL=1
      01001DB5H   LINE      CODE     ---       #23
      01001DB5H   LINE      CODE     ---       #24
      01001DB5H   LINE      CODE     ---       #28
      01001DBCH   LINE      CODE     ---       #29
      01001DCAH   LINE      CODE     ---       #31
      01001DD1H   LINE      CODE     ---       #32
      ---         BLOCKEND  ---      ---       LVL=0

      ---         MODULE    ---      ---       SYSTEMINIT
      01001D76H   PUBLIC    CODE     ---       SystemInit
      000000E2H   SFRSYM    DATA     BYTE      SV_USL
      000000ABH   SFRSYM    DATA     BYTE      TIM2_CNTRH
      000000B0H.4 SFRSYM    DATA     BIT       GP34
      000000A0H.5 SFRSYM    DATA     BIT       GP25
      00000090H.6 SFRSYM    DATA     BIT       GP16
      00000080H.7 SFRSYM    DATA     BIT       GP07
      00000088H.1 SFRSYM    DATA     BIT       IT01
      00000088H.3 SFRSYM    DATA     BIT       IT10
      000000F6H   SFRSYM    DATA     WORD      PI_UKMIN
      000000C2H   SFRSYM    DATA     WORD      MD_MA
      000000A3H   SFRSYM    DATA     BYTE      TIM3_CNTRH
      000000B0H.5 SFRSYM    DATA     BIT       GP35
      000000A0H.6 SFRSYM    DATA     BIT       GP26
      00000090H.7 SFRSYM    DATA     BIT       GP17
      00000080H   SFRSYM    DATA     BYTE      P0
      00000088H.4 SFRSYM    DATA     BIT       IT11
      000000CAH   SFRSYM    DATA     WORD      MD_MB
      00000093H   SFRSYM    DATA     BYTE      TIM4_CNTRH
      000000B0H.6 SFRSYM    DATA     BIT       GP36
      000000A0H.7 SFRSYM    DATA     BIT       GP27
LX51 LINKER/LOCATER V4.66.1.0                                                         03/23/2017  15:15:44  PAGE 132


      00000090H   SFRSYM    DATA     BYTE      P1
      000000D9H   SFRSYM    DATA     BYTE      EVT_FILT
      000000F4H   SFRSYM    DATA     WORD      PI_UKMAX
      0000008BH   SFRSYM    DATA     BYTE      TIM5_CNTRH
      000000B2H   SFRSYM    DATA     BYTE      TIM2_CMTRL
      000000B0H.7 SFRSYM    DATA     BIT       GP37
      000000A0H   SFRSYM    DATA     BYTE      P2
      000000AAH   SFRSYM    DATA     BYTE      TIM2_CNTRL
      000000B0H   SFRSYM    DATA     BYTE      P3
      000000A2H   SFRSYM    DATA     BYTE      TIM3_CNTRL
      000000D0H.6 SFRSYM    DATA     BIT       AC
      00000092H   SFRSYM    DATA     BYTE      TIM4_CNTRL
      0000008AH   SFRSYM    DATA     BYTE      TIM5_CNTRL
      000000B6H   SFRSYM    DATA     WORD      TIM0_CCR1
      000000A8H.7 SFRSYM    DATA     BIT       EA
      000000D5H   SFRSYM    DATA     BYTE      CMP_CR0
      000000BAH   SFRSYM    DATA     WORD      TIM0_CCR2
      000000D6H   SFRSYM    DATA     BYTE      CMP_CR1
      000000BCH   SFRSYM    DATA     WORD      TIM0_CCR3
      00000085H   SFRSYM    DATA     BYTE      PSCTL
      000000DAH   SFRSYM    DATA     BYTE      CMP_CR2
      000000BEH   SFRSYM    DATA     WORD      TIM0_CCR4
      000000B8H.2 SFRSYM    DATA     BIT       PX00
      000000EAH   SFRSYM    DATA     WORD      PI_EK
      000000F8H   SFRSYM    DATA     BIT       OISUH
      000000B8H.3 SFRSYM    DATA     BIT       PX01
      000000B8H.4 SFRSYM    DATA     BIT       PX10
      000000F8H.2 SFRSYM    DATA     BIT       OISVH
      000000B8H.5 SFRSYM    DATA     BIT       PX11
      000000F8H.4 SFRSYM    DATA     BIT       OISWH
      000000DCH   SFRSYM    DATA     WORD      LPF_K
      000000F2H   SFRSYM    DATA     WORD      PI_KI
      000000F8H.1 SFRSYM    DATA     BIT       OISUL
      000000A8H   SFRSYM    DATA     BYTE      IE
      000000F8H.3 SFRSYM    DATA     BIT       OISVL
      000000F8H.5 SFRSYM    DATA     BIT       OISWL
      000000D1H   SFRSYM    DATA     BYTE      P1IE
      00000098H.6 SFRSYM    DATA     BIT       MOD0
      000000D3H   SFRSYM    DATA     BYTE      P2IE
      000000D2H   SFRSYM    DATA     BYTE      P1IF
      000000F9H   SFRSYM    DATA     BYTE      PL_CR
      00000098H.7 SFRSYM    DATA     BIT       MOD1
      000000D4H   SFRSYM    DATA     BYTE      P2IF
      000000ACH   SFRSYM    DATA     WORD      TIM2_DR
      00000082H   SFRSYM    DATA     WORD      DP
      000000EEH   SFRSYM    DATA     WORD      PI_KP
      000000A4H   SFRSYM    DATA     WORD      TIM3_DR
      00000094H   SFRSYM    DATA     WORD      TIM4_DR
      0000008CH   SFRSYM    DATA     WORD      TIM5_DR
      000000F1H   SFRSYM    DATA     BYTE      OSC_CFG
      000000C1H   SFRSYM    DATA     BYTE      MD_MODE
      000000ECH   SFRSYM    DATA     WORD      PI_UK
      000000DEH   SFRSYM    DATA     WORD      LPF_X
      00000098H   SFRSYM    DATA     BIT       RI
      000000E6H   SFRSYM    DATA     WORD      LPF_Y
      000000C0H   SFRSYM    DATA     BIT       PTIM00
      000000D0H.7 SFRSYM    DATA     BIT       CY
      00000098H.1 SFRSYM    DATA     BIT       TI
      000000C0H.1 SFRSYM    DATA     BIT       PTIM01
      000000C0H.2 SFRSYM    DATA     BIT       PTIM10
      000000C0H.3 SFRSYM    DATA     BIT       PTIM11
      000000E1H   SFRSYM    DATA     BYTE      SV_CR
      00000098H   SFRSYM    DATA     BYTE      UT_CR
      00000099H   SFRSYM    DATA     BYTE      UT_DR
      000000F8H.6 SFRSYM    DATA     BIT       OIS4
LX51 LINKER/LOCATER V4.66.1.0                                                         03/23/2017  15:15:44  PAGE 133


      00000081H   SFRSYM    DATA     BYTE      SP
      000000D0H.2 SFRSYM    DATA     BIT       OV
      000000C4H   SFRSYM    DATA     BYTE      MD_DA0
      0000009AH   SFRSYM    DATA     WORD      UT_BAUD
      000000CCH   SFRSYM    DATA     BYTE      MD_DB0
      000000C5H   SFRSYM    DATA     BYTE      MD_DA1
      000000CDH   SFRSYM    DATA     BYTE      MD_DB1
      000000C6H   SFRSYM    DATA     BYTE      MD_DA2
      000000CEH   SFRSYM    DATA     BYTE      MD_DB2
      000000C7H   SFRSYM    DATA     BYTE      MD_DA3
      000000B4H   SFRSYM    DATA     WORD      TIM2_ADTR
      000000CFH   SFRSYM    DATA     BYTE      MD_DB3
      000000AFH   SFRSYM    DATA     BYTE      TIM2_ARRH
      000000A7H   SFRSYM    DATA     BYTE      TIM3_ARRH
      00000097H   SFRSYM    DATA     BYTE      TIM4_ARRH
      0000008FH   SFRSYM    DATA     BYTE      TIM5_ARRH
      000000AEH   SFRSYM    DATA     BYTE      TIM2_ARRL
      000000A6H   SFRSYM    DATA     BYTE      TIM3_ARRL
      00000087H   SFRSYM    DATA     BYTE      PCON
      000000E2H   SFRSYM    DATA     WORD      SV_US
      00000096H   SFRSYM    DATA     BYTE      TIM4_ARRL
      0000008EH   SFRSYM    DATA     BYTE      TIM5_ARRL
      000000B2H   SFRSYM    DATA     WORD      TIM2_CMTR
      00000088H   SFRSYM    DATA     BYTE      TCON
      000000AAH   SFRSYM    DATA     WORD      TIM2_CNTR
      000000A2H   SFRSYM    DATA     WORD      TIM3_CNTR
      00000092H   SFRSYM    DATA     WORD      TIM4_CNTR
      0000008AH   SFRSYM    DATA     WORD      TIM5_CNTR
      000000E5H   SFRSYM    DATA     BYTE      SV_ANGLEH
      000000D8H   SFRSYM    DATA     BIT       PUART0
      000000E4H   SFRSYM    DATA     BYTE      SV_ANGLEL
      000000C6H   SFRSYM    DATA     WORD      MD_DAH
      000000D8H.1 SFRSYM    DATA     BIT       PUART1
      000000D8H.2 SFRSYM    DATA     BIT       PI2C0
      00000088H.2 SFRSYM    DATA     BIT       IF0
      000000CEH   SFRSYM    DATA     WORD      MD_DBH
      000000D8H.3 SFRSYM    DATA     BIT       PI2C1
      000000F0H   SFRSYM    DATA     BYTE      B
      000000C4H   SFRSYM    DATA     WORD      MD_DAL
      000000A1H   SFRSYM    DATA     BYTE      TIM2_CR0
      000000CCH   SFRSYM    DATA     WORD      MD_DBL
      0000009CH   SFRSYM    DATA     BYTE      TIM3_CR0
      000000A9H   SFRSYM    DATA     BYTE      TIM2_CR1
      0000009EH   SFRSYM    DATA     BYTE      TIM4_CR0
      0000009DH   SFRSYM    DATA     BYTE      TIM3_CR1
      00000089H   SFRSYM    DATA     BYTE      TIM5_CR0
      0000009FH   SFRSYM    DATA     BYTE      TIM4_CR1
      000000F8H   SFRSYM    DATA     BYTE      DRV_OUT
      00000091H   SFRSYM    DATA     BYTE      TIM5_CR1
      000000E0H   SFRSYM    DATA     BYTE      ACC
      000000F7H   SFRSYM    DATA     BYTE      PI_UKMINH
      000000C3H   SFRSYM    DATA     BYTE      MD_MAH
      000000A8H.4 SFRSYM    DATA     BIT       ES0
      000000DBH   SFRSYM    DATA     BYTE      LVSR
      000000CBH   SFRSYM    DATA     BYTE      MD_MBH
      000000C0H.4 SFRSYM    DATA     BIT       PADC0
      000000B8H   SFRSYM    DATA     BYTE      IP0
      000000F5H   SFRSYM    DATA     BYTE      PI_UKMAXH
      000000C0H.5 SFRSYM    DATA     BIT       PADC1
      000000C0H   SFRSYM    DATA     BYTE      IP1
      000000C8H   SFRSYM    DATA     BYTE      IP2
      000000F6H   SFRSYM    DATA     BYTE      PI_UKMINL
      000000C2H   SFRSYM    DATA     BYTE      MD_MAL
      00000098H.2 SFRSYM    DATA     BIT       RB8
      000000D8H   SFRSYM    DATA     BYTE      IP3
LX51 LINKER/LOCATER V4.66.1.0                                                         03/23/2017  15:15:44  PAGE 134


      000000CAH   SFRSYM    DATA     BYTE      MD_MBL
      000000A8H   SFRSYM    DATA     BIT       EX0
      000000F4H   SFRSYM    DATA     BYTE      PI_UKMAXL
      00000098H.3 SFRSYM    DATA     BIT       TB8
      000000B7H   SFRSYM    DATA     BYTE      TIM0_CCR1H
      000000A8H.2 SFRSYM    DATA     BIT       EX1
      000000BBH   SFRSYM    DATA     BYTE      TIM0_CCR2H
      000000D0H   SFRSYM    DATA     BIT       P
      000000BDH   SFRSYM    DATA     BYTE      TIM0_CCR3H
      000000BFH   SFRSYM    DATA     BYTE      TIM0_CCR4H
      000000C8H.2 SFRSYM    DATA     BIT       PTIM230
      000000EBH   SFRSYM    DATA     BYTE      PI_EKH
      00000098H.5 SFRSYM    DATA     BIT       SM2
      000000B6H   SFRSYM    DATA     BYTE      TIM0_CCR1L
      000000B1H   SFRSYM    DATA     BYTE      TIM0_SR1
      000000C8H.3 SFRSYM    DATA     BIT       PTIM231
      000000BAH   SFRSYM    DATA     BYTE      TIM0_CCR2L
      000000BCH   SFRSYM    DATA     BYTE      TIM0_CCR3L
      000000BEH   SFRSYM    DATA     BYTE      TIM0_CCR4L
      000000D8H.6 SFRSYM    DATA     BIT       PMCD0
      000000C8H.4 SFRSYM    DATA     BIT       PTIM450
      000000D0H.3 SFRSYM    DATA     BIT       RS0
      000000DDH   SFRSYM    DATA     BYTE      LPF_KH
      000000F3H   SFRSYM    DATA     BYTE      PI_KIH
      000000EAH   SFRSYM    DATA     BYTE      PI_EKL
      000000E8H   SFRSYM    DATA     BYTE      FOC_SET0
      000000D8H.7 SFRSYM    DATA     BIT       PMCD1
      000000C8H.5 SFRSYM    DATA     BIT       PTIM451
      000000D0H.4 SFRSYM    DATA     BIT       RS1
      000000E9H   SFRSYM    DATA     BYTE      FOC_SET1
      000000B8H.6 SFRSYM    DATA     BIT       PFOC0
      000000DCH   SFRSYM    DATA     BYTE      LPF_KL
      000000F2H   SFRSYM    DATA     BYTE      PI_KIL
      000000B8H.7 SFRSYM    DATA     BIT       PFOC1
      000000ADH   SFRSYM    DATA     BYTE      TIM2_DRH
      000000B9H   SFRSYM    DATA     BYTE      TIM0_IER
      00000083H   SFRSYM    DATA     BYTE      DPH
      000000EFH   SFRSYM    DATA     BYTE      PI_KPH
      000000A5H   SFRSYM    DATA     BYTE      TIM3_DRH
      00000095H   SFRSYM    DATA     BYTE      TIM4_DRH
      0000008DH   SFRSYM    DATA     BYTE      TIM5_DRH
      000000ACH   SFRSYM    DATA     BYTE      TIM2_DRL
      00000082H   SFRSYM    DATA     BYTE      DPL
      000000EEH   SFRSYM    DATA     BYTE      PI_KPL
      000000A4H   SFRSYM    DATA     BYTE      TIM3_DRL
      000000F8H.7 SFRSYM    DATA     BIT       MOE
      000000C0H.6 SFRSYM    DATA     BIT       PCMP0
      000000EDH   SFRSYM    DATA     BYTE      PI_UKH
      00000094H   SFRSYM    DATA     BYTE      TIM4_DRL
      000000C0H.7 SFRSYM    DATA     BIT       PCMP1
      000000DFH   SFRSYM    DATA     BYTE      LPF_XH
      0000008CH   SFRSYM    DATA     BYTE      TIM5_DRL
      000000AEH   SFRSYM    DATA     WORD      TIM2_ARR
      000000A8H.5 SFRSYM    DATA     BIT       MCDIE
      000000C9H   SFRSYM    DATA     BYTE      RSTSRC
      000000E7H   SFRSYM    DATA     BYTE      LPF_YH
      000000A6H   SFRSYM    DATA     WORD      TIM3_ARR
      00000088H.6 SFRSYM    DATA     BIT       MCDIF
      00000098H.4 SFRSYM    DATA     BIT       REN
      00000096H   SFRSYM    DATA     WORD      TIM4_ARR
      000000ECH   SFRSYM    DATA     BYTE      PI_UKL
      000000D7H   SFRSYM    DATA     BYTE      CMP_SR
      0000008EH   SFRSYM    DATA     WORD      TIM5_ARR
      000000DEH   SFRSYM    DATA     BYTE      LPF_XL
      000000E6H   SFRSYM    DATA     BYTE      LPF_YL
LX51 LINKER/LOCATER V4.66.1.0                                                         03/23/2017  15:15:44  PAGE 135


      000000C8H   SFRSYM    DATA     BIT       PRTC0
      000000C8H.1 SFRSYM    DATA     BIT       PRTC1
      000000E8H.7 SFRSYM    DATA     BIT       FOCEN
      000000C8H.6 SFRSYM    DATA     BIT       PTSD0
      000000D8H.4 SFRSYM    DATA     BIT       PSPI0
      000000C8H.7 SFRSYM    DATA     BIT       PTSD1
      000000D8H.5 SFRSYM    DATA     BIT       PSPI1
      0000009BH   SFRSYM    DATA     BYTE      UT_BAUDH
      000000E4H   SFRSYM    DATA     WORD      SV_ANGLE
      000000B5H   SFRSYM    DATA     BYTE      TIM2_ADTRH
      0000009AH   SFRSYM    DATA     BYTE      UT_BAUDL
      000000FCH   SFRSYM    DATA     BYTE      P0_OE
      000000FDH   SFRSYM    DATA     BYTE      P1_OE
      000000D0H.5 SFRSYM    DATA     BIT       F0
      000000B4H   SFRSYM    DATA     BYTE      TIM2_ADTRL
      000000FEH   SFRSYM    DATA     BYTE      P2_OE
      000000D0H.1 SFRSYM    DATA     BIT       F1
      00000080H   SFRSYM    DATA     BIT       GP00
      000000FFH   SFRSYM    DATA     BYTE      P3_OE
      00000090H   SFRSYM    DATA     BIT       GP10
      00000080H.1 SFRSYM    DATA     BIT       GP01
      000000A8H.6 SFRSYM    DATA     BIT       RTCIE
      000000A0H   SFRSYM    DATA     BIT       GP20
      00000090H.1 SFRSYM    DATA     BIT       GP11
      00000080H.2 SFRSYM    DATA     BIT       GP02
      000000E3H   SFRSYM    DATA     BYTE      SV_USH
      000000B0H   SFRSYM    DATA     BIT       GP30
      000000A0H.1 SFRSYM    DATA     BIT       GP21
      00000090H.2 SFRSYM    DATA     BIT       GP12
      00000080H.3 SFRSYM    DATA     BIT       GP03
      000000B8H   SFRSYM    DATA     BIT       PLVW0
      000000A8H.1 SFRSYM    DATA     BIT       TSDIE
      000000D0H   SFRSYM    DATA     BYTE      PSW
      000000B0H.1 SFRSYM    DATA     BIT       GP31
      000000A0H.2 SFRSYM    DATA     BIT       GP22
      00000090H.3 SFRSYM    DATA     BIT       GP13
      00000080H.4 SFRSYM    DATA     BIT       GP04
      000000B8H.1 SFRSYM    DATA     BIT       PLVW1
      000000A8H.3 SFRSYM    DATA     BIT       SPIIE
      00000088H.5 SFRSYM    DATA     BIT       TSDIF
      000000B0H.2 SFRSYM    DATA     BIT       GP32
      000000A0H.3 SFRSYM    DATA     BIT       GP23
      00000090H.4 SFRSYM    DATA     BIT       GP14
      00000080H.5 SFRSYM    DATA     BIT       GP05
      00000084H   SFRSYM    DATA     BYTE      FLKEY
      000000B3H   SFRSYM    DATA     BYTE      TIM2_CMTRH
      000000B0H.3 SFRSYM    DATA     BIT       GP33
      000000A0H.4 SFRSYM    DATA     BIT       GP24
      00000090H.5 SFRSYM    DATA     BIT       GP15
      00000080H.6 SFRSYM    DATA     BIT       GP06
      00000088H   SFRSYM    DATA     BIT       IT00

      01001D76H   BLOCK     CODE     ---       LVL=0
      01001D76H   LINE      CODE     ---       #23
      01001D76H   LINE      CODE     ---       #24
      01001D76H   LINE      CODE     ---       #32
      01001D7BH   LINE      CODE     ---       #33
      01001D80H   LINE      CODE     ---       #39
      01001D87H   LINE      CODE     ---       #40
      01001D8EH   LINE      CODE     ---       #47
      ---         BLOCKEND  ---      ---       LVL=0

      ---         MODULE    ---      ---       INTERRUPTINIT
      01001CC8H   PUBLIC    CODE     ---       InterruptInit
      000000E2H   SFRSYM    DATA     BYTE      SV_USL
LX51 LINKER/LOCATER V4.66.1.0                                                         03/23/2017  15:15:44  PAGE 136


      000000ABH   SFRSYM    DATA     BYTE      TIM2_CNTRH
      000000B0H.4 SFRSYM    DATA     BIT       GP34
      000000A0H.5 SFRSYM    DATA     BIT       GP25
      00000090H.6 SFRSYM    DATA     BIT       GP16
      00000080H.7 SFRSYM    DATA     BIT       GP07
      00000088H.1 SFRSYM    DATA     BIT       IT01
      00000088H.3 SFRSYM    DATA     BIT       IT10
      000000F6H   SFRSYM    DATA     WORD      PI_UKMIN
      000000C2H   SFRSYM    DATA     WORD      MD_MA
      000000A3H   SFRSYM    DATA     BYTE      TIM3_CNTRH
      000000B0H.5 SFRSYM    DATA     BIT       GP35
      000000A0H.6 SFRSYM    DATA     BIT       GP26
      00000090H.7 SFRSYM    DATA     BIT       GP17
      00000080H   SFRSYM    DATA     BYTE      P0
      00000088H.4 SFRSYM    DATA     BIT       IT11
      000000CAH   SFRSYM    DATA     WORD      MD_MB
      00000093H   SFRSYM    DATA     BYTE      TIM4_CNTRH
      000000B0H.6 SFRSYM    DATA     BIT       GP36
      000000A0H.7 SFRSYM    DATA     BIT       GP27
      00000090H   SFRSYM    DATA     BYTE      P1
      000000D9H   SFRSYM    DATA     BYTE      EVT_FILT
      000000F4H   SFRSYM    DATA     WORD      PI_UKMAX
      0000008BH   SFRSYM    DATA     BYTE      TIM5_CNTRH
      000000B2H   SFRSYM    DATA     BYTE      TIM2_CMTRL
      000000B0H.7 SFRSYM    DATA     BIT       GP37
      000000A0H   SFRSYM    DATA     BYTE      P2
      000000AAH   SFRSYM    DATA     BYTE      TIM2_CNTRL
      000000B0H   SFRSYM    DATA     BYTE      P3
      000000A2H   SFRSYM    DATA     BYTE      TIM3_CNTRL
      000000D0H.6 SFRSYM    DATA     BIT       AC
      00000092H   SFRSYM    DATA     BYTE      TIM4_CNTRL
      0000008AH   SFRSYM    DATA     BYTE      TIM5_CNTRL
      000000B6H   SFRSYM    DATA     WORD      TIM0_CCR1
      000000A8H.7 SFRSYM    DATA     BIT       EA
      000000D5H   SFRSYM    DATA     BYTE      CMP_CR0
      000000BAH   SFRSYM    DATA     WORD      TIM0_CCR2
      000000D6H   SFRSYM    DATA     BYTE      CMP_CR1
      000000BCH   SFRSYM    DATA     WORD      TIM0_CCR3
      00000085H   SFRSYM    DATA     BYTE      PSCTL
      000000DAH   SFRSYM    DATA     BYTE      CMP_CR2
      000000BEH   SFRSYM    DATA     WORD      TIM0_CCR4
      000000B8H.2 SFRSYM    DATA     BIT       PX00
      000000EAH   SFRSYM    DATA     WORD      PI_EK
      000000F8H   SFRSYM    DATA     BIT       OISUH
      000000B8H.3 SFRSYM    DATA     BIT       PX01
      000000B8H.4 SFRSYM    DATA     BIT       PX10
      000000F8H.2 SFRSYM    DATA     BIT       OISVH
      000000B8H.5 SFRSYM    DATA     BIT       PX11
      000000F8H.4 SFRSYM    DATA     BIT       OISWH
      000000DCH   SFRSYM    DATA     WORD      LPF_K
      000000F2H   SFRSYM    DATA     WORD      PI_KI
      000000F8H.1 SFRSYM    DATA     BIT       OISUL
      000000A8H   SFRSYM    DATA     BYTE      IE
      000000F8H.3 SFRSYM    DATA     BIT       OISVL
      000000F8H.5 SFRSYM    DATA     BIT       OISWL
      000000D1H   SFRSYM    DATA     BYTE      P1IE
      00000098H.6 SFRSYM    DATA     BIT       MOD0
      000000D3H   SFRSYM    DATA     BYTE      P2IE
      000000D2H   SFRSYM    DATA     BYTE      P1IF
      000000F9H   SFRSYM    DATA     BYTE      PL_CR
      00000098H.7 SFRSYM    DATA     BIT       MOD1
      000000D4H   SFRSYM    DATA     BYTE      P2IF
      000000ACH   SFRSYM    DATA     WORD      TIM2_DR
      00000082H   SFRSYM    DATA     WORD      DP
      000000EEH   SFRSYM    DATA     WORD      PI_KP
LX51 LINKER/LOCATER V4.66.1.0                                                         03/23/2017  15:15:44  PAGE 137


      000000A4H   SFRSYM    DATA     WORD      TIM3_DR
      00000094H   SFRSYM    DATA     WORD      TIM4_DR
      0000008CH   SFRSYM    DATA     WORD      TIM5_DR
      000000F1H   SFRSYM    DATA     BYTE      OSC_CFG
      000000C1H   SFRSYM    DATA     BYTE      MD_MODE
      000000ECH   SFRSYM    DATA     WORD      PI_UK
      000000DEH   SFRSYM    DATA     WORD      LPF_X
      00000098H   SFRSYM    DATA     BIT       RI
      000000E6H   SFRSYM    DATA     WORD      LPF_Y
      000000C0H   SFRSYM    DATA     BIT       PTIM00
      000000D0H.7 SFRSYM    DATA     BIT       CY
      00000098H.1 SFRSYM    DATA     BIT       TI
      000000C0H.1 SFRSYM    DATA     BIT       PTIM01
      000000C0H.2 SFRSYM    DATA     BIT       PTIM10
      000000C0H.3 SFRSYM    DATA     BIT       PTIM11
      000000E1H   SFRSYM    DATA     BYTE      SV_CR
      00000098H   SFRSYM    DATA     BYTE      UT_CR
      00000099H   SFRSYM    DATA     BYTE      UT_DR
      000000F8H.6 SFRSYM    DATA     BIT       OIS4
      00000081H   SFRSYM    DATA     BYTE      SP
      000000D0H.2 SFRSYM    DATA     BIT       OV
      000000C4H   SFRSYM    DATA     BYTE      MD_DA0
      0000009AH   SFRSYM    DATA     WORD      UT_BAUD
      000000CCH   SFRSYM    DATA     BYTE      MD_DB0
      000000C5H   SFRSYM    DATA     BYTE      MD_DA1
      000000CDH   SFRSYM    DATA     BYTE      MD_DB1
      000000C6H   SFRSYM    DATA     BYTE      MD_DA2
      000000CEH   SFRSYM    DATA     BYTE      MD_DB2
      000000C7H   SFRSYM    DATA     BYTE      MD_DA3
      000000B4H   SFRSYM    DATA     WORD      TIM2_ADTR
      000000CFH   SFRSYM    DATA     BYTE      MD_DB3
      000000AFH   SFRSYM    DATA     BYTE      TIM2_ARRH
      000000A7H   SFRSYM    DATA     BYTE      TIM3_ARRH
      00000097H   SFRSYM    DATA     BYTE      TIM4_ARRH
      0000008FH   SFRSYM    DATA     BYTE      TIM5_ARRH
      000000AEH   SFRSYM    DATA     BYTE      TIM2_ARRL
      000000A6H   SFRSYM    DATA     BYTE      TIM3_ARRL
      00000087H   SFRSYM    DATA     BYTE      PCON
      000000E2H   SFRSYM    DATA     WORD      SV_US
      00000096H   SFRSYM    DATA     BYTE      TIM4_ARRL
      0000008EH   SFRSYM    DATA     BYTE      TIM5_ARRL
      000000B2H   SFRSYM    DATA     WORD      TIM2_CMTR
      00000088H   SFRSYM    DATA     BYTE      TCON
      000000AAH   SFRSYM    DATA     WORD      TIM2_CNTR
      000000A2H   SFRSYM    DATA     WORD      TIM3_CNTR
      00000092H   SFRSYM    DATA     WORD      TIM4_CNTR
      0000008AH   SFRSYM    DATA     WORD      TIM5_CNTR
      000000E5H   SFRSYM    DATA     BYTE      SV_ANGLEH
      000000D8H   SFRSYM    DATA     BIT       PUART0
      000000E4H   SFRSYM    DATA     BYTE      SV_ANGLEL
      000000C6H   SFRSYM    DATA     WORD      MD_DAH
      000000D8H.1 SFRSYM    DATA     BIT       PUART1
      000000D8H.2 SFRSYM    DATA     BIT       PI2C0
      00000088H.2 SFRSYM    DATA     BIT       IF0
      000000CEH   SFRSYM    DATA     WORD      MD_DBH
      000000D8H.3 SFRSYM    DATA     BIT       PI2C1
      000000F0H   SFRSYM    DATA     BYTE      B
      000000C4H   SFRSYM    DATA     WORD      MD_DAL
      000000A1H   SFRSYM    DATA     BYTE      TIM2_CR0
      000000CCH   SFRSYM    DATA     WORD      MD_DBL
      0000009CH   SFRSYM    DATA     BYTE      TIM3_CR0
      000000A9H   SFRSYM    DATA     BYTE      TIM2_CR1
      0000009EH   SFRSYM    DATA     BYTE      TIM4_CR0
      0000009DH   SFRSYM    DATA     BYTE      TIM3_CR1
      00000089H   SFRSYM    DATA     BYTE      TIM5_CR0
LX51 LINKER/LOCATER V4.66.1.0                                                         03/23/2017  15:15:44  PAGE 138


      0000009FH   SFRSYM    DATA     BYTE      TIM4_CR1
      000000F8H   SFRSYM    DATA     BYTE      DRV_OUT
      00000091H   SFRSYM    DATA     BYTE      TIM5_CR1
      000000E0H   SFRSYM    DATA     BYTE      ACC
      000000F7H   SFRSYM    DATA     BYTE      PI_UKMINH
      000000C3H   SFRSYM    DATA     BYTE      MD_MAH
      000000A8H.4 SFRSYM    DATA     BIT       ES0
      000000DBH   SFRSYM    DATA     BYTE      LVSR
      000000CBH   SFRSYM    DATA     BYTE      MD_MBH
      000000C0H.4 SFRSYM    DATA     BIT       PADC0
      000000B8H   SFRSYM    DATA     BYTE      IP0
      000000F5H   SFRSYM    DATA     BYTE      PI_UKMAXH
      000000C0H.5 SFRSYM    DATA     BIT       PADC1
      000000C0H   SFRSYM    DATA     BYTE      IP1
      000000C8H   SFRSYM    DATA     BYTE      IP2
      000000F6H   SFRSYM    DATA     BYTE      PI_UKMINL
      000000C2H   SFRSYM    DATA     BYTE      MD_MAL
      00000098H.2 SFRSYM    DATA     BIT       RB8
      000000D8H   SFRSYM    DATA     BYTE      IP3
      000000CAH   SFRSYM    DATA     BYTE      MD_MBL
      000000A8H   SFRSYM    DATA     BIT       EX0
      000000F4H   SFRSYM    DATA     BYTE      PI_UKMAXL
      00000098H.3 SFRSYM    DATA     BIT       TB8
      000000B7H   SFRSYM    DATA     BYTE      TIM0_CCR1H
      000000A8H.2 SFRSYM    DATA     BIT       EX1
      000000BBH   SFRSYM    DATA     BYTE      TIM0_CCR2H
      000000D0H   SFRSYM    DATA     BIT       P
      000000BDH   SFRSYM    DATA     BYTE      TIM0_CCR3H
      000000BFH   SFRSYM    DATA     BYTE      TIM0_CCR4H
      000000C8H.2 SFRSYM    DATA     BIT       PTIM230
      000000EBH   SFRSYM    DATA     BYTE      PI_EKH
      00000098H.5 SFRSYM    DATA     BIT       SM2
      000000B6H   SFRSYM    DATA     BYTE      TIM0_CCR1L
      000000B1H   SFRSYM    DATA     BYTE      TIM0_SR1
      000000C8H.3 SFRSYM    DATA     BIT       PTIM231
      000000BAH   SFRSYM    DATA     BYTE      TIM0_CCR2L
      000000BCH   SFRSYM    DATA     BYTE      TIM0_CCR3L
      000000BEH   SFRSYM    DATA     BYTE      TIM0_CCR4L
      000000D8H.6 SFRSYM    DATA     BIT       PMCD0
      000000C8H.4 SFRSYM    DATA     BIT       PTIM450
      000000D0H.3 SFRSYM    DATA     BIT       RS0
      000000DDH   SFRSYM    DATA     BYTE      LPF_KH
      000000F3H   SFRSYM    DATA     BYTE      PI_KIH
      000000EAH   SFRSYM    DATA     BYTE      PI_EKL
      000000E8H   SFRSYM    DATA     BYTE      FOC_SET0
      000000D8H.7 SFRSYM    DATA     BIT       PMCD1
      000000C8H.5 SFRSYM    DATA     BIT       PTIM451
      000000D0H.4 SFRSYM    DATA     BIT       RS1
      000000E9H   SFRSYM    DATA     BYTE      FOC_SET1
      000000B8H.6 SFRSYM    DATA     BIT       PFOC0
      000000DCH   SFRSYM    DATA     BYTE      LPF_KL
      000000F2H   SFRSYM    DATA     BYTE      PI_KIL
      000000B8H.7 SFRSYM    DATA     BIT       PFOC1
      000000ADH   SFRSYM    DATA     BYTE      TIM2_DRH
      000000B9H   SFRSYM    DATA     BYTE      TIM0_IER
      00000083H   SFRSYM    DATA     BYTE      DPH
      000000EFH   SFRSYM    DATA     BYTE      PI_KPH
      000000A5H   SFRSYM    DATA     BYTE      TIM3_DRH
      00000095H   SFRSYM    DATA     BYTE      TIM4_DRH
      0000008DH   SFRSYM    DATA     BYTE      TIM5_DRH
      000000ACH   SFRSYM    DATA     BYTE      TIM2_DRL
      00000082H   SFRSYM    DATA     BYTE      DPL
      000000EEH   SFRSYM    DATA     BYTE      PI_KPL
      000000A4H   SFRSYM    DATA     BYTE      TIM3_DRL
      000000F8H.7 SFRSYM    DATA     BIT       MOE
LX51 LINKER/LOCATER V4.66.1.0                                                         03/23/2017  15:15:44  PAGE 139


      000000C0H.6 SFRSYM    DATA     BIT       PCMP0
      000000EDH   SFRSYM    DATA     BYTE      PI_UKH
      00000094H   SFRSYM    DATA     BYTE      TIM4_DRL
      000000C0H.7 SFRSYM    DATA     BIT       PCMP1
      000000DFH   SFRSYM    DATA     BYTE      LPF_XH
      0000008CH   SFRSYM    DATA     BYTE      TIM5_DRL
      000000AEH   SFRSYM    DATA     WORD      TIM2_ARR
      000000A8H.5 SFRSYM    DATA     BIT       MCDIE
      000000C9H   SFRSYM    DATA     BYTE      RSTSRC
      000000E7H   SFRSYM    DATA     BYTE      LPF_YH
      000000A6H   SFRSYM    DATA     WORD      TIM3_ARR
      00000088H.6 SFRSYM    DATA     BIT       MCDIF
      00000098H.4 SFRSYM    DATA     BIT       REN
      00000096H   SFRSYM    DATA     WORD      TIM4_ARR
      000000ECH   SFRSYM    DATA     BYTE      PI_UKL
      000000D7H   SFRSYM    DATA     BYTE      CMP_SR
      0000008EH   SFRSYM    DATA     WORD      TIM5_ARR
      000000DEH   SFRSYM    DATA     BYTE      LPF_XL
      000000E6H   SFRSYM    DATA     BYTE      LPF_YL
      000000C8H   SFRSYM    DATA     BIT       PRTC0
      000000C8H.1 SFRSYM    DATA     BIT       PRTC1
      000000E8H.7 SFRSYM    DATA     BIT       FOCEN
      000000C8H.6 SFRSYM    DATA     BIT       PTSD0
      000000D8H.4 SFRSYM    DATA     BIT       PSPI0
      000000C8H.7 SFRSYM    DATA     BIT       PTSD1
      000000D8H.5 SFRSYM    DATA     BIT       PSPI1
      0000009BH   SFRSYM    DATA     BYTE      UT_BAUDH
      000000E4H   SFRSYM    DATA     WORD      SV_ANGLE
      000000B5H   SFRSYM    DATA     BYTE      TIM2_ADTRH
      0000009AH   SFRSYM    DATA     BYTE      UT_BAUDL
      000000FCH   SFRSYM    DATA     BYTE      P0_OE
      000000FDH   SFRSYM    DATA     BYTE      P1_OE
      000000D0H.5 SFRSYM    DATA     BIT       F0
      000000B4H   SFRSYM    DATA     BYTE      TIM2_ADTRL
      000000FEH   SFRSYM    DATA     BYTE      P2_OE
      000000D0H.1 SFRSYM    DATA     BIT       F1
      00000080H   SFRSYM    DATA     BIT       GP00
      000000FFH   SFRSYM    DATA     BYTE      P3_OE
      00000090H   SFRSYM    DATA     BIT       GP10
      00000080H.1 SFRSYM    DATA     BIT       GP01
      000000A8H.6 SFRSYM    DATA     BIT       RTCIE
      000000A0H   SFRSYM    DATA     BIT       GP20
      00000090H.1 SFRSYM    DATA     BIT       GP11
      00000080H.2 SFRSYM    DATA     BIT       GP02
      000000E3H   SFRSYM    DATA     BYTE      SV_USH
      000000B0H   SFRSYM    DATA     BIT       GP30
      000000A0H.1 SFRSYM    DATA     BIT       GP21
      00000090H.2 SFRSYM    DATA     BIT       GP12
      00000080H.3 SFRSYM    DATA     BIT       GP03
      000000B8H   SFRSYM    DATA     BIT       PLVW0
      000000A8H.1 SFRSYM    DATA     BIT       TSDIE
      000000D0H   SFRSYM    DATA     BYTE      PSW
      000000B0H.1 SFRSYM    DATA     BIT       GP31
      000000A0H.2 SFRSYM    DATA     BIT       GP22
      00000090H.3 SFRSYM    DATA     BIT       GP13
      00000080H.4 SFRSYM    DATA     BIT       GP04
      000000B8H.1 SFRSYM    DATA     BIT       PLVW1
      000000A8H.3 SFRSYM    DATA     BIT       SPIIE
      00000088H.5 SFRSYM    DATA     BIT       TSDIF
      000000B0H.2 SFRSYM    DATA     BIT       GP32
      000000A0H.3 SFRSYM    DATA     BIT       GP23
      00000090H.4 SFRSYM    DATA     BIT       GP14
      00000080H.5 SFRSYM    DATA     BIT       GP05
      00000084H   SFRSYM    DATA     BYTE      FLKEY
      000000B3H   SFRSYM    DATA     BYTE      TIM2_CMTRH
LX51 LINKER/LOCATER V4.66.1.0                                                         03/23/2017  15:15:44  PAGE 140


      000000B0H.3 SFRSYM    DATA     BIT       GP33
      000000A0H.4 SFRSYM    DATA     BIT       GP24
      00000090H.5 SFRSYM    DATA     BIT       GP15
      00000080H.6 SFRSYM    DATA     BIT       GP06
      00000088H   SFRSYM    DATA     BIT       IT00

      01001CC8H   BLOCK     CODE     ---       LVL=0
      01001CC8H   LINE      CODE     ---       #23
      01001CC8H   LINE      CODE     ---       #24
      01001CC8H   LINE      CODE     ---       #25
      01001CCAH   LINE      CODE     ---       #28
      01001CCCH   LINE      CODE     ---       #29
      01001CCEH   LINE      CODE     ---       #32
      01001CD0H   LINE      CODE     ---       #33
      01001CD2H   LINE      CODE     ---       #36
      01001CD4H   LINE      CODE     ---       #37
      01001CD6H   LINE      CODE     ---       #40
      01001CD8H   LINE      CODE     ---       #41
      01001CDAH   LINE      CODE     ---       #44
      01001CDCH   LINE      CODE     ---       #45
      01001CDEH   LINE      CODE     ---       #48
      01001CE0H   LINE      CODE     ---       #49
      01001CE2H   LINE      CODE     ---       #52
      01001CE4H   LINE      CODE     ---       #53
      01001CE6H   LINE      CODE     ---       #56
      01001CE8H   LINE      CODE     ---       #57
      01001CEAH   LINE      CODE     ---       #60
      01001CECH   LINE      CODE     ---       #61
      ---         BLOCKEND  ---      ---       LVL=0

      ---         MODULE    ---      ---       FU68XX_SYSTEM
      01001EA7H   PUBLIC    CODE     ---       WatchDogRefresh
      00000020H.0 PUBLIC    BIT      BIT       ?_WatchDogConfig?BIT
      01001B1DH   PUBLIC    CODE     ---       _WatchDogConfig
      00000020H.0 PUBLIC    BIT      BIT       ?VHALFConfig?BIT
      01001D97H   PUBLIC    CODE     ---       VHALFConfig
      00000020H.0 PUBLIC    BIT      BIT       ?_VREFConfig?BIT
      01001974H   PUBLIC    CODE     ---       _VREFConfig
      00000020H.0 PUBLIC    BIT      BIT       ?ExternalSlowClockConfig?BIT
      01001E4FH   PUBLIC    CODE     ---       ExternalSlowClockConfig
      00000020H.0 PUBLIC    BIT      BIT       ?SystemFastClockConfig?BIT
      01001E8AH   PUBLIC    CODE     ---       SystemFastClockConfig
      000000E2H   SFRSYM    DATA     BYTE      SV_USL
      000000ABH   SFRSYM    DATA     BYTE      TIM2_CNTRH
      000000B0H.4 SFRSYM    DATA     BIT       GP34
      000000A0H.5 SFRSYM    DATA     BIT       GP25
      00000090H.6 SFRSYM    DATA     BIT       GP16
      00000080H.7 SFRSYM    DATA     BIT       GP07
      00000088H.1 SFRSYM    DATA     BIT       IT01
      00000088H.3 SFRSYM    DATA     BIT       IT10
      000000F6H   SFRSYM    DATA     WORD      PI_UKMIN
      000000C2H   SFRSYM    DATA     WORD      MD_MA
      000000A3H   SFRSYM    DATA     BYTE      TIM3_CNTRH
      000000B0H.5 SFRSYM    DATA     BIT       GP35
      000000A0H.6 SFRSYM    DATA     BIT       GP26
      00000090H.7 SFRSYM    DATA     BIT       GP17
      00000080H   SFRSYM    DATA     BYTE      P0
      00000088H.4 SFRSYM    DATA     BIT       IT11
      000000CAH   SFRSYM    DATA     WORD      MD_MB
      00000093H   SFRSYM    DATA     BYTE      TIM4_CNTRH
      000000B0H.6 SFRSYM    DATA     BIT       GP36
      000000A0H.7 SFRSYM    DATA     BIT       GP27
      00000090H   SFRSYM    DATA     BYTE      P1
      000000D9H   SFRSYM    DATA     BYTE      EVT_FILT
      000000F4H   SFRSYM    DATA     WORD      PI_UKMAX
LX51 LINKER/LOCATER V4.66.1.0                                                         03/23/2017  15:15:44  PAGE 141


      0000008BH   SFRSYM    DATA     BYTE      TIM5_CNTRH
      000000B2H   SFRSYM    DATA     BYTE      TIM2_CMTRL
      000000B0H.7 SFRSYM    DATA     BIT       GP37
      000000A0H   SFRSYM    DATA     BYTE      P2
      000000AAH   SFRSYM    DATA     BYTE      TIM2_CNTRL
      000000B0H   SFRSYM    DATA     BYTE      P3
      000000A2H   SFRSYM    DATA     BYTE      TIM3_CNTRL
      000000D0H.6 SFRSYM    DATA     BIT       AC
      00000092H   SFRSYM    DATA     BYTE      TIM4_CNTRL
      0000008AH   SFRSYM    DATA     BYTE      TIM5_CNTRL
      000000B6H   SFRSYM    DATA     WORD      TIM0_CCR1
      000000A8H.7 SFRSYM    DATA     BIT       EA
      000000D5H   SFRSYM    DATA     BYTE      CMP_CR0
      000000BAH   SFRSYM    DATA     WORD      TIM0_CCR2
      000000D6H   SFRSYM    DATA     BYTE      CMP_CR1
      000000BCH   SFRSYM    DATA     WORD      TIM0_CCR3
      00000085H   SFRSYM    DATA     BYTE      PSCTL
      000000DAH   SFRSYM    DATA     BYTE      CMP_CR2
      000000BEH   SFRSYM    DATA     WORD      TIM0_CCR4
      000000B8H.2 SFRSYM    DATA     BIT       PX00
      000000EAH   SFRSYM    DATA     WORD      PI_EK
      000000F8H   SFRSYM    DATA     BIT       OISUH
      000000B8H.3 SFRSYM    DATA     BIT       PX01
      000000B8H.4 SFRSYM    DATA     BIT       PX10
      000000F8H.2 SFRSYM    DATA     BIT       OISVH
      000000B8H.5 SFRSYM    DATA     BIT       PX11
      000000F8H.4 SFRSYM    DATA     BIT       OISWH
      000000DCH   SFRSYM    DATA     WORD      LPF_K
      000000F2H   SFRSYM    DATA     WORD      PI_KI
      000000F8H.1 SFRSYM    DATA     BIT       OISUL
      000000A8H   SFRSYM    DATA     BYTE      IE
      000000F8H.3 SFRSYM    DATA     BIT       OISVL
      000000F8H.5 SFRSYM    DATA     BIT       OISWL
      000000D1H   SFRSYM    DATA     BYTE      P1IE
      00000098H.6 SFRSYM    DATA     BIT       MOD0
      000000D3H   SFRSYM    DATA     BYTE      P2IE
      000000D2H   SFRSYM    DATA     BYTE      P1IF
      000000F9H   SFRSYM    DATA     BYTE      PL_CR
      00000098H.7 SFRSYM    DATA     BIT       MOD1
      000000D4H   SFRSYM    DATA     BYTE      P2IF
      000000ACH   SFRSYM    DATA     WORD      TIM2_DR
      00000082H   SFRSYM    DATA     WORD      DP
      000000EEH   SFRSYM    DATA     WORD      PI_KP
      000000A4H   SFRSYM    DATA     WORD      TIM3_DR
      00000094H   SFRSYM    DATA     WORD      TIM4_DR
      0000008CH   SFRSYM    DATA     WORD      TIM5_DR
      000000F1H   SFRSYM    DATA     BYTE      OSC_CFG
      000000C1H   SFRSYM    DATA     BYTE      MD_MODE
      000000ECH   SFRSYM    DATA     WORD      PI_UK
      000000DEH   SFRSYM    DATA     WORD      LPF_X
      00000098H   SFRSYM    DATA     BIT       RI
      000000E6H   SFRSYM    DATA     WORD      LPF_Y
      000000C0H   SFRSYM    DATA     BIT       PTIM00
      000000D0H.7 SFRSYM    DATA     BIT       CY
      00000098H.1 SFRSYM    DATA     BIT       TI
      000000C0H.1 SFRSYM    DATA     BIT       PTIM01
      000000C0H.2 SFRSYM    DATA     BIT       PTIM10
      000000C0H.3 SFRSYM    DATA     BIT       PTIM11
      000000E1H   SFRSYM    DATA     BYTE      SV_CR
      00000098H   SFRSYM    DATA     BYTE      UT_CR
      00000099H   SFRSYM    DATA     BYTE      UT_DR
      000000F8H.6 SFRSYM    DATA     BIT       OIS4
      00000081H   SFRSYM    DATA     BYTE      SP
      000000D0H.2 SFRSYM    DATA     BIT       OV
      000000C4H   SFRSYM    DATA     BYTE      MD_DA0
LX51 LINKER/LOCATER V4.66.1.0                                                         03/23/2017  15:15:44  PAGE 142


      0000009AH   SFRSYM    DATA     WORD      UT_BAUD
      000000CCH   SFRSYM    DATA     BYTE      MD_DB0
      000000C5H   SFRSYM    DATA     BYTE      MD_DA1
      000000CDH   SFRSYM    DATA     BYTE      MD_DB1
      000000C6H   SFRSYM    DATA     BYTE      MD_DA2
      000000CEH   SFRSYM    DATA     BYTE      MD_DB2
      000000C7H   SFRSYM    DATA     BYTE      MD_DA3
      000000B4H   SFRSYM    DATA     WORD      TIM2_ADTR
      000000CFH   SFRSYM    DATA     BYTE      MD_DB3
      000000AFH   SFRSYM    DATA     BYTE      TIM2_ARRH
      000000A7H   SFRSYM    DATA     BYTE      TIM3_ARRH
      00000097H   SFRSYM    DATA     BYTE      TIM4_ARRH
      0000008FH   SFRSYM    DATA     BYTE      TIM5_ARRH
      000000AEH   SFRSYM    DATA     BYTE      TIM2_ARRL
      000000A6H   SFRSYM    DATA     BYTE      TIM3_ARRL
      00000087H   SFRSYM    DATA     BYTE      PCON
      000000E2H   SFRSYM    DATA     WORD      SV_US
      00000096H   SFRSYM    DATA     BYTE      TIM4_ARRL
      0000008EH   SFRSYM    DATA     BYTE      TIM5_ARRL
      000000B2H   SFRSYM    DATA     WORD      TIM2_CMTR
      00000088H   SFRSYM    DATA     BYTE      TCON
      000000AAH   SFRSYM    DATA     WORD      TIM2_CNTR
      000000A2H   SFRSYM    DATA     WORD      TIM3_CNTR
      00000092H   SFRSYM    DATA     WORD      TIM4_CNTR
      0000008AH   SFRSYM    DATA     WORD      TIM5_CNTR
      000000E5H   SFRSYM    DATA     BYTE      SV_ANGLEH
      000000D8H   SFRSYM    DATA     BIT       PUART0
      000000E4H   SFRSYM    DATA     BYTE      SV_ANGLEL
      000000C6H   SFRSYM    DATA     WORD      MD_DAH
      000000D8H.1 SFRSYM    DATA     BIT       PUART1
      000000D8H.2 SFRSYM    DATA     BIT       PI2C0
      00000088H.2 SFRSYM    DATA     BIT       IF0
      000000CEH   SFRSYM    DATA     WORD      MD_DBH
      000000D8H.3 SFRSYM    DATA     BIT       PI2C1
      000000F0H   SFRSYM    DATA     BYTE      B
      000000C4H   SFRSYM    DATA     WORD      MD_DAL
      000000A1H   SFRSYM    DATA     BYTE      TIM2_CR0
      000000CCH   SFRSYM    DATA     WORD      MD_DBL
      0000009CH   SFRSYM    DATA     BYTE      TIM3_CR0
      000000A9H   SFRSYM    DATA     BYTE      TIM2_CR1
      0000009EH   SFRSYM    DATA     BYTE      TIM4_CR0
      0000009DH   SFRSYM    DATA     BYTE      TIM3_CR1
      00000089H   SFRSYM    DATA     BYTE      TIM5_CR0
      0000009FH   SFRSYM    DATA     BYTE      TIM4_CR1
      000000F8H   SFRSYM    DATA     BYTE      DRV_OUT
      00000091H   SFRSYM    DATA     BYTE      TIM5_CR1
      000000E0H   SFRSYM    DATA     BYTE      ACC
      000000F7H   SFRSYM    DATA     BYTE      PI_UKMINH
      000000C3H   SFRSYM    DATA     BYTE      MD_MAH
      000000A8H.4 SFRSYM    DATA     BIT       ES0
      000000DBH   SFRSYM    DATA     BYTE      LVSR
      000000CBH   SFRSYM    DATA     BYTE      MD_MBH
      000000C0H.4 SFRSYM    DATA     BIT       PADC0
      000000B8H   SFRSYM    DATA     BYTE      IP0
      000000F5H   SFRSYM    DATA     BYTE      PI_UKMAXH
      000000C0H.5 SFRSYM    DATA     BIT       PADC1
      000000C0H   SFRSYM    DATA     BYTE      IP1
      000000C8H   SFRSYM    DATA     BYTE      IP2
      000000F6H   SFRSYM    DATA     BYTE      PI_UKMINL
      000000C2H   SFRSYM    DATA     BYTE      MD_MAL
      00000098H.2 SFRSYM    DATA     BIT       RB8
      000000D8H   SFRSYM    DATA     BYTE      IP3
      000000CAH   SFRSYM    DATA     BYTE      MD_MBL
      000000A8H   SFRSYM    DATA     BIT       EX0
      000000F4H   SFRSYM    DATA     BYTE      PI_UKMAXL
LX51 LINKER/LOCATER V4.66.1.0                                                         03/23/2017  15:15:44  PAGE 143


      00000098H.3 SFRSYM    DATA     BIT       TB8
      000000B7H   SFRSYM    DATA     BYTE      TIM0_CCR1H
      000000A8H.2 SFRSYM    DATA     BIT       EX1
      000000BBH   SFRSYM    DATA     BYTE      TIM0_CCR2H
      000000D0H   SFRSYM    DATA     BIT       P
      000000BDH   SFRSYM    DATA     BYTE      TIM0_CCR3H
      000000BFH   SFRSYM    DATA     BYTE      TIM0_CCR4H
      000000C8H.2 SFRSYM    DATA     BIT       PTIM230
      000000EBH   SFRSYM    DATA     BYTE      PI_EKH
      00000098H.5 SFRSYM    DATA     BIT       SM2
      000000B6H   SFRSYM    DATA     BYTE      TIM0_CCR1L
      000000B1H   SFRSYM    DATA     BYTE      TIM0_SR1
      000000C8H.3 SFRSYM    DATA     BIT       PTIM231
      000000BAH   SFRSYM    DATA     BYTE      TIM0_CCR2L
      000000BCH   SFRSYM    DATA     BYTE      TIM0_CCR3L
      000000BEH   SFRSYM    DATA     BYTE      TIM0_CCR4L
      000000D8H.6 SFRSYM    DATA     BIT       PMCD0
      000000C8H.4 SFRSYM    DATA     BIT       PTIM450
      000000D0H.3 SFRSYM    DATA     BIT       RS0
      000000DDH   SFRSYM    DATA     BYTE      LPF_KH
      000000F3H   SFRSYM    DATA     BYTE      PI_KIH
      000000EAH   SFRSYM    DATA     BYTE      PI_EKL
      000000E8H   SFRSYM    DATA     BYTE      FOC_SET0
      000000D8H.7 SFRSYM    DATA     BIT       PMCD1
      000000C8H.5 SFRSYM    DATA     BIT       PTIM451
      000000D0H.4 SFRSYM    DATA     BIT       RS1
      000000E9H   SFRSYM    DATA     BYTE      FOC_SET1
      000000B8H.6 SFRSYM    DATA     BIT       PFOC0
      000000DCH   SFRSYM    DATA     BYTE      LPF_KL
      000000F2H   SFRSYM    DATA     BYTE      PI_KIL
      000000B8H.7 SFRSYM    DATA     BIT       PFOC1
      000000ADH   SFRSYM    DATA     BYTE      TIM2_DRH
      000000B9H   SFRSYM    DATA     BYTE      TIM0_IER
      00000083H   SFRSYM    DATA     BYTE      DPH
      000000EFH   SFRSYM    DATA     BYTE      PI_KPH
      000000A5H   SFRSYM    DATA     BYTE      TIM3_DRH
      00000095H   SFRSYM    DATA     BYTE      TIM4_DRH
      0000008DH   SFRSYM    DATA     BYTE      TIM5_DRH
      000000ACH   SFRSYM    DATA     BYTE      TIM2_DRL
      00000082H   SFRSYM    DATA     BYTE      DPL
      000000EEH   SFRSYM    DATA     BYTE      PI_KPL
      000000A4H   SFRSYM    DATA     BYTE      TIM3_DRL
      000000F8H.7 SFRSYM    DATA     BIT       MOE
      000000C0H.6 SFRSYM    DATA     BIT       PCMP0
      000000EDH   SFRSYM    DATA     BYTE      PI_UKH
      00000094H   SFRSYM    DATA     BYTE      TIM4_DRL
      000000C0H.7 SFRSYM    DATA     BIT       PCMP1
      000000DFH   SFRSYM    DATA     BYTE      LPF_XH
      0000008CH   SFRSYM    DATA     BYTE      TIM5_DRL
      000000AEH   SFRSYM    DATA     WORD      TIM2_ARR
      000000A8H.5 SFRSYM    DATA     BIT       MCDIE
      000000C9H   SFRSYM    DATA     BYTE      RSTSRC
      000000E7H   SFRSYM    DATA     BYTE      LPF_YH
      000000A6H   SFRSYM    DATA     WORD      TIM3_ARR
      00000088H.6 SFRSYM    DATA     BIT       MCDIF
      00000098H.4 SFRSYM    DATA     BIT       REN
      00000096H   SFRSYM    DATA     WORD      TIM4_ARR
      000000ECH   SFRSYM    DATA     BYTE      PI_UKL
      000000D7H   SFRSYM    DATA     BYTE      CMP_SR
      0000008EH   SFRSYM    DATA     WORD      TIM5_ARR
      000000DEH   SFRSYM    DATA     BYTE      LPF_XL
      000000E6H   SFRSYM    DATA     BYTE      LPF_YL
      000000C8H   SFRSYM    DATA     BIT       PRTC0
      000000C8H.1 SFRSYM    DATA     BIT       PRTC1
      000000E8H.7 SFRSYM    DATA     BIT       FOCEN
LX51 LINKER/LOCATER V4.66.1.0                                                         03/23/2017  15:15:44  PAGE 144


      000000C8H.6 SFRSYM    DATA     BIT       PTSD0
      000000D8H.4 SFRSYM    DATA     BIT       PSPI0
      000000C8H.7 SFRSYM    DATA     BIT       PTSD1
      000000D8H.5 SFRSYM    DATA     BIT       PSPI1
      0000009BH   SFRSYM    DATA     BYTE      UT_BAUDH
      000000E4H   SFRSYM    DATA     WORD      SV_ANGLE
      000000B5H   SFRSYM    DATA     BYTE      TIM2_ADTRH
      0000009AH   SFRSYM    DATA     BYTE      UT_BAUDL
      000000FCH   SFRSYM    DATA     BYTE      P0_OE
      000000FDH   SFRSYM    DATA     BYTE      P1_OE
      000000D0H.5 SFRSYM    DATA     BIT       F0
      000000B4H   SFRSYM    DATA     BYTE      TIM2_ADTRL
      000000FEH   SFRSYM    DATA     BYTE      P2_OE
      000000D0H.1 SFRSYM    DATA     BIT       F1
      00000080H   SFRSYM    DATA     BIT       GP00
      000000FFH   SFRSYM    DATA     BYTE      P3_OE
      00000090H   SFRSYM    DATA     BIT       GP10
      00000080H.1 SFRSYM    DATA     BIT       GP01
      000000A8H.6 SFRSYM    DATA     BIT       RTCIE
      000000A0H   SFRSYM    DATA     BIT       GP20
      00000090H.1 SFRSYM    DATA     BIT       GP11
      00000080H.2 SFRSYM    DATA     BIT       GP02
      000000E3H   SFRSYM    DATA     BYTE      SV_USH
      000000B0H   SFRSYM    DATA     BIT       GP30
      000000A0H.1 SFRSYM    DATA     BIT       GP21
      00000090H.2 SFRSYM    DATA     BIT       GP12
      00000080H.3 SFRSYM    DATA     BIT       GP03
      000000B8H   SFRSYM    DATA     BIT       PLVW0
      000000A8H.1 SFRSYM    DATA     BIT       TSDIE
      000000D0H   SFRSYM    DATA     BYTE      PSW
      000000B0H.1 SFRSYM    DATA     BIT       GP31
      000000A0H.2 SFRSYM    DATA     BIT       GP22
      00000090H.3 SFRSYM    DATA     BIT       GP13
      00000080H.4 SFRSYM    DATA     BIT       GP04
      000000B8H.1 SFRSYM    DATA     BIT       PLVW1
      000000A8H.3 SFRSYM    DATA     BIT       SPIIE
      00000088H.5 SFRSYM    DATA     BIT       TSDIF
      000000B0H.2 SFRSYM    DATA     BIT       GP32
      000000A0H.3 SFRSYM    DATA     BIT       GP23
      00000090H.4 SFRSYM    DATA     BIT       GP14
      00000080H.5 SFRSYM    DATA     BIT       GP05
      00000084H   SFRSYM    DATA     BYTE      FLKEY
      000000B3H   SFRSYM    DATA     BYTE      TIM2_CMTRH
      000000B0H.3 SFRSYM    DATA     BIT       GP33
      000000A0H.4 SFRSYM    DATA     BIT       GP24
      00000090H.5 SFRSYM    DATA     BIT       GP15
      00000080H.6 SFRSYM    DATA     BIT       GP06
      00000088H   SFRSYM    DATA     BIT       IT00

      01001E8AH   BLOCK     CODE     ---       LVL=0
      00000020H.0 SYMBOL    BIT      BIT       Mode
      01001E8AH   LINE      CODE     ---       #39
      01001E8AH   LINE      CODE     ---       #40
      01001E8AH   LINE      CODE     ---       #41
      01001E98H   LINE      CODE     ---       #42
      ---         BLOCKEND  ---      ---       LVL=0

      01001E4FH   BLOCK     CODE     ---       LVL=0
      00000020H.0 SYMBOL    BIT      BIT       Status
      01001E4FH   LINE      CODE     ---       #52
      01001E4FH   LINE      CODE     ---       #53
      01001E4FH   LINE      CODE     ---       #54
      01001E5AH   LINE      CODE     ---       #55
      01001E64H   LINE      CODE     ---       #56
      ---         BLOCKEND  ---      ---       LVL=0
LX51 LINKER/LOCATER V4.66.1.0                                                         03/23/2017  15:15:44  PAGE 145



      01001974H   BLOCK     CODE     ---       LVL=0
      00000007H   SYMBOL    DATA     BYTE      Value
      00000020H.0 SYMBOL    BIT      BIT       Status
      01001974H   LINE      CODE     ---       #101
      01001974H   LINE      CODE     ---       #102
      01001974H   LINE      CODE     ---       #103
      01001982H   LINE      CODE     ---       #104
      01001982H   LINE      CODE     ---       #105
      01001982H   LINE      CODE     ---       #106
      01001988H   LINE      CODE     ---       #107
      01001988H   LINE      CODE     ---       #108
      0100198AH   LINE      CODE     ---       #109
      0100198AH   LINE      CODE     ---       #110
      01001990H   LINE      CODE     ---       #111
      01001990H   LINE      CODE     ---       #112
      01001992H   LINE      CODE     ---       #113
      01001992H   LINE      CODE     ---       #114
      01001999H   LINE      CODE     ---       #115
      0100199DH   LINE      CODE     ---       #116
      0100199FH   LINE      CODE     ---       #117
      0100199FH   LINE      CODE     ---       #118
      010019A6H   LINE      CODE     ---       #119
      010019AAH   LINE      CODE     ---       #120
      010019AAH   LINE      CODE     ---       #121
      010019AAH   LINE      CODE     ---       #122
      010019AAH   LINE      CODE     ---       #123
      010019AAH   LINE      CODE     ---       #124
      010019B8H   LINE      CODE     ---       #125
      ---         BLOCKEND  ---      ---       LVL=0

      01001D97H   BLOCK     CODE     ---       LVL=0
      00000020H.0 SYMBOL    BIT      BIT       Mode
      00000020H.1 SYMBOL    BIT      BIT       Status
      01001D97H   LINE      CODE     ---       #136
      01001D97H   LINE      CODE     ---       #137
      01001D97H   LINE      CODE     ---       #138
      01001DA6H   LINE      CODE     ---       #139
      01001DB4H   LINE      CODE     ---       #140
      ---         BLOCKEND  ---      ---       LVL=0

      01001B1DH   BLOCK     CODE     ---       LVL=0
      00000006H   SYMBOL    DATA     WORD      Value
      00000020H.0 SYMBOL    BIT      BIT       Status
      01001B1DH   LINE      CODE     ---       #152
      01001B1DH   LINE      CODE     ---       #153
      01001B1DH   LINE      CODE     ---       #154
      01001B2CH   LINE      CODE     ---       #155
      01001B48H   LINE      CODE     ---       #156
      01001B4FH   LINE      CODE     ---       #157
      01001B53H   LINE      CODE     ---       #158
      ---         BLOCKEND  ---      ---       LVL=0

      01001EA7H   BLOCK     CODE     ---       LVL=0
      01001EA7H   LINE      CODE     ---       #167
      01001EA7H   LINE      CODE     ---       #168
      01001EA7H   LINE      CODE     ---       #169
      01001EAEH   LINE      CODE     ---       #170
      ---         BLOCKEND  ---      ---       LVL=0
      00000082H   SYMBOL    DATA     ---       FlashAddress
      00000082H   SYMBOL    DATA     ---       FlashAddress
      00000005H   SYMBOL    DATA     BYTE      FlashData

      ---         MODULE    ---      ---       ?C?FPADD
      0100006DH   PUBLIC    CODE     ---       ?C?FPADD
LX51 LINKER/LOCATER V4.66.1.0                                                         03/23/2017  15:15:44  PAGE 146


      01000069H   PUBLIC    CODE     ---       ?C?FPSUB

      ---         MODULE    ---      ---       ?C?FPMUL
      0100015EH   PUBLIC    CODE     ---       ?C?FPMUL

      ---         MODULE    ---      ---       ?C?FPDIV
      01000267H   PUBLIC    CODE     ---       ?C?FPDIV

      ---         MODULE    ---      ---       ?C?FCAST
      0100030EH   PUBLIC    CODE     ---       ?C?FCASTC
      01000309H   PUBLIC    CODE     ---       ?C?FCASTI
      01000304H   PUBLIC    CODE     ---       ?C?FCASTL

      ---         MODULE    ---      ---       ?C?CASTF
      01000342H   PUBLIC    CODE     ---       ?C?CASTF

      ---         MODULE    ---      ---       ?C?FPGETOPN
      01000379H   PUBLIC    CODE     ---       ?C?FPGETOPN2
      010003AEH   PUBLIC    CODE     ---       ?C?FPNANRESULT
      010003B8H   PUBLIC    CODE     ---       ?C?FPOVERFLOW
      01000390H   PUBLIC    CODE     ---       ?C?FPRESULT
      010003A4H   PUBLIC    CODE     ---       ?C?FPRESULT2
      010003B5H   PUBLIC    CODE     ---       ?C?FPUNDERFLOW

      ---         MODULE    ---      ---       ?C_STARTUP
      01000000H   PUBLIC    CODE     ---       ?C_STARTUP

      ---         MODULE    ---      ---       ?C?ULDIV
      010003FFH   PUBLIC    CODE     ---       ?C?ULDIV

      ---         MODULE    ---      ---       ?C?LNEG
      01000491H   PUBLIC    CODE     ---       ?C?LNEG

      ---         MODULE    ---      ---       ?C?SLCMP
      0100049FH   PUBLIC    CODE     ---       ?C?SLCMP

      ---         MODULE    ---      ---       ?C?ULCMP
      010004B5H   PUBLIC    CODE     ---       ?C?ULCMP

      ---         MODULE    ---      ---       ?C?SLSHR
      010004C6H   PUBLIC    CODE     ---       ?C?SLSHR

      ---         MODULE    ---      ---       ?C?LSTXDATA
      010004DAH   PUBLIC    CODE     ---       ?C?LSTXDATA

      ---         MODULE    ---      ---       ?C?LSTKXDATA
      010004E6H   PUBLIC    CODE     ---       ?C?LSTKXDATA

      ---         MODULE    ---      ---       ?C?ICASE
      01000517H   PUBLIC    CODE     ---       ?C?ICASE

      ---         MODULE    ---      ---       ?C?LIMUL
      01000544H   PUBLIC    CODE     ---       ?C?LIMUL

      ---         MODULE    ---      ---       ?C_INIT
      010015AAH   PUBLIC    CODE     ---       ?C_START



*** WARNING L25: DATA TYPES DIFFERENT
    SYMBOL:  MDUInit
    MODULE:  .\Output\main.obj (MAIN)
   DEFINED:  .\Output\MDU.obj (MDU)

Program Size: data=65.3 xdata=400 const=0 code=7846
LX51 LINKER/LOCATER V4.66.1.0                                                         03/23/2017  15:15:44  PAGE 147


LX51 RUN COMPLETE.  1 WARNING(S),  0 ERROR(S)
